 fontmanager

 Timestamp is ffffffff (Sun Feb  7 06:28:15 2106)

 Preferred load address is 10000000

 Start         Length     Name                   Class
 0001:00000000 00083a80H .text$mn                CODE
 0002:00000000 00000210H .idata$5                DATA
 0002:00000210 00000004H .00cfg                  DATA
 0002:00000214 00000004H .CRT$XCA                DATA
 0002:00000218 00000004H .CRT$XCZ                DATA
 0002:0000021c 00000004H .CRT$XIA                DATA
 0002:00000220 00000004H .CRT$XIZ                DATA
 0002:00000224 00000004H .CRT$XLA                DATA
 0002:00000228 00000004H .CRT$XLZ                DATA
 0002:0000022c 00000004H .CRT$XPA                DATA
 0002:00000230 00000004H .CRT$XPZ                DATA
 0002:00000234 00000004H .CRT$XTA                DATA
 0002:00000238 00000008H .CRT$XTZ                DATA
 0002:0000023c 00000000H .gfids$y                DATA
 0002:00000240 0002ef00H .rdata                  DATA
 0002:0002f140 00000020H .rdata$T                DATA
 0002:0002f160 00000004H .rdata$sxdata           DATA
 0002:0002f164 000002e8H .rdata$zzzdbg           DATA
 0002:0002f44c 00000004H .rtc$IAA                DATA
 0002:0002f450 00000004H .rtc$IZZ                DATA
 0002:0002f454 00000004H .rtc$TAA                DATA
 0002:0002f458 00000004H .rtc$TZZ                DATA
 0002:0002f45c 00000001H .tls                    DATA
 0002:0002f45d 00000003H .tls$ZZZ                DATA
 0002:0002f460 00000080H .xdata$x                DATA
 0002:0002f4e0 000008dcH .edata                  DATA
 0002:0002fdbc 0000012cH .idata$2                DATA
 0002:0002fee8 00000014H .idata$3                DATA
 0002:0002fefc 00000210H .idata$4                DATA
 0002:0003010c 00000a36H .idata$6                DATA
 0003:00000000 00000900H .data                   DATA
 0003:00000900 00000da0H .bss                    DATA
 0004:00000000 00000060H .rsrc$01                DATA
 0004:00000060 00000320H .rsrc$02                DATA

  Address         Publics by Value              Rva+Base       Lib:Object

 0000:00000000       ___volatile_metadata       00000000     <absolute>
 0000:00000000       ___enclave_config          00000000     <absolute>
 0000:00000000       ___guard_longjmp_count     00000000     <absolute>
 0000:00000000       ___guard_longjmp_table     00000000     <absolute>
 0000:00000000       ___hybrid_code_map         00000000     <absolute>
 0000:00000000       ___hybrid_auxiliary_iat    00000000     <absolute>
 0000:00000000       ___guard_fids_table        00000000     <absolute>
 0000:00000000       ___dynamic_value_reloc_table 00000000     <absolute>
 0000:00000000       ___guard_iat_count         00000000     <absolute>
 0000:00000000       ___guard_fids_count        00000000     <absolute>
 0000:00000000       ___hybrid_code_map_count   00000000     <absolute>
 0000:00000000       ___guard_iat_table         00000000     <absolute>
 0000:00000001       ___safe_se_handler_count   00000001     <absolute>
 0000:0000002c       __tls_array                0000002c     <absolute>
 0000:00000100       ___guard_flags             00000100     <absolute>
 0000:00000000       ___ImageBase               10000000     <linker-defined>
 0001:00000000       _Java_sun_java2d_loops_DrawGlyphListAA_DrawGlyphListAA@20 10001000 f   DrawGlyphList.obj
 0001:00000000       _Java_sun_java2d_loops_DrawGlyphList_DrawGlyphList@20 10001000 f   DrawGlyphList.obj
 0001:00000070       _Java_sun_java2d_loops_DrawGlyphListLCD_DrawGlyphListLCD@20 10001070 f   DrawGlyphList.obj
 0001:00000120       _RefineBounds              10001120 f   DrawGlyphList.obj
 0001:000005e0       _initLCDGammaTables        100015e0 f   DrawGlyphList.obj
 0001:00000620       _initLUT                   10001620 f   DrawGlyphList.obj
 0001:00000750       _setupBlitVector           10001750 f   DrawGlyphList.obj
 0001:00000b60       _setupLCDBlitVector        10001b60 f   DrawGlyphList.obj
 0001:00001120       _Java_sun_font_SunLayoutEngine_shape@68 10002120 f   HBShaper.obj
 0001:000014f0       _storeGVData               100024f0 f   HBShaper.obj
 0001:00001ef0       _Java_sun_awt_Win32FontManager_getFontPath@12 10002ef0 f   fontpath.obj
 0001:00002070       _Java_sun_awt_Win32FontManager_populateFontFileNameMap0@24 10003070 f   fontpath.obj
 0001:00002490       _StringCchCatA@12          10003490 f i fontpath.obj
 0001:000029d0       _Java_sun_font_FreetypeFontScaler_createScalerContextNative@36 100039d0 f   freetypeScaler.obj
 0001:00002bc0       _Java_sun_font_FreetypeFontScaler_disposeNativeScaler@20 10003bc0 f   freetypeScaler.obj
 0001:00002bf0       _Java_sun_font_FreetypeFontScaler_getFontMetricsNative@28 10003bf0 f   freetypeScaler.obj
 0001:00002f30       _Java_sun_font_FreetypeFontScaler_getGlyphAdvanceNative@32 10003f30 f   freetypeScaler.obj
 0001:00002f90       _Java_sun_font_FreetypeFontScaler_getGlyphCodeNative@24 10003f90 f   freetypeScaler.obj
 0001:00003000       _Java_sun_font_FreetypeFontScaler_getGlyphImageNative@32 10004000 f   freetypeScaler.obj
 0001:00003030       _Java_sun_font_FreetypeFontScaler_getGlyphMetricsNative@36 10004030 f   freetypeScaler.obj
 0001:000030f0       _Java_sun_font_FreetypeFontScaler_getGlyphOutlineBoundsNative@32 100040f0 f   freetypeScaler.obj
 0001:00003270       _Java_sun_font_FreetypeFontScaler_getGlyphOutlineNative@40 10004270 f   freetypeScaler.obj
 0001:000033e0       _Java_sun_font_FreetypeFontScaler_getGlyphPointNative@36 100043e0 f   freetypeScaler.obj
 0001:000034b0       _Java_sun_font_FreetypeFontScaler_getGlyphVectorOutlineNative@44 100044b0 f   freetypeScaler.obj
 0001:000036b0       _Java_sun_font_FreetypeFontScaler_getMissingGlyphCodeNative@16 100046b0 f   freetypeScaler.obj
 0001:000036c0       _Java_sun_font_FreetypeFontScaler_getNumGlyphsNative@16 100046c0 f   freetypeScaler.obj
 0001:00003710       _Java_sun_font_FreetypeFontScaler_getUnitsPerEMNative@16 10004710 f   freetypeScaler.obj
 0001:00003730       _Java_sun_font_FreetypeFontScaler_initIDs@12 10004730 f   freetypeScaler.obj
 0001:00003760       _Java_sun_font_FreetypeFontScaler_initNativeScaler@28 10004760 f   freetypeScaler.obj
 0001:00004530       ?fini@hb_user_data_array_t@@QAEXXZ 10005530 f i gsubgpos-context.obj
 0001:00004640       ?to_int@?$FixedVersion@U?$IntType@G$01@OT@@@OT@@QBEIXZ 10005640 f i gsubgpos-context.obj
 0001:00004640       ??B?$IntType@I$03@OT@@QBEIXZ 10005640 f i hb-aat-layout.obj
 0001:00004660       ??$?0PBU?$ChainSubtable@UExtendedTypes@AAT@@@AAT@@@hb_sanitize_with_object_t@@QAE@PAUhb_sanitize_context_t@@ABQBU?$ChainSubtable@UExtendedTypes@AAT@@@AAT@@@Z 10005660 f i hb-aat-layout.obj
 0001:00004660       ??$?0PBUKerxSubTable@AAT@@@hb_sanitize_with_object_t@@QAE@PAUhb_sanitize_context_t@@ABQBUKerxSubTable@AAT@@@Z 10005660 f i hb-aat-layout.obj
 0001:00004660       ??$?0PBU?$KernSubTable@UKernAATSubTableHeader@OT@@@OT@@@hb_sanitize_with_object_t@@QAE@PAUhb_sanitize_context_t@@ABQBU?$KernSubTable@UKernAATSubTableHeader@OT@@@OT@@@Z 10005660 f i hb-ot-layout.obj
 0001:000046f0       ??$?0PBU?$ChainSubtable@UObsoleteTypes@AAT@@@AAT@@@hb_sanitize_with_object_t@@QAE@PAUhb_sanitize_context_t@@ABQBU?$ChainSubtable@UObsoleteTypes@AAT@@@AAT@@@Z 100056f0 f i hb-aat-layout.obj
 0001:000047e0       __hb_ot_shaper_face_data_destroy 100057e0 f   hb-ot-shape.obj
 0001:000047e0       ?hb_ot_layout_position_finish_advances@@YAXPAUhb_font_t@@PAUhb_buffer_t@@@Z 100057e0 f   hb-ot-layout.obj
 0001:000047e0       __hb_ot_shaper_font_data_destroy 100057e0 f   hb-ot-shape.obj
 0001:000047e0       __hb_fallback_shaper_face_data_destroy 100057e0 f   hb-fallback-shape.obj
 0001:000047e0       @_guard_check_icall_nop@4  100057e0 f   MSVCRT:guard_support.obj
 0001:000047e0       __hb_fallback_shaper_font_data_destroy 100057e0 f   hb-fallback-shape.obj
 0001:000047f0       ??$bsearch@I@?$hb_sorted_array_t@$$CBU?$RangeRecord@USmallTypes@Layout@OT@@@Common@Layout@OT@@@@QAEPBU?$RangeRecord@USmallTypes@Layout@OT@@@Common@Layout@OT@@ABIPBU1234@@Z 100057f0 f i hb-aat-layout.obj
 0001:00004870       ??$check_array@U?$Entry@X@AAT@@@hb_sanitize_context_t@@QBE_NPBU?$Entry@X@AAT@@I@Z 10005870 f i hb-aat-layout.obj
 0001:00004900       ??$check_array@U?$IntType@G$01@OT@@@hb_sanitize_context_t@@QBE_NPBU?$IntType@G$01@OT@@I@Z 10005900 f i hb-aat-layout.obj
 0001:00004920       ??$check_array@UFeature@AAT@@@hb_sanitize_context_t@@QBE_NPBUFeature@AAT@@I@Z 10005920 f i hb-aat-layout.obj
 0001:000049b0       ??$check_array@UHBGlyphID16@OT@@@hb_sanitize_context_t@@QBE_NPBUHBGlyphID16@OT@@I@Z 100059b0 f i hb-aat-layout.obj
 0001:00004a40       ??$check_range@U?$IntType@G$01@OT@@@hb_sanitize_context_t@@QBE_NPBU?$IntType@G$01@OT@@II@Z 10005a40 f i hb-aat-layout.obj
 0001:00004a40       ??$check_range@U?$IntType@E$00@OT@@@hb_sanitize_context_t@@QBE_NPBU?$IntType@E$00@OT@@II@Z 10005a40 f i hb-aat-layout.obj
 0001:00004a40       ??$check_range@U?$IntType@F$01@OT@@@hb_sanitize_context_t@@QBE_NPBU?$IntType@F$01@OT@@II@Z 10005a40 f i hb-aat-layout.obj
 0001:00004ae0       ??$collect_coverage@U?$hb_set_digest_combiner_t@U?$hb_set_digest_bits_pattern_t@K$03@@U?$hb_set_digest_combiner_t@U?$hb_set_digest_bits_pattern_t@K$0A@@@U?$hb_set_digest_bits_pattern_t@K$08@@@@@@@?$CoverageFormat2_4@USmallTypes@Layout@OT@@@Common@Layout@OT@@ABE_NPAU?$hb_set_digest_combiner_t@U?$hb_set_digest_bits_pattern_t@K$03@@U?$hb_set_digest_combiner_t@U?$hb_set_digest_bits_pattern_t@K$0A@@@U?$hb_set_digest_bits_pattern_t@K$08@@@@@@@Z 10005ae0 f i hb-aat-layout.obj
 0001:00004c70       ??$collect_coverage@U?$hb_set_digest_combiner_t@U?$hb_set_digest_bits_pattern_t@K$03@@U?$hb_set_digest_combiner_t@U?$hb_set_digest_bits_pattern_t@K$0A@@@U?$hb_set_digest_bits_pattern_t@K$08@@@@@@@Coverage@Common@Layout@OT@@QBE_NPAU?$hb_set_digest_combiner_t@U?$hb_set_digest_bits_pattern_t@K$03@@U?$hb_set_digest_combiner_t@U?$hb_set_digest_bits_pattern_t@K$0A@@@U?$hb_set_digest_bits_pattern_t@K$08@@@@@@@Z 10005c70 f i hb-aat-layout.obj
 0001:00004d30       ??$collect_coverage@U?$hb_set_digest_combiner_t@U?$hb_set_digest_bits_pattern_t@K$03@@U?$hb_set_digest_combiner_t@U?$hb_set_digest_bits_pattern_t@K$0A@@@U?$hb_set_digest_bits_pattern_t@K$08@@@@@@@MarkGlyphSetsFormat1@OT@@QBEXAAU?$hb_vector_t@U?$hb_set_digest_combiner_t@U?$hb_set_digest_bits_pattern_t@K$03@@U?$hb_set_digest_combiner_t@U?$hb_set_digest_bits_pattern_t@K$0A@@@U?$hb_set_digest_bits_pattern_t@K$08@@@@@@$0A@@@@Z 10005d30 f i hb-aat-layout.obj
 0001:00004f30       ??$dispatch@U?$ClassTable@U?$IntType@E$00@OT@@@AAT@@$$V@hb_sanitize_context_t@@QAE_NABU?$ClassTable@U?$IntType@E$00@OT@@@AAT@@@Z 10005f30 f i hb-aat-layout.obj
 0001:00004fb0       ??$dispatch@U?$UnsizedArrayOf@U?$OffsetTo@U?$ArrayOf@UAnchor@AAT@@U?$IntType@I$03@OT@@@OT@@U?$IntType@G$01@2@$0A@@OT@@@OT@@IAAPBX@hb_sanitize_context_t@@QAE_NABU?$UnsizedArrayOf@U?$OffsetTo@U?$ArrayOf@UAnchor@AAT@@U?$IntType@I$03@OT@@@OT@@U?$IntType@G$01@2@$0A@@OT@@@OT@@$$QAIAAPBX@Z 10005fb0 f i hb-aat-layout.obj
 0001:00005030       ??$dispatch@UAttachList@OT@@$$V@hb_sanitize_context_t@@QAE_NABUAttachList@OT@@@Z 10006030 f i hb-aat-layout.obj
 0001:00005140       ??$dispatch@UClassDef@OT@@$$V@hb_sanitize_context_t@@QAE_NABUClassDef@OT@@@Z 10006140 f i hb-aat-layout.obj
 0001:00005200       ??$dispatch@UCoverage@Common@Layout@OT@@$$V@hb_sanitize_context_t@@QAE_NABUCoverage@Common@Layout@OT@@@Z 10006200 f i hb-aat-layout.obj
 0001:00005260       ??$dispatch@ULigCaretList@OT@@$$V@hb_sanitize_context_t@@QAE_NABULigCaretList@OT@@@Z 10006260 f i hb-aat-layout.obj
 0001:00005370       ??$dispatch@ULigGlyph@OT@@$$V@hb_sanitize_context_t@@QAE_NABULigGlyph@OT@@@Z 10006370 f i hb-aat-layout.obj
 0001:00005420       ??$dispatch@UMarkGlyphSets@OT@@$$V@hb_sanitize_context_t@@QAE_NABUMarkGlyphSets@OT@@@Z 10006420 f i hb-aat-layout.obj
 0001:00005500       ??$dispatch@UVarData@OT@@$$V@hb_sanitize_context_t@@QAE_NABUVarData@OT@@@Z 10006500 f i hb-aat-layout.obj
 0001:000055e0       ??$dispatch@UVarRegionList@OT@@$$V@hb_sanitize_context_t@@QAE_NABUVarRegionList@OT@@@Z 100065e0 f i hb-aat-layout.obj
 0001:00005680       ??$dispatch@Uhb_aat_apply_context_t@AAT@@$$V@?$ChainSubtable@UExtendedTypes@AAT@@@AAT@@QBE_NPAUhb_aat_apply_context_t@1@@Z 10006680 f i hb-aat-layout.obj
 0001:00005990       ??$dispatch@Uhb_aat_apply_context_t@AAT@@$$V@?$ChainSubtable@UObsoleteTypes@AAT@@@AAT@@QBE_NPAUhb_aat_apply_context_t@1@@Z 10006990 f i hb-aat-layout.obj
 0001:00005c40       ??$dispatch@Uhb_aat_apply_context_t@AAT@@$$V@KerxSubTable@AAT@@QBE_NPAUhb_aat_apply_context_t@1@@Z 10006c40 f i hb-aat-layout.obj
 0001:00005f00       ??$dispatch@Uhb_sanitize_context_t@@$$V@?$ChainSubtable@UExtendedTypes@AAT@@@AAT@@QBE_NPAUhb_sanitize_context_t@@@Z 10006f00 f i hb-aat-layout.obj
 0001:000061d0       ??$dispatch@Uhb_sanitize_context_t@@$$V@?$ChainSubtable@UObsoleteTypes@AAT@@@AAT@@QBE_NPAUhb_sanitize_context_t@@@Z 100071d0 f i hb-aat-layout.obj
 0001:000063b0       ??$dispatch@Uhb_sanitize_context_t@@$$V@KerxSubTable@AAT@@QBE_NPAUhb_sanitize_context_t@@@Z 100073b0 f i hb-aat-layout.obj
 0001:00006500       ??$drive@Udriver_context_t@?$ContextualSubtable@UExtendedTypes@AAT@@@AAT@@@?$StateTableDriver@UExtendedTypes@AAT@@UEntryData@?$ContextualSubtable@UExtendedTypes@AAT@@@2@@AAT@@QAEXPAUdriver_context_t@?$ContextualSubtable@UExtendedTypes@AAT@@@1@PAUhb_aat_apply_context_t@1@@Z 10007500 f i hb-aat-layout.obj
 0001:00006850       ??$drive@Udriver_context_t@?$ContextualSubtable@UObsoleteTypes@AAT@@@AAT@@@?$StateTableDriver@UObsoleteTypes@AAT@@UEntryData@?$ContextualSubtable@UObsoleteTypes@AAT@@@2@@AAT@@QAEXPAUdriver_context_t@?$ContextualSubtable@UObsoleteTypes@AAT@@@1@PAUhb_aat_apply_context_t@1@@Z 10007850 f i hb-aat-layout.obj
 0001:00006b00       ??$drive@Udriver_context_t@?$InsertionSubtable@UExtendedTypes@AAT@@@AAT@@@?$StateTableDriver@UExtendedTypes@AAT@@UEntryData@?$InsertionSubtable@UExtendedTypes@AAT@@@2@@AAT@@QAEXPAUdriver_context_t@?$InsertionSubtable@UExtendedTypes@AAT@@@1@PAUhb_aat_apply_context_t@1@@Z 10007b00 f i hb-aat-layout.obj
 0001:00006f50       ??$drive@Udriver_context_t@?$InsertionSubtable@UObsoleteTypes@AAT@@@AAT@@@?$StateTableDriver@UObsoleteTypes@AAT@@UEntryData@?$InsertionSubtable@UObsoleteTypes@AAT@@@2@@AAT@@QAEXPAUdriver_context_t@?$InsertionSubtable@UObsoleteTypes@AAT@@@1@PAUhb_aat_apply_context_t@1@@Z 10007f50 f i hb-aat-layout.obj
 0001:00007210       ??$drive@Udriver_context_t@?$KerxSubTableFormat1@UKerxSubTableHeader@AAT@@@AAT@@@?$StateTableDriver@UExtendedTypes@AAT@@UEntryData@?$Format1Entry@$00@2@@AAT@@QAEXPAUdriver_context_t@?$KerxSubTableFormat1@UKerxSubTableHeader@AAT@@@1@PAUhb_aat_apply_context_t@1@@Z 10008210 f i hb-aat-layout.obj
 0001:000075c0       ??$drive@Udriver_context_t@?$KerxSubTableFormat4@UKerxSubTableHeader@AAT@@@AAT@@@?$StateTableDriver@UExtendedTypes@AAT@@UEntryData@?$KerxSubTableFormat4@UKerxSubTableHeader@AAT@@@2@@AAT@@QAEXPAUdriver_context_t@?$KerxSubTableFormat4@UKerxSubTableHeader@AAT@@@1@PAUhb_aat_apply_context_t@1@@Z 100085c0 f i hb-aat-layout.obj
 0001:00007970       ??$drive@Udriver_context_t@?$LigatureSubtable@UExtendedTypes@AAT@@@AAT@@@?$StateTableDriver@UExtendedTypes@AAT@@UEntryData@?$LigatureEntry@$00@2@@AAT@@QAEXPAUdriver_context_t@?$LigatureSubtable@UExtendedTypes@AAT@@@1@PAUhb_aat_apply_context_t@1@@Z 10008970 f i hb-aat-layout.obj
 0001:00007d00       ??$drive@Udriver_context_t@?$LigatureSubtable@UObsoleteTypes@AAT@@@AAT@@@?$StateTableDriver@UObsoleteTypes@AAT@@X@AAT@@QAEXPAUdriver_context_t@?$LigatureSubtable@UObsoleteTypes@AAT@@@1@PAUhb_aat_apply_context_t@1@@Z 10008d00 f i hb-aat-layout.obj
 0001:000080e0       ??$drive@Udriver_context_t@?$RearrangementSubtable@UExtendedTypes@AAT@@@AAT@@@?$StateTableDriver@UExtendedTypes@AAT@@X@AAT@@QAEXPAUdriver_context_t@?$RearrangementSubtable@UExtendedTypes@AAT@@@1@PAUhb_aat_apply_context_t@1@@Z 100090e0 f i hb-aat-layout.obj
 0001:00008430       ??$drive@Udriver_context_t@?$RearrangementSubtable@UObsoleteTypes@AAT@@@AAT@@@?$StateTableDriver@UObsoleteTypes@AAT@@X@AAT@@QAEXPAUdriver_context_t@?$RearrangementSubtable@UObsoleteTypes@AAT@@@1@PAUhb_aat_apply_context_t@1@@Z 10009430 f i hb-aat-layout.obj
 0001:00008860       ??$replace_glyphs@I@hb_buffer_t@@QAE_NIIPBI@Z 10009860 f i hb-aat-layout.obj
 0001:00008910       ??$replace_glyphs@UHBGlyphID16@OT@@@hb_buffer_t@@QAE_NIIPBUHBGlyphID16@OT@@@Z 10009910 f i hb-aat-layout.obj
 0001:000089e0       ??$sanitize@$$V@?$UnsizedListOfOffset16To@U?$Lookup@UHBGlyphID16@OT@@@AAT@@U?$IntType@G$01@OT@@$0A@@OT@@QBE_NPAUhb_sanitize_context_t@@I@Z 100099e0 f i hb-aat-layout.obj
 0001:00008a50       ??$sanitize@$$V@?$UnsizedListOfOffset16To@U?$Lookup@UHBGlyphID16@OT@@@AAT@@U?$IntType@I$03@OT@@$0A@@OT@@QBE_NPAUhb_sanitize_context_t@@I@Z 10009a50 f i hb-aat-layout.obj
 0001:00008ad0       ??$sanitize_blob@UGDEF@OT@@@hb_sanitize_context_t@@QAEPAUhb_blob_t@@PAU1@@Z 10009ad0 f i hb-aat-layout.obj
 0001:00008c80       ??$sanitize_blob@Uankr@AAT@@@hb_sanitize_context_t@@QAEPAUhb_blob_t@@PAU1@@Z 10009c80 f i hb-aat-layout.obj
 0001:00008f80       ??$sanitize_blob@Ufeat@AAT@@@hb_sanitize_context_t@@QAEPAUhb_blob_t@@PAU1@@Z 10009f80 f i hb-aat-layout.obj
 0001:00009110       ??$sanitize_blob@Ukerx@AAT@@@hb_sanitize_context_t@@QAEPAUhb_blob_t@@PAU1@@Z 1000a110 f i hb-aat-layout.obj
 0001:000092a0       ??$sanitize_blob@Ultag@AAT@@@hb_sanitize_context_t@@QAEPAUhb_blob_t@@PAU1@@Z 1000a2a0 f i hb-aat-layout.obj
 0001:00009430       ??$sanitize_blob@Umort@AAT@@@hb_sanitize_context_t@@QAEPAUhb_blob_t@@PAU1@@Z 1000a430 f i hb-aat-layout.obj
 0001:00009880       ??$sanitize_blob@Umorx@AAT@@@hb_sanitize_context_t@@QAEPAUhb_blob_t@@PAU1@@Z 1000a880 f i hb-aat-layout.obj
 0001:00009ad0       ??$sanitize_blob@Utrak@AAT@@@hb_sanitize_context_t@@QAEPAUhb_blob_t@@PAU1@@Z 1000aad0 f i hb-aat-layout.obj
 0001:00009d80       ??0hb_aat_apply_context_t@AAT@@QAE@PBUhb_ot_shape_plan_t@@PAUhb_font_t@@PAUhb_buffer_t@@PAUhb_blob_t@@@Z 1000ad80 f   hb-aat-layout.obj
 0001:00009e80       ??0hb_ot_apply_context_t@OT@@QAE@IPAUhb_font_t@@PAUhb_buffer_t@@PAUhb_blob_t@@@Z 1000ae80 f i hb-aat-layout.obj
 0001:0000a1e0       ??1hb_aat_apply_context_t@AAT@@QAE@XZ 1000b1e0 f   hb-aat-layout.obj
 0001:0000a230       ??C?$hb_lazy_loader_t@Ufeat@AAT@@U?$hb_table_lazy_loader_t@Ufeat@AAT@@$0CC@$0A@@@Uhb_face_t@@$0CC@Uhb_blob_t@@@@QBEPBUfeat@AAT@@XZ 1000b230 f i hb-aat-layout.obj
 0001:0000a370       ??C?$hb_lazy_loader_t@Ultag@AAT@@U?$hb_table_lazy_loader_t@Ultag@AAT@@$0CB@$0A@@@Uhb_face_t@@$0CB@Uhb_blob_t@@@@QBEPBUltag@AAT@@XZ 1000b370 f i hb-aat-layout.obj
 0001:0000a4b0       ??R<lambda_ed1e1ccc2d0221af3ceea6d64221943e>@@QBE_NXZ 1000b4b0 f i hb-aat-layout.obj
 0001:0000a6a0       ??R<lambda_f16c60a149bb02a89ef922852cd447f9>@@QBE_NXZ 1000b6a0 f i hb-aat-layout.obj
 0001:0000a860       ?_Atomic_compare_exchange_strong_4@std@@YAHPCKPAKKW4memory_order@1@2@Z 1000b860 f i hb-aat-layout.obj
 0001:0000a8f0       ?_infos_find_min_cluster@hb_buffer_t@@QAEIPBUhb_glyph_info_t@@III@Z 1000b8f0 f i hb-aat-layout.obj
 0001:0000a980       ?_infos_set_glyph_flags@hb_buffer_t@@QAEXPAUhb_glyph_info_t@@IIII@Z 1000b980 f i hb-aat-layout.obj
 0001:0000aa50       ?_set_glyph_flags@hb_buffer_t@@QAEXIII_N0@Z 1000ba50 f i hb-aat-layout.obj
 0001:0000abb0       ?alloc@?$hb_vector_t@U?$hb_vector_t@Urange_flags_t@hb_aat_map_t@@$00@@$0A@@@QAE_NI_N@Z 1000bbb0 f i hb-aat-layout.obj
 0001:0000ad50       ?apply@?$Chain@UExtendedTypes@AAT@@@AAT@@QBEXPAUhb_aat_apply_context_t@2@@Z 1000bd50 f i hb-aat-layout.obj
 0001:0000afb0       ?apply@?$Chain@UObsoleteTypes@AAT@@@AAT@@QBEXPAUhb_aat_apply_context_t@2@@Z 1000bfb0 f i hb-aat-layout.obj
 0001:0000b1e0       ?apply@?$KerxTable@Ukerx@AAT@@@AAT@@QBE_NPAUhb_aat_apply_context_t@2@@Z 1000c1e0 f i hb-aat-layout.obj
 0001:0000b460       ?apply@?$NoncontextualSubtable@UObsoleteTypes@AAT@@@AAT@@QBE_NPAUhb_aat_apply_context_t@2@@Z 1000c460 f i hb-aat-layout.obj
 0001:0000b460       ?apply@?$NoncontextualSubtable@UExtendedTypes@AAT@@@AAT@@QBE_NPAUhb_aat_apply_context_t@2@@Z 1000c460 f i hb-aat-layout.obj
 0001:0000b5a0       ?apply@trak@AAT@@QBE_NPAUhb_aat_apply_context_t@2@@Z 1000c5a0 f i hb-aat-layout.obj
 0001:0000b8c0       ?backtrack_len@hb_buffer_t@@QBEIXZ 1000c8c0 f i hb-aat-layout.obj
 0001:0000b8d0       ?compile_flags@?$Chain@UExtendedTypes@AAT@@@AAT@@QBEIPBUhb_aat_map_builder_t@@@Z 1000c8d0 f i hb-aat-layout.obj
 0001:0000bb00       ?compile_flags@?$Chain@UObsoleteTypes@AAT@@@AAT@@QBEIPBUhb_aat_map_builder_t@@@Z 1000cb00 f i hb-aat-layout.obj
 0001:0000bd10       ?compile_flags@?$mortmorx@UExtendedTypes@AAT@@$0GNGPHCHI@@AAT@@QBEXPBUhb_aat_map_builder_t@@PAUhb_aat_map_t@@@Z 1000cd10 f i hb-aat-layout.obj
 0001:0000bf00       ?compile_flags@?$mortmorx@UObsoleteTypes@AAT@@$0GNGPHCHE@@AAT@@QBEXPBUhb_aat_map_builder_t@@PAUhb_aat_map_t@@@Z 1000cf00 f i hb-aat-layout.obj
 0001:0000c0f0       ?copy_glyph@hb_buffer_t@@QAE_NXZ 1000d0f0 f i hb-aat-layout.obj
 0001:0000c150       ?create@?$hb_lazy_loader_t@UGDEF_accelerator_t@OT@@U?$hb_face_lazy_loader_t@UGDEF_accelerator_t@OT@@$0BI@@@Uhb_face_t@@$0BI@U12@@@SAPAUGDEF_accelerator_t@OT@@PAUhb_face_t@@@Z 1000d150 f i hb-aat-layout.obj
 0001:0000c2e0       ?create_cache@VariationStore@OT@@QBEPAMXZ 1000d2e0 f i hb-aat-layout.obj
 0001:0000c350       ?do_destroy@?$hb_lazy_loader_t@UGDEF_accelerator_t@OT@@U?$hb_face_lazy_loader_t@UGDEF_accelerator_t@OT@@$0BI@@@Uhb_face_t@@$0BI@U12@@@SAXPAUGDEF_accelerator_t@OT@@@Z 1000d350 f i hb-aat-layout.obj
 0001:0000c3b0       ?em_scale_x@hb_font_t@@QAEHF@Z 1000d3b0 f i hb-aat-layout.obj
 0001:0000c3e0       ?em_scale_y@hb_font_t@@QAEHF@Z 1000d3e0 f i hb-aat-layout.obj
 0001:0000c410       ?em_scalef_x@hb_font_t@@QAEHM@Z 1000d410 f i hb-aat-layout.obj
 0001:0000c460       ?em_scalef_y@hb_font_t@@QAEHM@Z 1000d460 f i hb-aat-layout.obj
 0001:0000c4b0       ?end_processing@hb_sanitize_context_t@@QAEXXZ 1000d4b0 f i hb-aat-layout.obj
 0001:0000c500       ?get@?$hb_lazy_loader_t@UGDEF_accelerator_t@OT@@U?$hb_face_lazy_loader_t@UGDEF_accelerator_t@OT@@$0BI@@@Uhb_face_t@@$0BI@U12@@@QBEPBUGDEF_accelerator_t@OT@@XZ 1000d500 f i hb-aat-layout.obj
 0001:0000c5c0       ?get@?$hb_lazy_loader_t@Utrak@AAT@@U?$hb_table_lazy_loader_t@Utrak@AAT@@$0CA@$0A@@@Uhb_face_t@@$0CA@Uhb_blob_t@@@@QBEPBUtrak@AAT@@XZ 1000d5c0 f i hb-aat-layout.obj
 0001:0000c700       ?get_anchor@ankr@AAT@@QBEABUAnchor@2@III@Z 1000d700 f i hb-aat-layout.obj
 0001:0000c7b0       ?get_class@ClassDef@OT@@QBEII@Z 1000d7b0 f i hb-aat-layout.obj
 0001:0000c880       ?get_coverage@?$CoverageFormat1_3@USmallTypes@Layout@OT@@@Common@Layout@OT@@ABEII@Z 1000d880 f i hb-aat-layout.obj
 0001:0000c8e0       ?get_coverage@?$CoverageFormat2_4@USmallTypes@Layout@OT@@@Common@Layout@OT@@ABEII@Z 1000d8e0 f i hb-aat-layout.obj
 0001:0000c970       ?get_entry@?$StateTable@UExtendedTypes@AAT@@UEntryData@?$ContextualSubtable@UExtendedTypes@AAT@@@2@@AAT@@QBEABU?$Entry@UEntryData@?$ContextualSubtable@UExtendedTypes@AAT@@@AAT@@@2@HI@Z 1000d970 f i hb-aat-layout.obj
 0001:0000c970       ?get_entry@?$StateTable@UExtendedTypes@AAT@@UEntryData@?$InsertionSubtable@UExtendedTypes@AAT@@@2@@AAT@@QBEABU?$Entry@UEntryData@?$InsertionSubtable@UExtendedTypes@AAT@@@AAT@@@2@HI@Z 1000d970 f i hb-aat-layout.obj
 0001:0000ca10       ?get_entry@?$StateTable@UExtendedTypes@AAT@@UEntryData@?$LigatureEntry@$00@2@@AAT@@QBEABU?$Entry@UEntryData@?$LigatureEntry@$00@AAT@@@2@HI@Z 1000da10 f i hb-aat-layout.obj
 0001:0000ca10       ?get_entry@?$StateTable@UExtendedTypes@AAT@@UEntryData@?$Format1Entry@$00@2@@AAT@@QBEABU?$Entry@UEntryData@?$Format1Entry@$00@AAT@@@2@HI@Z 1000da10 f i hb-aat-layout.obj
 0001:0000ca10       ?get_entry@?$StateTable@UExtendedTypes@AAT@@UEntryData@?$KerxSubTableFormat4@UKerxSubTableHeader@AAT@@@2@@AAT@@QBEABU?$Entry@UEntryData@?$KerxSubTableFormat4@UKerxSubTableHeader@AAT@@@AAT@@@2@HI@Z 1000da10 f i hb-aat-layout.obj
 0001:0000cab0       ?get_entry@?$StateTable@UExtendedTypes@AAT@@X@AAT@@QBEABU?$Entry@X@2@HI@Z 1000dab0 f i hb-aat-layout.obj
 0001:0000cb50       ?get_feature@feat@AAT@@QBEABUFeatureName@2@W4hb_aat_layout_feature_type_t@@@Z 1000db50 f i hb-aat-layout.obj
 0001:0000cbc0       ?get_glyph_contour_point_for_origin@hb_font_t@@QAEHIIW4hb_direction_t@@PAH1@Z 1000dbc0 f i hb-aat-layout.obj
 0001:0000cd70       ?get_glyph_h_advance@hb_font_t@@QAEHI@Z 1000dd70 f i hb-aat-layout.obj
 0001:0000cdb0       ?get_glyph_h_origin_with_fallback@hb_font_t@@QAEXIPAH0@Z 1000ddb0 f i hb-aat-layout.obj
 0001:0000ce40       ?get_glyph_props@GDEF@OT@@QBEII@Z 1000de40 f i hb-aat-layout.obj
 0001:0000cf10       ?get_glyph_v_origin_with_fallback@hb_font_t@@QAEXIPAH0@Z 1000df10 f i hb-aat-layout.obj
 0001:0000cfa0       ?get_h_extents_with_fallback@hb_font_t@@QAEXPAUhb_font_extents_t@@@Z 1000dfa0 f i hb-aat-layout.obj
 0001:0000d000       ?get_kerning@?$KerxSubTableFormat0@UKerxSubTableHeader@AAT@@@AAT@@QBEHIIPAUhb_aat_apply_context_t@2@@Z 1000e000 f i hb-aat-layout.obj
 0001:0000d130       ?get_kerning@?$KerxSubTableFormat2@UKerxSubTableHeader@AAT@@@AAT@@QBEHIIPAUhb_aat_apply_context_t@2@@Z 1000e130 f i hb-aat-layout.obj
 0001:0000d270       ?get_kerning@?$KerxSubTableFormat6@UKerxSubTableHeader@AAT@@@AAT@@QBEHIIPAUhb_aat_apply_context_t@2@@Z 1000e270 f i hb-aat-layout.obj
 0001:0000d480       ?get_language@ltag@AAT@@QBEPBUhb_language_impl_t@@I@Z 1000e480 f i hb-aat-layout.obj
 0001:0000d4e0       ?get_length@?$VarSizedBinSearchArrayOf@U?$LookupSegmentSingle@U?$IntType@G$01@OT@@@AAT@@@OT@@QBEIXZ 1000e4e0 f i hb-aat-layout.obj
 0001:0000d4e0       ?get_length@?$VarSizedBinSearchArrayOf@U?$LookupSegmentArray@U?$IntType@G$01@OT@@@AAT@@@OT@@QBEIXZ 1000e4e0 f i hb-aat-layout.obj
 0001:0000d4e0       ?get_length@?$VarSizedBinSearchArrayOf@U?$LookupSegmentSingle@U?$IntType@I$03@OT@@@AAT@@@OT@@QBEIXZ 1000e4e0 f i hb-aat-layout.obj
 0001:0000d4e0       ?get_length@?$VarSizedBinSearchArrayOf@U?$LookupSegmentArray@UHBGlyphID16@OT@@@AAT@@@OT@@QBEIXZ 1000e4e0 f i hb-aat-layout.obj
 0001:0000d4e0       ?get_length@?$VarSizedBinSearchArrayOf@U?$LookupSegmentSingle@U?$OffsetTo@U?$ArrayOf@UAnchor@AAT@@U?$IntType@I$03@OT@@@OT@@U?$IntType@G$01@2@$0A@@OT@@@AAT@@@OT@@QBEIXZ 1000e4e0 f i hb-aat-layout.obj
 0001:0000d4e0       ?get_length@?$VarSizedBinSearchArrayOf@U?$LookupSegmentArray@U?$IntType@I$03@OT@@@AAT@@@OT@@QBEIXZ 1000e4e0 f i hb-aat-layout.obj
 0001:0000d4e0       ?get_length@?$VarSizedBinSearchArrayOf@U?$LookupSegmentSingle@UHBGlyphID16@OT@@@AAT@@@OT@@QBEIXZ 1000e4e0 f i hb-aat-layout.obj
 0001:0000d4e0       ?get_length@?$VarSizedBinSearchArrayOf@U?$LookupSegmentArray@U?$OffsetTo@U?$ArrayOf@UAnchor@AAT@@U?$IntType@I$03@OT@@@OT@@U?$IntType@G$01@2@$0A@@OT@@@AAT@@@OT@@QBEIXZ 1000e4e0 f i hb-aat-layout.obj
 0001:0000d560       ?get_length@?$VarSizedBinSearchArrayOf@U?$LookupSingle@UHBGlyphID16@OT@@@AAT@@@OT@@QBEIXZ 1000e560 f i hb-aat-layout.obj
 0001:0000d560       ?get_length@?$VarSizedBinSearchArrayOf@U?$LookupSingle@U?$OffsetTo@U?$ArrayOf@UAnchor@AAT@@U?$IntType@I$03@OT@@@OT@@U?$IntType@G$01@2@$0A@@OT@@@AAT@@@OT@@QBEIXZ 1000e560 f i hb-aat-layout.obj
 0001:0000d560       ?get_length@?$VarSizedBinSearchArrayOf@U?$LookupSingle@U?$IntType@I$03@OT@@@AAT@@@OT@@QBEIXZ 1000e560 f i hb-aat-layout.obj
 0001:0000d560       ?get_length@?$VarSizedBinSearchArrayOf@U?$LookupSingle@U?$IntType@G$01@OT@@@AAT@@@OT@@QBEIXZ 1000e560 f i hb-aat-layout.obj
 0001:0000d5e0       ?get_mark_glyph_sets@GDEF@OT@@QBEABUMarkGlyphSets@2@XZ 1000e5e0 f i hb-aat-layout.obj
 0001:0000d640       ?get_row_size@VarData@OT@@QBEIXZ 1000e640 f i hb-aat-layout.obj
 0001:0000d690       ?get_size@HintingDevice@OT@@QBEIXZ 1000e690 f i hb-aat-layout.obj
 0001:0000d700       ?get_stored@?$hb_lazy_loader_t@Ukerx@AAT@@U?$hb_table_lazy_loader_t@Ukerx@AAT@@$0BO@$0A@@@Uhb_face_t@@$0BO@Uhb_blob_t@@@@QBEPAUhb_blob_t@@XZ 1000e700 f i hb-aat-layout.obj
 0001:0000d870       ?get_stored@?$hb_lazy_loader_t@Umort@AAT@@U?$hb_table_lazy_loader_t@Umort@AAT@@$0BN@$0A@@@Uhb_face_t@@$0BN@Uhb_blob_t@@@@QBEPAUhb_blob_t@@XZ 1000e870 f i hb-aat-layout.obj
 0001:0000d9e0       ?get_stored@?$hb_lazy_loader_t@Umorx@AAT@@U?$hb_table_lazy_loader_t@Umorx@AAT@@$0BM@$0A@@@Uhb_face_t@@$0BM@Uhb_blob_t@@@@QBEPAUhb_blob_t@@XZ 1000e9e0 f i hb-aat-layout.obj
 0001:0000db50       ?get_tracking@TrackData@AAT@@QBEHPBXM@Z 1000eb50 f i hb-aat-layout.obj
 0001:0000dcf0       ?get_value@?$Lookup@U?$IntType@G$01@OT@@@AAT@@QBEPBU?$IntType@G$01@OT@@II@Z 1000ecf0 f i hb-aat-layout.obj
 0001:0000dcf0       ?get_value@?$Lookup@UHBGlyphID16@OT@@@AAT@@QBEPBUHBGlyphID16@OT@@II@Z 1000ecf0 f i hb-aat-layout.obj
 0001:0000dcf0       ?get_value@?$Lookup@U?$OffsetTo@U?$ArrayOf@UAnchor@AAT@@U?$IntType@I$03@OT@@@OT@@U?$IntType@G$01@2@$0A@@OT@@@AAT@@QBEPBU?$OffsetTo@U?$ArrayOf@UAnchor@AAT@@U?$IntType@I$03@OT@@@OT@@U?$IntType@G$01@2@$0A@@OT@@II@Z 1000ecf0 f i hb-aat-layout.obj
 0001:0000df10       ?get_value@?$Lookup@U?$IntType@I$03@OT@@@AAT@@QBEPBU?$IntType@I$03@OT@@II@Z 1000ef10 f i hb-aat-layout.obj
 0001:0000e130       ?get_value_or_null@?$Lookup@U?$IntType@G$01@OT@@@AAT@@QBE?BGII@Z 1000f130 f i hb-aat-layout.obj
 0001:0000e200       ?get_value_or_null@?$Lookup@U?$IntType@I$03@OT@@@AAT@@QBE?BIII@Z 1000f200 f i hb-aat-layout.obj
 0001:0000e2f0       ?guess_v_origin_minus_h_origin@hb_font_t@@QAEXIPAH0@Z 1000f2f0 f i hb-aat-layout.obj
 0001:0000e3a0       ?hb_aat_layout_compile_map@@YAXPBUhb_aat_map_builder_t@@PAUhb_aat_map_t@@@Z 1000f3a0 f   hb-aat-layout.obj
 0001:0000e420       ?hb_aat_layout_find_feature_mapping@@YAPBUhb_aat_feature_mapping_t@@I@Z 1000f420 f   hb-aat-layout.obj
 0001:0000e470       ?hb_aat_layout_position@@YAXPBUhb_ot_shape_plan_t@@PAUhb_font_t@@PAUhb_buffer_t@@@Z 1000f470 f   hb-aat-layout.obj
 0001:0000e670       ?hb_aat_layout_remove_deleted_glyphs@@YAXPAUhb_buffer_t@@@Z 1000f670 f   hb-aat-layout.obj
 0001:0000e680       ?hb_aat_layout_substitute@@YAXPBUhb_ot_shape_plan_t@@PAUhb_font_t@@PAUhb_buffer_t@@PBUhb_feature_t@@I@Z 1000f680 f   hb-aat-layout.obj
 0001:0000ea80       ?hb_aat_layout_track@@YAXPBUhb_ot_shape_plan_t@@PAUhb_font_t@@PAUhb_buffer_t@@@Z 1000fa80 f   hb-aat-layout.obj
 0001:0000eb00       ?hb_aat_layout_zero_width_deleted_glyphs@@YAXPAUhb_buffer_t@@@Z 1000fb00 f   hb-aat-layout.obj
 0001:0000eb50       ?init_iters@hb_ot_apply_context_t@OT@@QAEXXZ 1000fb50 f i hb-aat-layout.obj
 0001:0000ec30       ?interpolate_at@TrackData@AAT@@QBEMIMABUTrackTableEntry@2@PBX@Z 1000fc30 f i hb-aat-layout.obj
 0001:0000eda0       ?is_actionable@driver_context_t@?$ContextualSubtable@UObsoleteTypes@AAT@@@AAT@@QAE_NPAU?$StateTableDriver@UObsoleteTypes@AAT@@UEntryData@?$ContextualSubtable@UObsoleteTypes@AAT@@@2@@3@ABU?$Entry@UEntryData@?$ContextualSubtable@UObsoleteTypes@AAT@@@AAT@@@3@@Z 1000fda0 f i hb-aat-layout.obj
 0001:0000eda0       ?is_actionable@driver_context_t@?$ContextualSubtable@UExtendedTypes@AAT@@@AAT@@QAE_NPAU?$StateTableDriver@UExtendedTypes@AAT@@UEntryData@?$ContextualSubtable@UExtendedTypes@AAT@@@2@@3@ABU?$Entry@UEntryData@?$ContextualSubtable@UExtendedTypes@AAT@@@AAT@@@3@@Z 1000fda0 f i hb-aat-layout.obj
 0001:0000ee00       ?is_actionable@driver_context_t@?$InsertionSubtable@UObsoleteTypes@AAT@@@AAT@@QAE_NPAU?$StateTableDriver@UObsoleteTypes@AAT@@UEntryData@?$InsertionSubtable@UObsoleteTypes@AAT@@@2@@3@ABU?$Entry@UEntryData@?$InsertionSubtable@UObsoleteTypes@AAT@@@AAT@@@3@@Z 1000fe00 f i hb-aat-layout.obj
 0001:0000ee70       ?kern@?$hb_kern_machine_t@Uaccelerator_t@?$KerxSubTableFormat0@UKerxSubTableHeader@AAT@@@AAT@@@OT@@QBEXPAUhb_font_t@@PAUhb_buffer_t@@I_N@Z 1000fe70 f i hb-aat-layout.obj
 0001:0000f360       ?kern@?$hb_kern_machine_t@Uaccelerator_t@?$KerxSubTableFormat2@UKerxSubTableHeader@AAT@@@AAT@@@OT@@QBEXPAUhb_font_t@@PAUhb_buffer_t@@I_N@Z 10010360 f i hb-aat-layout.obj
 0001:0000f850       ?kern@?$hb_kern_machine_t@Uaccelerator_t@?$KerxSubTableFormat6@UKerxSubTableHeader@AAT@@@AAT@@@OT@@QBEXPAUhb_font_t@@PAUhb_buffer_t@@I_N@Z 10010850 f i hb-aat-layout.obj
 0001:0000fda0       ?mark_set_covers@accelerator_t@GDEF@OT@@QBE_NII@Z 10010da0 f i hb-aat-layout.obj
 0001:0000fef0       ?match_properties_mark@hb_ot_apply_context_t@OT@@QBE_NIII@Z 10010ef0 f i hb-aat-layout.obj
 0001:0000ff30       ?may_edit@hb_sanitize_context_t@@QAE_NPBXI@Z 10010f30 f i hb-aat-layout.obj
 0001:0000ff90       ?merge_clusters@hb_buffer_t@@QAEXII@Z 10010f90 f i hb-aat-layout.obj
 0001:0000ffb0       ?message@hb_buffer_t@@QAA_NPAUhb_font_t@@PBDZZ 10010fb0 f i hb-aat-layout.obj
 0001:0000ffe0       ?next_glyph@hb_buffer_t@@QAE_NXZ 10010fe0 f i hb-aat-layout.obj
 0001:00010040       ?replace_glyph@hb_buffer_t@@QAE_NI@Z 10011040 f i hb-aat-layout.obj
 0001:000100b0       ?reverse_range@hb_buffer_t@@QAEXII@Z 100110b0 f i hb-aat-layout.obj
 0001:00010180       ?sanitize@?$Chain@UExtendedTypes@AAT@@@AAT@@QBE_NPAUhb_sanitize_context_t@@I@Z 10011180 f i hb-aat-layout.obj
 0001:000103e0       ?sanitize@?$Chain@UObsoleteTypes@AAT@@@AAT@@QBE_NPAUhb_sanitize_context_t@@I@Z 100113e0 f i hb-aat-layout.obj
 0001:00010510       ?sanitize@?$ChainSubtable@UObsoleteTypes@AAT@@@AAT@@QBE_NPAUhb_sanitize_context_t@@@Z 10011510 f i hb-aat-layout.obj
 0001:00010600       ?sanitize@?$FixedVersion@U?$IntType@G$01@OT@@@OT@@QBE_NPAUhb_sanitize_context_t@@@Z 10011600 f i hb-aat-layout.obj
 0001:00010600       ?sanitize@?$IntType@H$03@OT@@QBE_NPAUhb_sanitize_context_t@@@Z 10011600 f i hb-aat-layout.obj
 0001:00010600       ?sanitize@?$IntType@I$03@OT@@QBE_NPAUhb_sanitize_context_t@@@Z 10011600 f i hb-aat-layout.obj
 0001:00010670       ?sanitize@?$GDEFVersion1_2@USmallTypes@Layout@OT@@@OT@@QBE_NPAUhb_sanitize_context_t@@@Z 10011670 f i hb-aat-layout.obj
 0001:000108e0       ?sanitize@?$IntType@E$00@OT@@QBE_NPAUhb_sanitize_context_t@@@Z 100118e0 f i hb-aat-layout.obj
 0001:00010950       ?sanitize@?$IntType@G$01@OT@@QBE_NPAUhb_sanitize_context_t@@@Z 10011950 f i hb-aat-layout.obj
 0001:00010950       ?sanitize@?$IntType@F$01@OT@@QBE_NPAUhb_sanitize_context_t@@@Z 10011950 f i hb-aat-layout.obj
 0001:000109c0       ?sanitize@?$KerxSubTableFormat2@UKerxSubTableHeader@AAT@@@AAT@@QBE_NPAUhb_sanitize_context_t@@@Z 100119c0 f i hb-aat-layout.obj
 0001:00010b40       ?sanitize@?$KerxSubTableFormat6@UKerxSubTableHeader@AAT@@@AAT@@QBE_NPAUhb_sanitize_context_t@@@Z 10011b40 f i hb-aat-layout.obj
 0001:00010de0       ?sanitize@?$KerxTable@Ukerx@AAT@@@AAT@@QBE_NPAUhb_sanitize_context_t@@@Z 10011de0 f i hb-aat-layout.obj
 0001:00010fc0       ?sanitize@?$Lookup@U?$IntType@G$01@OT@@@AAT@@QBE_NPAUhb_sanitize_context_t@@@Z 10011fc0 f i hb-aat-layout.obj
 0001:00011210       ?sanitize@?$Lookup@U?$IntType@I$03@OT@@@AAT@@QBE_NPAUhb_sanitize_context_t@@@Z 10012210 f i hb-aat-layout.obj
 0001:00011460       ?sanitize@?$Lookup@U?$OffsetTo@U?$ArrayOf@UAnchor@AAT@@U?$IntType@I$03@OT@@@OT@@U?$IntType@G$01@2@$0A@@OT@@@AAT@@QBE_NPAUhb_sanitize_context_t@@PBX@Z 10012460 f i hb-aat-layout.obj
 0001:00011630       ?sanitize@?$Lookup@UHBGlyphID16@OT@@@AAT@@QBE_NPAUhb_sanitize_context_t@@@Z 10012630 f i hb-aat-layout.obj
 0001:00011870       ?sanitize@?$LookupFormat2@U?$OffsetTo@U?$ArrayOf@UAnchor@AAT@@U?$IntType@I$03@OT@@@OT@@U?$IntType@G$01@2@$0A@@OT@@@AAT@@ABE_NPAUhb_sanitize_context_t@@PBX@Z 10012870 f i hb-aat-layout.obj
 0001:000119d0       ?sanitize@?$LookupFormat4@U?$IntType@G$01@OT@@@AAT@@ABE_NPAUhb_sanitize_context_t@@@Z 100129d0 f i hb-aat-layout.obj
 0001:00011b90       ?sanitize@?$LookupFormat4@U?$IntType@I$03@OT@@@AAT@@ABE_NPAUhb_sanitize_context_t@@@Z 10012b90 f i hb-aat-layout.obj
 0001:00011d50       ?sanitize@?$LookupFormat4@U?$OffsetTo@U?$ArrayOf@UAnchor@AAT@@U?$IntType@I$03@OT@@@OT@@U?$IntType@G$01@2@$0A@@OT@@@AAT@@ABE_NPAUhb_sanitize_context_t@@PBX@Z 10012d50 f i hb-aat-layout.obj
 0001:00011f00       ?sanitize@?$LookupFormat4@UHBGlyphID16@OT@@@AAT@@ABE_NPAUhb_sanitize_context_t@@@Z 10012f00 f i hb-aat-layout.obj
 0001:000120c0       ?sanitize@?$LookupFormat6@U?$OffsetTo@U?$ArrayOf@UAnchor@AAT@@U?$IntType@I$03@OT@@@OT@@U?$IntType@G$01@2@$0A@@OT@@@AAT@@ABE_NPAUhb_sanitize_context_t@@PBX@Z 100130c0 f i hb-aat-layout.obj
 0001:00012220       ?sanitize@?$StateTable@UExtendedTypes@AAT@@UEntryData@?$ContextualSubtable@UExtendedTypes@AAT@@@2@@AAT@@QBE_NPAUhb_sanitize_context_t@@PAI@Z 10013220 f i hb-aat-layout.obj
 0001:00012220       ?sanitize@?$StateTable@UExtendedTypes@AAT@@UEntryData@?$InsertionSubtable@UExtendedTypes@AAT@@@2@@AAT@@QBE_NPAUhb_sanitize_context_t@@PAI@Z 10013220 f i hb-aat-layout.obj
 0001:000125f0       ?sanitize@?$StateTable@UExtendedTypes@AAT@@UEntryData@?$Format1Entry@$00@2@@AAT@@QBE_NPAUhb_sanitize_context_t@@PAI@Z 100135f0 f i hb-aat-layout.obj
 0001:000125f0       ?sanitize@?$StateTable@UExtendedTypes@AAT@@UEntryData@?$LigatureEntry@$00@2@@AAT@@QBE_NPAUhb_sanitize_context_t@@PAI@Z 100135f0 f i hb-aat-layout.obj
 0001:000125f0       ?sanitize@?$StateTable@UExtendedTypes@AAT@@UEntryData@?$KerxSubTableFormat4@UKerxSubTableHeader@AAT@@@2@@AAT@@QBE_NPAUhb_sanitize_context_t@@PAI@Z 100135f0 f i hb-aat-layout.obj
 0001:000129c0       ?sanitize@?$StateTable@UExtendedTypes@AAT@@X@AAT@@QBE_NPAUhb_sanitize_context_t@@PAI@Z 100139c0 f i hb-aat-layout.obj
 0001:00012d00       ?sanitize@?$StateTable@UObsoleteTypes@AAT@@UEntryData@?$ContextualSubtable@UObsoleteTypes@AAT@@@2@@AAT@@QBE_NPAUhb_sanitize_context_t@@PAI@Z 10013d00 f i hb-aat-layout.obj
 0001:00012d00       ?sanitize@?$StateTable@UObsoleteTypes@AAT@@UEntryData@?$InsertionSubtable@UObsoleteTypes@AAT@@@2@@AAT@@QBE_NPAUhb_sanitize_context_t@@PAI@Z 10013d00 f i hb-aat-layout.obj
 0001:00013090       ?sanitize@?$StateTable@UObsoleteTypes@AAT@@X@AAT@@QBE_NPAUhb_sanitize_context_t@@PAI@Z 10014090 f i hb-aat-layout.obj
 0001:00013380       ?sanitize@?$mortmorx@UExtendedTypes@AAT@@$0GNGPHCHI@@AAT@@QBE_NPAUhb_sanitize_context_t@@@Z 10014380 f i hb-aat-layout.obj
 0001:00013450       ?sanitize@?$mortmorx@UObsoleteTypes@AAT@@$0GNGPHCHE@@AAT@@QBE_NPAUhb_sanitize_context_t@@@Z 10014450 f i hb-aat-layout.obj
 0001:00013520       ?sanitize@CaretValue@OT@@QBE_NPAUhb_sanitize_context_t@@@Z 10014520 f i hb-aat-layout.obj
 0001:00013680       ?sanitize@Device@OT@@QBE_NPAUhb_sanitize_context_t@@@Z 10014680 f i hb-aat-layout.obj
 0001:000137f0       ?sanitize@GDEF@OT@@QBE_NPAUhb_sanitize_context_t@@@Z 100147f0 f i hb-aat-layout.obj
 0001:00013830       ?sanitize@KerxSubTableHeader@AAT@@QBE_NPAUhb_sanitize_context_t@@@Z 10014830 f i hb-aat-layout.obj
 0001:00013830       ?sanitize@SBitLineMetrics@OT@@QBE_NPAUhb_sanitize_context_t@@@Z 10014830 f i hb-ot-color.obj
 0001:000138a0       ?sanitize@TrackData@AAT@@QBE_NPAUhb_sanitize_context_t@@PBX@Z 100148a0 f i hb-aat-layout.obj
 0001:00013a70       ?sanitize@VarSizedBinSearchHeader@OT@@QBE_NPAUhb_sanitize_context_t@@@Z 10014a70 f i hb-aat-layout.obj
 0001:00013ae0       ?sanitize@VariationStore@OT@@QBE_NPAUhb_sanitize_context_t@@@Z 10014ae0 f i hb-aat-layout.obj
 0001:00013c70       ?sanitize@ankr@AAT@@QBE_NPAUhb_sanitize_context_t@@@Z 10014c70 f i hb-aat-layout.obj
 0001:00013e00       ?sanitize@feat@AAT@@QBE_NPAUhb_sanitize_context_t@@@Z 10014e00 f i hb-aat-layout.obj
 0001:00013f90       ?sanitize@ltag@AAT@@QBE_NPAUhb_sanitize_context_t@@@Z 10014f90 f i hb-aat-layout.obj
 0001:00014110       ?sanitize@trak@AAT@@QBE_NPAUhb_sanitize_context_t@@@Z 10015110 f i hb-aat-layout.obj
 0001:00014250       ?sanitize_shallow@?$ArrayOf@U?$IntType@E$00@OT@@U?$IntType@G$01@2@@OT@@QBE_NPAUhb_sanitize_context_t@@@Z 10015250 f i hb-aat-layout.obj
 0001:000142f0       ?sanitize_shallow@?$ArrayOf@U?$Offset@U?$IntType@G$01@OT@@$00@OT@@U?$IntType@G$01@2@@OT@@QBE_NPAUhb_sanitize_context_t@@@Z 100152f0 f i hb-ot-layout.obj
 0001:000142f0       ?sanitize_shallow@?$ArrayOf@U?$OffsetTo@U?$ChainRule@USmallTypes@Layout@OT@@@OT@@U?$IntType@G$01@2@$00@OT@@U?$IntType@G$01@2@@OT@@QBE_NPAUhb_sanitize_context_t@@@Z 100152f0 f i hb-ot-layout.obj
 0001:000142f0       ?sanitize_shallow@?$ArrayOf@U?$OffsetTo@U?$Ligature@USmallTypes@Layout@OT@@@GSUB_impl@Layout@OT@@U?$IntType@G$01@4@$00@OT@@U?$IntType@G$01@2@@OT@@QBE_NPAUhb_sanitize_context_t@@@Z 100152f0 f i hb-ot-layout.obj
 0001:000142f0       ?sanitize_shallow@?$ArrayOf@U?$OffsetTo@UAttachPoint@OT@@U?$IntType@G$01@2@$00@OT@@U?$IntType@G$01@2@@OT@@QBE_NPAUhb_sanitize_context_t@@@Z 100152f0 f i hb-aat-layout.obj
 0001:000142f0       ?sanitize_shallow@?$ArrayOf@UHBGlyphID16@OT@@U?$IntType@G$01@2@@OT@@QBE_NPAUhb_sanitize_context_t@@@Z 100152f0 f i hb-aat-layout.obj
 0001:000142f0       ?sanitize_shallow@?$ArrayOf@U?$OffsetTo@ULigGlyph@OT@@U?$IntType@G$01@2@$00@OT@@U?$IntType@G$01@2@@OT@@QBE_NPAUhb_sanitize_context_t@@@Z 100152f0 f i hb-aat-layout.obj
 0001:000142f0       ?sanitize_shallow@?$ArrayOf@UIndex@OT@@U?$IntType@G$01@2@@OT@@QBE_NPAUhb_sanitize_context_t@@@Z 100152f0 f i hb-ot-layout.obj
 0001:000142f0       ?sanitize_shallow@?$ArrayOf@U?$OffsetTo@U?$ChainRuleSet@USmallTypes@Layout@OT@@@OT@@U?$IntType@G$01@2@$00@OT@@U?$IntType@G$01@2@@OT@@QBE_NPAUhb_sanitize_context_t@@@Z 100152f0 f i hb-ot-layout.obj
 0001:000142f0       ?sanitize_shallow@?$ArrayOf@U?$IntType@G$01@OT@@U12@@OT@@QBE_NPAUhb_sanitize_context_t@@@Z 100152f0 f i hb-aat-layout.obj
 0001:000142f0       ?sanitize_shallow@?$ArrayOf@U?$OffsetTo@USubstLookup@GSUB_impl@Layout@OT@@U?$IntType@G$01@4@$00@OT@@U?$IntType@G$01@2@@OT@@QBE_NPAUhb_sanitize_context_t@@@Z 100152f0 f i hb-ot-layout.obj
 0001:000142f0       ?sanitize_shallow@?$ArrayOf@U?$OffsetTo@U?$AlternateSet@USmallTypes@Layout@OT@@@GSUB_impl@Layout@OT@@U?$IntType@G$01@4@$00@OT@@U?$IntType@G$01@2@@OT@@QBE_NPAUhb_sanitize_context_t@@@Z 100152f0 f i hb-ot-layout.obj
 0001:000142f0       ?sanitize_shallow@?$ArrayOf@U?$OffsetTo@USubstLookupSubTable@GSUB_impl@Layout@OT@@U?$IntType@G$01@4@$00@OT@@U?$IntType@G$01@2@@OT@@QBE_NPAUhb_sanitize_context_t@@@Z 100152f0 f i hb-ot-layout.obj
 0001:000142f0       ?sanitize_shallow@?$ArrayOf@U?$OffsetTo@UPosLookupSubTable@GPOS_impl@Layout@OT@@U?$IntType@G$01@4@$00@OT@@U?$IntType@G$01@2@@OT@@QBE_NPAUhb_sanitize_context_t@@@Z 100152f0 f i hb-ot-layout.obj
 0001:000142f0       ?sanitize_shallow@?$ArrayOf@U?$OffsetTo@UPosLookup@GPOS_impl@Layout@OT@@U?$IntType@G$01@4@$00@OT@@U?$IntType@G$01@2@@OT@@QBE_NPAUhb_sanitize_context_t@@@Z 100152f0 f i hb-ot-layout.obj
 0001:000142f0       ?sanitize_shallow@?$ArrayOf@U?$OffsetTo@U?$PairSet@USmallTypes@Layout@OT@@@GPOS_impl@Layout@OT@@U?$IntType@G$01@4@$00@OT@@U?$IntType@G$01@2@@OT@@QBE_NPAUhb_sanitize_context_t@@@Z 100152f0 f i hb-ot-layout.obj
 0001:000142f0       ?sanitize_shallow@?$ArrayOf@U?$OffsetTo@UAnchorMatrix@GPOS_impl@Layout@OT@@U?$IntType@G$01@4@$00@OT@@U?$IntType@G$01@2@@OT@@QBE_NPAUhb_sanitize_context_t@@@Z 100152f0 f i hb-ot-layout.obj
 0001:000142f0       ?sanitize_shallow@?$ArrayOf@U?$OffsetTo@U?$LigatureSet@USmallTypes@Layout@OT@@@GSUB_impl@Layout@OT@@U?$IntType@G$01@4@$00@OT@@U?$IntType@G$01@2@@OT@@QBE_NPAUhb_sanitize_context_t@@@Z 100152f0 f i hb-ot-layout.obj
 0001:000142f0       ?sanitize_shallow@?$ArrayOf@U?$OffsetTo@U?$RuleSet@USmallTypes@Layout@OT@@@OT@@U?$IntType@G$01@2@$00@OT@@U?$IntType@G$01@2@@OT@@QBE_NPAUhb_sanitize_context_t@@@Z 100152f0 f i hb-ot-layout.obj
 0001:000142f0       ?sanitize_shallow@?$ArrayOf@U?$OffsetTo@UCoverage@Common@Layout@OT@@U?$IntType@G$01@4@$00@OT@@U?$IntType@G$01@2@@OT@@QBE_NPAUhb_sanitize_context_t@@@Z 100152f0 f i hb-ot-layout.obj
 0001:000142f0       ?sanitize_shallow@?$ArrayOf@U?$OffsetTo@U?$Rule@USmallTypes@Layout@OT@@@OT@@U?$IntType@G$01@2@$00@OT@@U?$IntType@G$01@2@@OT@@QBE_NPAUhb_sanitize_context_t@@@Z 100152f0 f i hb-ot-layout.obj
 0001:000142f0       ?sanitize_shallow@?$ArrayOf@U?$OffsetTo@UCaretValue@OT@@U?$IntType@G$01@2@$00@OT@@U?$IntType@G$01@2@@OT@@QBE_NPAUhb_sanitize_context_t@@@Z 100152f0 f i hb-aat-layout.obj
 0001:000142f0       ?sanitize_shallow@?$ArrayOf@U?$OffsetTo@U?$Sequence@USmallTypes@Layout@OT@@@GSUB_impl@Layout@OT@@U?$IntType@G$01@4@$00@OT@@U?$IntType@G$01@2@@OT@@QBE_NPAUhb_sanitize_context_t@@@Z 100152f0 f i hb-ot-layout.obj
 0001:00014390       ?sanitize_shallow@?$ArrayOf@UMarkRecord@GPOS_impl@Layout@OT@@U?$IntType@G$01@4@@OT@@QBE_NPAUhb_sanitize_context_t@@@Z 10015390 f i hb-ot-layout.obj
 0001:00014390       ?sanitize_shallow@?$ArrayOf@UAxisValueMap@OT@@U?$IntType@G$01@2@@OT@@QBE_NPAUhb_sanitize_context_t@@@Z 10015390 f i hb-font.obj
 0001:00014390       ?sanitize_shallow@?$ArrayOf@ULookupRecord@OT@@U?$IntType@G$01@2@@OT@@QBE_NPAUhb_sanitize_context_t@@@Z 10015390 f i hb-ot-layout.obj
 0001:00014390       ?sanitize_shallow@?$ArrayOf@U?$OffsetTo@UVarData@OT@@U?$IntType@I$03@2@$00@OT@@U?$IntType@G$01@2@@OT@@QBE_NPAUhb_sanitize_context_t@@@Z 10015390 f i hb-aat-layout.obj
 0001:00014390       ?sanitize_shallow@?$ArrayOf@U?$OffsetTo@UCondition@OT@@U?$IntType@I$03@2@$00@OT@@U?$IntType@G$01@2@@OT@@QBE_NPAUhb_sanitize_context_t@@@Z 10015390 f i hb-ot-layout.obj
 0001:00014390       ?sanitize_shallow@?$ArrayOf@UEntryExitRecord@GPOS_impl@Layout@OT@@U?$IntType@G$01@4@@OT@@QBE_NPAUhb_sanitize_context_t@@@Z 10015390 f i hb-ot-layout.obj
 0001:00014390       ?sanitize_shallow@?$ArrayOf@U?$OffsetTo@UCoverage@Common@Layout@OT@@U?$IntType@I$03@4@$00@OT@@U?$IntType@G$01@2@@OT@@QBE_NPAUhb_sanitize_context_t@@@Z 10015390 f i hb-aat-layout.obj
 0001:00014390       ?sanitize_shallow@?$ArrayOf@UVertOriginMetric@OT@@U?$IntType@G$01@2@@OT@@QBE_NPAUhb_sanitize_context_t@@@Z 10015390 f i hb-ot-font.obj
 0001:00014430       ?sanitize_shallow@?$ArrayOf@U?$Record@UScript@OT@@@OT@@U?$IntType@G$01@2@@OT@@QBE_NPAUhb_sanitize_context_t@@@Z 10015430 f i hb-ot-layout.obj
 0001:00014430       ?sanitize_shallow@?$ArrayOf@U?$NoVariable@UColorStop@OT@@@OT@@U?$IntType@G$01@2@@OT@@QBE_NPAUhb_sanitize_context_t@@@Z 10015430 f i hb-ot-color.obj
 0001:00014430       ?sanitize_shallow@?$ArrayOf@U?$Record@ULangSys@OT@@@OT@@U?$IntType@G$01@2@@OT@@QBE_NPAUhb_sanitize_context_t@@@Z 10015430 f i hb-ot-layout.obj
 0001:00014430       ?sanitize_shallow@?$ArrayOf@UFeatureTableSubstitutionRecord@OT@@U?$IntType@G$01@2@@OT@@QBE_NPAUhb_sanitize_context_t@@@Z 10015430 f i hb-ot-layout.obj
 0001:00014430       ?sanitize_shallow@?$ArrayOf@U?$Record@UFeature@OT@@@OT@@U?$IntType@G$01@2@@OT@@QBE_NPAUhb_sanitize_context_t@@@Z 10015430 f i hb-ot-layout.obj
 0001:00014430       ?sanitize_shallow@?$ArrayOf@U?$RangeRecord@USmallTypes@Layout@OT@@@Common@Layout@OT@@U?$IntType@G$01@4@@OT@@QBE_NPAUhb_sanitize_context_t@@@Z 10015430 f i hb-aat-layout.obj
 0001:000144e0       ?sanitize_shallow@?$ArrayOf@UAnchor@AAT@@U?$IntType@I$03@OT@@@OT@@QBE_NPAUhb_sanitize_context_t@@@Z 100154e0 f i hb-aat-layout.obj
 0001:000144e0       ?sanitize_shallow@?$ArrayOf@U?$OffsetTo@USBIXStrike@OT@@U?$IntType@I$03@2@$00@OT@@U?$IntType@I$03@2@@OT@@QBE_NPAUhb_sanitize_context_t@@@Z 100154e0 f i hb-ot-color.obj
 0001:000144e0       ?sanitize_shallow@?$ArrayOf@U?$OffsetTo@UPaint@OT@@U?$IntType@I$03@2@$00@OT@@U?$IntType@I$03@2@@OT@@QBE_NPAUhb_sanitize_context_t@@@Z 100154e0 f i hb-ot-color.obj
 0001:000144e0       ?sanitize_shallow@?$ArrayOf@UFTStringRange@AAT@@U?$IntType@I$03@OT@@@OT@@QBE_NPAUhb_sanitize_context_t@@@Z 100154e0 f i hb-aat-layout.obj
 0001:000144e0       ?sanitize_shallow@?$ArrayOf@UUnicodeValueRange@OT@@U?$IntType@I$03@2@@OT@@QBE_NPAUhb_sanitize_context_t@@@Z 100154e0 f i hb-face.obj
 0001:000145a0       ?sanitize_shallow@?$ArrayOf@UKernPair@AAT@@U?$BinSearchHeader@U?$IntType@I$03@OT@@@OT@@@OT@@QBE_NPAUhb_sanitize_context_t@@@Z 100155a0 f i hb-aat-layout.obj
 0001:000146b0       ?sanitize_shallow@?$OffsetTo@USubstLookupSubTable@GSUB_impl@Layout@OT@@U?$IntType@G$01@4@$00@OT@@QBE_NPAUhb_sanitize_context_t@@PBX@Z 100156b0 f i hb-ot-layout.obj
 0001:000146b0       ?sanitize_shallow@?$OffsetTo@UAttachList@OT@@U?$IntType@G$01@2@$00@OT@@QBE_NPAUhb_sanitize_context_t@@PBX@Z 100156b0 f i hb-aat-layout.obj
 0001:000146b0       ?sanitize_shallow@?$OffsetTo@UCoverage@Common@Layout@OT@@U?$IntType@G$01@4@$00@OT@@QBE_NPAUhb_sanitize_context_t@@PBX@Z 100156b0 f i hb-aat-layout.obj
 0001:000146b0       ?sanitize_shallow@?$OffsetTo@UScript@OT@@U?$IntType@G$01@2@$00@OT@@QBE_NPAUhb_sanitize_context_t@@PBX@Z 100156b0 f i hb-ot-layout.obj
 0001:000146b0       ?sanitize_shallow@?$OffsetTo@USubstLookup@GSUB_impl@Layout@OT@@U?$IntType@G$01@4@$00@OT@@QBE_NPAUhb_sanitize_context_t@@PBX@Z 100156b0 f i hb-ot-layout.obj
 0001:000146b0       ?sanitize_shallow@?$OffsetTo@U?$Sequence@USmallTypes@Layout@OT@@@GSUB_impl@Layout@OT@@U?$IntType@G$01@4@$00@OT@@QBE_NPAUhb_sanitize_context_t@@PBX@Z 100156b0 f i hb-ot-layout.obj
 0001:000146b0       ?sanitize_shallow@?$OffsetTo@U?$UnsizedArrayOf@UHBGlyphID16@OT@@@OT@@U?$IntType@G$01@2@$0A@@OT@@QBE_NPAUhb_sanitize_context_t@@PBX@Z 100156b0 f i hb-aat-layout.obj
 0001:000146b0       ?sanitize_shallow@?$OffsetTo@UVariationStore@OT@@U?$IntType@G$01@2@$00@OT@@QBE_NPAUhb_sanitize_context_t@@PBX@Z 100156b0 f i hb-ot-metrics.obj
 0001:000146b0       ?sanitize_shallow@?$OffsetTo@UFeatureParams@OT@@U?$IntType@G$01@2@$00@OT@@QBE_NPAUhb_sanitize_context_t@@PBX@Z 100156b0 f i hb-ot-layout.obj
 0001:000146b0       ?sanitize_shallow@?$OffsetTo@UFeature@OT@@U?$IntType@G$01@2@$00@OT@@QBE_NPAUhb_sanitize_context_t@@PBX@Z 100156b0 f i hb-ot-layout.obj
 0001:000146b0       ?sanitize_shallow@?$OffsetTo@UMarkGlyphSets@OT@@U?$IntType@G$01@2@$00@OT@@QBE_NPAUhb_sanitize_context_t@@PBX@Z 100156b0 f i hb-aat-layout.obj
 0001:000146b0       ?sanitize_shallow@?$OffsetTo@UTrackData@AAT@@U?$IntType@G$01@OT@@$00@OT@@QBE_NPAUhb_sanitize_context_t@@PBX@Z 100156b0 f i hb-aat-layout.obj
 0001:000146b0       ?sanitize_shallow@?$OffsetTo@ULigGlyph@OT@@U?$IntType@G$01@2@$00@OT@@QBE_NPAUhb_sanitize_context_t@@PBX@Z 100156b0 f i hb-aat-layout.obj
 0001:000146b0       ?sanitize_shallow@?$OffsetTo@U?$ClassTable@U?$IntType@E$00@OT@@@AAT@@U?$IntType@G$01@OT@@$0A@@OT@@QBE_NPAUhb_sanitize_context_t@@PBX@Z 100156b0 f i hb-aat-layout.obj
 0001:000146b0       ?sanitize_shallow@?$OffsetTo@U?$ChainRuleSet@USmallTypes@Layout@OT@@@OT@@U?$IntType@G$01@2@$00@OT@@QBE_NPAUhb_sanitize_context_t@@PBX@Z 100156b0 f i hb-ot-layout.obj
 0001:000146b0       ?sanitize_shallow@?$OffsetTo@U?$Rule@USmallTypes@Layout@OT@@@OT@@U?$IntType@G$01@2@$00@OT@@QBE_NPAUhb_sanitize_context_t@@PBX@Z 100156b0 f i hb-ot-layout.obj
 0001:000146b0       ?sanitize_shallow@?$OffsetTo@U?$UnsizedArrayOf@U?$OffsetTo@U?$ArrayOf@UAnchor@AAT@@U?$IntType@I$03@OT@@@OT@@U?$IntType@G$01@2@$0A@@OT@@@OT@@U?$IntType@G$01@2@$0A@@OT@@QBE_NPAUhb_sanitize_context_t@@PBX@Z 100156b0 f i hb-aat-layout.obj
 0001:000146b0       ?sanitize_shallow@?$OffsetTo@U?$List16OfOffsetTo@USubstLookup@GSUB_impl@Layout@OT@@U?$IntType@G$01@4@@OT@@U?$IntType@G$01@2@$00@OT@@QBE_NPAUhb_sanitize_context_t@@PBX@Z 100156b0 f i hb-ot-layout.obj
 0001:000146b0       ?sanitize_shallow@?$OffsetTo@UPosLookup@GPOS_impl@Layout@OT@@U?$IntType@G$01@4@$00@OT@@QBE_NPAUhb_sanitize_context_t@@PBX@Z 100156b0 f i hb-ot-layout.obj
 0001:000146b0       ?sanitize_shallow@?$OffsetTo@ULigatureArray@GPOS_impl@Layout@OT@@U?$IntType@G$01@4@$00@OT@@QBE_NPAUhb_sanitize_context_t@@PBX@Z 100156b0 f i hb-ot-layout.obj
 0001:000146b0       ?sanitize_shallow@?$OffsetTo@U?$UnsizedArrayOf@U?$IntType@F$01@OT@@@OT@@U?$IntType@G$01@2@$0A@@OT@@QBE_NPAUhb_sanitize_context_t@@PBX@Z 100156b0 f i hb-aat-layout.obj
 0001:000146b0       ?sanitize_shallow@?$OffsetTo@U?$UnsizedArrayOf@U?$IntType@G$01@OT@@@OT@@U?$IntType@G$01@2@$0A@@OT@@QBE_NPAUhb_sanitize_context_t@@PBX@Z 100156b0 f i hb-aat-layout.obj
 0001:000146b0       ?sanitize_shallow@?$OffsetTo@U?$UnsizedListOfOffset16To@U?$Lookup@UHBGlyphID16@OT@@@AAT@@U?$IntType@G$01@OT@@$0A@@OT@@U?$IntType@G$01@2@$0A@@OT@@QBE_NPAUhb_sanitize_context_t@@PBX@Z 100156b0 f i hb-aat-layout.obj
 0001:000146b0       ?sanitize_shallow@?$OffsetTo@U?$RecordListOf@UFeature@OT@@@OT@@U?$IntType@G$01@2@$00@OT@@QBE_NPAUhb_sanitize_context_t@@PBX@Z 100156b0 f i hb-ot-layout.obj
 0001:000146b0       ?sanitize_shallow@?$OffsetTo@U?$Lookup@UHBGlyphID16@OT@@@AAT@@U?$IntType@G$01@OT@@$0A@@OT@@QBE_NPAUhb_sanitize_context_t@@PBX@Z 100156b0 f i hb-aat-layout.obj
 0001:000146b0       ?sanitize_shallow@?$OffsetTo@UAnchor@GPOS_impl@Layout@OT@@U?$IntType@G$01@4@$00@OT@@QBE_NPAUhb_sanitize_context_t@@PBX@Z 100156b0 f i hb-ot-layout.obj
 0001:000146b0       ?sanitize_shallow@?$OffsetTo@U?$Ligature@USmallTypes@Layout@OT@@@GSUB_impl@Layout@OT@@U?$IntType@G$01@4@$00@OT@@QBE_NPAUhb_sanitize_context_t@@PBX@Z 100156b0 f i hb-ot-layout.obj
 0001:000146b0       ?sanitize_shallow@?$OffsetTo@UCaretValue@OT@@U?$IntType@G$01@2@$00@OT@@QBE_NPAUhb_sanitize_context_t@@PBX@Z 100156b0 f i hb-aat-layout.obj
 0001:000146b0       ?sanitize_shallow@?$OffsetTo@UMarkArray@GPOS_impl@Layout@OT@@U?$IntType@G$01@4@$00@OT@@QBE_NPAUhb_sanitize_context_t@@PBX@Z 100156b0 f i hb-ot-layout.obj
 0001:000146b0       ?sanitize_shallow@?$OffsetTo@UAttachPoint@OT@@U?$IntType@G$01@2@$00@OT@@QBE_NPAUhb_sanitize_context_t@@PBX@Z 100156b0 f i hb-aat-layout.obj
 0001:000146b0       ?sanitize_shallow@?$OffsetTo@UDevice@OT@@U?$IntType@G$01@2@$00@OT@@QBE_NPAUhb_sanitize_context_t@@PBX@Z 100156b0 f i hb-aat-layout.obj
 0001:000146b0       ?sanitize_shallow@?$OffsetTo@U?$RuleSet@USmallTypes@Layout@OT@@@OT@@U?$IntType@G$01@2@$00@OT@@QBE_NPAUhb_sanitize_context_t@@PBX@Z 100156b0 f i hb-ot-layout.obj
 0001:000146b0       ?sanitize_shallow@?$OffsetTo@URecordListOfScript@OT@@U?$IntType@G$01@2@$00@OT@@QBE_NPAUhb_sanitize_context_t@@PBX@Z 100156b0 f i hb-ot-layout.obj
 0001:000146b0       ?sanitize_shallow@?$OffsetTo@U?$ClassTable@U?$IntType@G$01@OT@@@AAT@@U?$IntType@G$01@OT@@$0A@@OT@@QBE_NPAUhb_sanitize_context_t@@PBX@Z 100156b0 f i hb-ot-layout.obj
 0001:000146b0       ?sanitize_shallow@?$OffsetTo@U?$List16OfOffsetTo@UPosLookup@GPOS_impl@Layout@OT@@U?$IntType@G$01@4@@OT@@U?$IntType@G$01@2@$00@OT@@QBE_NPAUhb_sanitize_context_t@@PBX@Z 100156b0 f i hb-ot-layout.obj
 0001:000146b0       ?sanitize_shallow@?$OffsetTo@ULigCaretList@OT@@U?$IntType@G$01@2@$00@OT@@QBE_NPAUhb_sanitize_context_t@@PBX@Z 100156b0 f i hb-aat-layout.obj
 0001:000146b0       ?sanitize_shallow@?$OffsetTo@U?$UnsizedArrayOf@U?$IntType@I$03@OT@@@OT@@U?$IntType@G$01@2@$0A@@OT@@QBE_NPAUhb_sanitize_context_t@@PBX@Z 100156b0 f i hb-aat-layout.obj
 0001:000146b0       ?sanitize_shallow@?$OffsetTo@UClassDef@OT@@U?$IntType@G$01@2@$00@OT@@QBE_NPAUhb_sanitize_context_t@@PBX@Z 100156b0 f i hb-aat-layout.obj
 0001:000146b0       ?sanitize_shallow@?$OffsetTo@U?$PairSet@USmallTypes@Layout@OT@@@GPOS_impl@Layout@OT@@U?$IntType@G$01@4@$00@OT@@QBE_NPAUhb_sanitize_context_t@@PBX@Z 100156b0 f i hb-ot-layout.obj
 0001:000146b0       ?sanitize_shallow@?$OffsetTo@U?$LigatureSet@USmallTypes@Layout@OT@@@GSUB_impl@Layout@OT@@U?$IntType@G$01@4@$00@OT@@QBE_NPAUhb_sanitize_context_t@@PBX@Z 100156b0 f i hb-ot-layout.obj
 0001:000146b0       ?sanitize_shallow@?$OffsetTo@UPosLookupSubTable@GPOS_impl@Layout@OT@@U?$IntType@G$01@4@$00@OT@@QBE_NPAUhb_sanitize_context_t@@PBX@Z 100156b0 f i hb-ot-layout.obj
 0001:000146b0       ?sanitize_shallow@?$OffsetTo@U?$ChainRule@USmallTypes@Layout@OT@@@OT@@U?$IntType@G$01@2@$00@OT@@QBE_NPAUhb_sanitize_context_t@@PBX@Z 100156b0 f i hb-ot-layout.obj
 0001:000146b0       ?sanitize_shallow@?$OffsetTo@U?$AlternateSet@USmallTypes@Layout@OT@@@GSUB_impl@Layout@OT@@U?$IntType@G$01@4@$00@OT@@QBE_NPAUhb_sanitize_context_t@@PBX@Z 100156b0 f i hb-ot-layout.obj
 0001:000146b0       ?sanitize_shallow@?$OffsetTo@U?$ArrayOf@UAnchor@AAT@@U?$IntType@I$03@OT@@@OT@@U?$IntType@G$01@2@$0A@@OT@@QBE_NPAUhb_sanitize_context_t@@PBX@Z 100156b0 f i hb-aat-layout.obj
 0001:000146b0       ?sanitize_shallow@?$OffsetTo@UAnchorMatrix@GPOS_impl@Layout@OT@@U?$IntType@G$01@4@$00@OT@@QBE_NPAUhb_sanitize_context_t@@PBX@Z 100156b0 f i hb-ot-layout.obj
 0001:000146b0       ?sanitize_shallow@?$OffsetTo@ULangSys@OT@@U?$IntType@G$01@2@$00@OT@@QBE_NPAUhb_sanitize_context_t@@PBX@Z 100156b0 f i hb-ot-layout.obj
 0001:00014740       ?sanitize_shallow@?$OffsetTo@U?$Lookup@UHBGlyphID16@OT@@@AAT@@U?$IntType@I$03@OT@@$0A@@OT@@QBE_NPAUhb_sanitize_context_t@@PBX@Z 10015740 f i hb-aat-layout.obj
 0001:00014740       ?sanitize_shallow@?$OffsetTo@UCoverage@Common@Layout@OT@@U?$IntType@I$03@4@$00@OT@@QBE_NPAUhb_sanitize_context_t@@PBX@Z 10015740 f i hb-aat-layout.obj
 0001:00014740       ?sanitize_shallow@?$OffsetTo@UIndexSubtableArray@OT@@U?$IntType@I$03@2@$0A@@OT@@QBE_NPAUhb_sanitize_context_t@@PBX@Z 10015740 f i hb-ot-color.obj
 0001:00014740       ?sanitize_shallow@?$OffsetTo@UCmapSubtable@OT@@U?$IntType@I$03@2@$00@OT@@QBE_NPAUhb_sanitize_context_t@@PBX@Z 10015740 f i hb-face.obj
 0001:00014740       ?sanitize_shallow@?$OffsetTo@UClipList@OT@@U?$IntType@I$03@2@$00@OT@@QBE_NPAUhb_sanitize_context_t@@PBX@Z 10015740 f i hb-ot-color.obj
 0001:00014740       ?sanitize_shallow@?$OffsetTo@ULayerList@OT@@U?$IntType@I$03@2@$00@OT@@QBE_NPAUhb_sanitize_context_t@@PBX@Z 10015740 f i hb-ot-color.obj
 0001:00014740       ?sanitize_shallow@?$OffsetTo@UNonDefaultUVS@OT@@U?$IntType@I$03@2@$00@OT@@QBE_NPAUhb_sanitize_context_t@@PBX@Z 10015740 f i hb-face.obj
 0001:00014740       ?sanitize_shallow@?$OffsetTo@UCondition@OT@@U?$IntType@I$03@2@$00@OT@@QBE_NPAUhb_sanitize_context_t@@PBX@Z 10015740 f i hb-ot-layout.obj
 0001:00014740       ?sanitize_shallow@?$OffsetTo@UVariationStore@OT@@U?$IntType@I$03@2@$00@OT@@QBE_NPAUhb_sanitize_context_t@@PBX@Z 10015740 f i hb-aat-layout.obj
 0001:00014740       ?sanitize_shallow@?$OffsetTo@UPaint@OT@@U?$IntType@I$03@2@$00@OT@@QBE_NPAUhb_sanitize_context_t@@PBX@Z 10015740 f i hb-ot-color.obj
 0001:00014740       ?sanitize_shallow@?$OffsetTo@UIndexSubtable@OT@@U?$IntType@I$03@2@$00@OT@@QBE_NPAUhb_sanitize_context_t@@PBX@Z 10015740 f i hb-ot-color.obj
 0001:00014740       ?sanitize_shallow@?$OffsetTo@UDefaultUVS@OT@@U?$IntType@I$03@2@$00@OT@@QBE_NPAUhb_sanitize_context_t@@PBX@Z 10015740 f i hb-face.obj
 0001:00014740       ?sanitize_shallow@?$OffsetTo@U?$UnsizedArrayOf@U?$HBFixed@U?$IntType@H$03@OT@@$0BA@@OT@@@OT@@U?$IntType@I$03@2@$0A@@OT@@QBE_NPAUhb_sanitize_context_t@@PBX@Z 10015740 f i hb-aat-layout.obj
 0001:00014740       ?sanitize_shallow@?$OffsetTo@UVarRegionList@OT@@U?$IntType@I$03@2@$00@OT@@QBE_NPAUhb_sanitize_context_t@@PBX@Z 10015740 f i hb-aat-layout.obj
 0001:00014740       ?sanitize_shallow@?$OffsetTo@U?$Lookup@U?$IntType@G$01@OT@@@AAT@@U?$IntType@I$03@OT@@$0A@@OT@@QBE_NPAUhb_sanitize_context_t@@PBX@Z 10015740 f i hb-aat-layout.obj
 0001:00014740       ?sanitize_shallow@?$OffsetTo@U?$UnsizedArrayOf@U?$HBFixed@U?$IntType@F$01@OT@@$0O@@OT@@@OT@@U?$IntType@I$03@2@$0A@@OT@@QBE_NPAUhb_sanitize_context_t@@PBX@Z 10015740 f i hb-common.obj
 0001:00014740       ?sanitize_shallow@?$OffsetTo@UVarData@OT@@U?$IntType@I$03@2@$00@OT@@QBE_NPAUhb_sanitize_context_t@@PBX@Z 10015740 f i hb-aat-layout.obj
 0001:00014740       ?sanitize_shallow@?$OffsetTo@UConditionSet@OT@@U?$IntType@I$03@2@$00@OT@@QBE_NPAUhb_sanitize_context_t@@PBX@Z 10015740 f i hb-ot-layout.obj
 0001:00014740       ?sanitize_shallow@?$OffsetTo@UFeatureVariations@OT@@U?$IntType@I$03@2@$00@OT@@QBE_NPAUhb_sanitize_context_t@@PBX@Z 10015740 f i hb-ot-layout.obj
 0001:00014740       ?sanitize_shallow@?$OffsetTo@UFeature@OT@@U?$IntType@I$03@2@$00@OT@@QBE_NPAUhb_sanitize_context_t@@PBX@Z 10015740 f i hb-ot-layout.obj
 0001:00014740       ?sanitize_shallow@?$OffsetTo@UBaseGlyphList@OT@@U?$IntType@I$03@2@$00@OT@@QBE_NPAUhb_sanitize_context_t@@PBX@Z 10015740 f i hb-ot-color.obj
 0001:00014740       ?sanitize_shallow@?$OffsetTo@U?$Lookup@U?$OffsetTo@U?$ArrayOf@UAnchor@AAT@@U?$IntType@I$03@OT@@@OT@@U?$IntType@G$01@2@$0A@@OT@@@AAT@@U?$IntType@I$03@OT@@$00@OT@@QBE_NPAUhb_sanitize_context_t@@PBX@Z 10015740 f i hb-aat-layout.obj
 0001:00014740       ?sanitize_shallow@?$OffsetTo@UFeatureTableSubstitution@OT@@U?$IntType@I$03@2@$00@OT@@QBE_NPAUhb_sanitize_context_t@@PBX@Z 10015740 f i hb-ot-layout.obj
 0001:00014740       ?sanitize_shallow@?$OffsetTo@U?$UnsizedListOfOffset16To@U?$Lookup@UHBGlyphID16@OT@@@AAT@@U?$IntType@I$03@OT@@$0A@@OT@@U?$IntType@I$03@2@$0A@@OT@@QBE_NPAUhb_sanitize_context_t@@PBX@Z 10015740 f i hb-aat-layout.obj
 0001:00014740       ?sanitize_shallow@?$OffsetTo@UDeltaSetIndexMap@OT@@U?$IntType@I$03@2@$00@OT@@QBE_NPAUhb_sanitize_context_t@@PBX@Z 10015740 f i hb-common.obj
 0001:00014740       ?sanitize_shallow@?$OffsetTo@USBIXStrike@OT@@U?$IntType@I$03@2@$00@OT@@QBE_NPAUhb_sanitize_context_t@@PBX@Z 10015740 f i hb-ot-color.obj
 0001:00014740       ?sanitize_shallow@?$OffsetTo@U?$Lookup@U?$IntType@I$03@OT@@@AAT@@U?$IntType@I$03@OT@@$0A@@OT@@QBE_NPAUhb_sanitize_context_t@@PBX@Z 10015740 f i hb-aat-layout.obj
 0001:000147e0       ?sanitize_shallow@?$UnsizedArrayOf@ULayerRecord@OT@@@OT@@QBE_NPAUhb_sanitize_context_t@@I@Z 100157e0 f i hb-ot-color.obj
 0001:000147e0       ?sanitize_shallow@?$UnsizedArrayOf@USettingName@AAT@@@OT@@QBE_NPAUhb_sanitize_context_t@@I@Z 100157e0 f i hb-aat-layout.obj
 0001:000147e0       ?sanitize_shallow@?$UnsizedArrayOf@U?$HBFixed@U?$IntType@H$03@OT@@$0BA@@OT@@@OT@@QBE_NPAUhb_sanitize_context_t@@I@Z 100157e0 f i hb-aat-layout.obj
 0001:000147e0       ?sanitize_shallow@?$UnsizedArrayOf@U?$OffsetTo@U?$Lookup@UHBGlyphID16@OT@@@AAT@@U?$IntType@I$03@OT@@$0A@@OT@@@OT@@QBE_NPAUhb_sanitize_context_t@@I@Z 100157e0 f i hb-aat-layout.obj
 0001:000147e0       ?sanitize_shallow@?$UnsizedArrayOf@U?$Offset@U?$IntType@I$03@OT@@$00@OT@@@OT@@QBE_NPAUhb_sanitize_context_t@@I@Z 100157e0 f i hb-ot-color.obj
 0001:000147e0       ?sanitize_shallow@?$UnsizedArrayOf@U?$IntType@I$03@OT@@@OT@@QBE_NPAUhb_sanitize_context_t@@I@Z 100157e0 f i hb-aat-layout.obj
 0001:00014870       ?sanitize_shallow@?$UnsizedArrayOf@U?$IntType@G$01@OT@@@OT@@QBE_NPAUhb_sanitize_context_t@@I@Z 10015870 f i hb-aat-layout.obj
 0001:00014890       ?sanitize_shallow@?$UnsizedArrayOf@U?$Offset@U?$IntType@G$01@OT@@$00@OT@@@OT@@QBE_NPAUhb_sanitize_context_t@@I@Z 10015890 f i hb-ot-color.obj
 0001:00014890       ?sanitize_shallow@?$UnsizedArrayOf@UIndex@OT@@@OT@@QBE_NPAUhb_sanitize_context_t@@I@Z 10015890 f i hb-ot-color.obj
 0001:00014890       ?sanitize_shallow@?$UnsizedArrayOf@U?$OffsetTo@U?$ArrayOf@UAnchor@AAT@@U?$IntType@I$03@OT@@@OT@@U?$IntType@G$01@2@$0A@@OT@@@OT@@QBE_NPAUhb_sanitize_context_t@@I@Z 10015890 f i hb-aat-layout.obj
 0001:00014890       ?sanitize_shallow@?$UnsizedArrayOf@U?$OffsetTo@U?$Lookup@UHBGlyphID16@OT@@@AAT@@U?$IntType@G$01@OT@@$0A@@OT@@@OT@@QBE_NPAUhb_sanitize_context_t@@I@Z 10015890 f i hb-aat-layout.obj
 0001:00014890       ?sanitize_shallow@?$UnsizedArrayOf@U?$HBFixed@U?$IntType@F$01@OT@@$0O@@OT@@@OT@@QBE_NPAUhb_sanitize_context_t@@I@Z 10015890 f i hb-common.obj
 0001:00014920       ?sanitize_shallow@?$UnsizedArrayOf@UFeatureName@AAT@@@OT@@QBE_NPAUhb_sanitize_context_t@@I@Z 10015920 f i hb-aat-layout.obj
 0001:000149b0       ?sanitize_shallow@?$UnsizedArrayOf@UTrackTableEntry@AAT@@@OT@@QBE_NPAUhb_sanitize_context_t@@I@Z 100159b0 f i hb-aat-layout.obj
 0001:000149b0       ?sanitize_shallow@?$UnsizedArrayOf@UIndexSubtableRecord@OT@@@OT@@QBE_NPAUhb_sanitize_context_t@@I@Z 100159b0 f i hb-ot-color.obj
 0001:00014a40       ?sanitize_shallow@?$UnsizedArrayOf@UBaseGlyphRecord@OT@@@OT@@QBE_NPAUhb_sanitize_context_t@@I@Z 10015a40 f i hb-ot-color.obj
 0001:00014a40       ?sanitize_shallow@?$UnsizedArrayOf@UVarRegionAxis@OT@@@OT@@QBE_NPAUhb_sanitize_context_t@@I@Z 10015a40 f i hb-aat-layout.obj
 0001:00014ad0       ?shrink_vector@?$hb_vector_t@U?$hb_vector_t@Urange_flags_t@hb_aat_map_t@@$00@@$0A@@@QAEXI@Z 10015ad0 f i hb-aat-layout.obj
 0001:00014b50       ?start_processing@hb_sanitize_context_t@@QAEXXZ 10015b50 f i hb-aat-layout.obj
 0001:00014c00       ?transition@driver_context_t@?$ContextualSubtable@UExtendedTypes@AAT@@@AAT@@QAEXPAU?$StateTableDriver@UExtendedTypes@AAT@@UEntryData@?$ContextualSubtable@UExtendedTypes@AAT@@@2@@3@ABU?$Entry@UEntryData@?$ContextualSubtable@UExtendedTypes@AAT@@@AAT@@@3@@Z 10015c00 f i hb-aat-layout.obj
 0001:00014e30       ?transition@driver_context_t@?$ContextualSubtable@UObsoleteTypes@AAT@@@AAT@@QAEXPAU?$StateTableDriver@UObsoleteTypes@AAT@@UEntryData@?$ContextualSubtable@UObsoleteTypes@AAT@@@2@@3@ABU?$Entry@UEntryData@?$ContextualSubtable@UObsoleteTypes@AAT@@@AAT@@@3@@Z 10015e30 f i hb-aat-layout.obj
 0001:00015050       ?transition@driver_context_t@?$InsertionSubtable@UObsoleteTypes@AAT@@@AAT@@QAEXPAU?$StateTableDriver@UObsoleteTypes@AAT@@UEntryData@?$InsertionSubtable@UObsoleteTypes@AAT@@@2@@3@ABU?$Entry@UEntryData@?$InsertionSubtable@UObsoleteTypes@AAT@@@AAT@@@3@@Z 10016050 f i hb-aat-layout.obj
 0001:00015050       ?transition@driver_context_t@?$InsertionSubtable@UExtendedTypes@AAT@@@AAT@@QAEXPAU?$StateTableDriver@UExtendedTypes@AAT@@UEntryData@?$InsertionSubtable@UExtendedTypes@AAT@@@2@@3@ABU?$Entry@UEntryData@?$InsertionSubtable@UExtendedTypes@AAT@@@AAT@@@3@@Z 10016050 f i hb-aat-layout.obj
 0001:00015270       ?transition@driver_context_t@?$KerxSubTableFormat1@UKerxSubTableHeader@AAT@@@AAT@@QAEXPAU?$StateTableDriver@UExtendedTypes@AAT@@UEntryData@?$Format1Entry@$00@2@@3@ABU?$Entry@UEntryData@?$Format1Entry@$00@AAT@@@3@@Z 10016270 f i hb-aat-layout.obj
 0001:00015560       ?transition@driver_context_t@?$KerxSubTableFormat4@UKerxSubTableHeader@AAT@@@AAT@@QAEXPAU?$StateTableDriver@UExtendedTypes@AAT@@UEntryData@?$KerxSubTableFormat4@UKerxSubTableHeader@AAT@@@2@@3@ABU?$Entry@UEntryData@?$KerxSubTableFormat4@UKerxSubTableHeader@AAT@@@AAT@@@3@@Z 10016560 f i hb-aat-layout.obj
 0001:00015970       ?transition@driver_context_t@?$LigatureSubtable@UExtendedTypes@AAT@@@AAT@@QAEXPAU?$StateTableDriver@UExtendedTypes@AAT@@UEntryData@?$LigatureEntry@$00@2@@3@ABU?$Entry@UEntryData@?$LigatureEntry@$00@AAT@@@3@@Z 10016970 f i hb-aat-layout.obj
 0001:00015ce0       ?transition@driver_context_t@?$LigatureSubtable@UObsoleteTypes@AAT@@@AAT@@QAEXPAU?$StateTableDriver@UObsoleteTypes@AAT@@X@3@ABU?$Entry@X@3@@Z 10016ce0 f i hb-aat-layout.obj
 0001:00016090       ?transition@driver_context_t@?$RearrangementSubtable@UObsoleteTypes@AAT@@@AAT@@QAEXPAU?$StateTableDriver@UObsoleteTypes@AAT@@X@3@ABU?$Entry@X@3@@Z 10017090 f i hb-aat-layout.obj
 0001:00016090       ?transition@driver_context_t@?$RearrangementSubtable@UExtendedTypes@AAT@@@AAT@@QAEXPAU?$StateTableDriver@UExtendedTypes@AAT@@X@3@ABU?$Entry@X@3@@Z 10017090 f i hb-aat-layout.obj
 0001:00016310       ?unsafe_to_break@hb_buffer_t@@QAEXII@Z 10017310 f i hb-aat-layout.obj
 0001:00016360       ?unsafe_to_break_from_outbuffer@hb_buffer_t@@QAEXII@Z 10017360 f i hb-aat-layout.obj
 0001:00016400       _hb_aat_layout_has_positioning 10017400 f   hb-aat-layout.obj
 0001:00016440       _hb_aat_layout_has_substitution 10017440 f   hb-aat-layout.obj
 0001:000164b0       _hb_aat_layout_has_tracking 100174b0 f   hb-aat-layout.obj
 0001:000168e0       ?add_feature@hb_aat_map_builder_t@@QAEXABUhb_feature_t@@@Z 100178e0 f   hb-aat-map.obj
 0001:00016a50       ?alloc@?$hb_vector_t@Ufeature_info_t@hb_aat_map_builder_t@@$00@@QAE_NI_N@Z 10017a50 f i hb-aat-map.obj
 0001:00016b00       ?cmp@feature_event_t@hb_aat_map_builder_t@@SAHPBX0@Z 10017b00 f i hb-aat-map.obj
 0001:00016b50       ?cmp@feature_info_t@hb_aat_map_builder_t@@SAHPBX0@Z 10017b50 f i hb-aat-map.obj
 0001:00016bc0       ?compile@hb_aat_map_builder_t@@QAEXAAUhb_aat_map_t@@@Z 10017bc0 f   hb-aat-map.obj
 0001:00017310       ?push@?$hb_vector_t@Ufeature_range_t@hb_aat_map_builder_t@@$00@@QAEPAUfeature_range_t@hb_aat_map_builder_t@@XZ 10018310 f i hb-aat-map.obj
 0001:00017310       ?push@?$hb_vector_t@Ufeature_event_t@hb_aat_map_builder_t@@$0A@@@QAEPAUfeature_event_t@hb_aat_map_builder_t@@XZ 10018310 f i hb-aat-map.obj
 0001:00017430       ??$replace_or_insert@Uhb_user_data_item_t@hb_user_data_array_t@@@?$hb_lockable_set_t@Uhb_user_data_item_t@hb_user_data_array_t@@Uhb_mutex_t@@@@QAEPAUhb_user_data_item_t@hb_user_data_array_t@@U12@AAUhb_mutex_t@@_N@Z 10018430 f i hb-blob.obj
 0001:000175b0       ?try_make_writable@hb_blob_t@@QAE_NXZ 100185b0 f   hb-blob.obj
 0001:00017670       _hb_blob_create            10018670 f   hb-blob.obj
 0001:000176c0       _hb_blob_create_or_fail    100186c0 f   hb-blob.obj
 0001:000177a0       _hb_blob_create_sub_blob   100187a0 f   hb-blob.obj
 0001:00017840       _hb_blob_destroy           10018840 f   hb-blob.obj
 0001:000178b0       _hb_blob_get_data_writable 100188b0 f   hb-blob.obj
 0001:000178f0       _hb_blob_get_empty         100188f0 f   hb-blob.obj
 0001:00017900       _hb_paint_funcs_make_immutable 10018900 f   hb-paint.obj
 0001:00017900       _hb_font_funcs_make_immutable 10018900 f   hb-font.obj
 0001:00017900       _hb_blob_make_immutable    10018900 f   hb-blob.obj
 0001:00017900       _hb_unicode_funcs_make_immutable 10018900 f   hb-unicode.obj
 0001:00017900       _hb_face_make_immutable    10018900 f   hb-face.obj
 0001:00017900       _hb_draw_funcs_make_immutable 10018900 f   hb-draw.obj
 0001:00017920       _hb_face_reference         10018920 f   hb-face.obj
 0001:00017920       _hb_unicode_funcs_reference 10018920 f   hb-unicode.obj
 0001:00017920       _hb_blob_reference         10018920 f   hb-blob.obj
 0001:00017940       ___local_stdio_printf_options 10018940 f i hb-buffer-serialize.obj
 0001:00017950       _hb_buffer_serialize_unicode 10018950 f   hb-buffer-serialize.obj
 0001:00017c30       _snprintf                  10018c30 f i hb-buffer-serialize.obj
 0001:000182b0       ?verify@hb_buffer_t@@QAE_NPAU1@PAUhb_font_t@@PBUhb_feature_t@@IPBQBD@Z 100192b0 f   hb-buffer-verify.obj
 0001:00018470       _fprintf                   10019470 f i hb-buffer-verify.obj
 0001:000186b0       ??$reverse_groups@$$A6A_NABUhb_glyph_info_t@@0@Z@hb_buffer_t@@QAEXA6A_NABUhb_glyph_info_t@@0@Z_N@Z 100196b0 f i hb-buffer.obj
 0001:00018840       ?_cluster_group_func@hb_buffer_t@@SA_NABUhb_glyph_info_t@@0@Z 10019840 f i hb-buffer.obj
 0001:00018860       ?clear@hb_buffer_t@@QAEXXZ 10019860 f   hb-buffer.obj
 0001:000188c0       ?clear_output@hb_buffer_t@@QAEXXZ 100198c0 f   hb-buffer.obj
 0001:000188e0       ?clear_positions@hb_buffer_t@@QAEXXZ 100198e0 f   hb-buffer.obj
 0001:00018910       ?delete_glyph@hb_buffer_t@@QAEXXZ 10019910 f   hb-buffer.obj
 0001:000189a0       ?delete_glyphs_inplace@hb_buffer_t@@QAEXP6A_NPBUhb_glyph_info_t@@@Z@Z 100199a0 f   hb-buffer.obj
 0001:00018ac0       ?enlarge@hb_buffer_t@@QAE_NI@Z 10019ac0 f   hb-buffer.obj
 0001:00018b90       ?ensure@hb_buffer_t@@QAE_NI@Z 10019b90 f i hb-buffer.obj
 0001:00018c80       ?enter@hb_buffer_t@@QAEXXZ 10019c80 f   hb-buffer.obj
 0001:00018ce0       ?leave@hb_buffer_t@@QAEXXZ 10019ce0 f   hb-buffer.obj
 0001:00018d00       ?make_room_for@hb_buffer_t@@QAE_NII@Z 10019d00 f   hb-buffer.obj
 0001:00018d60       ?merge_clusters_impl@hb_buffer_t@@QAEXII@Z 10019d60 f   hb-buffer.obj
 0001:00018f10       ?merge_out_clusters@hb_buffer_t@@QAEXII@Z 10019f10 f   hb-buffer.obj
 0001:00019060       ?message_impl@hb_buffer_t@@QAE_NPAUhb_font_t@@PBDPAD@Z 1001a060 f   hb-buffer.obj
 0001:000190e0       ?move_to@hb_buffer_t@@QAE_NI@Z 1001a0e0 f   hb-buffer.obj
 0001:00019240       ?next@?$hb_utf16_xe_t@G@@SAPBGPBG0PAII@Z 1001a240 f i hb-buffer.obj
 0001:000192b0       ?set_masks@hb_buffer_t@@QAEXIIII@Z 1001a2b0 f   hb-buffer.obj
 0001:00019300       ?sort@hb_buffer_t@@QAEXIIP6AHPBUhb_glyph_info_t@@0@Z@Z 1001a300 f   hb-buffer.obj
 0001:000193f0       ?sync@hb_buffer_t@@QAE_NXZ 1001a3f0 f   hb-buffer.obj
 0001:000194a0       ?sync_so_far@hb_buffer_t@@QAEHXZ 1001a4a0 f   hb-buffer.obj
 0001:00019560       _hb_buffer_add_utf16       1001a560 f   hb-buffer.obj
 0001:00019570       _hb_buffer_append          1001a570 f   hb-buffer.obj
 0001:00019850       _hb_buffer_clear_contents  1001a850 f   hb-buffer.obj
 0001:00019860       _hb_buffer_create          1001a860 f   hb-buffer.obj
 0001:00019920       _hb_buffer_create_similar  1001a920 f   hb-buffer.obj
 0001:00019a20       _hb_buffer_destroy         1001aa20 f   hb-buffer.obj
 0001:00019aa0       _hb_buffer_diff            1001aaa0 f   hb-buffer.obj
 0001:00019c20       _hb_buffer_get_direction   1001ac20 f   hb-buffer.obj
 0001:00019c30       _hb_buffer_get_flags       1001ac30 f   hb-buffer.obj
 0001:00019c40       _hb_buffer_get_glyph_infos 1001ac40 f   hb-buffer.obj
 0001:00019c60       _hb_buffer_get_glyph_positions 1001ac60 f   hb-buffer.obj
 0001:00019cc0       _hb_buffer_get_length      1001acc0 f   hb-buffer.obj
 0001:00019cd0       _hb_buffer_get_segment_properties 1001acd0 f   hb-buffer.obj
 0001:00019cf0       _hb_buffer_reverse         1001acf0 f   hb-buffer.obj
 0001:00019d00       _hb_buffer_set_cluster_level 1001ad00 f   hb-buffer.obj
 0001:00019d20       _hb_buffer_set_direction   1001ad20 f   hb-buffer.obj
 0001:00019d40       _hb_buffer_set_flags       1001ad40 f   hb-buffer.obj
 0001:00019d60       _hb_buffer_set_language    1001ad60 f   hb-buffer.obj
 0001:00019d80       _hb_buffer_set_length      1001ad80 f   hb-buffer.obj
 0001:00019e30       _hb_buffer_set_script      1001ae30 f   hb-buffer.obj
 0001:00019e50       _hb_buffer_set_segment_properties 1001ae50 f   hb-buffer.obj
 0001:00019e70       _hb_segment_properties_equal 1001ae70 f   hb-buffer.obj
 0001:00019eb0       ??$?HU?$hb_blob_ptr_t@Ugvar@OT@@@@$0A@@OT@@YAABU?$UnsizedArrayOf@U?$HBFixed@U?$IntType@F$01@OT@@$0O@@OT@@@0@ABU?$hb_blob_ptr_t@Ugvar@OT@@@@ABU?$OffsetTo@U?$UnsizedArrayOf@U?$HBFixed@U?$IntType@F$01@OT@@$0O@@OT@@@OT@@U?$IntType@I$03@2@$0A@@0@@Z 1001aeb0 f i hb-common.obj
 0001:00019f00       ??$get_points@Uglyf_accelerator_t@OT@@@Glyph@glyf_impl@OT@@QBE_NPAUhb_font_t@@ABUglyf_accelerator_t@2@AAUcontour_point_vector_t@@PAU5@PAUhead_maxp_info_t@@PAI_N66U?$hb_array_t@H@@PAUhb_map_t@@I5@Z 1001af00 f i hb-common.obj
 0001:0001b040       ??$get_points@Upoints_aggregator_t@glyf_accelerator_t@OT@@@glyf_accelerator_t@OT@@IBE_NPAUhb_font_t@@IUpoints_aggregator_t@01@@Z 1001c040 f i hb-common.obj
 0001:0001b370       ??$push@AAI@?$hb_vector_t@I$0A@@@QAEPAIAAI@Z 1001c370 f i hb-common.obj
 0001:0001b3c0       ??$sanitize_blob@UHVAR@OT@@@hb_sanitize_context_t@@QAEPAUhb_blob_t@@PAU1@@Z 1001c3c0 f i hb-common.obj
 0001:0001b550       ??$sanitize_blob@UVVAR@OT@@@hb_sanitize_context_t@@QAEPAUhb_blob_t@@PAU1@@Z 1001c550 f i hb-common.obj
 0001:0001b740       ??$sanitize_blob@Ugvar@OT@@@hb_sanitize_context_t@@QAEPAUhb_blob_t@@PAU1@@Z 1001c740 f i hb-common.obj
 0001:0001b8d0       ??$sanitize_blob@Uhead@OT@@@hb_sanitize_context_t@@QAEPAUhb_blob_t@@PAU1@@Z 1001c8d0 f i hb-common.obj
 0001:0001bae0       ??$sanitize_blob@Uvhea@OT@@@hb_sanitize_context_t@@QAEPAUhb_blob_t@@PAU1@@Z 1001cae0 f i hb-common.obj
 0001:0001bae0       ??$sanitize_blob@Uhhea@OT@@@hb_sanitize_context_t@@QAEPAUhb_blob_t@@PAU1@@Z 1001cae0 f i hb-common.obj
 0001:0001bcd0       ??$sanitize_blob@Umaxp@OT@@@hb_sanitize_context_t@@QAEPAUhb_blob_t@@PAU1@@Z 1001ccd0 f i hb-common.obj
 0001:0001bf30       ??$set_with_hash@ABIABI@?$hb_hashmap_t@II$00@@QAE_NABII0_N@Z 1001cf30 f i hb-common.obj
 0001:0001bf30       ??$set_with_hash@ABIAAI@?$hb_hashmap_t@II$00@@QAE_NABIIAAI_N@Z 1001cf30 f i hb-face.obj
 0001:0001c070       ??0?$composite_iter_tmpl@UCompositeGlyphRecord@glyf_impl@OT@@@glyf_impl@OT@@QAE@U?$hb_array_t@$$CBD@@PBUCompositeGlyphRecord@12@@Z 1001d070 f i hb-common.obj
 0001:0001c0f0       ??0Glyph@glyf_impl@OT@@QAE@U?$hb_array_t@$$CBD@@I@Z 1001d0f0 f i hb-common.obj
 0001:0001c160       ??0accelerator_t@?$hmtxvmtx@Uhmtx@OT@@Uhhea@2@UHVAR@2@@OT@@QAE@PAUhb_face_t@@@Z 1001d160 f i hb-common.obj
 0001:0001c4d0       ??0accelerator_t@?$hmtxvmtx@Uvmtx@OT@@Uvhea@2@UVVAR@2@@OT@@QAE@PAUhb_face_t@@@Z 1001d4d0 f i hb-common.obj
 0001:0001c830       ??0accelerator_t@gvar@OT@@QAE@PAUhb_face_t@@@Z 1001d830 f i hb-common.obj
 0001:0001cb60       ??0glyf_accelerator_t@OT@@QAE@PAUhb_face_t@@@Z 1001db60 f i hb-common.obj
 0001:0001d020       ??0hb_map_t@@QAE@XZ        1001e020 f i hb-common.obj
 0001:0001d080       ??A?$hb_iter_t@U?$hb_array_t@I@@AAI@@QBEAAII@Z 1001e080 f i hb-common.obj
 0001:0001d0b0       ??A?$hb_iter_t@U?$hb_array_t@Ucontour_point_t@@@@AAUcontour_point_t@@@@QAEAAUcontour_point_t@@I@Z 1001e0b0 f i hb-common.obj
 0001:0001d0f0       ??A?$hb_vector_t@Ucontour_point_t@@$0A@@@QAEAAUcontour_point_t@@H@Z 1001e0f0 f i hb-common.obj
 0001:0001d130       ??C?$hb_lazy_loader_t@Uglyf_accelerator_t@OT@@U?$hb_face_lazy_loader_t@Uglyf_accelerator_t@OT@@$0P@@@Uhb_face_t@@$0P@U12@@@QBEPBUglyf_accelerator_t@OT@@XZ 1001e130 f i hb-common.obj
 0001:0001d1d0       ??C?$hb_lazy_loader_t@Uhhea@OT@@U?$hb_table_lazy_loader_t@Uhhea@OT@@$03$00@@Uhb_face_t@@$03Uhb_blob_t@@@@QBEPBUhhea@OT@@XZ 1001e1d0 f i hb-common.obj
 0001:0001d2e0       ??C?$hb_lazy_loader_t@Umaxp@OT@@U?$hb_table_lazy_loader_t@Umaxp@OT@@$01$00@@Uhb_face_t@@$01Uhb_blob_t@@@@QBEPBUmaxp@OT@@XZ 1001e2e0 f i hb-common.obj
 0001:0001d3f0       ??C?$hb_lazy_loader_t@Uvhea@OT@@U?$hb_table_lazy_loader_t@Uvhea@OT@@$0L@$00@@Uhb_face_t@@$0L@Uhb_blob_t@@@@QBEPBUvhea@OT@@XZ 1001e3f0 f i hb-common.obj
 0001:0001d500       ?_glyf_get_advance_with_var_unscaled@@YAIPAUhb_font_t@@I_N@Z 1001e500 f   hb-common.obj
 0001:0001d690       ?_glyf_get_leading_bearing_with_var_unscaled@@YA_NPAUhb_font_t@@I_NPAH@Z 1001e690 f   hb-common.obj
 0001:0001d7d0       ?_hb_options_init@@YAXXZ   1001e7d0 f   hb-common.obj
 0001:0001d870       ?alloc@?$hb_hashmap_t@II$00@@QAE_NI@Z 1001e870 f i hb-common.obj
 0001:0001dc30       ?alloc@?$hb_vector_t@I$0A@@@QAE_NI_N@Z 1001ec30 f i hb-common.obj
 0001:0001dc30       ?alloc@?$hb_vector_t@PAUobject_t@hb_serialize_context_t@@$0A@@@QAE_NI_N@Z 1001ec30 f i hb-face-builder.obj
 0001:0001dc30       ?alloc@?$hb_vector_t@PAUchunk_t@?$hb_pool_t@Uobject_t@hb_serialize_context_t@@$0CA@@@$0A@@@QAE_NI_N@Z 1001ec30 f i hb-face-builder.obj
 0001:0001dc30       ?alloc@?$hb_vector_t@H$0A@@@QAE_NI_N@Z 1001ec30 f i hb-common.obj
 0001:0001dce0       ?alloc@?$hb_vector_t@Ulink_t@object_t@hb_serialize_context_t@@$0A@@@QAE_NI_N@Z 1001ece0 f i hb-face-builder.obj
 0001:0001dce0       ?alloc@?$hb_vector_t@Ucontour_point_t@@$0A@@@QAE_NI_N@Z 1001ece0 f i hb-common.obj
 0001:0001dce0       ?alloc@?$hb_vector_t@Uhb_outline_point_t@@$0A@@@QAE_NI_N@Z 1001ece0 f i hb-outline.obj
 0001:0001dce0       ?alloc@?$hb_vector_t@Ulookup_map_t@hb_ot_map_t@@$0A@@@QAE_NI_N@Z 1001ece0 f i hb-ot-map.obj
 0001:0001dd90       ?apply_deltas_to_points@accelerator_t@gvar@OT@@QBE_NIU?$hb_array_t@H@@U?$hb_array_t@Ucontour_point_t@@@@_N@Z 1001ed90 f i hb-common.obj
 0001:0001ec20       ?calculate_scalar@TupleVariationHeader@OT@@QBEMU?$hb_array_t@H@@IU?$hb_array_t@$$CBU?$HBFixed@U?$IntType@F$01@OT@@$0O@@OT@@@@PBU?$hb_vector_t@U?$hb_pair_t@HH@@$0A@@@@Z 1001fc20 f i hb-common.obj
 0001:0001eef0       ?del@?$hb_hashmap_t@II$00@@QAEXABI@Z 1001fef0 f i hb-common.obj
 0001:0001ef30       ?do_destroy@?$hb_lazy_loader_t@Ugvar_accelerator_t@OT@@U?$hb_face_lazy_loader_t@Ugvar_accelerator_t@OT@@$0BF@@@Uhb_face_t@@$0BF@U12@@@SAXPAUgvar_accelerator_t@OT@@@Z 1001ff30 f i hb-common.obj
 0001:0001ef90       ?end@?$hb_iter_t@U?$composite_iter_tmpl@UCompositeGlyphRecord@glyf_impl@OT@@@glyf_impl@OT@@ABUCompositeGlyphRecord@23@@@QBE?AU?$composite_iter_tmpl@UCompositeGlyphRecord@glyf_impl@OT@@@glyf_impl@OT@@XZ 1001ff90 f i hb-common.obj
 0001:0001efd0       ?extend@contour_point_vector_t@@QAEXABU?$hb_array_t@Ucontour_point_t@@@@@Z 1001ffd0 f i hb-common.obj
 0001:0001f030       ?fetch_item@?$hb_hashmap_t@II$00@@QBEPAUitem_t@1@ABII@Z 10020030 f i hb-common.obj
 0001:0001f0a0       ?get@?$hb_lazy_loader_t@Uhead@OT@@U?$hb_table_lazy_loader_t@Uhead@OT@@$00$00@@Uhb_face_t@@$00Uhb_blob_t@@@@QBEPBUhead@OT@@XZ 100200a0 f i hb-common.obj
 0001:0001f1b0       ?get@?$hb_lazy_loader_t@Uhmtx_accelerator_t@OT@@U?$hb_face_lazy_loader_t@Uhmtx_accelerator_t@OT@@$04@@Uhb_face_t@@$04U12@@@QBEPBUhmtx_accelerator_t@OT@@XZ 100201b0 f i hb-common.obj
 0001:0001f260       ?get@?$hb_lazy_loader_t@Uvmtx_accelerator_t@OT@@U?$hb_face_lazy_loader_t@Uvmtx_accelerator_t@OT@@$0M@@@Uhb_face_t@@$0M@U12@@@QBEPBUvmtx_accelerator_t@OT@@XZ 10020260 f i hb-common.obj
 0001:0001f310       ?get_advance_without_var_unscaled@accelerator_t@?$hmtxvmtx@Uhmtx@OT@@Uhhea@2@UHVAR@2@@OT@@QBEII@Z 10020310 f i hb-common.obj
 0001:0001f310       ?get_advance_without_var_unscaled@accelerator_t@?$hmtxvmtx@Uvmtx@OT@@Uvhea@2@UVVAR@2@@OT@@QBEII@Z 10020310 f i hb-common.obj
 0001:0001f370       ?get_composite_iterator@Glyph@glyf_impl@OT@@QBE?AU?$composite_iter_tmpl@UCompositeGlyphRecord@glyf_impl@OT@@@23@XZ 10020370 f i hb-common.obj
 0001:0001f3d0       ?get_contour_points@SimpleGlyph@glyf_impl@OT@@QBE_NAAUcontour_point_vector_t@@_N@Z 100203d0 f i hb-common.obj
 0001:0001f670       ?get_glyph_var_data_bytes@gvar@OT@@IBE?BU?$hb_array_t@$$CBD@@PAUhb_blob_t@@II@Z 10020670 f i hb-common.obj
 0001:0001f7d0       ?get_leading_bearing_without_var_unscaled@accelerator_t@?$hmtxvmtx@Uvmtx@OT@@Uvhea@2@UVVAR@2@@OT@@QBE_NIPAH@Z 100207d0 f i hb-common.obj
 0001:0001f7d0       ?get_leading_bearing_without_var_unscaled@accelerator_t@?$hmtxvmtx@Uhmtx@OT@@Uhhea@2@UHVAR@2@@OT@@QBE_NIPAH@Z 100207d0 f i hb-common.obj
 0001:0001f860       ?get_transformation@CompositeGlyphRecord@glyf_impl@OT@@QBE_NAAY03MAAUcontour_point_t@@@Z 10020860 f i hb-common.obj
 0001:0001fab0       ?get_tuple_iterator@TupleVariationData@OT@@SA_NU?$hb_array_t@$$CBD@@IPBXAAU?$hb_vector_t@I$0A@@@PAUtuple_iterator_t@12@@Z 10020ab0 f i hb-common.obj
 0001:0001fb80       ?glyph_for_gid@glyf_accelerator_t@OT@@QBE?BUGlyph@glyf_impl@2@I_N@Z 10020b80 f i hb-common.obj
 0001:0001fd40       ?is_valid@tuple_iterator_t@TupleVariationData@OT@@QBE_NXZ 10020d40 f i hb-common.obj
 0001:0001ff20       ?load_num_glyphs@hb_face_t@@ABEIXZ 10020f20 f   hb-common.obj
 0001:0001ff60       ?load_upem@hb_face_t@@ABEIXZ 10020f60 f   hb-common.obj
 0001:00020340       ?read_points@SimpleGlyph@glyf_impl@OT@@SA_NAAPBU?$IntType@E$00@3@U?$hb_array_t@Ucontour_point_t@@@@PBU43@PQcontour_point_t@@MW4simple_glyph_flag_t@123@4@Z 10021340 f i hb-common.obj
 0001:00020420       ?resize@?$hb_vector_t@Ucontour_point_t@@$0A@@@QAE_NH_N0@Z 10021420 f i hb-common.obj
 0001:00020480       ?sanitize@?$_hea@Uvhea@OT@@@OT@@QBE_NPAUhb_sanitize_context_t@@@Z 10021480 f i hb-common.obj
 0001:00020480       ?sanitize@?$_hea@Uhhea@OT@@@OT@@QBE_NPAUhb_sanitize_context_t@@@Z 10021480 f i hb-common.obj
 0001:00020510       ?sanitize@DeltaSetIndexMap@OT@@QBE_NPAUhb_sanitize_context_t@@@Z 10021510 f i hb-common.obj
 0001:00020670       ?sanitize@HVARVVAR@OT@@QBE_NPAUhb_sanitize_context_t@@@Z 10021670 f i hb-common.obj
 0001:00020830       ?sanitize@VVAR@OT@@QBE_NPAUhb_sanitize_context_t@@@Z 10021830 f i hb-common.obj
 0001:000208b0       ?sanitize@head@OT@@QBE_NPAUhb_sanitize_context_t@@@Z 100218b0 f i hb-common.obj
 0001:00020960       ?sanitize@maxp@OT@@QBE_NPAUhb_sanitize_context_t@@@Z 10021960 f i hb-common.obj
 0001:00020a70       ?sanitize_shallow@gvar@OT@@QBE_NPAUhb_sanitize_context_t@@@Z 10021a70 f i hb-common.obj
 0001:00020c80       ?scale_glyph_extents@hb_font_t@@QAEXPAUhb_glyph_extents_t@@@Z 10021c80 f i hb-common.obj
 0001:00020e60       ?set_current@?$composite_iter_tmpl@UCompositeGlyphRecord@glyf_impl@OT@@@glyf_impl@OT@@QAEXPBUCompositeGlyphRecord@23@@Z 10021e60 f i hb-common.obj
 0001:00020ec0       ?transform@CompositeGlyphRecord@glyf_impl@OT@@SAXAAY03$$CBMU?$hb_array_t@Ucontour_point_t@@@@@Z 10021ec0 f i hb-common.obj
 0001:00020f60       ?translate@CompositeGlyphRecord@glyf_impl@OT@@SAXABUcontour_point_t@@U?$hb_array_t@Ucontour_point_t@@@@@Z 10021f60 f i hb-common.obj
 0001:00021010       ?trim_padding@SimpleGlyph@glyf_impl@OT@@QBE?BU?$hb_array_t@$$CBD@@XZ 10022010 f i hb-common.obj
 0001:00021160       ?unpack_deltas@TupleVariationData@OT@@SA_NAAPBU?$IntType@E$00@2@AAU?$hb_vector_t@H$0A@@@PBU32@@Z 10022160 f i hb-common.obj
 0001:000212c0       ?unpack_points@TupleVariationData@OT@@SA_NAAPBU?$IntType@E$00@2@AAU?$hb_vector_t@I$0A@@@PBU32@@Z 100222c0 f i hb-common.obj
 0001:000213c0       _hb_feature_from_string    100223c0 f   hb-common.obj
 0001:00021420       _hb_language_from_string   10022420 f   hb-common.obj
 0001:000214c0       _hb_language_matches       100224c0 f   hb-common.obj
 0001:00021530       _hb_language_to_string     10022530 f   hb-common.obj
 0001:00021540       _hb_script_get_horizontal_direction 10022540 f   hb-common.obj
 0001:000216d0       _hb_tag_from_string        100226d0 f   hb-common.obj
 0001:00021770       _hb_tag_to_string          10022770 f   hb-common.obj
 0001:000218a0       _hb_draw_funcs_create      100228a0 f   hb-draw.obj
 0001:00021930       _hb_draw_funcs_destroy     10022930 f   hb-draw.obj
 0001:00021a20       _hb_draw_funcs_get_empty   10022a20 f   hb-draw.obj
 0001:00021a30       _hb_draw_funcs_set_close_path_func 10022a30 f   hb-draw.obj
 0001:00021ae0       _hb_draw_funcs_set_cubic_to_func 10022ae0 f   hb-draw.obj
 0001:00021b90       _hb_draw_funcs_set_line_to_func 10022b90 f   hb-draw.obj
 0001:00021c40       _hb_draw_funcs_set_move_to_func 10022c40 f   hb-draw.obj
 0001:00021ce0       _hb_draw_funcs_set_quadratic_to_func 10022ce0 f   hb-draw.obj
 0001:00021d90       ??$propagate_error@AAU?$hb_hashmap_t@PBUobject_t@hb_serialize_context_t@@I$0A@@@@hb_serialize_context_t@@QAE_NAAU?$hb_hashmap_t@PBUobject_t@hb_serialize_context_t@@I$0A@@@@Z 10022d90 f i hb-face-builder.obj
 0001:00021dc0       ??$set_with_hash@AAPAUobject_t@hb_serialize_context_t@@AAI@?$hb_hashmap_t@PBUobject_t@hb_serialize_context_t@@I$0A@@@QAE_NAAPAUobject_t@hb_serialize_context_t@@IAAI_N@Z 10022dc0 f i hb-face-builder.obj
 0001:00021dc0       ??$set_with_hash@PBUobject_t@hb_serialize_context_t@@I@?$hb_hashmap_t@PBUobject_t@hb_serialize_context_t@@I$0A@@@QAE_N$$QAPBUobject_t@hb_serialize_context_t@@I$$QAI_N@Z 10022dc0 f i hb-face-builder.obj
 0001:00021fa0       ??0hb_serialize_context_t@@QAE@PAXI@Z 10022fa0 f i hb-face-builder.obj
 0001:000220f0       ??1?$hb_pool_t@Uobject_t@hb_serialize_context_t@@$0CA@@@QAE@XZ 100230f0 f i hb-face-builder.obj
 0001:00022180       ??1hb_serialize_context_t@@QAE@XZ 10023180 f i hb-face-builder.obj
 0001:00022210       ?alloc@?$hb_hashmap_t@PBUobject_t@hb_serialize_context_t@@I$0A@@@QAE_NI@Z 10023210 f i hb-face-builder.obj
 0001:00022490       ?alloc@?$hb_pool_t@Uobject_t@hb_serialize_context_t@@$0CA@@@QAEPAUobject_t@hb_serialize_context_t@@XZ 10023490 f i hb-face-builder.obj
 0001:00022540       ?end_serialize@hb_serialize_context_t@@QAEXXZ 10023540 f i hb-face-builder.obj
 0001:00022870       ?fetch_item@?$hb_hashmap_t@PBUobject_t@hb_serialize_context_t@@I$0A@@@QBEPAUitem_t@1@ABQBUobject_t@hb_serialize_context_t@@I@Z 10023870 f i hb-face-builder.obj
 0001:00022980       ?fini@hb_serialize_context_t@@QAEXXZ 10023980 f i hb-face-builder.obj
 0001:00022b50       ?fini@object_t@hb_serialize_context_t@@QAEXXZ 10023b50 f i hb-face-builder.obj
 0001:00022c30       ?pop_pack@hb_serialize_context_t@@QAEI_N@Z 10023c30 f i hb-face-builder.obj
 0001:00022ee0       ?resolve_links@hb_serialize_context_t@@QAEXXZ 10023ee0 f i hb-face-builder.obj
 0001:00023130       ??$bsearch@I@?$SortedArrayOf@UCmapSubtableLongGroup@OT@@U?$IntType@I$03@2@@OT@@QBEABUCmapSubtableLongGroup@1@ABIABU21@@Z 10024130 f i hb-face.obj
 0001:000231e0       ??$bsearch@I@?$SortedArrayOf@UVariationSelectorRecord@OT@@U?$IntType@I$03@2@@OT@@QBEABUVariationSelectorRecord@1@ABIABU21@@Z 100241e0 f i hb-face.obj
 0001:00023260       ??$get_glyph_from@UCmapSubtable@OT@@@accelerator_t@cmap@OT@@KA_NPBXIPAI@Z 10024260 f i hb-face.obj
 0001:00023280       ??$get_glyph_from@UCmapSubtableFormat12@OT@@@accelerator_t@cmap@OT@@KA_NPBXIPAI@Z 10024280 f i hb-face.obj
 0001:000237e0       ??$sanitize_blob@UOS2@OT@@@hb_sanitize_context_t@@QAEPAUhb_blob_t@@PAU1@@Z 100247e0 f i hb-face.obj
 0001:00023970       ??$sanitize_blob@Ucmap@OT@@@hb_sanitize_context_t@@QAEPAUhb_blob_t@@PAU1@@Z 10024970 f i hb-face.obj
 0001:00023b00       ??0accelerator_t@cmap@OT@@QAE@PAUhb_face_t@@@Z 10024b00 f i hb-face.obj
 0001:00023f00       ??A?$ArrayOf@UHBGlyphID16@OT@@U?$IntType@G$01@2@@OT@@QBEABUHBGlyphID16@1@H@Z 10024f00 f i hb-face.obj
 0001:00023f30       ??A?$hb_vector_t@I$0A@@@QBEABIH@Z 10024f30 f i hb-face.obj
 0001:00023f50       ??C?$hb_lazy_loader_t@UOS2@OT@@U?$hb_table_lazy_loader_t@UOS2@OT@@$05$00@@Uhb_face_t@@$05Uhb_blob_t@@@@QBEPBUOS2@OT@@XZ 10024f50 f i hb-face.obj
 0001:00024070       ??C?$hb_lazy_loader_t@Ucmap_accelerator_t@OT@@U?$hb_face_lazy_loader_t@Ucmap_accelerator_t@OT@@$02@@Uhb_face_t@@$02U12@@@QBEPBUcmap_accelerator_t@OT@@XZ 10025070 f i hb-face.obj
 0001:00024210       ?find_subtable@cmap@OT@@IBEPBUCmapSubtable@2@II@Z 10025210 f i hb-face.obj
 0001:000243b0       ?get_glyph@?$CmapSubtableLongSegmented@UCmapSubtableFormat12@OT@@@OT@@QBE_NIPAI@Z 100253b0 f i hb-face.obj
 0001:000243f0       ?get_glyph@CmapSubtable@OT@@QBE_NIPAI@Z 100253f0 f i hb-face.obj
 0001:000245f0       ?get_glyph@accelerator_t@CmapSubtableFormat4@OT@@QBE_NIPAI@Z 100255f0 f i hb-face.obj
 0001:00024710       ?get_glyph_func@accelerator_t@CmapSubtableFormat4@OT@@SA_NPBXIPAI@Z 10025710 f i hb-face.obj
 0001:00024730       ?group_get_glyph@CmapSubtableFormat12@OT@@SAIABUCmapSubtableLongGroup@2@I@Z 10025730 f i hb-face.obj
 0001:000247d0       ?init@accelerator_t@CmapSubtableFormat4@OT@@QAEXPBU23@@Z 100257d0 f i hb-face.obj
 0001:00024830       ?sanitize@CmapSubtable@OT@@QBE_NPAUhb_sanitize_context_t@@@Z 10025830 f i hb-face.obj
 0001:00024b20       ?sanitize@CmapSubtableFormat4@OT@@QBE_NPAUhb_sanitize_context_t@@@Z 10025b20 f i hb-face.obj
 0001:00024c70       ?sanitize@OS2@OT@@QBE_NPAUhb_sanitize_context_t@@@Z 10025c70 f i hb-face.obj
 0001:00024e40       ?sanitize@VariationSelectorRecord@OT@@QBE_NPAUhb_sanitize_context_t@@PBX@Z 10025e40 f i hb-face.obj
 0001:00024f80       ?sanitize@cmap@OT@@QBE_NPAUhb_sanitize_context_t@@@Z 10025f80 f i hb-face.obj
 0001:00025120       ?sanitize_shallow@?$ArrayOf@UCmapSubtableLongGroup@OT@@U?$IntType@I$03@2@@OT@@QBE_NPAUhb_sanitize_context_t@@@Z 10026120 f i hb-face.obj
 0001:000251e0       ?sanitize_shallow@?$ArrayOf@UEncodingRecord@OT@@U?$IntType@G$01@2@@OT@@QBE_NPAUhb_sanitize_context_t@@@Z 100261e0 f i hb-face.obj
 0001:00025280       ?sanitize_shallow@?$ArrayOf@UHBGlyphID16@OT@@U?$IntType@I$03@2@@OT@@QBE_NPAUhb_sanitize_context_t@@@Z 10026280 f i hb-face.obj
 0001:00025340       ?sanitize_shallow@?$ArrayOf@UUVSMapping@OT@@U?$IntType@I$03@2@@OT@@QBE_NPAUhb_sanitize_context_t@@@Z 10026340 f i hb-face.obj
 0001:00025400       ?sanitize_shallow@?$ArrayOf@UVariationSelectorRecord@OT@@U?$IntType@I$03@2@@OT@@QBE_NPAUhb_sanitize_context_t@@@Z 10026400 f i hb-face.obj
 0001:000254c0       _hb_face_create_for_tables 100264c0 f   hb-face.obj
 0001:00025520       _hb_face_destroy           10026520 f   hb-face.obj
 0001:000255f0       _hb_face_get_empty         100265f0 f   hb-face.obj
 0001:00025600       _hb_face_get_glyph_count   10026600 f   hb-face.obj
 0001:00025620       _hb_face_get_upem          10026620 f   hb-face.obj
 0001:00025630       _hb_face_get_user_data     10026630 f   hb-face.obj
 0001:000256c0       _hb_face_reference_table   100266c0 f   hb-face.obj
 0001:000256f0       _hb_face_set_user_data     100266f0 f   hb-face.obj
 0001:00025710       ?get_glyph_v_advance@hb_font_t@@QAEHI@Z 10026710 f i hb-fallback-shape.obj
 0001:00025750       __hb_fallback_shape        10026750 f   hb-fallback-shape.obj
 0001:00025b40       __hb_ot_shaper_face_data_create 10026b40 f   hb-ot-shape.obj
 0001:00025b40       __hb_fallback_shaper_font_data_create 10026b40 f   hb-fallback-shape.obj
 0001:00025b40       __hb_ot_shaper_font_data_create 10026b40 f   hb-ot-shape.obj
 0001:00025b40       __hb_fallback_shaper_face_data_create 10026b40 f   hb-fallback-shape.obj
 0001:00025b50       ??$sanitize_blob@Uavar@OT@@@hb_sanitize_context_t@@QAEPAUhb_blob_t@@PAU1@@Z 10026b50 f i hb-font.obj
 0001:00025ce0       ??$sanitize_blob@Ufvar@OT@@@hb_sanitize_context_t@@QAEPAUhb_blob_t@@PAU1@@Z 10026ce0 f i hb-font.obj
 0001:00025e70       ??C?$hb_lazy_loader_t@Uavar@OT@@U?$hb_table_lazy_loader_t@Uavar@OT@@$0BD@$00@@Uhb_face_t@@$0BD@Uhb_blob_t@@@@QBEPBUavar@OT@@XZ 10026e70 f i hb-font.obj
 0001:000260e0       ?get@?$hb_lazy_loader_t@Ufvar@OT@@U?$hb_table_lazy_loader_t@Ufvar@OT@@$0BC@$00@@Uhb_face_t@@$0BC@Uhb_blob_t@@@@QBEPBUfvar@OT@@XZ 100270e0 f i hb-font.obj
 0001:000261f0       ?get_axes@fvar@OT@@QBE?AU?$hb_array_t@$$CBUAxisRecord@OT@@@@XZ 100271f0 f i hb-font.obj
 0001:00026240       ?get_coordinates@AxisRecord@OT@@QBEXAAM00@Z 10027240 f i hb-font.obj
 0001:00026320       ?has_func@hb_font_t@@QAE_NI@Z 10027320 f   hb-font.obj
 0001:00026c40       ___scrt_stub_for_is_c_termination_complete 10027c40 f   MSVCRT:ucrt_stubs.obj
 0001:00026c40       __is_c_termination_complete 10027c40 f   MSVCRT:ucrt_stubs.obj
 0001:00027210       ?map@SegmentMaps@OT@@QBEHHII@Z 10028210 f i hb-font.obj
 0001:00027480       ?mults_changed@hb_font_t@@QAEXXZ 10028480 f i hb-font.obj
 0001:00027660       ?parent_scale_position@hb_font_t@@QAEXPAH0@Z 10028660 f i hb-font.obj
 0001:000276d0       ?sanitize@avar@OT@@QBE_NPAUhb_sanitize_context_t@@@Z 100286d0 f i hb-font.obj
 0001:00027890       ?sanitize@fvar@OT@@QBE_NPAUhb_sanitize_context_t@@@Z 10028890 f i hb-font.obj
 0001:00027ac0       _hb_font_create            10028ac0 f   hb-font.obj
 0001:00027b10       _hb_font_destroy           10028b10 f   hb-font.obj
 0001:00027be0       _hb_font_draw_glyph        10028be0 f   hb-font.obj
 0001:00027c10       _hb_font_funcs_create      10028c10 f   hb-font.obj
 0001:00027cb0       _hb_font_funcs_destroy     10028cb0 f   hb-font.obj
 0001:00027f10       _hb_font_funcs_get_empty   10028f10 f   hb-font.obj
 0001:00027f20       _hb_font_funcs_set_draw_glyph_func 10028f20 f   hb-font.obj
 0001:00027fd0       _hb_font_funcs_set_font_h_extents_func 10028fd0 f   hb-font.obj
 0001:00028070       _hb_font_funcs_set_font_v_extents_func 10029070 f   hb-font.obj
 0001:00028120       _hb_font_funcs_set_glyph_contour_point_func 10029120 f   hb-font.obj
 0001:000281d0       _hb_font_funcs_set_glyph_extents_func 100291d0 f   hb-font.obj
 0001:00028280       _hb_font_funcs_set_glyph_from_name_func 10029280 f   hb-font.obj
 0001:00028330       _hb_font_funcs_set_glyph_h_advance_func 10029330 f   hb-font.obj
 0001:000283e0       _hb_font_funcs_set_glyph_h_advances_func 100293e0 f   hb-font.obj
 0001:00028490       _hb_font_funcs_set_glyph_h_kerning_func 10029490 f   hb-font.obj
 0001:00028540       _hb_font_funcs_set_glyph_h_origin_func 10029540 f   hb-font.obj
 0001:000285f0       _hb_font_funcs_set_glyph_name_func 100295f0 f   hb-font.obj
 0001:000286a0       _hb_font_funcs_set_glyph_v_advance_func 100296a0 f   hb-font.obj
 0001:00028750       _hb_font_funcs_set_glyph_v_advances_func 10029750 f   hb-font.obj
 0001:00028800       _hb_font_funcs_set_glyph_v_kerning_func 10029800 f   hb-font.obj
 0001:000288b0       _hb_font_funcs_set_glyph_v_origin_func 100298b0 f   hb-font.obj
 0001:00028960       _hb_font_funcs_set_nominal_glyph_func 10029960 f   hb-font.obj
 0001:00028a10       _hb_font_funcs_set_nominal_glyphs_func 10029a10 f   hb-font.obj
 0001:00028ac0       _hb_font_funcs_set_paint_glyph_func 10029ac0 f   hb-font.obj
 0001:00028b70       _hb_font_funcs_set_variation_glyph_func 10029b70 f   hb-font.obj
 0001:00028c20       _hb_font_get_face          10029c20 f   hb-font.obj
 0001:00028c30       _hb_font_get_glyph         10029c30 f   hb-font.obj
 0001:00028ca0       _hb_font_get_glyph_extents 10029ca0 f   hb-font.obj
 0001:00028cf0       _hb_font_get_glyph_h_advance 10029cf0 f   hb-font.obj
 0001:00028d30       _hb_font_get_nominal_glyph 10029d30 f   hb-font.obj
 0001:00028d80       _hb_font_set_funcs         10029d80 f   hb-font.obj
 0001:00028e00       _hb_font_set_scale         10029e00 f   hb-font.obj
 0001:00028e30       _hb_font_set_var_coords_normalized 10029e30 f   hb-font.obj
 0001:00029170       _hb_font_set_variations    1002a170 f   hb-font.obj
 0001:00029390       ?CallIntMethod@JNIEnv_@@QAAJPAV_jobject@@PAU_jmethodID@@ZZ 1002a390 f i hb-jdk-font.obj
 0001:000293b0       ?CallObjectMethod@JNIEnv_@@QAAPAV_jobject@@PAV2@PAU_jmethodID@@ZZ 1002a3b0 f i hb-jdk-font.obj
 0001:00029720       _Java_sun_font_SunLayoutEngine_createFace@20 1002a720 f   hb-jdk-font.obj
 0001:000297a0       _Java_sun_font_SunLayoutEngine_disposeFace@16 1002a7a0 f   hb-jdk-font.obj
 0001:000297b0       _hb_jdk_font_create        1002a7b0 f   hb-jdk-font.obj
 0001:00029930       ?hb_parse_double@@YA_NPAPBDPBDPAN_N@Z 1002a930 f   hb-number.obj
 0001:00029980       ?hb_parse_int@@YA_NPAPBDPBDPAH_N@Z 1002a980 f   hb-number.obj
 0001:00029d80       ??$?0$$CBUaccelerator_t@cff1@OT@@@cff1_cs_interp_env_t@CFF@@QAE@ABU?$hb_array_t@$$CBE@@ABUaccelerator_t@cff1@OT@@IPBHI@Z 1002ad80 f i hb-ot-cff1-table.obj
 0001:00029df0       ??$bsearch@I@?$hb_sorted_array_t@$$CBUsid_to_gid_t@@@@QAEPBUsid_to_gid_t@@ABIPBU1@@Z 1002adf0 f i hb-ot-cff1-table.obj
 0001:00029e60       ??0?$cs_interp_env_t@Unumber_t@CFF@@U?$Subrs@U?$IntType@G$01@OT@@@2@@CFF@@QAE@ABU?$hb_array_t@$$CBE@@PBU?$Subrs@U?$IntType@G$01@OT@@@1@1@Z 1002ae60 f i hb-ot-cff1-table.obj
 0001:0002a000       ??0?$interp_env_t@Unumber_t@CFF@@@CFF@@QAE@ABU?$hb_array_t@$$CBE@@@Z 1002b000 f i hb-ot-cff1-table.obj
 0001:0002a050       ??A?$CFFIndex@U?$IntType@G$01@OT@@@CFF@@QBE?AU?$hb_array_t@$$CBE@@I@Z 1002b050 f i hb-ot-cff1-table.obj
 0001:0002a310       ?call_subr@?$cs_interp_env_t@Unumber_t@CFF@@U?$Subrs@U?$IntType@G$01@OT@@@2@@CFF@@QAEXABU?$biased_subrs_t@U?$Subrs@U?$IntType@G$01@OT@@@CFF@@@2@W4cs_type_t@2@@Z 1002b310 f i hb-ot-cff1-table.obj
 0001:0002a460       ?check_width@?$cff1_cs_opset_t@Ucff1_cs_opset_extents_t@@Ucff1_extents_param_t@@Ucff1_path_procs_extents_t@@@CFF@@SAXIAAUcff1_cs_interp_env_t@2@AAUcff1_extents_param_t@@@Z 1002b460 f i hb-ot-cff1-table.obj
 0001:0002a460       ?check_width@?$cff1_cs_opset_t@Ucff1_cs_opset_path_t@@Ucff1_path_param_t@@Ucff1_path_procs_path_t@@@CFF@@SAXIAAUcff1_cs_interp_env_t@2@AAUcff1_path_param_t@@@Z 1002b460 f i hb-ot-cff1-table.obj
 0001:0002a4f0       ?clear_args@?$interp_env_t@Unumber_t@CFF@@@CFF@@QAEXXZ 1002b4f0 f i hb-ot-cff1-table.obj
 0001:0002a510       ?cubic_to@cff1_path_param_t@@QAEXABUpoint_t@CFF@@00@Z 1002b510 f i hb-ot-cff1-table.obj
 0001:0002a7c0       ?curve@cff1_path_procs_extents_t@@SAXAAUcff1_cs_interp_env_t@CFF@@AAUcff1_extents_param_t@@ABUpoint_t@3@22@Z 1002b7c0 f i hb-ot-cff1-table.obj
 0001:0002a9d0       ?end_path@cff1_path_param_t@@QAEXXZ 1002b9d0 f i hb-ot-cff1-table.obj
 0001:0002aa70       ?flex1@?$path_procs_t@Ucff1_path_procs_extents_t@@Ucff1_cs_interp_env_t@CFF@@Ucff1_extents_param_t@@@CFF@@SAXAAUcff1_cs_interp_env_t@2@AAUcff1_extents_param_t@@@Z 1002ba70 f i hb-ot-cff1-table.obj
 0001:0002ae50       ?flex1@?$path_procs_t@Ucff1_path_procs_path_t@@Ucff1_cs_interp_env_t@CFF@@Ucff1_path_param_t@@@CFF@@SAXAAUcff1_cs_interp_env_t@2@AAUcff1_path_param_t@@@Z 1002be50 f i hb-ot-cff1-table.obj
 0001:0002b250       ?flex@?$path_procs_t@Ucff1_path_procs_extents_t@@Ucff1_cs_interp_env_t@CFF@@Ucff1_extents_param_t@@@CFF@@SAXAAUcff1_cs_interp_env_t@2@AAUcff1_extents_param_t@@@Z 1002c250 f i hb-ot-cff1-table.obj
 0001:0002b580       ?flex@?$path_procs_t@Ucff1_path_procs_path_t@@Ucff1_cs_interp_env_t@CFF@@Ucff1_path_param_t@@@CFF@@SAXAAUcff1_cs_interp_env_t@2@AAUcff1_path_param_t@@@Z 1002c580 f i hb-ot-cff1-table.obj
 0001:0002b8f0       ?flush_args_and_op@?$cs_opset_t@Unumber_t@CFF@@Ucff1_cs_opset_extents_t@@Ucff1_cs_interp_env_t@2@Ucff1_extents_param_t@@Ucff1_path_procs_extents_t@@@CFF@@SAXIAAUcff1_cs_interp_env_t@2@AAUcff1_extents_param_t@@@Z 1002c8f0 f i hb-ot-cff1-table.obj
 0001:0002b8f0       ?process_post_flex@?$cs_opset_t@Unumber_t@CFF@@Ucff1_cs_opset_path_t@@Ucff1_cs_interp_env_t@2@Ucff1_path_param_t@@Ucff1_path_procs_path_t@@@CFF@@SAXIAAUcff1_cs_interp_env_t@2@AAUcff1_path_param_t@@@Z 1002c8f0 f i hb-ot-cff1-table.obj
 0001:0002b8f0       ?flush_args_and_op@?$cs_opset_t@Unumber_t@CFF@@Ucff1_cs_opset_path_t@@Ucff1_cs_interp_env_t@2@Ucff1_path_param_t@@Ucff1_path_procs_path_t@@@CFF@@SAXIAAUcff1_cs_interp_env_t@2@AAUcff1_path_param_t@@@Z 1002c8f0 f i hb-ot-cff1-table.obj
 0001:0002b8f0       ?process_post_flex@?$cs_opset_t@Unumber_t@CFF@@Ucff1_cs_opset_extents_t@@Ucff1_cs_interp_env_t@2@Ucff1_extents_param_t@@Ucff1_path_procs_extents_t@@@CFF@@SAXIAAUcff1_cs_interp_env_t@2@AAUcff1_extents_param_t@@@Z 1002c8f0 f i hb-ot-cff1-table.obj
 0001:0002b8f0       ?process_post_path@?$cs_opset_t@Unumber_t@CFF@@Ucff1_cs_opset_extents_t@@Ucff1_cs_interp_env_t@2@Ucff1_extents_param_t@@Ucff1_path_procs_extents_t@@@CFF@@SAXIAAUcff1_cs_interp_env_t@2@AAUcff1_extents_param_t@@@Z 1002c8f0 f i hb-ot-cff1-table.obj
 0001:0002b8f0       ?process_post_path@?$cs_opset_t@Unumber_t@CFF@@Ucff1_cs_opset_path_t@@Ucff1_cs_interp_env_t@2@Ucff1_path_param_t@@Ucff1_path_procs_path_t@@@CFF@@SAXIAAUcff1_cs_interp_env_t@2@AAUcff1_path_param_t@@@Z 1002c8f0 f i hb-ot-cff1-table.obj
 0001:0002b930       ?get_extents@accelerator_t@cff1@OT@@QBE_NPAUhb_font_t@@IPAUhb_glyph_extents_t@@@Z 1002c930 f   hb-ot-cff1-table.obj
 0001:0002bc90       ?get_fd@FDSelect@CFF@@QBEII@Z 1002cc90 f i hb-ot-cff1-table.obj
 0001:0002bd80       ?get_glyph@Charset@CFF@@QBEIII@Z 1002cd80 f i hb-ot-cff1-table.obj
 0001:0002bec0       ?get_path@accelerator_t@cff1@OT@@QBE_NPAUhb_font_t@@IAAUhb_draw_session_t@@@Z 1002cec0 f   hb-ot-cff1-table.obj
 0001:0002bef0       ?hflex1@?$path_procs_t@Ucff1_path_procs_extents_t@@Ucff1_cs_interp_env_t@CFF@@Ucff1_extents_param_t@@@CFF@@SAXAAUcff1_cs_interp_env_t@2@AAUcff1_extents_param_t@@@Z 1002cef0 f i hb-ot-cff1-table.obj
 0001:0002c180       ?hflex1@?$path_procs_t@Ucff1_path_procs_path_t@@Ucff1_cs_interp_env_t@CFF@@Ucff1_path_param_t@@@CFF@@SAXAAUcff1_cs_interp_env_t@2@AAUcff1_path_param_t@@@Z 1002d180 f i hb-ot-cff1-table.obj
 0001:0002c420       ?hflex@?$path_procs_t@Ucff1_path_procs_extents_t@@Ucff1_cs_interp_env_t@CFF@@Ucff1_extents_param_t@@@CFF@@SAXAAUcff1_cs_interp_env_t@2@AAUcff1_extents_param_t@@@Z 1002d420 f i hb-ot-cff1-table.obj
 0001:0002c650       ?hflex@?$path_procs_t@Ucff1_path_procs_path_t@@Ucff1_cs_interp_env_t@CFF@@Ucff1_path_param_t@@@CFF@@SAXAAUcff1_cs_interp_env_t@2@AAUcff1_path_param_t@@@Z 1002d650 f i hb-ot-cff1-table.obj
 0001:0002c890       ?hhcurveto@?$path_procs_t@Ucff1_path_procs_extents_t@@Ucff1_cs_interp_env_t@CFF@@Ucff1_extents_param_t@@@CFF@@SAXAAUcff1_cs_interp_env_t@2@AAUcff1_extents_param_t@@@Z 1002d890 f i hb-ot-cff1-table.obj
 0001:0002cbf0       ?hhcurveto@?$path_procs_t@Ucff1_path_procs_path_t@@Ucff1_cs_interp_env_t@CFF@@Ucff1_path_param_t@@@CFF@@SAXAAUcff1_cs_interp_env_t@2@AAUcff1_path_param_t@@@Z 1002dbf0 f i hb-ot-cff1-table.obj
 0001:0002cda0       ?hlineto@?$path_procs_t@Ucff1_path_procs_extents_t@@Ucff1_cs_interp_env_t@CFF@@Ucff1_extents_param_t@@@CFF@@SAXAAUcff1_cs_interp_env_t@2@AAUcff1_extents_param_t@@@Z 1002dda0 f i hb-ot-cff1-table.obj
 0001:0002d120       ?hvcurveto@?$path_procs_t@Ucff1_path_procs_extents_t@@Ucff1_cs_interp_env_t@CFF@@Ucff1_extents_param_t@@@CFF@@SAXAAUcff1_cs_interp_env_t@2@AAUcff1_extents_param_t@@@Z 1002e120 f i hb-ot-cff1-table.obj
 0001:0002dea0       ?hvcurveto@?$path_procs_t@Ucff1_path_procs_path_t@@Ucff1_cs_interp_env_t@CFF@@Ucff1_path_param_t@@@CFF@@SAXAAUcff1_cs_interp_env_t@2@AAUcff1_path_param_t@@@Z 1002eea0 f i hb-ot-cff1-table.obj
 0001:0002e5a0       ?interpret@?$cs_interpreter_t@Ucff1_cs_interp_env_t@CFF@@Ucff1_cs_opset_extents_t@@Ucff1_extents_param_t@@@CFF@@QAE_NAAUcff1_extents_param_t@@@Z 1002f5a0 f i hb-ot-cff1-table.obj
 0001:0002e6f0       ?interpret@?$cs_interpreter_t@Ucff1_cs_interp_env_t@CFF@@Ucff1_cs_opset_path_t@@Ucff1_path_param_t@@@CFF@@QAE_NAAUcff1_path_param_t@@@Z 1002f6f0 f i hb-ot-cff1-table.obj
 0001:0002e840       ?line@cff1_path_procs_extents_t@@SAXAAUcff1_cs_interp_env_t@CFF@@AAUcff1_extents_param_t@@ABUpoint_t@3@@Z 1002f840 f i hb-ot-cff1-table.obj
 0001:0002e980       ?line_to@cff1_path_param_t@@QAEXABUpoint_t@CFF@@@Z 1002f980 f i hb-ot-cff1-table.obj
 0001:0002eb20       ?lookup_expert_charset_for_glyph@cff1@OT@@KAII@Z 1002fb20 f   hb-ot-cff1-table.obj
 0001:0002eb60       ?lookup_expert_charset_for_sid@cff1@OT@@KAII@Z 1002fb60 f   hb-ot-cff1-table.obj
 0001:0002eb80       ?lookup_expert_subset_charset_for_glyph@cff1@OT@@KAII@Z 1002fb80 f   hb-ot-cff1-table.obj
 0001:0002ebc0       ?lookup_expert_subset_charset_for_sid@cff1@OT@@KAII@Z 1002fbc0 f   hb-ot-cff1-table.obj
 0001:0002ebe0       ?merge@bounds_t@@QAEXABU1@@Z 1002fbe0 f i hb-ot-cff1-table.obj
 0001:0002ec90       ?move_to@cff1_path_param_t@@QAEXABUpoint_t@CFF@@@Z 1002fc90 f i hb-ot-cff1-table.obj
 0001:0002edb0       ?offset_at@?$CFFIndex@U?$IntType@G$01@OT@@@CFF@@ABEII@Z 1002fdb0 f i hb-ot-cff1-table.obj
 0001:0002ee50       ?process_op@?$cs_opset_t@Unumber_t@CFF@@Ucff1_cs_opset_extents_t@@Ucff1_cs_interp_env_t@2@Ucff1_extents_param_t@@Ucff1_path_procs_extents_t@@@CFF@@SAXIAAUcff1_cs_interp_env_t@2@AAUcff1_extents_param_t@@@Z 1002fe50 f i hb-ot-cff1-table.obj
 0001:0002f480       ?process_op@?$cs_opset_t@Unumber_t@CFF@@Ucff1_cs_opset_path_t@@Ucff1_cs_interp_env_t@2@Ucff1_path_param_t@@Ucff1_path_procs_path_t@@@CFF@@SAXIAAUcff1_cs_interp_env_t@2@AAUcff1_path_param_t@@@Z 10030480 f i hb-ot-cff1-table.obj
 0001:0002fe60       ?process_op@?$opset_t@Unumber_t@CFF@@@CFF@@SAXIAAU?$interp_env_t@Unumber_t@CFF@@@2@@Z 10030e60 f i hb-ot-cff1-table.obj
 0001:00030150       ?process_post_move@?$cs_opset_t@Unumber_t@CFF@@Ucff1_cs_opset_extents_t@@Ucff1_cs_interp_env_t@2@Ucff1_extents_param_t@@Ucff1_path_procs_extents_t@@@CFF@@SAXIAAUcff1_cs_interp_env_t@2@AAUcff1_extents_param_t@@@Z 10031150 f i hb-ot-cff1-table.obj
 0001:00030150       ?process_post_move@?$cs_opset_t@Unumber_t@CFF@@Ucff1_cs_opset_path_t@@Ucff1_cs_interp_env_t@2@Ucff1_path_param_t@@Ucff1_path_procs_path_t@@@CFF@@SAXIAAUcff1_cs_interp_env_t@2@AAUcff1_path_param_t@@@Z 10031150 f i hb-ot-cff1-table.obj
 0001:000301d0       ?process_seac@cff1_cs_opset_extents_t@@SAXAAUcff1_cs_interp_env_t@CFF@@AAUcff1_extents_param_t@@@Z 100311d0 f i hb-ot-cff1-table.obj
 0001:00030450       ?process_seac@cff1_cs_opset_path_t@@SAXAAUcff1_cs_interp_env_t@CFF@@AAUcff1_path_param_t@@@Z 10031450 f i hb-ot-cff1-table.obj
 0001:00030640       ?push_fixed_from_substr@?$arg_stack_t@Unumber_t@CFF@@@CFF@@QAE_NAAUbyte_str_ref_t@2@@Z 10031640 f i hb-ot-cff1-table.obj
 0001:000306d0       ?rcurveline@?$path_procs_t@Ucff1_path_procs_extents_t@@Ucff1_cs_interp_env_t@CFF@@Ucff1_extents_param_t@@@CFF@@SAXAAUcff1_cs_interp_env_t@2@AAUcff1_extents_param_t@@@Z 100316d0 f i hb-ot-cff1-table.obj
 0001:00030b00       ?rcurveline@?$path_procs_t@Ucff1_path_procs_path_t@@Ucff1_cs_interp_env_t@CFF@@Ucff1_path_param_t@@@CFF@@SAXAAUcff1_cs_interp_env_t@2@AAUcff1_path_param_t@@@Z 10031b00 f i hb-ot-cff1-table.obj
 0001:00030dc0       ?return_from_subr@?$cs_interp_env_t@Unumber_t@CFF@@U?$Subrs@U?$IntType@I$03@OT@@@2@@CFF@@QAEXXZ 10031dc0 f i hb-ot-cff2-table.obj
 0001:00030dc0       ?return_from_subr@?$cs_interp_env_t@Unumber_t@CFF@@U?$Subrs@U?$IntType@G$01@OT@@@2@@CFF@@QAEXXZ 10031dc0 f i hb-ot-cff1-table.obj
 0001:00030e40       ?rlinecurve@?$path_procs_t@Ucff1_path_procs_extents_t@@Ucff1_cs_interp_env_t@CFF@@Ucff1_extents_param_t@@@CFF@@SAXAAUcff1_cs_interp_env_t@2@AAUcff1_extents_param_t@@@Z 10031e40 f i hb-ot-cff1-table.obj
 0001:000311d0       ?rlinecurve@?$path_procs_t@Ucff1_path_procs_path_t@@Ucff1_cs_interp_env_t@CFF@@Ucff1_path_param_t@@@CFF@@SAXAAUcff1_cs_interp_env_t@2@AAUcff1_path_param_t@@@Z 100321d0 f i hb-ot-cff1-table.obj
 0001:00031490       ?rlineto@?$path_procs_t@Ucff1_path_procs_extents_t@@Ucff1_cs_interp_env_t@CFF@@Ucff1_extents_param_t@@@CFF@@SAXAAUcff1_cs_interp_env_t@2@AAUcff1_extents_param_t@@@Z 10032490 f i hb-ot-cff1-table.obj
 0001:00031690       ?rrcurveto@?$path_procs_t@Ucff1_path_procs_extents_t@@Ucff1_cs_interp_env_t@CFF@@Ucff1_extents_param_t@@@CFF@@SAXAAUcff1_cs_interp_env_t@2@AAUcff1_extents_param_t@@@Z 10032690 f i hb-ot-cff1-table.obj
 0001:00031a10       ?rrcurveto@?$path_procs_t@Ucff1_path_procs_path_t@@Ucff1_cs_interp_env_t@CFF@@Ucff1_path_param_t@@@CFF@@SAXAAUcff1_cs_interp_env_t@2@AAUcff1_path_param_t@@@Z 10032a10 f i hb-ot-cff1-table.obj
 0001:00031c00       ?set_width@cff1_cs_interp_env_t@CFF@@QAEX_N@Z 10032c00 f i hb-ot-cff1-table.obj
 0001:00031c80       ?vhcurveto@?$path_procs_t@Ucff1_path_procs_extents_t@@Ucff1_cs_interp_env_t@CFF@@Ucff1_extents_param_t@@@CFF@@SAXAAUcff1_cs_interp_env_t@2@AAUcff1_extents_param_t@@@Z 10032c80 f i hb-ot-cff1-table.obj
 0001:000329e0       ?vhcurveto@?$path_procs_t@Ucff1_path_procs_path_t@@Ucff1_cs_interp_env_t@CFF@@Ucff1_path_param_t@@@CFF@@SAXAAUcff1_cs_interp_env_t@2@AAUcff1_path_param_t@@@Z 100339e0 f i hb-ot-cff1-table.obj
 0001:000330d0       ?vlineto@?$path_procs_t@Ucff1_path_procs_extents_t@@Ucff1_cs_interp_env_t@CFF@@Ucff1_extents_param_t@@@CFF@@SAXAAUcff1_cs_interp_env_t@2@AAUcff1_extents_param_t@@@Z 100340d0 f i hb-ot-cff1-table.obj
 0001:00033450       ?vvcurveto@?$path_procs_t@Ucff1_path_procs_extents_t@@Ucff1_cs_interp_env_t@CFF@@Ucff1_extents_param_t@@@CFF@@SAXAAUcff1_cs_interp_env_t@2@AAUcff1_extents_param_t@@@Z 10034450 f i hb-ot-cff1-table.obj
 0001:000337b0       ?vvcurveto@?$path_procs_t@Ucff1_path_procs_path_t@@Ucff1_cs_interp_env_t@CFF@@Ucff1_path_param_t@@@CFF@@SAXAAUcff1_cs_interp_env_t@2@AAUcff1_path_param_t@@@Z 100347b0 f i hb-ot-cff1-table.obj
 0001:00033980       ??$?0$$CBUaccelerator_t@cff2@OT@@@?$cff2_cs_interp_env_t@Unumber_t@CFF@@@CFF@@QAE@ABU?$hb_array_t@$$CBE@@ABUaccelerator_t@cff2@OT@@IPBHI@Z 10034980 f i hb-ot-cff2-table.obj
 0001:00033a90       ??0?$cs_interp_env_t@Unumber_t@CFF@@U?$Subrs@U?$IntType@I$03@OT@@@2@@CFF@@QAE@ABU?$hb_array_t@$$CBE@@PBU?$Subrs@U?$IntType@I$03@OT@@@1@1@Z 10034a90 f i hb-ot-cff2-table.obj
 0001:00033c50       ??1?$cff2_cs_interp_env_t@Unumber_t@CFF@@@CFF@@QAE@XZ 10034c50 f i hb-ot-cff2-table.obj
 0001:00033ca0       ??A?$ArrayOf@U?$FDSelect3_4_Range@U?$IntType@I$03@OT@@U?$IntType@G$01@2@@CFF@@U?$IntType@I$03@OT@@@OT@@QBEABU?$FDSelect3_4_Range@U?$IntType@I$03@OT@@U?$IntType@G$01@2@@CFF@@H@Z 10034ca0 f i hb-ot-cff2-table.obj
 0001:00033ce0       ??A?$CFFIndex@U?$IntType@I$03@OT@@@CFF@@QBE?AU?$hb_array_t@$$CBE@@I@Z 10034ce0 f i hb-ot-cff2-table.obj
 0001:00033d90       ?blend_deltas@?$cff2_cs_interp_env_t@Unumber_t@CFF@@@CFF@@QBENU?$hb_array_t@$$CBUnumber_t@CFF@@@@@Z 10034d90 f i hb-ot-cff2-table.obj
 0001:00033e80       ?call_subr@?$cs_interp_env_t@Unumber_t@CFF@@U?$Subrs@U?$IntType@I$03@OT@@@2@@CFF@@QAEXABU?$biased_subrs_t@U?$Subrs@U?$IntType@I$03@OT@@@CFF@@@2@W4cs_type_t@2@@Z 10034e80 f i hb-ot-cff2-table.obj
 0001:00034000       ?cubic_to@cff2_path_param_t@@QAEXABUpoint_t@CFF@@00@Z 10035000 f i hb-ot-cff2-table.obj
 0001:00034240       ?curve@cff2_path_procs_extents_t@@SAXAAU?$cff2_cs_interp_env_t@Unumber_t@CFF@@@CFF@@AAUcff2_extents_param_t@@ABUpoint_t@3@22@Z 10035240 f i hb-ot-cff2-table.obj
 0001:00034460       ?data_base@?$CFFIndex@U?$IntType@I$03@OT@@@CFF@@ABEPBEXZ 10035460 f i hb-ot-cff2-table.obj
 0001:00034490       ?evaluate@VarRegionList@OT@@QBEMIPBHIPAM@Z 10035490 f i hb-ot-cff2-table.obj
 0001:00034650       ?flex1@?$path_procs_t@Ucff2_path_procs_extents_t@@U?$cff2_cs_interp_env_t@Unumber_t@CFF@@@CFF@@Ucff2_extents_param_t@@@CFF@@SAXAAU?$cff2_cs_interp_env_t@Unumber_t@CFF@@@2@AAUcff2_extents_param_t@@@Z 10035650 f i hb-ot-cff2-table.obj
 0001:00034a30       ?flex1@?$path_procs_t@Ucff2_path_procs_path_t@@U?$cff2_cs_interp_env_t@Unumber_t@CFF@@@CFF@@Ucff2_path_param_t@@@CFF@@SAXAAU?$cff2_cs_interp_env_t@Unumber_t@CFF@@@2@AAUcff2_path_param_t@@@Z 10035a30 f i hb-ot-cff2-table.obj
 0001:00034e30       ?flex@?$path_procs_t@Ucff2_path_procs_extents_t@@U?$cff2_cs_interp_env_t@Unumber_t@CFF@@@CFF@@Ucff2_extents_param_t@@@CFF@@SAXAAU?$cff2_cs_interp_env_t@Unumber_t@CFF@@@2@AAUcff2_extents_param_t@@@Z 10035e30 f i hb-ot-cff2-table.obj
 0001:00035160       ?flex@?$path_procs_t@Ucff2_path_procs_path_t@@U?$cff2_cs_interp_env_t@Unumber_t@CFF@@@CFF@@Ucff2_path_param_t@@@CFF@@SAXAAU?$cff2_cs_interp_env_t@Unumber_t@CFF@@@2@AAUcff2_path_param_t@@@Z 10036160 f i hb-ot-cff2-table.obj
 0001:000354d0       ?process_post_path@?$cs_opset_t@Unumber_t@CFF@@Ucff2_cs_opset_path_t@@U?$cff2_cs_interp_env_t@Unumber_t@CFF@@@2@Ucff2_path_param_t@@Ucff2_path_procs_path_t@@@CFF@@SAXIAAU?$cff2_cs_interp_env_t@Unumber_t@CFF@@@2@AAUcff2_path_param_t@@@Z 100364d0 f i hb-ot-cff2-table.obj
 0001:000354d0       ?flush_args_and_op@?$cs_opset_t@Unumber_t@CFF@@Ucff2_cs_opset_path_t@@U?$cff2_cs_interp_env_t@Unumber_t@CFF@@@2@Ucff2_path_param_t@@Ucff2_path_procs_path_t@@@CFF@@SAXIAAU?$cff2_cs_interp_env_t@Unumber_t@CFF@@@2@AAUcff2_path_param_t@@@Z 100364d0 f i hb-ot-cff2-table.obj
 0001:000354d0       ?process_post_path@?$cs_opset_t@Unumber_t@CFF@@Ucff2_cs_opset_extents_t@@U?$cff2_cs_interp_env_t@Unumber_t@CFF@@@2@Ucff2_extents_param_t@@Ucff2_path_procs_extents_t@@@CFF@@SAXIAAU?$cff2_cs_interp_env_t@Unumber_t@CFF@@@2@AAUcff2_extents_param_t@@@Z 100364d0 f i hb-ot-cff2-table.obj
 0001:000354d0       ?flush_args_and_op@?$cs_opset_t@Unumber_t@CFF@@Ucff2_cs_opset_extents_t@@U?$cff2_cs_interp_env_t@Unumber_t@CFF@@@2@Ucff2_extents_param_t@@Ucff2_path_procs_extents_t@@@CFF@@SAXIAAU?$cff2_cs_interp_env_t@Unumber_t@CFF@@@2@AAUcff2_extents_param_t@@@Z 100364d0 f i hb-ot-cff2-table.obj
 0001:000354f0       ?get_extents@accelerator_t@cff2@OT@@QBE_NPAUhb_font_t@@IPAUhb_glyph_extents_t@@@Z 100364f0 f   hb-ot-cff2-table.obj
 0001:000359c0       ?get_fd@CFF2FDSelect@CFF@@QBEII@Z 100369c0 f i hb-ot-cff2-table.obj
 0001:00035bf0       ?get_path@accelerator_t@cff2@OT@@QBE_NPAUhb_font_t@@IAAUhb_draw_session_t@@@Z 10036bf0 f   hb-ot-cff2-table.obj
 0001:00035d50       ?get_region_scalars@VarData@OT@@QBEXPBHIABUVarRegionList@2@PAMI@Z 10036d50 f i hb-ot-cff2-table.obj
 0001:00035f20       ?hflex1@?$path_procs_t@Ucff2_path_procs_extents_t@@U?$cff2_cs_interp_env_t@Unumber_t@CFF@@@CFF@@Ucff2_extents_param_t@@@CFF@@SAXAAU?$cff2_cs_interp_env_t@Unumber_t@CFF@@@2@AAUcff2_extents_param_t@@@Z 10036f20 f i hb-ot-cff2-table.obj
 0001:000361b0       ?hflex1@?$path_procs_t@Ucff2_path_procs_path_t@@U?$cff2_cs_interp_env_t@Unumber_t@CFF@@@CFF@@Ucff2_path_param_t@@@CFF@@SAXAAU?$cff2_cs_interp_env_t@Unumber_t@CFF@@@2@AAUcff2_path_param_t@@@Z 100371b0 f i hb-ot-cff2-table.obj
 0001:00036460       ?hflex@?$path_procs_t@Ucff2_path_procs_extents_t@@U?$cff2_cs_interp_env_t@Unumber_t@CFF@@@CFF@@Ucff2_extents_param_t@@@CFF@@SAXAAU?$cff2_cs_interp_env_t@Unumber_t@CFF@@@2@AAUcff2_extents_param_t@@@Z 10037460 f i hb-ot-cff2-table.obj
 0001:00036690       ?hflex@?$path_procs_t@Ucff2_path_procs_path_t@@U?$cff2_cs_interp_env_t@Unumber_t@CFF@@@CFF@@Ucff2_path_param_t@@@CFF@@SAXAAU?$cff2_cs_interp_env_t@Unumber_t@CFF@@@2@AAUcff2_path_param_t@@@Z 10037690 f i hb-ot-cff2-table.obj
 0001:000368d0       ?hhcurveto@?$path_procs_t@Ucff2_path_procs_extents_t@@U?$cff2_cs_interp_env_t@Unumber_t@CFF@@@CFF@@Ucff2_extents_param_t@@@CFF@@SAXAAU?$cff2_cs_interp_env_t@Unumber_t@CFF@@@2@AAUcff2_extents_param_t@@@Z 100378d0 f i hb-ot-cff2-table.obj
 0001:00036c40       ?hhcurveto@?$path_procs_t@Ucff2_path_procs_path_t@@U?$cff2_cs_interp_env_t@Unumber_t@CFF@@@CFF@@Ucff2_path_param_t@@@CFF@@SAXAAU?$cff2_cs_interp_env_t@Unumber_t@CFF@@@2@AAUcff2_path_param_t@@@Z 10037c40 f i hb-ot-cff2-table.obj
 0001:00036df0       ?hlineto@?$path_procs_t@Ucff2_path_procs_extents_t@@U?$cff2_cs_interp_env_t@Unumber_t@CFF@@@CFF@@Ucff2_extents_param_t@@@CFF@@SAXAAU?$cff2_cs_interp_env_t@Unumber_t@CFF@@@2@AAUcff2_extents_param_t@@@Z 10037df0 f i hb-ot-cff2-table.obj
 0001:00037170       ?hlineto@?$path_procs_t@Ucff2_path_procs_path_t@@U?$cff2_cs_interp_env_t@Unumber_t@CFF@@@CFF@@Ucff2_path_param_t@@@CFF@@SAXAAU?$cff2_cs_interp_env_t@Unumber_t@CFF@@@2@AAUcff2_path_param_t@@@Z 10038170 f i hb-ot-cff2-table.obj
 0001:000375a0       ?hvcurveto@?$path_procs_t@Ucff2_path_procs_extents_t@@U?$cff2_cs_interp_env_t@Unumber_t@CFF@@@CFF@@Ucff2_extents_param_t@@@CFF@@SAXAAU?$cff2_cs_interp_env_t@Unumber_t@CFF@@@2@AAUcff2_extents_param_t@@@Z 100385a0 f i hb-ot-cff2-table.obj
 0001:00038350       ?hvcurveto@?$path_procs_t@Ucff2_path_procs_path_t@@U?$cff2_cs_interp_env_t@Unumber_t@CFF@@@CFF@@Ucff2_path_param_t@@@CFF@@SAXAAU?$cff2_cs_interp_env_t@Unumber_t@CFF@@@2@AAUcff2_path_param_t@@@Z 10039350 f i hb-ot-cff2-table.obj
 0001:00038a50       ?in_error@?$cs_interp_env_t@Unumber_t@CFF@@U?$Subrs@U?$IntType@I$03@OT@@@2@@CFF@@QBE_NXZ 10039a50 f i hb-ot-cff2-table.obj
 0001:00038a70       ?line@cff2_path_procs_extents_t@@SAXAAU?$cff2_cs_interp_env_t@Unumber_t@CFF@@@CFF@@AAUcff2_extents_param_t@@ABUpoint_t@3@@Z 10039a70 f i hb-ot-cff2-table.obj
 0001:00038bb0       ?line@cff2_path_procs_path_t@@SAXAAU?$cff2_cs_interp_env_t@Unumber_t@CFF@@@CFF@@AAUcff2_path_param_t@@ABUpoint_t@3@@Z 10039bb0 f i hb-ot-cff2-table.obj
 0001:00038d30       ?move_to@cff2_path_param_t@@QAEXABUpoint_t@CFF@@@Z 10039d30 f i hb-ot-cff2-table.obj
 0001:00038e20       ?offset_at@?$CFFIndex@U?$IntType@I$03@OT@@@CFF@@ABEII@Z 10039e20 f i hb-ot-cff2-table.obj
 0001:00038ec0       ?pop_uint@?$arg_stack_t@Unumber_t@CFF@@@CFF@@QAEIXZ 10039ec0 f i hb-ot-cff2-table.obj
 0001:00038f00       ?process_blend@?$cff2_cs_interp_env_t@Unumber_t@CFF@@@CFF@@QAEXXZ 10039f00 f i hb-ot-cff2-table.obj
 0001:00039190       ?process_op@?$cff2_cs_opset_t@Ucff2_cs_opset_extents_t@@Ucff2_extents_param_t@@Unumber_t@CFF@@Ucff2_path_procs_extents_t@@@CFF@@SAXIAAU?$cff2_cs_interp_env_t@Unumber_t@CFF@@@2@AAUcff2_extents_param_t@@@Z 1003a190 f i hb-ot-cff2-table.obj
 0001:00039380       ?process_op@?$cff2_cs_opset_t@Ucff2_cs_opset_path_t@@Ucff2_path_param_t@@Unumber_t@CFF@@Ucff2_path_procs_path_t@@@CFF@@SAXIAAU?$cff2_cs_interp_env_t@Unumber_t@CFF@@@2@AAUcff2_path_param_t@@@Z 1003a380 f i hb-ot-cff2-table.obj
 0001:00039570       ?process_op@?$cs_opset_t@Unumber_t@CFF@@Ucff2_cs_opset_extents_t@@U?$cff2_cs_interp_env_t@Unumber_t@CFF@@@2@Ucff2_extents_param_t@@Ucff2_path_procs_extents_t@@@CFF@@SAXIAAU?$cff2_cs_interp_env_t@Unumber_t@CFF@@@2@AAUcff2_extents_param_t@@@Z 1003a570 f i hb-ot-cff2-table.obj
 0001:00039ad0       ?process_op@?$cs_opset_t@Unumber_t@CFF@@Ucff2_cs_opset_path_t@@U?$cff2_cs_interp_env_t@Unumber_t@CFF@@@2@Ucff2_path_param_t@@Ucff2_path_procs_path_t@@@CFF@@SAXIAAU?$cff2_cs_interp_env_t@Unumber_t@CFF@@@2@AAUcff2_path_param_t@@@Z 1003aad0 f i hb-ot-cff2-table.obj
 0001:0003a0a0       ?process_post_move@?$cs_opset_t@Unumber_t@CFF@@Ucff2_cs_opset_path_t@@U?$cff2_cs_interp_env_t@Unumber_t@CFF@@@2@Ucff2_path_param_t@@Ucff2_path_procs_path_t@@@CFF@@SAXIAAU?$cff2_cs_interp_env_t@Unumber_t@CFF@@@2@AAUcff2_path_param_t@@@Z 1003b0a0 f i hb-ot-cff2-table.obj
 0001:0003a0a0       ?process_post_move@?$cs_opset_t@Unumber_t@CFF@@Ucff2_cs_opset_extents_t@@U?$cff2_cs_interp_env_t@Unumber_t@CFF@@@2@Ucff2_extents_param_t@@Ucff2_path_procs_extents_t@@@CFF@@SAXIAAU?$cff2_cs_interp_env_t@Unumber_t@CFF@@@2@AAUcff2_extents_param_t@@@Z 1003b0a0 f i hb-ot-cff2-table.obj
 0001:0003a100       ?process_vsindex@?$cff2_cs_interp_env_t@Unumber_t@CFF@@@CFF@@QAEXXZ 1003b100 f i hb-ot-cff2-table.obj
 0001:0003a170       ?rcurveline@?$path_procs_t@Ucff2_path_procs_extents_t@@U?$cff2_cs_interp_env_t@Unumber_t@CFF@@@CFF@@Ucff2_extents_param_t@@@CFF@@SAXAAU?$cff2_cs_interp_env_t@Unumber_t@CFF@@@2@AAUcff2_extents_param_t@@@Z 1003b170 f i hb-ot-cff2-table.obj
 0001:0003a5c0       ?rcurveline@?$path_procs_t@Ucff2_path_procs_path_t@@U?$cff2_cs_interp_env_t@Unumber_t@CFF@@@CFF@@Ucff2_path_param_t@@@CFF@@SAXAAU?$cff2_cs_interp_env_t@Unumber_t@CFF@@@2@AAUcff2_path_param_t@@@Z 1003b5c0 f i hb-ot-cff2-table.obj
 0001:0003a860       ?rlinecurve@?$path_procs_t@Ucff2_path_procs_extents_t@@U?$cff2_cs_interp_env_t@Unumber_t@CFF@@@CFF@@Ucff2_extents_param_t@@@CFF@@SAXAAU?$cff2_cs_interp_env_t@Unumber_t@CFF@@@2@AAUcff2_extents_param_t@@@Z 1003b860 f i hb-ot-cff2-table.obj
 0001:0003abf0       ?rlinecurve@?$path_procs_t@Ucff2_path_procs_path_t@@U?$cff2_cs_interp_env_t@Unumber_t@CFF@@@CFF@@Ucff2_path_param_t@@@CFF@@SAXAAU?$cff2_cs_interp_env_t@Unumber_t@CFF@@@2@AAUcff2_path_param_t@@@Z 1003bbf0 f i hb-ot-cff2-table.obj
 0001:0003b010       ?rlineto@?$path_procs_t@Ucff2_path_procs_extents_t@@U?$cff2_cs_interp_env_t@Unumber_t@CFF@@@CFF@@Ucff2_extents_param_t@@@CFF@@SAXAAU?$cff2_cs_interp_env_t@Unumber_t@CFF@@@2@AAUcff2_extents_param_t@@@Z 1003c010 f i hb-ot-cff2-table.obj
 0001:0003b210       ?rlineto@?$path_procs_t@Ucff2_path_procs_path_t@@U?$cff2_cs_interp_env_t@Unumber_t@CFF@@@CFF@@Ucff2_path_param_t@@@CFF@@SAXAAU?$cff2_cs_interp_env_t@Unumber_t@CFF@@@2@AAUcff2_path_param_t@@@Z 1003c210 f i hb-ot-cff2-table.obj
 0001:0003b470       ?rrcurveto@?$path_procs_t@Ucff2_path_procs_extents_t@@U?$cff2_cs_interp_env_t@Unumber_t@CFF@@@CFF@@Ucff2_extents_param_t@@@CFF@@SAXAAU?$cff2_cs_interp_env_t@Unumber_t@CFF@@@2@AAUcff2_extents_param_t@@@Z 1003c470 f i hb-ot-cff2-table.obj
 0001:0003b810       ?rrcurveto@?$path_procs_t@Ucff2_path_procs_path_t@@U?$cff2_cs_interp_env_t@Unumber_t@CFF@@@CFF@@Ucff2_path_param_t@@@CFF@@SAXAAU?$cff2_cs_interp_env_t@Unumber_t@CFF@@@2@AAUcff2_path_param_t@@@Z 1003c810 f i hb-ot-cff2-table.obj
 0001:0003ba00       ?vhcurveto@?$path_procs_t@Ucff2_path_procs_extents_t@@U?$cff2_cs_interp_env_t@Unumber_t@CFF@@@CFF@@Ucff2_extents_param_t@@@CFF@@SAXAAU?$cff2_cs_interp_env_t@Unumber_t@CFF@@@2@AAUcff2_extents_param_t@@@Z 1003ca00 f i hb-ot-cff2-table.obj
 0001:0003c7c0       ?vhcurveto@?$path_procs_t@Ucff2_path_procs_path_t@@U?$cff2_cs_interp_env_t@Unumber_t@CFF@@@CFF@@Ucff2_path_param_t@@@CFF@@SAXAAU?$cff2_cs_interp_env_t@Unumber_t@CFF@@@2@AAUcff2_path_param_t@@@Z 1003d7c0 f i hb-ot-cff2-table.obj
 0001:0003ceb0       ?vlineto@?$path_procs_t@Ucff2_path_procs_extents_t@@U?$cff2_cs_interp_env_t@Unumber_t@CFF@@@CFF@@Ucff2_extents_param_t@@@CFF@@SAXAAU?$cff2_cs_interp_env_t@Unumber_t@CFF@@@2@AAUcff2_extents_param_t@@@Z 1003deb0 f i hb-ot-cff2-table.obj
 0001:0003d230       ?vlineto@?$path_procs_t@Ucff2_path_procs_path_t@@U?$cff2_cs_interp_env_t@Unumber_t@CFF@@@CFF@@Ucff2_path_param_t@@@CFF@@SAXAAU?$cff2_cs_interp_env_t@Unumber_t@CFF@@@2@AAUcff2_path_param_t@@@Z 1003e230 f i hb-ot-cff2-table.obj
 0001:0003d660       ?vvcurveto@?$path_procs_t@Ucff2_path_procs_extents_t@@U?$cff2_cs_interp_env_t@Unumber_t@CFF@@@CFF@@Ucff2_extents_param_t@@@CFF@@SAXAAU?$cff2_cs_interp_env_t@Unumber_t@CFF@@@2@AAUcff2_extents_param_t@@@Z 1003e660 f i hb-ot-cff2-table.obj
 0001:0003d9d0       ?vvcurveto@?$path_procs_t@Ucff2_path_procs_path_t@@U?$cff2_cs_interp_env_t@Unumber_t@CFF@@@CFF@@Ucff2_path_param_t@@@CFF@@SAXAAU?$cff2_cs_interp_env_t@Unumber_t@CFF@@@2@AAUcff2_path_param_t@@@Z 1003e9d0 f i hb-ot-cff2-table.obj
 0001:0003dba0       ??$_dispatch@UIndexSubtableRecord@OT@@PBUIndexSubtableArray@2@@hb_sanitize_context_t@@AAE_NABUIndexSubtableRecord@OT@@U?$hb_priority@$00@@$$QAPBUIndexSubtableArray@2@@Z 1003eba0 f i hb-ot-color.obj
 0001:0003dcc0       ??$dispatch@U?$ColorLine@UNoVariable@OT@@@OT@@$$V@hb_sanitize_context_t@@QAE_NABU?$ColorLine@UNoVariable@OT@@@OT@@@Z 1003ecc0 f i hb-ot-color.obj
 0001:0003dd40       ??$dispatch@U?$ColorLine@UVariable@OT@@@OT@@$$V@hb_sanitize_context_t@@QAE_NABU?$ColorLine@UVariable@OT@@@OT@@@Z 1003ed40 f i hb-ot-color.obj
 0001:0003ddc0       ??$dispatch@U?$NoVariable@UAffine2x3@OT@@@OT@@$$V@hb_sanitize_context_t@@QAE_NABU?$NoVariable@UAffine2x3@OT@@@OT@@@Z 1003edc0 f i hb-ot-color.obj
 0001:0003de40       ??$dispatch@U?$Variable@UAffine2x3@OT@@@OT@@$$V@hb_sanitize_context_t@@QAE_NABU?$Variable@UAffine2x3@OT@@@OT@@@Z 1003ee40 f i hb-ot-color.obj
 0001:0003dec0       ??$dispatch@UClipBox@OT@@$$V@hb_sanitize_context_t@@QAE_NABUClipBox@OT@@@Z 1003eec0 f i hb-ot-color.obj
 0001:0003df70       ??$dispatch@UIndexSubtableArray@OT@@ABU?$IntType@I$03@2@@hb_sanitize_context_t@@QAE_NABUIndexSubtableArray@OT@@ABU?$IntType@I$03@2@@Z 1003ef70 f i hb-ot-color.obj
 0001:0003dff0       ??$dispatch@ULayerList@OT@@$$V@hb_sanitize_context_t@@QAE_NABULayerList@OT@@@Z 1003eff0 f i hb-ot-color.obj
 0001:0003e0d0       ??$dispatch@USBIXStrike@OT@@$$V@hb_sanitize_context_t@@QAE_NABUSBIXStrike@OT@@@Z 1003f0d0 f i hb-ot-color.obj
 0001:0003e1c0       ??$dispatch@Uhb_sanitize_context_t@@$$V@Paint@OT@@QBE_NPAUhb_sanitize_context_t@@@Z 1003f1c0 f i hb-ot-color.obj
 0001:0003ec50       ??$sanitize@$$V@Paint@OT@@QBE_NPAUhb_sanitize_context_t@@@Z 1003fc50 f i hb-ot-color.obj
 0001:0003ec80       ??$sanitize_blob@UCBDT@OT@@@hb_sanitize_context_t@@QAEPAUhb_blob_t@@PAU1@@Z 1003fc80 f i hb-ot-color.obj
 0001:0003ee70       ??$sanitize_blob@UCBLC@OT@@@hb_sanitize_context_t@@QAEPAUhb_blob_t@@PAU1@@Z 1003fe70 f i hb-ot-color.obj
 0001:0003f000       ??$sanitize_blob@UCOLR@OT@@@hb_sanitize_context_t@@QAEPAUhb_blob_t@@PAU1@@Z 10040000 f i hb-ot-color.obj
 0001:0003f190       ??$sanitize_blob@UCPAL@OT@@@hb_sanitize_context_t@@QAEPAUhb_blob_t@@PAU1@@Z 10040190 f i hb-ot-color.obj
 0001:0003f410       ??$sanitize_blob@USVG@OT@@@hb_sanitize_context_t@@QAEPAUhb_blob_t@@PAU1@@Z 10040410 f i hb-ot-color.obj
 0001:0003f6a0       ??$sanitize_blob@Usbix@OT@@@hb_sanitize_context_t@@QAEPAUhb_blob_t@@PAU1@@Z 100406a0 f i hb-ot-color.obj
 0001:0003f950       ??C?$hb_lazy_loader_t@UCOLR@OT@@U?$hb_table_lazy_loader_t@UCOLR@OT@@$0CD@$00@@Uhb_face_t@@$0CD@Uhb_blob_t@@@@QBEPBUCOLR@OT@@XZ 10040950 f i hb-ot-color.obj
 0001:0003fa90       ??C?$hb_lazy_loader_t@UCPAL@OT@@U?$hb_table_lazy_loader_t@UCPAL@OT@@$0CE@$00@@Uhb_face_t@@$0CE@Uhb_blob_t@@@@QBEPBUCPAL@OT@@XZ 10040a90 f i hb-ot-color.obj
 0001:0003fbb0       ??C?$hb_lazy_loader_t@Usbix_accelerator_t@OT@@U?$hb_face_lazy_loader_t@Usbix_accelerator_t@OT@@$0CG@@@Uhb_face_t@@$0CG@U12@@@QBEPBUsbix_accelerator_t@OT@@XZ 10040bb0 f i hb-ot-color.obj
 0001:0003fd30       ?choose_strike@CBLC@OT@@IBEABUBitmapSizeTable@2@PAUhb_font_t@@@Z 10040d30 f i hb-ot-color.obj
 0001:0003fe50       ?choose_strike@accelerator_t@sbix@OT@@ABEABUSBIXStrike@3@PAUhb_font_t@@@Z 10040e50 f i hb-ot-color.obj
 0001:00040000       ?find_table@BitmapSizeTable@OT@@QBEPBUIndexSubtableRecord@2@IPBXPAPBX@Z 10041000 f i hb-ot-color.obj
 0001:00040080       ?find_table@IndexSubtableArray@OT@@QBEPBUIndexSubtableRecord@2@II@Z 10041080 f i hb-ot-color.obj
 0001:000400e0       ?get_base_glyph_paint@COLR@OT@@QBEPBUPaint@2@I@Z 100410e0 f i hb-ot-color.obj
 0001:00040210       ?get_glyph_blob@SBIXStrike@OT@@QBEPAUhb_blob_t@@IPAU3@IPAH1IPAI@Z 10041210 f i hb-ot-color.obj
 0001:00040400       ?get_image_data@IndexSubtable@OT@@QBE_NIPAI00@Z 10041400 f i hb-ot-color.obj
 0001:000405a0       ?get_image_data@IndexSubtableRecord@OT@@QBE_NIPBXPAI11@Z 100415a0 f i hb-ot-color.obj
 0001:00040620       ?get_palette_colors@CPAL@OT@@QBEIIIPAI0@Z 10041620 f i hb-ot-color.obj
 0001:000407a0       ?get_stored@?$hb_lazy_loader_t@UCBDT_accelerator_t@OT@@U?$hb_face_lazy_loader_t@UCBDT_accelerator_t@OT@@$0CF@@@Uhb_face_t@@$0CF@U12@@@QBEPAUCBDT_accelerator_t@OT@@XZ 100417a0 f i hb-ot-color.obj
 0001:000409d0       ?get_strike@sbix@OT@@QBEABUSBIXStrike@2@I@Z 100419d0 f i hb-ot-color.obj
 0001:00040a70       ?neuter@?$OffsetTo@U?$NoVariable@UAffine2x3@OT@@@OT@@U?$IntType@I$02@2@$00@OT@@QBE_NPAUhb_sanitize_context_t@@@Z 10041a70 f i hb-ot-color.obj
 0001:00040a70       ?neuter@?$OffsetTo@U?$ColorLine@UNoVariable@OT@@@OT@@U?$IntType@I$02@2@$00@OT@@QBE_NPAUhb_sanitize_context_t@@@Z 10041a70 f i hb-ot-color.obj
 0001:00040a70       ?neuter@?$OffsetTo@U?$ColorLine@UVariable@OT@@@OT@@U?$IntType@I$02@2@$00@OT@@QBE_NPAUhb_sanitize_context_t@@@Z 10041a70 f i hb-ot-color.obj
 0001:00040a70       ?neuter@?$OffsetTo@UClipBox@OT@@U?$IntType@I$02@2@$00@OT@@QBE_NPAUhb_sanitize_context_t@@@Z 10041a70 f i hb-ot-color.obj
 0001:00040a70       ?neuter@?$OffsetTo@U?$Variable@UAffine2x3@OT@@@OT@@U?$IntType@I$02@2@$00@OT@@QBE_NPAUhb_sanitize_context_t@@@Z 10041a70 f i hb-ot-color.obj
 0001:00040a70       ?neuter@?$OffsetTo@UPaint@OT@@U?$IntType@I$02@2@$00@OT@@QBE_NPAUhb_sanitize_context_t@@@Z 10041a70 f i hb-ot-color.obj
 0001:00040ab0       ?reference_blob_for_glyph@accelerator_t@SVG@OT@@QBEPAUhb_blob_t@@I@Z 10041ab0 f i hb-ot-color.obj
 0001:00040c00       ?reference_png@accelerator_t@CBDT@OT@@QBEPAUhb_blob_t@@PAUhb_font_t@@I@Z 10041c00 f i hb-ot-color.obj
 0001:00040da0       ?sanitize@?$NoVariable@U?$PaintLinearGradient@UNoVariable@OT@@@OT@@@OT@@QBE_NPAUhb_sanitize_context_t@@@Z 10041da0 f i hb-ot-color.obj
 0001:00040da0       ?sanitize@?$NoVariable@U?$PaintRadialGradient@UNoVariable@OT@@@OT@@@OT@@QBE_NPAUhb_sanitize_context_t@@@Z 10041da0 f i hb-ot-color.obj
 0001:00040eb0       ?sanitize@?$NoVariable@U?$PaintSweepGradient@UNoVariable@OT@@@OT@@@OT@@QBE_NPAUhb_sanitize_context_t@@@Z 10041eb0 f i hb-ot-color.obj
 0001:00040fc0       ?sanitize@?$Variable@U?$PaintLinearGradient@UVariable@OT@@@OT@@@OT@@QBE_NPAUhb_sanitize_context_t@@@Z 10041fc0 f i hb-ot-color.obj
 0001:00040fc0       ?sanitize@?$Variable@U?$PaintRadialGradient@UVariable@OT@@@OT@@@OT@@QBE_NPAUhb_sanitize_context_t@@@Z 10041fc0 f i hb-ot-color.obj
 0001:000410d0       ?sanitize@?$Variable@U?$PaintSweepGradient@UVariable@OT@@@OT@@@OT@@QBE_NPAUhb_sanitize_context_t@@@Z 100420d0 f i hb-ot-color.obj
 0001:000411e0       ?sanitize@Affine2x3@OT@@QBE_NPAUhb_sanitize_context_t@@@Z 100421e0 f i hb-ot-color.obj
 0001:00041250       ?sanitize@BaseGlyphList@OT@@QBE_NPAUhb_sanitize_context_t@@@Z 10042250 f i hb-ot-color.obj
 0001:000413b0       ?sanitize@CBDT@OT@@QBE_NPAUhb_sanitize_context_t@@@Z 100423b0 f i hb-ot-color.obj
 0001:00041440       ?sanitize@CBLC@OT@@QBE_NPAUhb_sanitize_context_t@@@Z 10042440 f i hb-ot-color.obj
 0001:00041600       ?sanitize@COLR@OT@@QBE_NPAUhb_sanitize_context_t@@@Z 10042600 f i hb-ot-color.obj
 0001:00041900       ?sanitize@CPAL@OT@@QBE_NPAUhb_sanitize_context_t@@@Z 10042900 f i hb-ot-color.obj
 0001:00041a20       ?sanitize@CPALV1Tail@OT@@QBE_NPAUhb_sanitize_context_t@@PBXII@Z 10042a20 f i hb-ot-color.obj
 0001:00041b30       ?sanitize@ClipBoxFormat1@OT@@QBE_NPAUhb_sanitize_context_t@@@Z 10042b30 f i hb-ot-color.obj
 0001:00041ba0       ?sanitize@ClipList@OT@@QBE_NPAUhb_sanitize_context_t@@@Z 10042ba0 f i hb-ot-color.obj
 0001:00041d20       ?sanitize@IndexSubtable@OT@@QBE_NPAUhb_sanitize_context_t@@I@Z 10042d20 f i hb-ot-color.obj
 0001:00041e90       ?sanitize@PaintComposite@OT@@QBE_NPAUhb_sanitize_context_t@@@Z 10042e90 f i hb-ot-color.obj
 0001:00041fb0       ?sanitize@PaintRotate@OT@@QBE_NPAUhb_sanitize_context_t@@@Z 10042fb0 f i hb-ot-color.obj
 0001:00041fb0       ?sanitize@PaintScaleUniform@OT@@QBE_NPAUhb_sanitize_context_t@@@Z 10042fb0 f i hb-ot-color.obj
 0001:00042070       ?sanitize@PaintRotateAroundCenter@OT@@QBE_NPAUhb_sanitize_context_t@@@Z 10043070 f i hb-ot-color.obj
 0001:00042070       ?sanitize@PaintScaleUniformAroundCenter@OT@@QBE_NPAUhb_sanitize_context_t@@@Z 10043070 f i hb-ot-color.obj
 0001:00042130       ?sanitize@PaintSkew@OT@@QBE_NPAUhb_sanitize_context_t@@@Z 10043130 f i hb-ot-color.obj
 0001:00042130       ?sanitize@PaintScale@OT@@QBE_NPAUhb_sanitize_context_t@@@Z 10043130 f i hb-ot-color.obj
 0001:00042130       ?sanitize@PaintTranslate@OT@@QBE_NPAUhb_sanitize_context_t@@@Z 10043130 f i hb-ot-color.obj
 0001:000421f0       ?sanitize@PaintScaleAroundCenter@OT@@QBE_NPAUhb_sanitize_context_t@@@Z 100431f0 f i hb-ot-color.obj
 0001:000421f0       ?sanitize@PaintSkewAroundCenter@OT@@QBE_NPAUhb_sanitize_context_t@@@Z 100431f0 f i hb-ot-color.obj
 0001:000422b0       ?sanitize@PaintSolid@OT@@QBE_NPAUhb_sanitize_context_t@@@Z 100432b0 f i hb-ot-color.obj
 0001:00042320       ?sanitize@SVG@OT@@QBE_NPAUhb_sanitize_context_t@@@Z 10043320 f i hb-ot-color.obj
 0001:00042450       ?sanitize@sbix@OT@@QBE_NPAUhb_sanitize_context_t@@@Z 10043450 f i hb-ot-color.obj
 0001:00042590       ?sanitize_shallow@?$ArrayOf@U?$Variable@UColorStop@OT@@@OT@@U?$IntType@G$01@2@@OT@@QBE_NPAUhb_sanitize_context_t@@@Z 10043590 f i hb-ot-color.obj
 0001:00042640       ?sanitize_shallow@?$ArrayOf@UBaseGlyphPaintRecord@OT@@U?$IntType@I$03@2@@OT@@QBE_NPAUhb_sanitize_context_t@@@Z 10043640 f i hb-ot-color.obj
 0001:00042640       ?sanitize_shallow@?$ArrayOf@U?$FDSelect3_4_Range@U?$IntType@I$03@OT@@U?$IntType@G$01@2@@CFF@@U?$IntType@I$03@OT@@@OT@@QBE_NPAUhb_sanitize_context_t@@@Z 10043640 f i hb-ot-font.obj
 0001:00042700       ?sanitize_shallow@?$ArrayOf@UBitmapSizeTable@OT@@U?$IntType@I$03@2@@OT@@QBE_NPAUhb_sanitize_context_t@@@Z 10043700 f i hb-ot-color.obj
 0001:000427c0       ?sanitize_shallow@?$ArrayOf@UClipRecord@OT@@U?$IntType@I$03@2@@OT@@QBE_NPAUhb_sanitize_context_t@@@Z 100437c0 f i hb-ot-color.obj
 0001:00042880       ?sanitize_shallow@?$OffsetTo@UPaint@OT@@U?$IntType@I$02@2@$00@OT@@QBE_NPAUhb_sanitize_context_t@@PBX@Z 10043880 f i hb-ot-color.obj
 0001:00042880       ?sanitize_shallow@?$OffsetTo@U?$Variable@UAffine2x3@OT@@@OT@@U?$IntType@I$02@2@$00@OT@@QBE_NPAUhb_sanitize_context_t@@PBX@Z 10043880 f i hb-ot-color.obj
 0001:00042880       ?sanitize_shallow@?$OffsetTo@U?$ColorLine@UVariable@OT@@@OT@@U?$IntType@I$02@2@$00@OT@@QBE_NPAUhb_sanitize_context_t@@PBX@Z 10043880 f i hb-ot-color.obj
 0001:00042880       ?sanitize_shallow@?$OffsetTo@U?$ColorLine@UNoVariable@OT@@@OT@@U?$IntType@I$02@2@$00@OT@@QBE_NPAUhb_sanitize_context_t@@PBX@Z 10043880 f i hb-ot-color.obj
 0001:00042880       ?sanitize_shallow@?$OffsetTo@U?$NoVariable@UAffine2x3@OT@@@OT@@U?$IntType@I$02@2@$00@OT@@QBE_NPAUhb_sanitize_context_t@@PBX@Z 10043880 f i hb-ot-color.obj
 0001:00042880       ?sanitize_shallow@?$OffsetTo@UClipBox@OT@@U?$IntType@I$02@2@$00@OT@@QBE_NPAUhb_sanitize_context_t@@PBX@Z 10043880 f i hb-ot-color.obj
 0001:00042910       ?sub_array@?$hb_array_t@$$CBU?$IntType@I$03@OT@@@@QBE?AU1@IPAI@Z 10043910 f i hb-ot-color.obj
 0001:00042970       ?v1@CPAL@OT@@ABEABUCPALV1Tail@2@XZ 10043970 f i hb-ot-color.obj
 0001:000429b0       _hb_ot_color_palette_get_colors 100439b0 f   hb-ot-color.obj
 0001:000429e0       ??1?$accelerator_templ_t@Ucff1_private_dict_opset_t@CFF@@U?$cff1_private_dict_values_base_t@Udict_val_t@CFF@@@2@@cff1@OT@@QAE@XZ 100439e0 f i hb-ot-face.obj
 0001:00042aa0       ??1?$accelerator_templ_t@Ucff2_private_dict_opset_t@CFF@@U?$cff2_private_dict_values_base_t@Udict_val_t@CFF@@@2@@cff2@OT@@QAE@XZ 10043aa0 f i hb-ot-face.obj
 0001:00042b50       ?_fini@?$accelerator_templ_t@Ucff1_private_dict_opset_t@CFF@@U?$cff1_private_dict_values_base_t@Udict_val_t@CFF@@@2@@cff1@OT@@QAEXXZ 10043b50 f i hb-ot-face.obj
 0001:00042c50       ?_fini@?$accelerator_templ_t@Ucff2_private_dict_opset_t@CFF@@U?$cff2_private_dict_values_base_t@Udict_val_t@CFF@@@2@@cff2@OT@@QAEXXZ 10043c50 f i hb-ot-face.obj
 0001:00042d50       ?fini@hb_ot_face_t@@QAEXXZ 10043d50 f   hb-ot-face.obj
 0001:00043400       ?init0@hb_ot_face_t@@QAEXPAUhb_face_t@@@Z 10044400 f   hb-ot-face.obj
 0001:00043410       ?shrink_vector@?$hb_vector_t@U?$cff1_private_dict_values_base_t@Udict_val_t@CFF@@@CFF@@$0A@@@QAEXI@Z 10044410 f i hb-ot-face.obj
 0001:00043490       ?shrink_vector@?$hb_vector_t@Ucff2_font_dict_values_t@CFF@@$0A@@@QAEXI@Z 10044490 f i hb-ot-face.obj
 0001:00043490       ?shrink_vector@?$hb_vector_t@U?$cff2_private_dict_values_base_t@Udict_val_t@CFF@@@CFF@@$0A@@@QAEXI@Z 10044490 f i hb-ot-face.obj
 0001:00043510       ?shrink_vector@?$hb_vector_t@Ucff1_font_dict_values_t@CFF@@$0A@@@QAEXI@Z 10044510 f i hb-ot-face.obj
 0001:000435b0       ??$bfind@I@?$hb_sorted_array_t@$$CBUUnicodeValueRange@OT@@@@QBE_NABIPAIW4hb_not_found_t@@I@Z 100445b0 f i hb-ot-font.obj
 0001:00043650       ??$check_array@U?$IntType@E$00@OT@@@hb_sanitize_context_t@@QBE_NPBU?$IntType@E$00@OT@@II@Z 10044650 f i hb-ot-font.obj
 0001:00043690       ??$dispatch@Uhb_paint_context_t@OT@@$$V@Paint@OT@@QBE?AUhb_empty_t@@PAUhb_paint_context_t@1@@Z 10044690 f i hb-ot-font.obj
 0001:00043d30       ??$get_extents_without_var_scaled@Uglyf_accelerator_t@OT@@@GlyphHeader@glyf_impl@OT@@QBE_NPAUhb_font_t@@ABUglyf_accelerator_t@2@IPAUhb_glyph_extents_t@@@Z 10044d30 f i hb-ot-font.obj
 0001:00043f20       ??$get_points@Upath_builder_t@glyf_impl@OT@@@glyf_accelerator_t@OT@@IBE_NPAUhb_font_t@@IUpath_builder_t@glyf_impl@1@@Z 10044f20 f i hb-ot-font.obj
 0001:000457d0       ??$push@Uhb_bounds_t@@@?$hb_vector_t@Uhb_bounds_t@@$0A@@@QAEPAUhb_bounds_t@@$$QAU1@@Z 100467d0 f i hb-ot-font.obj
 0001:00045890       ??$sanitize@Uhb_sanitize_context_t@@@?$hb_array_t@$$CBE@@QBE_NPAUhb_sanitize_context_t@@@Z 10046890 f i hb-ot-font.obj
 0001:00045920       ??$sanitize_blob@UVORG@OT@@@hb_sanitize_context_t@@QAEPAUhb_blob_t@@PAU1@@Z 10046920 f i hb-ot-font.obj
 0001:00045b20       ??$sanitize_blob@Ucff1@OT@@@hb_sanitize_context_t@@QAEPAUhb_blob_t@@PAU1@@Z 10046b20 f i hb-ot-font.obj
 0001:00045cf0       ??$sanitize_blob@Ucff2@OT@@@hb_sanitize_context_t@@QAEPAUhb_blob_t@@PAU1@@Z 10046cf0 f i hb-ot-font.obj
 0001:00045ec0       ??$sanitize_blob@Upost@OT@@@hb_sanitize_context_t@@QAEPAUhb_blob_t@@PAU1@@Z 10046ec0 f i hb-ot-font.obj
 0001:00046500       ??0?$accelerator_templ_t@Ucff1_private_dict_opset_t@CFF@@U?$cff1_private_dict_values_base_t@Udict_val_t@CFF@@@2@@cff1@OT@@QAE@PAUhb_face_t@@@Z 10047500 f i hb-ot-font.obj
 0001:00046ba0       ??0?$accelerator_templ_t@Ucff2_private_dict_opset_t@CFF@@U?$cff2_private_dict_values_base_t@Udict_val_t@CFF@@@2@@cff2@OT@@QAE@PAUhb_face_t@@@Z 10047ba0 f i hb-ot-font.obj
 0001:00047100       ??0accelerator_t@post@OT@@QAE@PAUhb_face_t@@@Z 10048100 f i hb-ot-font.obj
 0001:00047320       ??0cff1_top_dict_interp_env_t@CFF@@QAE@ABU?$hb_array_t@$$CBE@@@Z 10048320 f i hb-ot-font.obj
 0001:00047380       ??0cff2_priv_dict_interp_env_t@CFF@@QAE@ABU?$hb_array_t@$$CBE@@@Z 10048380 f i hb-ot-font.obj
 0001:000473e0       ??0hb_paint_extents_context_t@@QAE@XZ 100483e0 f i hb-ot-font.obj
 0001:000474e0       ??1hb_paint_extents_context_t@@QAE@XZ 100484e0 f i hb-ot-font.obj
 0001:00047570       ??A?$hb_vector_t@U?$cff1_private_dict_values_base_t@Udict_val_t@CFF@@@CFF@@$0A@@@QAEAAU?$cff1_private_dict_values_base_t@Udict_val_t@CFF@@@CFF@@H@Z 10048570 f i hb-ot-font.obj
 0001:000475b0       ??A?$hb_vector_t@U?$cff2_private_dict_values_base_t@Udict_val_t@CFF@@@CFF@@$0A@@@QAEAAU?$cff2_private_dict_values_base_t@Udict_val_t@CFF@@@CFF@@H@Z 100485b0 f i hb-ot-font.obj
 0001:00047600       ??C?$hb_lazy_loader_t@Ucff1_accelerator_t@OT@@U?$hb_face_lazy_loader_t@Ucff1_accelerator_t@OT@@$0BA@@@Uhb_face_t@@$0BA@U12@@@QBEPBUcff1_accelerator_t@OT@@XZ 10048600 f i hb-ot-font.obj
 0001:000476f0       ??C?$hb_lazy_loader_t@Ucff2_accelerator_t@OT@@U?$hb_face_lazy_loader_t@Ucff2_accelerator_t@OT@@$0BB@@@Uhb_face_t@@$0BB@U12@@@QBEPBUcff2_accelerator_t@OT@@XZ 100486f0 f i hb-ot-font.obj
 0001:00047790       ??C?$hb_lazy_loader_t@Upost_accelerator_t@OT@@U?$hb_face_lazy_loader_t@Upost_accelerator_t@OT@@$06@@Uhb_face_t@@$06U12@@@QBEPBUpost_accelerator_t@OT@@XZ 10048790 f i hb-ot-font.obj
 0001:00047870       ??RVarStoreInstancer@OT@@QBEMIG@Z 10048870 f i hb-ot-font.obj
 0001:00047910       ?_cached_get@accelerator_t@cmap@OT@@QBE_NIPAIPAU?$hb_cache_t@$0BF@$0BA@$07$00@@@Z 10048910 f i hb-ot-font.obj
 0001:000479f0       ?add_op@?$parsed_values_t@Uop_str_t@CFF@@@CFF@@QAEXIABUbyte_str_ref_t@2@ABUop_str_t@2@@Z 100489f0 f i hb-ot-font.obj
 0001:000479f0       ?add_op@?$parsed_values_t@Udict_val_t@CFF@@@CFF@@QAEXIABUbyte_str_ref_t@2@ABUdict_val_t@2@@Z 100489f0 f i hb-ot-font.obj
 0001:00047b00       ?alloc@?$hb_vector_t@U?$cff1_private_dict_values_base_t@Udict_val_t@CFF@@@CFF@@$0A@@@QAE_NI_N@Z 10048b00 f i hb-ot-font.obj
 0001:00047cd0       ?alloc@?$hb_vector_t@U?$cff2_private_dict_values_base_t@Udict_val_t@CFF@@@CFF@@$0A@@@QAE_NI_N@Z 10048cd0 f i hb-ot-font.obj
 0001:00047ec0       ?alloc@?$hb_vector_t@Ucff1_font_dict_values_t@CFF@@$0A@@@QAE_NI_N@Z 10048ec0 f i hb-ot-font.obj
 0001:000480b0       ?alloc@?$hb_vector_t@Ucff2_font_dict_values_t@CFF@@$0A@@@QAE_NI_N@Z 100490b0 f i hb-ot-font.obj
 0001:00048290       ?alloc@?$hb_vector_t@Uhb_transform_t@@$0A@@@QAE_NI_N@Z 10049290 f i hb-ot-font.obj
 0001:00048370       ?cmp@gname_t@accelerator_t@cff1@OT@@SAHPBX0@Z 10049370 f i hb-ot-font.obj
 0001:000483b0       ?cmp_gids@accelerator_t@post@OT@@KAHPBX0PAX@Z 100493b0 f i hb-ot-font.obj
 0001:00048410       ?find_glyph_name@accelerator_t@post@OT@@IBE?AU?$hb_array_t@$$CBD@@I@Z 10049410 f i hb-ot-font.obj
 0001:00048530       ?get_advance_delta_unscaled@HVARVVAR@OT@@QBEMIPBHIPAM@Z 10049530 f i hb-ot-font.obj
 0001:000485b0       ?get_base_glyph_record@COLR@OT@@QBEPBUBaseGlyphRecord@2@I@Z 100495b0 f i hb-ot-font.obj
 0001:00048670       ?get_clip@COLR@OT@@QBE_NIPAUhb_glyph_extents_t@@UVarStoreInstancer@2@@Z 10049670 f i hb-ot-font.obj
 0001:000487b0       ?get_clip_box@ClipBoxFormat1@OT@@QBEXAAUClipBoxData@2@ABUVarStoreInstancer@2@@Z 100497b0 f i hb-ot-font.obj
 0001:00048830       ?get_clip_box@ClipBoxFormat2@OT@@QBEXAAUClipBoxData@2@ABUVarStoreInstancer@2@@Z 10049830 f i hb-ot-font.obj
 0001:000489f0       ?get_color@hb_paint_context_t@OT@@QAEIIMPAH@Z 100499f0 f i hb-ot-font.obj
 0001:00048aa0       ?get_color_stop@ColorStop@OT@@QBEXPAUhb_paint_context_t@2@PAUhb_color_stop_t@@IABUVarStoreInstancer@2@@Z 10049aa0 f i hb-ot-font.obj
 0001:00048b60       ?get_delta@VarData@OT@@QBEMIPBHIABUVarRegionList@2@PAM@Z 10049b60 f i hb-ot-font.obj
 0001:00048da0       ?get_delta@VariationStore@OT@@QBEMIPBHIPAM@Z 10049da0 f i hb-ot-font.obj
 0001:00048e50       ?get_extents@COLR@OT@@QBE_NPAUhb_font_t@@IPAUhb_glyph_extents_t@@@Z 10049e50 f i hb-ot-font.obj
 0001:00048fe0       ?get_extents@SmallGlyphMetrics@OT@@QBEXPAUhb_font_t@@PAUhb_glyph_extents_t@@_N@Z 10049fe0 f i hb-ot-font.obj
 0001:00049020       ?get_extents@accelerator_t@CBDT@OT@@QBE_NPAUhb_font_t@@IPAUhb_glyph_extents_t@@_N@Z 1004a020 f i hb-ot-font.obj
 0001:00049230       ?get_extents@glyf_accelerator_t@OT@@QBE_NPAUhb_font_t@@IPAUhb_glyph_extents_t@@@Z 1004a230 f i hb-ot-font.obj
 0001:00049320       ?get_extents@hb_paint_extents_context_t@@QAE?AUhb_extents_t@@XZ 1004a320 f i hb-ot-font.obj
 0001:00049380       ?get_glyph@VariationSelectorRecord@OT@@QBE?AW4glyph_variant_t@2@IPAIPBX@Z 1004a380 f i hb-ot-font.obj
 0001:000494e0       ?get_glyph_from_name@accelerator_t@cff1@OT@@QBE_NPBDHPAI@Z 1004a4e0 f i hb-ot-font.obj
 0001:000498c0       ?get_glyph_from_name@accelerator_t@post@OT@@QBE_NPBDHPAI@Z 1004a8c0 f i hb-ot-font.obj
 0001:00049a30       ?get_png_extents@accelerator_t@sbix@OT@@ABE_NPAUhb_font_t@@IPAUhb_glyph_extents_t@@_N@Z 1004aa30 f i hb-ot-font.obj
 0001:00049cb0       ?get_sid@Charset@CFF@@QBEIIIPAUcode_pair_t@2@@Z 1004acb0 f i hb-ot-font.obj
 0001:00049e10       ?get_size@?$CFFIndex@U?$IntType@G$01@OT@@@CFF@@QBEIXZ 1004ae10 f i hb-ot-font.obj
 0001:00049e60       ?glyph_to_sid@?$accelerator_templ_t@Ucff1_private_dict_opset_t@CFF@@U?$cff1_private_dict_values_base_t@Udict_val_t@CFF@@@2@@cff1@OT@@QBEIIPAUcode_pair_t@CFF@@@Z 1004ae60 f i hb-ot-font.obj
 0001:0004b650       ?image@hb_paint_funcs_t@@QAE_NPAXPAUhb_blob_t@@IIIMPAUhb_glyph_extents_t@@@Z 1004c650 f i hb-ot-font.obj
 0001:0004b690       ?init@?$cff1_private_dict_values_base_t@Udict_val_t@CFF@@@CFF@@QAEXXZ 1004c690 f i hb-ot-font.obj
 0001:0004b6c0       ?init@?$cff2_private_dict_values_base_t@Udict_val_t@CFF@@@CFF@@QAEXXZ 1004c6c0 f i hb-ot-font.obj
 0001:0004b700       ?init@cff1_font_dict_values_t@CFF@@QAEXXZ 1004c700 f i hb-ot-font.obj
 0001:0004b740       ?init@cff1_top_dict_values_t@CFF@@QAEXXZ 1004c740 f i hb-ot-font.obj
 0001:0004b7c0       ?init@cff2_font_dict_values_t@CFF@@QAEXXZ 1004c7c0 f i hb-ot-font.obj
 0001:0004b800       ?init@cff2_top_dict_values_t@CFF@@QAEXXZ 1004c800 f i hb-ot-font.obj
 0001:0004b840       ?interpret@?$dict_interpreter_t@Ucff1_font_dict_opset_t@CFF@@Ucff1_font_dict_values_t@2@U?$interp_env_t@Unumber_t@CFF@@@2@@CFF@@QAE_NAAUcff1_font_dict_values_t@2@@Z 1004c840 f i hb-ot-font.obj
 0001:0004ba70       ?interpret@?$dict_interpreter_t@Ucff1_private_dict_opset_t@CFF@@U?$cff1_private_dict_values_base_t@Udict_val_t@CFF@@@2@U?$interp_env_t@Unumber_t@CFF@@@2@@CFF@@QAE_NAAU?$cff1_private_dict_values_base_t@Udict_val_t@CFF@@@2@@Z 1004ca70 f i hb-ot-font.obj
 0001:0004bc10       ?interpret@?$dict_interpreter_t@Ucff1_top_dict_opset_t@CFF@@Ucff1_top_dict_values_t@2@Ucff1_top_dict_interp_env_t@2@@CFF@@QAE_NAAUcff1_top_dict_values_t@2@@Z 1004cc10 f i hb-ot-font.obj
 0001:0004bcb0       ?interpret@?$dict_interpreter_t@Ucff2_font_dict_opset_t@CFF@@Ucff2_font_dict_values_t@2@U?$interp_env_t@Unumber_t@CFF@@@2@@CFF@@QAE_NAAUcff2_font_dict_values_t@2@@Z 1004ccb0 f i hb-ot-font.obj
 0001:0004be70       ?interpret@?$dict_interpreter_t@Ucff2_private_dict_opset_t@CFF@@U?$cff2_private_dict_values_base_t@Udict_val_t@CFF@@@2@Ucff2_priv_dict_interp_env_t@2@@CFF@@QAE_NAAU?$cff2_private_dict_values_base_t@Udict_val_t@CFF@@@2@@Z 1004ce70 f i hb-ot-font.obj
 0001:0004c0d0       ?interpret@?$dict_interpreter_t@Ucff2_top_dict_opset_t@CFF@@Ucff2_top_dict_values_t@2@U?$interp_env_t@Unumber_t@CFF@@@2@@CFF@@QAE_NAAUcff2_top_dict_values_t@2@@Z 1004d0d0 f i hb-ot-font.obj
 0001:0004c3a0       ?map@DeltaSetIndexMap@OT@@QBEII@Z 1004d3a0 f i hb-ot-font.obj
 0001:0004c490       ?paint_glyph@?$PaintLinearGradient@UNoVariable@OT@@@OT@@QBEXPAUhb_paint_context_t@2@I@Z 1004d490 f i hb-ot-font.obj
 0001:0004c6e0       ?paint_glyph@?$PaintLinearGradient@UVariable@OT@@@OT@@QBEXPAUhb_paint_context_t@2@I@Z 1004d6e0 f i hb-ot-font.obj
 0001:0004c930       ?paint_glyph@?$PaintRadialGradient@UNoVariable@OT@@@OT@@QBEXPAUhb_paint_context_t@2@I@Z 1004d930 f i hb-ot-font.obj
 0001:0004cb90       ?paint_glyph@?$PaintRadialGradient@UVariable@OT@@@OT@@QBEXPAUhb_paint_context_t@2@I@Z 1004db90 f i hb-ot-font.obj
 0001:0004cdf0       ?paint_glyph@?$PaintSweepGradient@UNoVariable@OT@@@OT@@QBEXPAUhb_paint_context_t@2@I@Z 1004ddf0 f i hb-ot-font.obj
 0001:0004cfd0       ?paint_glyph@?$PaintSweepGradient@UVariable@OT@@@OT@@QBEXPAUhb_paint_context_t@2@I@Z 1004dfd0 f i hb-ot-font.obj
 0001:0004d1b0       ?paint_glyph@Affine2x3@OT@@QBEXPAUhb_paint_context_t@2@I@Z 1004e1b0 f i hb-ot-font.obj
 0001:0004d3e0       ?paint_glyph@COLR@OT@@QBE_NPAUhb_font_t@@IPAUhb_paint_funcs_t@@PAXII_N@Z 1004e3e0 f i hb-ot-font.obj
 0001:0004da90       ?paint_glyph@PaintColrGlyph@OT@@QBEXPAUhb_paint_context_t@2@@Z 1004ea90 f i hb-ot-font.obj
 0001:0004dce0       ?paint_glyph@PaintColrLayers@OT@@QBEXPAUhb_paint_context_t@2@@Z 1004ece0 f i hb-ot-font.obj
 0001:0004dee0       ?paint_glyph@PaintRotate@OT@@QBEXPAUhb_paint_context_t@2@I@Z 1004eee0 f i hb-ot-font.obj
 0001:0004e030       ?paint_glyph@PaintRotateAroundCenter@OT@@QBEXPAUhb_paint_context_t@2@I@Z 1004f030 f i hb-ot-font.obj
 0001:0004e350       ?paint_glyph@PaintScale@OT@@QBEXPAUhb_paint_context_t@2@I@Z 1004f350 f i hb-ot-font.obj
 0001:0004e4c0       ?paint_glyph@PaintScaleAroundCenter@OT@@QBEXPAUhb_paint_context_t@2@I@Z 1004f4c0 f i hb-ot-font.obj
 0001:0004e800       ?paint_glyph@PaintScaleUniform@OT@@QBEXPAUhb_paint_context_t@2@I@Z 1004f800 f i hb-ot-font.obj
 0001:0004e910       ?paint_glyph@PaintScaleUniformAroundCenter@OT@@QBEXPAUhb_paint_context_t@2@I@Z 1004f910 f i hb-ot-font.obj
 0001:0004ebe0       ?paint_glyph@PaintSkew@OT@@QBEXPAUhb_paint_context_t@2@I@Z 1004fbe0 f i hb-ot-font.obj
 0001:0004ed00       ?paint_glyph@PaintSkewAroundCenter@OT@@QBEXPAUhb_paint_context_t@2@I@Z 1004fd00 f i hb-ot-font.obj
 0001:0004efe0       ?paint_glyph@PaintSolid@OT@@QBEXPAUhb_paint_context_t@2@I@Z 1004ffe0 f i hb-ot-font.obj
 0001:0004f070       ?paint_glyph@PaintTranslate@OT@@QBEXPAUhb_paint_context_t@2@I@Z 10050070 f i hb-ot-font.obj
 0001:0004f1d0       ?parse_bcd@dict_opset_t@CFF@@SANAAUbyte_str_ref_t@2@@Z 100501d0 f i hb-ot-font.obj
 0001:0004f2e0       ?process_op@cff1_top_dict_opset_t@CFF@@SAXIAAUcff1_top_dict_interp_env_t@2@AAUcff1_top_dict_values_t@2@@Z 100502e0 f i hb-ot-font.obj
 0001:0004f6b0       ?process_op@dict_opset_t@CFF@@SAXIAAU?$interp_env_t@Unumber_t@CFF@@@2@@Z 100506b0 f i hb-ot-font.obj
 0001:0004f7f0       ?push@?$hb_vector_t@Ucff1_font_dict_values_t@CFF@@$0A@@@QAEPAUcff1_font_dict_values_t@CFF@@XZ 100507f0 f i hb-ot-font.obj
 0001:0004f890       ?push@?$hb_vector_t@Ucff2_font_dict_values_t@CFF@@$0A@@@QAEPAUcff2_font_dict_values_t@CFF@@XZ 10050890 f i hb-ot-font.obj
 0001:0004f950       ?push_clip_rectangle@hb_paint_funcs_t@@QAEXPAXMMMM@Z 10050950 f i hb-ot-font.obj
 0001:0004f9a0       ?push_inverse_root_transform@hb_paint_funcs_t@@QAEXPAXPAUhb_font_t@@@Z 100509a0 f i hb-ot-font.obj
 0001:0004fa80       ?push_root_transform@hb_paint_funcs_t@@QAEXPAXPBUhb_font_t@@@Z 10050a80 f i hb-ot-font.obj
 0001:0004fb20       ?push_skew@hb_paint_funcs_t@@QAE_NPAXMM@Z 10050b20 f i hb-ot-font.obj
 0001:0004fbe0       ?recurse@hb_paint_context_t@OT@@QAEXABUPaint@2@@Z 10050be0 f i hb-ot-font.obj
 0001:0004fc20       ?sanitize@?$CFFIndex@U?$IntType@G$01@OT@@@CFF@@QBE_NPAUhb_sanitize_context_t@@@Z 10050c20 f i hb-ot-font.obj
 0001:0004fd80       ?sanitize@?$CFFIndex@U?$IntType@I$03@OT@@@CFF@@QBE_NPAUhb_sanitize_context_t@@@Z 10050d80 f i hb-ot-font.obj
 0001:0004fef0       ?sanitize@?$FDSelect3_4@U?$IntType@G$01@OT@@U?$IntType@E$00@2@@CFF@@QBE_NPAUhb_sanitize_context_t@@I@Z 10050ef0 f i hb-ot-font.obj
 0001:00050140       ?sanitize@?$FDSelect3_4@U?$IntType@I$03@OT@@U?$IntType@G$01@2@@CFF@@QBE_NPAUhb_sanitize_context_t@@I@Z 10051140 f i hb-ot-font.obj
 0001:000503c0       ?sanitize@CFF2FDSelect@CFF@@QBE_NPAUhb_sanitize_context_t@@I@Z 100513c0 f i hb-ot-font.obj
 0001:00050460       ?sanitize@CFF2VariationStore@CFF@@QBE_NPAUhb_sanitize_context_t@@@Z 10051460 f i hb-ot-font.obj
 0001:00050550       ?sanitize@Charset@CFF@@QBE_NPAUhb_sanitize_context_t@@PAI@Z 10051550 f i hb-ot-font.obj
 0001:000507e0       ?sanitize@Encoding@CFF@@QBE_NPAUhb_sanitize_context_t@@@Z 100517e0 f i hb-ot-font.obj
 0001:000508a0       ?sanitize@FDSelect0@CFF@@QBE_NPAUhb_sanitize_context_t@@I@Z 100518a0 f i hb-ot-font.obj
 0001:00050910       ?sanitize@FDSelect@CFF@@QBE_NPAUhb_sanitize_context_t@@I@Z 10051910 f i hb-ot-font.obj
 0001:000509b0       ?sanitize@VORG@OT@@QBE_NPAUhb_sanitize_context_t@@@Z 100519b0 f i hb-ot-font.obj
 0001:00050a50       ?sanitize@cff1@OT@@QBE_NPAUhb_sanitize_context_t@@@Z 10051a50 f i hb-ot-font.obj
 0001:00050ad0       ?sanitize@cff2@OT@@QBE_NPAUhb_sanitize_context_t@@@Z 10051ad0 f i hb-ot-font.obj
 0001:00050b50       ?sanitize@post@OT@@QBE_NPAUhb_sanitize_context_t@@@Z 10051b50 f i hb-ot-font.obj
 0001:00050c40       ?sanitize_shallow@?$ArrayOf@U?$FDSelect3_4_Range@U?$IntType@G$01@OT@@U?$IntType@E$00@2@@CFF@@U?$IntType@G$01@OT@@@OT@@QBE_NPAUhb_sanitize_context_t@@@Z 10051c40 f i hb-ot-font.obj
 0001:00050c40       ?sanitize_shallow@?$ArrayOf@U?$IntType@I$02@OT@@U?$IntType@G$01@2@@OT@@QBE_NPAUhb_sanitize_context_t@@@Z 10051c40 f i hb-ot-layout.obj
 0001:00050ce0       ?sanitize_shallow@?$ArrayOf@U?$IntType@E$00@OT@@U12@@OT@@QBE_NPAUhb_sanitize_context_t@@@Z 10051ce0 f i hb-ot-font.obj
 0001:00050d70       ?sanitize_shallow@?$ArrayOf@UEncoding1_Range@CFF@@U?$IntType@E$00@OT@@@OT@@QBE_NPAUhb_sanitize_context_t@@@Z 10051d70 f i hb-ot-font.obj
 0001:00050e00       ?sanitize_shallow@?$ArrayOf@USuppEncoding@CFF@@U?$IntType@E$00@OT@@@OT@@QBE_NPAUhb_sanitize_context_t@@@Z 10051e00 f i hb-ot-font.obj
 0001:00050e90       ?sentinel@?$FDSelect3_4@U?$IntType@I$03@OT@@U?$IntType@G$01@2@@CFF@@QBEABU?$IntType@I$03@OT@@XZ 10051e90 f i hb-ot-font.obj
 0001:00050ee0       ?sid_to_glyph@?$accelerator_templ_t@Ucff1_private_dict_opset_t@CFF@@U?$cff1_private_dict_values_base_t@Udict_val_t@CFF@@@2@@cff1@OT@@QBEII@Z 10051ee0 f i hb-ot-font.obj
 0001:00051060       ?static_get_color_stops@?$ColorLine@UNoVariable@OT@@@OT@@SAIPAUhb_color_line_t@@PAXIPAIPAUhb_color_stop_t@@1@Z 10052060 f i hb-ot-font.obj
 0001:00051120       ?static_get_color_stops@?$ColorLine@UVariable@OT@@@OT@@SAIPAUhb_color_line_t@@PAXIPAIPAUhb_color_stop_t@@1@Z 10052120 f i hb-ot-font.obj
 0001:000511f0       ?static_get_extend@?$ColorLine@UVariable@OT@@@OT@@SA?AW4hb_paint_extend_t@@PAUhb_color_line_t@@PAX1@Z 100521f0 f i hb-ot-font.obj
 0001:000511f0       ?static_get_extend@?$ColorLine@UNoVariable@OT@@@OT@@SA?AW4hb_paint_extend_t@@PAUhb_color_line_t@@PAX1@Z 100521f0 f i hb-ot-font.obj
 0001:00051200       ?suppEncData@Encoding@CFF@@IBEABUCFF1SuppEncData@2@XZ 10052200 f i hb-ot-font.obj
 0001:00051250       _hb_ot_font_set_funcs      10052250 f   hb-ot-font.obj
 0001:00051450       ??$?0PBU?$KernSubTable@UKernOTSubTableHeader@OT@@@OT@@@hb_sanitize_with_object_t@@QAE@PAUhb_sanitize_context_t@@ABQBU?$KernSubTable@UKernOTSubTableHeader@OT@@@OT@@@Z 10052450 f i hb-ot-layout.obj
 0001:000514d0       ??$?HPBU?$MarkMarkPosFormat1_2@USmallTypes@Layout@OT@@@GPOS_impl@Layout@OT@@$0A@@OT@@YAABUMarkArray@GPOS_impl@Layout@0@ABQBU?$MarkMarkPosFormat1_2@USmallTypes@Layout@OT@@@230@ABU?$OffsetTo@UMarkArray@GPOS_impl@Layout@OT@@U?$IntType@G$01@4@$00@0@@Z 100524d0 f i hb-ot-layout.obj
 0001:000514d0       ??$?HPBU?$MarkMarkPosFormat1_2@USmallTypes@Layout@OT@@@GPOS_impl@Layout@OT@@$0A@@OT@@YAABUCoverage@Common@Layout@0@ABQBU?$MarkMarkPosFormat1_2@USmallTypes@Layout@OT@@@GPOS_impl@30@ABU?$OffsetTo@UCoverage@Common@Layout@OT@@U?$IntType@G$01@4@$00@0@@Z 100524d0 f i hb-ot-layout.obj
 0001:000514d0       ??$?HPBUCursivePosFormat1@GPOS_impl@Layout@OT@@$0A@@OT@@YAABUAnchor@GPOS_impl@Layout@0@ABQBUCursivePosFormat1@230@ABU?$OffsetTo@UAnchor@GPOS_impl@Layout@OT@@U?$IntType@G$01@4@$00@0@@Z 100524d0 f i hb-ot-layout.obj
 0001:000514d0       ??$?HPBU?$LigatureSet@USmallTypes@Layout@OT@@@GSUB_impl@Layout@OT@@$0A@@OT@@YAABU?$Ligature@USmallTypes@Layout@OT@@@GSUB_impl@Layout@0@ABQBU?$LigatureSet@USmallTypes@Layout@OT@@@230@ABU?$OffsetTo@U?$Ligature@USmallTypes@Layout@OT@@@GSUB_impl@Layout@OT@@U?$IntType@G$01@4@$00@0@@Z 100524d0 f i hb-ot-layout.obj
 0001:000514d0       ??$?HPBU?$MarkMarkPosFormat1_2@USmallTypes@Layout@OT@@@GPOS_impl@Layout@OT@@$0A@@OT@@YAABUAnchorMatrix@GPOS_impl@Layout@0@ABQBU?$MarkMarkPosFormat1_2@USmallTypes@Layout@OT@@@230@ABU?$OffsetTo@UAnchorMatrix@GPOS_impl@Layout@OT@@U?$IntType@G$01@4@$00@0@@Z 100524d0 f i hb-ot-layout.obj
 0001:00051670       ??$_dispatch@UFeatureParams@OT@@I@hb_sanitize_context_t@@AAE_NABUFeatureParams@OT@@U?$hb_priority@$00@@$$QAI@Z 10052670 f i hb-ot-layout.obj
 0001:00051780       ??$apply@UGPOSProxy@@@hb_ot_map_t@@QBEXABUGPOSProxy@@PBUhb_ot_shape_plan_t@@PAUhb_font_t@@PAUhb_buffer_t@@@Z 10052780 f i hb-ot-layout.obj
 0001:00051c30       ??$apply@UGSUBProxy@@@hb_ot_map_t@@QBEXABUGSUBProxy@@PBUhb_ot_shape_plan_t@@PAUhb_font_t@@PAUhb_buffer_t@@@Z 10052c30 f i hb-ot-layout.obj
 0001:00052140       ??$apply_to@U?$AlternateSubstFormat1_2@USmallTypes@Layout@OT@@@GSUB_impl@Layout@OT@@@hb_accelerate_subtables_context_t@OT@@SA_NPBXPAUhb_ot_apply_context_t@1@@Z 10053140 f i hb-ot-layout.obj
 0001:00052140       ??$apply_cached_to@U?$AlternateSubstFormat1_2@USmallTypes@Layout@OT@@@GSUB_impl@Layout@OT@@@hb_accelerate_subtables_context_t@OT@@SA_NPBXPAUhb_ot_apply_context_t@1@@Z 10053140 f i hb-ot-layout.obj
 0001:00052150       ??$apply_cached_to@U?$ChainContextFormat1_4@USmallTypes@Layout@OT@@@OT@@@hb_accelerate_subtables_context_t@OT@@SA_NPBXPAUhb_ot_apply_context_t@1@@Z 10053150 f i hb-ot-layout.obj
 0001:00052150       ??$apply_to@U?$ChainContextFormat1_4@USmallTypes@Layout@OT@@@OT@@@hb_accelerate_subtables_context_t@OT@@SA_NPBXPAUhb_ot_apply_context_t@1@@Z 10053150 f i hb-ot-layout.obj
 0001:00052160       ??$apply_cached_to@U?$ChainContextFormat2_5@USmallTypes@Layout@OT@@@OT@@@hb_accelerate_subtables_context_t@OT@@SA_NPBXPAUhb_ot_apply_context_t@1@@Z 10053160 f i hb-ot-layout.obj
 0001:00052170       ??$apply_to@U?$ContextFormat1_4@USmallTypes@Layout@OT@@@OT@@@hb_accelerate_subtables_context_t@OT@@SA_NPBXPAUhb_ot_apply_context_t@1@@Z 10053170 f i hb-ot-layout.obj
 0001:00052170       ??$apply_cached_to@U?$ContextFormat1_4@USmallTypes@Layout@OT@@@OT@@@hb_accelerate_subtables_context_t@OT@@SA_NPBXPAUhb_ot_apply_context_t@1@@Z 10053170 f i hb-ot-layout.obj
 0001:00052180       ??$apply_cached_to@U?$ContextFormat2_5@USmallTypes@Layout@OT@@@OT@@@hb_accelerate_subtables_context_t@OT@@SA_NPBXPAUhb_ot_apply_context_t@1@@Z 10053180 f i hb-ot-layout.obj
 0001:00052190       ??$apply_to@U?$LigatureSubstFormat1_2@USmallTypes@Layout@OT@@@GSUB_impl@Layout@OT@@@hb_accelerate_subtables_context_t@OT@@SA_NPBXPAUhb_ot_apply_context_t@1@@Z 10053190 f i hb-ot-layout.obj
 0001:00052190       ??$apply_cached_to@U?$LigatureSubstFormat1_2@USmallTypes@Layout@OT@@@GSUB_impl@Layout@OT@@@hb_accelerate_subtables_context_t@OT@@SA_NPBXPAUhb_ot_apply_context_t@1@@Z 10053190 f i hb-ot-layout.obj
 0001:000521a0       ??$apply_cached_to@U?$MarkBasePosFormat1_2@USmallTypes@Layout@OT@@@GPOS_impl@Layout@OT@@@hb_accelerate_subtables_context_t@OT@@SA_NPBXPAUhb_ot_apply_context_t@1@@Z 100531a0 f i hb-ot-layout.obj
 0001:000521a0       ??$apply_to@U?$MarkBasePosFormat1_2@USmallTypes@Layout@OT@@@GPOS_impl@Layout@OT@@@hb_accelerate_subtables_context_t@OT@@SA_NPBXPAUhb_ot_apply_context_t@1@@Z 100531a0 f i hb-ot-layout.obj
 0001:000521b0       ??$apply_cached_to@U?$MarkLigPosFormat1_2@USmallTypes@Layout@OT@@@GPOS_impl@Layout@OT@@@hb_accelerate_subtables_context_t@OT@@SA_NPBXPAUhb_ot_apply_context_t@1@@Z 100531b0 f i hb-ot-layout.obj
 0001:000521b0       ??$apply_to@U?$MarkLigPosFormat1_2@USmallTypes@Layout@OT@@@GPOS_impl@Layout@OT@@@hb_accelerate_subtables_context_t@OT@@SA_NPBXPAUhb_ot_apply_context_t@1@@Z 100531b0 f i hb-ot-layout.obj
 0001:000521c0       ??$apply_to@U?$MarkMarkPosFormat1_2@USmallTypes@Layout@OT@@@GPOS_impl@Layout@OT@@@hb_accelerate_subtables_context_t@OT@@SA_NPBXPAUhb_ot_apply_context_t@1@@Z 100531c0 f i hb-ot-layout.obj
 0001:000521c0       ??$apply_cached_to@U?$MarkMarkPosFormat1_2@USmallTypes@Layout@OT@@@GPOS_impl@Layout@OT@@@hb_accelerate_subtables_context_t@OT@@SA_NPBXPAUhb_ot_apply_context_t@1@@Z 100531c0 f i hb-ot-layout.obj
 0001:000521d0       ??$apply_to@U?$MultipleSubstFormat1_2@USmallTypes@Layout@OT@@@GSUB_impl@Layout@OT@@@hb_accelerate_subtables_context_t@OT@@SA_NPBXPAUhb_ot_apply_context_t@1@@Z 100531d0 f i hb-ot-layout.obj
 0001:000521d0       ??$apply_cached_to@U?$MultipleSubstFormat1_2@USmallTypes@Layout@OT@@@GSUB_impl@Layout@OT@@@hb_accelerate_subtables_context_t@OT@@SA_NPBXPAUhb_ot_apply_context_t@1@@Z 100531d0 f i hb-ot-layout.obj
 0001:000521e0       ??$apply_cached_to@U?$PairPosFormat1_3@USmallTypes@Layout@OT@@@GPOS_impl@Layout@OT@@@hb_accelerate_subtables_context_t@OT@@SA_NPBXPAUhb_ot_apply_context_t@1@@Z 100531e0 f i hb-ot-layout.obj
 0001:000521e0       ??$apply_to@U?$PairPosFormat1_3@USmallTypes@Layout@OT@@@GPOS_impl@Layout@OT@@@hb_accelerate_subtables_context_t@OT@@SA_NPBXPAUhb_ot_apply_context_t@1@@Z 100531e0 f i hb-ot-layout.obj
 0001:000521f0       ??$apply_to@U?$PairPosFormat2_4@USmallTypes@Layout@OT@@@GPOS_impl@Layout@OT@@@hb_accelerate_subtables_context_t@OT@@SA_NPBXPAUhb_ot_apply_context_t@1@@Z 100531f0 f i hb-ot-layout.obj
 0001:000521f0       ??$apply_cached_to@U?$PairPosFormat2_4@USmallTypes@Layout@OT@@@GPOS_impl@Layout@OT@@@hb_accelerate_subtables_context_t@OT@@SA_NPBXPAUhb_ot_apply_context_t@1@@Z 100531f0 f i hb-ot-layout.obj
 0001:00052200       ??$apply_to@U?$SingleSubstFormat1_3@USmallTypes@Layout@OT@@@GSUB_impl@Layout@OT@@@hb_accelerate_subtables_context_t@OT@@SA_NPBXPAUhb_ot_apply_context_t@1@@Z 10053200 f i hb-ot-layout.obj
 0001:00052200       ??$apply_cached_to@U?$SingleSubstFormat1_3@USmallTypes@Layout@OT@@@GSUB_impl@Layout@OT@@@hb_accelerate_subtables_context_t@OT@@SA_NPBXPAUhb_ot_apply_context_t@1@@Z 10053200 f i hb-ot-layout.obj
 0001:00052210       ??$apply_cached_to@U?$SingleSubstFormat2_4@USmallTypes@Layout@OT@@@GSUB_impl@Layout@OT@@@hb_accelerate_subtables_context_t@OT@@SA_NPBXPAUhb_ot_apply_context_t@1@@Z 10053210 f i hb-ot-layout.obj
 0001:00052210       ??$apply_to@U?$SingleSubstFormat2_4@USmallTypes@Layout@OT@@@GSUB_impl@Layout@OT@@@hb_accelerate_subtables_context_t@OT@@SA_NPBXPAUhb_ot_apply_context_t@1@@Z 10053210 f i hb-ot-layout.obj
 0001:00052220       ??$apply_to@UChainContextFormat3@OT@@@hb_accelerate_subtables_context_t@OT@@SA_NPBXPAUhb_ot_apply_context_t@1@@Z 10053220 f i hb-ot-layout.obj
 0001:00052220       ??$apply_cached_to@UChainContextFormat3@OT@@@hb_accelerate_subtables_context_t@OT@@SA_NPBXPAUhb_ot_apply_context_t@1@@Z 10053220 f i hb-ot-layout.obj
 0001:00052230       ??$apply_to@UContextFormat3@OT@@@hb_accelerate_subtables_context_t@OT@@SA_NPBXPAUhb_ot_apply_context_t@1@@Z 10053230 f i hb-ot-layout.obj
 0001:00052230       ??$apply_cached_to@UContextFormat3@OT@@@hb_accelerate_subtables_context_t@OT@@SA_NPBXPAUhb_ot_apply_context_t@1@@Z 10053230 f i hb-ot-layout.obj
 0001:00052240       ??$apply_to@UCursivePosFormat1@GPOS_impl@Layout@OT@@@hb_accelerate_subtables_context_t@OT@@SA_NPBXPAUhb_ot_apply_context_t@1@@Z 10053240 f i hb-ot-layout.obj
 0001:00052240       ??$apply_cached_to@UCursivePosFormat1@GPOS_impl@Layout@OT@@@hb_accelerate_subtables_context_t@OT@@SA_NPBXPAUhb_ot_apply_context_t@1@@Z 10053240 f i hb-ot-layout.obj
 0001:00052250       ??$apply_cached_to@UReverseChainSingleSubstFormat1@GSUB_impl@Layout@OT@@@hb_accelerate_subtables_context_t@OT@@SA_NPBXPAUhb_ot_apply_context_t@1@@Z 10053250 f i hb-ot-layout.obj
 0001:00052250       ??$apply_to@UReverseChainSingleSubstFormat1@GSUB_impl@Layout@OT@@@hb_accelerate_subtables_context_t@OT@@SA_NPBXPAUhb_ot_apply_context_t@1@@Z 10053250 f i hb-ot-layout.obj
 0001:00052260       ??$apply_to@USinglePosFormat1@GPOS_impl@Layout@OT@@@hb_accelerate_subtables_context_t@OT@@SA_NPBXPAUhb_ot_apply_context_t@1@@Z 10053260 f i hb-ot-layout.obj
 0001:00052260       ??$apply_cached_to@USinglePosFormat1@GPOS_impl@Layout@OT@@@hb_accelerate_subtables_context_t@OT@@SA_NPBXPAUhb_ot_apply_context_t@1@@Z 10053260 f i hb-ot-layout.obj
 0001:00052270       ??$apply_to@USinglePosFormat2@GPOS_impl@Layout@OT@@@hb_accelerate_subtables_context_t@OT@@SA_NPBXPAUhb_ot_apply_context_t@1@@Z 10053270 f i hb-ot-layout.obj
 0001:00052270       ??$apply_cached_to@USinglePosFormat2@GPOS_impl@Layout@OT@@@hb_accelerate_subtables_context_t@OT@@SA_NPBXPAUhb_ot_apply_context_t@1@@Z 10053270 f i hb-ot-layout.obj
 0001:00052360       ??$apply_to@U?$ChainContextFormat2_5@USmallTypes@Layout@OT@@@OT@@@hb_accelerate_subtables_context_t@OT@@SA_NPBXPAUhb_ot_apply_context_t@1@@Z 10053360 f i hb-ot-layout.obj
 0001:00052370       ??$apply_to@U?$ContextFormat2_5@USmallTypes@Layout@OT@@@OT@@@hb_accelerate_subtables_context_t@OT@@SA_NPBXPAUhb_ot_apply_context_t@1@@Z 10053370 f i hb-ot-layout.obj
 0001:00052380       ??$bsearch@Uhb_glyph_pair_t@AAT@@@?$SortedArrayOf@UKernPair@AAT@@U?$BinSearchHeader@U?$IntType@G$01@OT@@@OT@@@OT@@QBEABUKernPair@AAT@@ABUhb_glyph_pair_t@3@ABU23@@Z 10053380 f i hb-ot-layout.obj
 0001:00052430       ??$cache_func_to@U?$ContextFormat1_4@USmallTypes@Layout@OT@@@OT@@@hb_accelerate_subtables_context_t@OT@@SA_NPBXPAUhb_ot_apply_context_t@1@_N@Z 10053430 f i hb-ot-layout.obj
 0001:00052430       ??$cache_func_to@UChainContextFormat3@OT@@@hb_accelerate_subtables_context_t@OT@@SA_NPBXPAUhb_ot_apply_context_t@1@_N@Z 10053430 f i hb-ot-layout.obj
 0001:00052430       ??$cache_func_to@U?$MarkBasePosFormat1_2@USmallTypes@Layout@OT@@@GPOS_impl@Layout@OT@@@hb_accelerate_subtables_context_t@OT@@SA_NPBXPAUhb_ot_apply_context_t@1@_N@Z 10053430 f i hb-ot-layout.obj
 0001:00052430       ??$cache_func_to@U?$SingleSubstFormat1_3@USmallTypes@Layout@OT@@@GSUB_impl@Layout@OT@@@hb_accelerate_subtables_context_t@OT@@SA_NPBXPAUhb_ot_apply_context_t@1@_N@Z 10053430 f i hb-ot-layout.obj
 0001:00052430       ??$cache_func_to@U?$MarkMarkPosFormat1_2@USmallTypes@Layout@OT@@@GPOS_impl@Layout@OT@@@hb_accelerate_subtables_context_t@OT@@SA_NPBXPAUhb_ot_apply_context_t@1@_N@Z 10053430 f i hb-ot-layout.obj
 0001:00052430       ??$cache_func_to@USinglePosFormat2@GPOS_impl@Layout@OT@@@hb_accelerate_subtables_context_t@OT@@SA_NPBXPAUhb_ot_apply_context_t@1@_N@Z 10053430 f i hb-ot-layout.obj
 0001:00052430       ??$cache_func_to@U?$LigatureSubstFormat1_2@USmallTypes@Layout@OT@@@GSUB_impl@Layout@OT@@@hb_accelerate_subtables_context_t@OT@@SA_NPBXPAUhb_ot_apply_context_t@1@_N@Z 10053430 f i hb-ot-layout.obj
 0001:00052430       ??$cache_func_to@U?$SingleSubstFormat2_4@USmallTypes@Layout@OT@@@GSUB_impl@Layout@OT@@@hb_accelerate_subtables_context_t@OT@@SA_NPBXPAUhb_ot_apply_context_t@1@_N@Z 10053430 f i hb-ot-layout.obj
 0001:00052430       ??$cache_func_to@U?$MultipleSubstFormat1_2@USmallTypes@Layout@OT@@@GSUB_impl@Layout@OT@@@hb_accelerate_subtables_context_t@OT@@SA_NPBXPAUhb_ot_apply_context_t@1@_N@Z 10053430 f i hb-ot-layout.obj
 0001:00052430       ??$cache_func_to@U?$ChainContextFormat1_4@USmallTypes@Layout@OT@@@OT@@@hb_accelerate_subtables_context_t@OT@@SA_NPBXPAUhb_ot_apply_context_t@1@_N@Z 10053430 f i hb-ot-layout.obj
 0001:00052430       ??$cache_func_to@UCursivePosFormat1@GPOS_impl@Layout@OT@@@hb_accelerate_subtables_context_t@OT@@SA_NPBXPAUhb_ot_apply_context_t@1@_N@Z 10053430 f i hb-ot-layout.obj
 0001:00052430       ??$cache_func_to@USinglePosFormat1@GPOS_impl@Layout@OT@@@hb_accelerate_subtables_context_t@OT@@SA_NPBXPAUhb_ot_apply_context_t@1@_N@Z 10053430 f i hb-ot-layout.obj
 0001:00052430       ??$cache_func_to@U?$MarkLigPosFormat1_2@USmallTypes@Layout@OT@@@GPOS_impl@Layout@OT@@@hb_accelerate_subtables_context_t@OT@@SA_NPBXPAUhb_ot_apply_context_t@1@_N@Z 10053430 f i hb-ot-layout.obj
 0001:00052430       ??$cache_func_to@U?$PairPosFormat2_4@USmallTypes@Layout@OT@@@GPOS_impl@Layout@OT@@@hb_accelerate_subtables_context_t@OT@@SA_NPBXPAUhb_ot_apply_context_t@1@_N@Z 10053430 f i hb-ot-layout.obj
 0001:00052430       ??$cache_func_to@U?$AlternateSubstFormat1_2@USmallTypes@Layout@OT@@@GSUB_impl@Layout@OT@@@hb_accelerate_subtables_context_t@OT@@SA_NPBXPAUhb_ot_apply_context_t@1@_N@Z 10053430 f i hb-ot-layout.obj
 0001:00052430       ??$cache_func_to@UContextFormat3@OT@@@hb_accelerate_subtables_context_t@OT@@SA_NPBXPAUhb_ot_apply_context_t@1@_N@Z 10053430 f i hb-ot-layout.obj
 0001:00052430       ??$cache_func_to@U?$PairPosFormat1_3@USmallTypes@Layout@OT@@@GPOS_impl@Layout@OT@@@hb_accelerate_subtables_context_t@OT@@SA_NPBXPAUhb_ot_apply_context_t@1@_N@Z 10053430 f i hb-ot-layout.obj
 0001:00052430       ??$cache_func_to@UReverseChainSingleSubstFormat1@GSUB_impl@Layout@OT@@@hb_accelerate_subtables_context_t@OT@@SA_NPBXPAUhb_ot_apply_context_t@1@_N@Z 10053430 f i hb-ot-layout.obj
 0001:00052440       ??$cache_func_to@U?$ContextFormat2_5@USmallTypes@Layout@OT@@@OT@@@hb_accelerate_subtables_context_t@OT@@SA_NPBXPAUhb_ot_apply_context_t@1@_N@Z 10053440 f i hb-ot-layout.obj
 0001:00052440       ??$cache_func_to@U?$ChainContextFormat2_5@USmallTypes@Layout@OT@@@OT@@@hb_accelerate_subtables_context_t@OT@@SA_NPBXPAUhb_ot_apply_context_t@1@_N@Z 10053440 f i hb-ot-layout.obj
 0001:000524b0       ??$create@UPosLookup@GPOS_impl@Layout@OT@@@hb_ot_layout_lookup_accelerator_t@OT@@SAPAU01@ABUPosLookup@GPOS_impl@Layout@1@@Z 100534b0 f i hb-ot-layout.obj
 0001:00052630       ??$create@USubstLookup@GSUB_impl@Layout@OT@@@hb_ot_layout_lookup_accelerator_t@OT@@SAPAU01@ABUSubstLookup@GSUB_impl@Layout@1@@Z 10053630 f i hb-ot-layout.obj
 0001:000527b0       ??$dispatch@U?$ChainContextFormat2_5@USmallTypes@Layout@OT@@@OT@@@hb_accelerate_subtables_context_t@OT@@QAE?AUhb_empty_t@@ABU?$ChainContextFormat2_5@USmallTypes@Layout@OT@@@1@@Z 100537b0 f i hb-ot-layout.obj
 0001:000528d0       ??$dispatch@U?$ChainRule@USmallTypes@Layout@OT@@@OT@@$$V@hb_sanitize_context_t@@QAE_NABU?$ChainRule@USmallTypes@Layout@OT@@@OT@@@Z 100538d0 f i hb-ot-layout.obj
 0001:00052960       ??$dispatch@U?$ChainRuleSet@USmallTypes@Layout@OT@@@OT@@$$V@hb_sanitize_context_t@@QAE_NABU?$ChainRuleSet@USmallTypes@Layout@OT@@@OT@@@Z 10053960 f i hb-ot-layout.obj
 0001:00052a10       ??$dispatch@U?$ClassTable@U?$IntType@G$01@OT@@@AAT@@$$V@hb_sanitize_context_t@@QAE_NABU?$ClassTable@U?$IntType@G$01@OT@@@AAT@@@Z 10053a10 f i hb-ot-layout.obj
 0001:00052a90       ??$dispatch@U?$ContextFormat2_5@USmallTypes@Layout@OT@@@OT@@@hb_accelerate_subtables_context_t@OT@@QAE?AUhb_empty_t@@ABU?$ContextFormat2_5@USmallTypes@Layout@OT@@@1@@Z 10053a90 f i hb-ot-layout.obj
 0001:00052bb0       ??$dispatch@U?$LigatureSet@USmallTypes@Layout@OT@@@GSUB_impl@Layout@OT@@$$V@hb_sanitize_context_t@@QAE_NABU?$LigatureSet@USmallTypes@Layout@OT@@@GSUB_impl@Layout@OT@@@Z 10053bb0 f i hb-ot-layout.obj
 0001:00052c80       ??$dispatch@U?$List16OfOffsetTo@UPosLookup@GPOS_impl@Layout@OT@@U?$IntType@G$01@4@@OT@@$$V@hb_sanitize_context_t@@QAE_NABU?$List16OfOffsetTo@UPosLookup@GPOS_impl@Layout@OT@@U?$IntType@G$01@4@@OT@@@Z 10053c80 f i hb-ot-layout.obj
 0001:00052d30       ??$dispatch@U?$List16OfOffsetTo@USubstLookup@GSUB_impl@Layout@OT@@U?$IntType@G$01@4@@OT@@$$V@hb_sanitize_context_t@@QAE_NABU?$List16OfOffsetTo@USubstLookup@GSUB_impl@Layout@OT@@U?$IntType@G$01@4@@OT@@@Z 10053d30 f i hb-ot-layout.obj
 0001:00052de0       ??$dispatch@U?$RuleSet@USmallTypes@Layout@OT@@@OT@@$$V@hb_sanitize_context_t@@QAE_NABU?$RuleSet@USmallTypes@Layout@OT@@@OT@@@Z 10053de0 f i hb-ot-layout.obj
 0001:00052e90       ??$dispatch@UAnchor@GPOS_impl@Layout@OT@@$$V@hb_sanitize_context_t@@QAE_NABUAnchor@GPOS_impl@Layout@OT@@@Z 10053e90 f i hb-ot-layout.obj
 0001:00052f80       ??$dispatch@UCondition@OT@@$$V@hb_sanitize_context_t@@QAE_NABUCondition@OT@@@Z 10053f80 f i hb-ot-layout.obj
 0001:00053010       ??$dispatch@UConditionSet@OT@@$$V@hb_sanitize_context_t@@QAE_NABUConditionSet@OT@@@Z 10054010 f i hb-ot-layout.obj
 0001:000530c0       ??$dispatch@ULigatureArray@GPOS_impl@Layout@OT@@I@hb_sanitize_context_t@@QAE_NABULigatureArray@GPOS_impl@Layout@OT@@$$QAI@Z 100540c0 f i hb-ot-layout.obj
 0001:00053170       ??$dispatch@UMarkArray@GPOS_impl@Layout@OT@@$$V@hb_sanitize_context_t@@QAE_NABUMarkArray@GPOS_impl@Layout@OT@@@Z 10054170 f i hb-ot-layout.obj
 0001:00053290       ??$dispatch@URecordListOfScript@OT@@$$V@hb_sanitize_context_t@@QAE_NABURecordListOfScript@OT@@@Z 10054290 f i hb-ot-layout.obj
 0001:000533c0       ??$dispatch@Uhb_aat_apply_context_t@AAT@@$$V@?$KernSubTable@UKernAATSubTableHeader@OT@@@OT@@QBE_NPAUhb_aat_apply_context_t@AAT@@@Z 100543c0 f i hb-ot-layout.obj
 0001:00053590       ??$dispatch@Uhb_accelerate_subtables_context_t@OT@@$$V@ChainContext@OT@@QBE?AUhb_empty_t@@PAUhb_accelerate_subtables_context_t@1@@Z 10054590 f i hb-ot-layout.obj
 0001:000536d0       ??$dispatch@Uhb_accelerate_subtables_context_t@OT@@$$V@Context@OT@@QBE?AUhb_empty_t@@PAUhb_accelerate_subtables_context_t@1@@Z 100546d0 f i hb-ot-layout.obj
 0001:00053820       ??$dispatch@Uhb_accelerate_subtables_context_t@OT@@$$V@PosLookupSubTable@GPOS_impl@Layout@OT@@QBE?AUhb_empty_t@@PAUhb_accelerate_subtables_context_t@3@I@Z 10054820 f i hb-ot-layout.obj
 0001:00053bd0       ??$dispatch@Uhb_accelerate_subtables_context_t@OT@@$$V@SubstLookupSubTable@GSUB_impl@Layout@OT@@QBE?AUhb_empty_t@@PAUhb_accelerate_subtables_context_t@3@I@Z 10054bd0 f i hb-ot-layout.obj
 0001:00053f30       ??$dispatch@Uhb_sanitize_context_t@@$$V@?$KernSubTable@UKernAATSubTableHeader@OT@@@OT@@QBE_NPAUhb_sanitize_context_t@@@Z 10054f30 f i hb-ot-layout.obj
 0001:000540f0       ??$dispatch@Uhb_sanitize_context_t@@$$V@ChainContext@OT@@QBE_NPAUhb_sanitize_context_t@@@Z 100550f0 f i hb-ot-layout.obj
 0001:00054250       ??$dispatch@Uhb_sanitize_context_t@@$$V@Context@OT@@QBE_NPAUhb_sanitize_context_t@@@Z 10055250 f i hb-ot-layout.obj
 0001:000543b0       ??$dispatch@Uhb_sanitize_context_t@@$$V@PosLookupSubTable@GPOS_impl@Layout@OT@@QBE_NPAUhb_sanitize_context_t@@I@Z 100553b0 f i hb-ot-layout.obj
 0001:00054640       ??$dispatch@Uhb_sanitize_context_t@@$$V@SubstLookupSubTable@GSUB_impl@Layout@OT@@QBE_NPAUhb_sanitize_context_t@@I@Z 10055640 f i hb-ot-layout.obj
 0001:00054bc0       ??$dispatch@Uhb_would_apply_context_t@OT@@$$V@ChainContext@OT@@QBE_NPAUhb_would_apply_context_t@1@@Z 10055bc0 f i hb-ot-layout.obj
 0001:00054e60       ??$dispatch@Uhb_would_apply_context_t@OT@@$$V@Context@OT@@QBE_NPAUhb_would_apply_context_t@1@@Z 10055e60 f i hb-ot-layout.obj
 0001:00055030       ??$dispatch@Uhb_would_apply_context_t@OT@@$$V@SubstLookupSubTable@GSUB_impl@Layout@OT@@QBE_NPAUhb_would_apply_context_t@3@I@Z 10056030 f i hb-ot-layout.obj
 0001:00055260       ??$dispatch_recurse_func@Uhb_ot_apply_context_t@OT@@@PosLookup@GPOS_impl@Layout@OT@@SA_NPAUhb_ot_apply_context_t@3@I@Z 10056260 f i hb-ot-layout.obj
 0001:00055380       ??$dispatch_recurse_func@Uhb_ot_apply_context_t@OT@@@SubstLookup@GSUB_impl@Layout@OT@@SA_NPAUhb_ot_apply_context_t@3@I@Z 10056380 f i hb-ot-layout.obj
 0001:000554a0       ??$drive@Udriver_context_t@?$KerxSubTableFormat1@UKernAATSubTableHeader@OT@@@AAT@@@?$StateTableDriver@UObsoleteTypes@AAT@@X@AAT@@QAEXPAUdriver_context_t@?$KerxSubTableFormat1@UKernAATSubTableHeader@OT@@@1@PAUhb_aat_apply_context_t@1@@Z 100564a0 f i hb-ot-layout.obj
 0001:00055880       ??$get_subtable@UPosLookupSubTable@GPOS_impl@Layout@OT@@@Lookup@OT@@QBEABUPosLookupSubTable@GPOS_impl@Layout@1@I@Z 10056880 f i hb-ot-layout.obj
 0001:00055880       ??$get_subtable@USubstLookupSubTable@GSUB_impl@Layout@OT@@@Lookup@OT@@QBEABUSubstLookupSubTable@GSUB_impl@Layout@1@I@Z 10056880 f i hb-ot-layout.obj
 0001:000558e0       ??$sanitize@UPosLookup@GPOS_impl@Layout@OT@@@?$GSUBGPOSVersion1_2@USmallTypes@Layout@OT@@@OT@@QBE_NPAUhb_sanitize_context_t@@@Z 100568e0 f i hb-ot-layout.obj
 0001:00055a90       ??$sanitize@UPosLookupSubTable@GPOS_impl@Layout@OT@@@Lookup@OT@@QBE_NPAUhb_sanitize_context_t@@@Z 10056a90 f i hb-ot-layout.obj
 0001:00055c70       ??$sanitize@USubstLookup@GSUB_impl@Layout@OT@@@?$GSUBGPOSVersion1_2@USmallTypes@Layout@OT@@@OT@@QBE_NPAUhb_sanitize_context_t@@@Z 10056c70 f i hb-ot-layout.obj
 0001:00055e20       ??$sanitize@USubstLookupSubTable@GSUB_impl@Layout@OT@@@Lookup@OT@@QBE_NPAUhb_sanitize_context_t@@@Z 10056e20 f i hb-ot-layout.obj
 0001:00056000       ??$sanitize_blob@UGPOS@Layout@OT@@@hb_sanitize_context_t@@QAEPAUhb_blob_t@@PAU1@@Z 10057000 f i hb-ot-layout.obj
 0001:000561b0       ??$sanitize_blob@UGSUB@Layout@OT@@@hb_sanitize_context_t@@QAEPAUhb_blob_t@@PAU1@@Z 100571b0 f i hb-ot-layout.obj
 0001:00056360       ??$sanitize_blob@Ukern@OT@@@hb_sanitize_context_t@@QAEPAUhb_blob_t@@PAU1@@Z 10057360 f i hb-ot-layout.obj
 0001:000565c0       ??D?$hb_iter_t@U?$hb_map_iter_t@U?$hb_array_t@$$CBU?$OffsetTo@U?$ChainRule@USmallTypes@Layout@OT@@@OT@@U?$IntType@G$01@2@$00@OT@@@@U?$hb_partial_t@$01PBU<unnamed-type-hb_add>@@PBU?$ChainRuleSet@USmallTypes@Layout@OT@@@OT@@@@$0A@$0A@@@ABU?$ChainRule@USmallTypes@Layout@OT@@@OT@@@@QBEABU?$ChainRule@USmallTypes@Layout@OT@@@OT@@XZ 100575c0 f i hb-ot-layout.obj
 0001:00056600       ?_apply@?$ChainContextFormat2_5@USmallTypes@Layout@OT@@@OT@@QBE_NPAUhb_ot_apply_context_t@2@_N@Z 10057600 f i hb-ot-layout.obj
 0001:000567e0       ?_apply@?$ContextFormat2_5@USmallTypes@Layout@OT@@@OT@@QBE_NPAUhb_ot_apply_context_t@2@_N@Z 100577e0 f i hb-ot-layout.obj
 0001:00056b60       ?_set_glyph_class@hb_ot_apply_context_t@OT@@QAEXII_N0@Z 10057b60 f i hb-ot-layout.obj
 0001:00056c60       ?apply@?$AlternateSubstFormat1_2@USmallTypes@Layout@OT@@@GSUB_impl@Layout@OT@@QBE_NPAUhb_ot_apply_context_t@4@@Z 10057c60 f i hb-ot-layout.obj
 0001:00056e60       ?apply@?$ChainContextFormat1_4@USmallTypes@Layout@OT@@@OT@@QBE_NPAUhb_ot_apply_context_t@2@@Z 10057e60 f i hb-ot-layout.obj
 0001:00056f70       ?apply@?$ChainRule@USmallTypes@Layout@OT@@@OT@@QBE_NPAUhb_ot_apply_context_t@2@ABUChainContextApplyLookupContext@2@@Z 10057f70 f i hb-ot-layout.obj
 0001:00057850       ?apply@?$ChainRuleSet@USmallTypes@Layout@OT@@@OT@@QBE_NPAUhb_ot_apply_context_t@2@ABUChainContextApplyLookupContext@2@@Z 10058850 f i hb-ot-layout.obj
 0001:000581d0       ?apply@?$ContextFormat1_4@USmallTypes@Layout@OT@@@OT@@QBE_NPAUhb_ot_apply_context_t@2@@Z 100591d0 f i hb-ot-layout.obj
 0001:000582c0       ?apply@?$KerxTable@UKernAAT@OT@@@AAT@@QBE_NPAUhb_aat_apply_context_t@2@@Z 100592c0 f i hb-ot-layout.obj
 0001:00058510       ?apply@?$KerxTable@UKernOT@OT@@@AAT@@QBE_NPAUhb_aat_apply_context_t@2@@Z 10059510 f i hb-ot-layout.obj
 0001:000587b0       ?apply@?$Ligature@USmallTypes@Layout@OT@@@GSUB_impl@Layout@OT@@QBE_NPAUhb_ot_apply_context_t@4@@Z 100597b0 f i hb-ot-layout.obj
 0001:00058d90       ?apply@?$LigatureSet@USmallTypes@Layout@OT@@@GSUB_impl@Layout@OT@@QBE_NPAUhb_ot_apply_context_t@4@@Z 10059d90 f i hb-ot-layout.obj
 0001:00059180       ?apply@?$LigatureSubstFormat1_2@USmallTypes@Layout@OT@@@GSUB_impl@Layout@OT@@QBE_NPAUhb_ot_apply_context_t@4@@Z 1005a180 f i hb-ot-layout.obj
 0001:00059260       ?apply@?$MarkBasePosFormat1_2@USmallTypes@Layout@OT@@@GPOS_impl@Layout@OT@@QBE_NPAUhb_ot_apply_context_t@4@@Z 1005a260 f i hb-ot-layout.obj
 0001:00059790       ?apply@?$MarkLigPosFormat1_2@USmallTypes@Layout@OT@@@GPOS_impl@Layout@OT@@QBE_NPAUhb_ot_apply_context_t@4@@Z 1005a790 f i hb-ot-layout.obj
 0001:00059d30       ?apply@?$MarkMarkPosFormat1_2@USmallTypes@Layout@OT@@@GPOS_impl@Layout@OT@@QBE_NPAUhb_ot_apply_context_t@4@@Z 1005ad30 f i hb-ot-layout.obj
 0001:0005a2f0       ?apply@?$MultipleSubstFormat1_2@USmallTypes@Layout@OT@@@GSUB_impl@Layout@OT@@QBE_NPAUhb_ot_apply_context_t@4@@Z 1005b2f0 f i hb-ot-layout.obj
 0001:0005a3d0       ?apply@?$PairPosFormat1_3@USmallTypes@Layout@OT@@@GPOS_impl@Layout@OT@@QBE_NPAUhb_ot_apply_context_t@4@@Z 1005b3d0 f i hb-ot-layout.obj
 0001:0005a680       ?apply@?$PairPosFormat2_4@USmallTypes@Layout@OT@@@GPOS_impl@Layout@OT@@QBE_NPAUhb_ot_apply_context_t@4@@Z 1005b680 f i hb-ot-layout.obj
 0001:0005ab80       ?apply@?$PairSet@USmallTypes@Layout@OT@@@GPOS_impl@Layout@OT@@QBE_NPAUhb_ot_apply_context_t@4@PBUValueFormat@234@I@Z 1005bb80 f i hb-ot-layout.obj
 0001:0005ae30       ?apply@?$Rule@USmallTypes@Layout@OT@@@OT@@QBE_NPAUhb_ot_apply_context_t@2@ABUContextApplyLookupContext@2@@Z 1005be30 f i hb-ot-layout.obj
 0001:0005b2b0       ?apply@?$RuleSet@USmallTypes@Layout@OT@@@OT@@QBE_NPAUhb_ot_apply_context_t@2@ABUContextApplyLookupContext@2@@Z 1005c2b0 f i hb-ot-layout.obj
 0001:0005bac0       ?apply@?$Sequence@USmallTypes@Layout@OT@@@GSUB_impl@Layout@OT@@QBE_NPAUhb_ot_apply_context_t@4@@Z 1005cac0 f i hb-ot-layout.obj
 0001:0005bda0       ?apply@?$SingleSubstFormat1_3@USmallTypes@Layout@OT@@@GSUB_impl@Layout@OT@@QBE_NPAUhb_ot_apply_context_t@4@@Z 1005cda0 f i hb-ot-layout.obj
 0001:0005be90       ?apply@?$SingleSubstFormat2_4@USmallTypes@Layout@OT@@@GSUB_impl@Layout@OT@@QBE_NPAUhb_ot_apply_context_t@4@@Z 1005ce90 f i hb-ot-layout.obj
 0001:0005bfd0       ?apply@ChainContextFormat3@OT@@QBE_NPAUhb_ot_apply_context_t@2@@Z 1005cfd0 f i hb-ot-layout.obj
 0001:0005c910       ?apply@ContextFormat3@OT@@QBE_NPAUhb_ot_apply_context_t@2@@Z 1005d910 f i hb-ot-layout.obj
 0001:0005cdc0       ?apply@CursivePosFormat1@GPOS_impl@Layout@OT@@QBE_NPAUhb_ot_apply_context_t@4@@Z 1005ddc0 f i hb-ot-layout.obj
 0001:0005d680       ?apply@MarkArray@GPOS_impl@Layout@OT@@QBE_NPAUhb_ot_apply_context_t@4@IIABUAnchorMatrix@234@II@Z 1005e680 f i hb-ot-layout.obj
 0001:0005d950       ?apply@ReverseChainSingleSubstFormat1@GSUB_impl@Layout@OT@@QBE_NPAUhb_ot_apply_context_t@4@@Z 1005e950 f i hb-ot-layout.obj
 0001:0005df10       ?apply@SinglePosFormat1@GPOS_impl@Layout@OT@@QBE_NPAUhb_ot_apply_context_t@4@@Z 1005ef10 f i hb-ot-layout.obj
 0001:0005e000       ?apply@SinglePosFormat2@GPOS_impl@Layout@OT@@QBE_NPAUhb_ot_apply_context_t@4@@Z 1005f000 f i hb-ot-layout.obj
 0001:0005e880       ?apply_value@ValueFormat@GPOS_impl@Layout@OT@@QBE_NPAUhb_ot_apply_context_t@4@PBXPBU?$IntType@G$01@4@AAUhb_glyph_position_t@@@Z 1005f880 f i hb-ot-layout.obj
 0001:0005ebb0       ?find_index@FeatureVariations@OT@@QBE_NPBHIPAI@Z 1005fbb0 f i hb-ot-layout.obj
 0001:0005ed40       ?find_lang_sys_index@Script@OT@@QBE_NIPAI@Z 1005fd40 f i hb-ot-layout.obj
 0001:0005edd0       ?find_script_index@GSUBGPOS@OT@@QBE_NIPAI@Z 1005fdd0 f i hb-ot-layout.obj
 0001:0005eea0       ?get_accel@?$accelerator_t@UGPOS@Layout@OT@@@GSUBGPOS@OT@@QBEPAUhb_ot_layout_lookup_accelerator_t@3@I@Z 1005fea0 f i hb-ot-layout.obj
 0001:0005ef30       ?get_accel@?$accelerator_t@UGSUB@Layout@OT@@@GSUBGPOS@OT@@QBEPAUhb_ot_layout_lookup_accelerator_t@3@I@Z 1005ff30 f i hb-ot-layout.obj
 0001:0005efc0       ?get_anchor@Anchor@GPOS_impl@Layout@OT@@QBEXPAUhb_ot_apply_context_t@4@IPAM1@Z 1005ffc0 f i hb-ot-layout.obj
 0001:0005f170       ?get_anchor@AnchorFormat3@GPOS_impl@Layout@OT@@QBEXPAUhb_ot_apply_context_t@4@IPAM1@Z 10060170 f i hb-ot-layout.obj
 0001:0005f360       ?get_coverage@ChainContextFormat3@OT@@QBEABUCoverage@Common@Layout@2@XZ 10060360 f i hb-ot-layout.obj
 0001:0005f3d0       ?get_delta@HintingDevice@OT@@ABEHIH@Z 100603d0 f i hb-ot-layout.obj
 0001:0005f4c0       ?get_device@ValueFormat@GPOS_impl@Layout@OT@@CAABUDevice@4@PBU?$IntType@G$01@4@PA_NPBXAAUhb_sanitize_context_t@@@Z 100604c0 f i hb-ot-layout.obj
 0001:0005f570       ?get_feature@GSUBGPOS@OT@@QBEABUFeature@2@I@Z 10060570 f i hb-ot-layout.obj
 0001:0005f600       ?get_feature_tag@GSUBGPOS@OT@@QBEII@Z 10060600 f i hb-ot-layout.obj
 0001:0005f6a0       ?get_feature_variation@GSUBGPOS@OT@@QBEABUFeature@2@II@Z 100606a0 f i hb-ot-layout.obj
 0001:0005f7d0       ?get_feature_variations@GSUBGPOS@OT@@QBEABUFeatureVariations@2@XZ 100607d0 f i hb-ot-layout.obj
 0001:0005f830       ?get_glyph_props@accelerator_t@GDEF@OT@@QBEII@Z 10060830 f i hb-ot-layout.obj
 0001:0005f9e0       ?get_indexes@IndexArray@OT@@QBEIIPAI0@Z 100609e0 f i hb-ot-layout.obj
 0001:0005fad0       ?get_kerning@accelerator_t@?$KerxSubTableFormat2@UKernAATSubTableHeader@OT@@@AAT@@QBEHII@Z 10060ad0 f i hb-ot-layout.obj
 0001:0005fbd0       ?get_kerning@accelerator_t@?$KerxSubTableFormat2@UKernOTSubTableHeader@OT@@@AAT@@QBEHII@Z 10060bd0 f i hb-ot-layout.obj
 0001:0005fcd0       ?get_lang_sys@Script@OT@@QBEABULangSys@2@I@Z 10060cd0 f i hb-ot-layout.obj
 0001:0005fd40       ?get_len@ValueFormat@GPOS_impl@Layout@OT@@QBEIXZ 10060d40 f i hb-ot-layout.obj
 0001:0005fd80       ?get_lookup@GSUBGPOS@OT@@QBEABULookup@2@I@Z 10060d80 f i hb-ot-layout.obj
 0001:0005fe10       ?get_lookup_count@GSUBGPOS@OT@@QBEIXZ 10060e10 f i hb-ot-layout.obj
 0001:0005fe70       ?get_population@Coverage@Common@Layout@OT@@QBEIXZ 10060e70 f i hb-ot-layout.obj
 0001:0005ff10       ?get_props@Lookup@OT@@QBEIXZ 10060f10 f i hb-ot-layout.obj
 0001:0005ff60       ?get_script@GSUBGPOS@OT@@QBEABUScript@2@I@Z 10060f60 f i hb-ot-layout.obj
 0001:0005fff0       ?get_stored@?$hb_lazy_loader_t@UGPOS_accelerator_t@OT@@U?$hb_face_lazy_loader_t@UGPOS_accelerator_t@OT@@$0BK@@@Uhb_face_t@@$0BK@U12@@@QBEPAUGPOS_accelerator_t@OT@@XZ 10060ff0 f i hb-ot-layout.obj
 0001:000601d0       ?get_stored@?$hb_lazy_loader_t@UGSUB_accelerator_t@OT@@U?$hb_face_lazy_loader_t@UGSUB_accelerator_t@OT@@$0BJ@@@Uhb_face_t@@$0BJ@U12@@@QBEPAUGSUB_accelerator_t@OT@@XZ 100611d0 f i hb-ot-layout.obj
 0001:000603b0       ?get_stored@?$hb_lazy_loader_t@Ukern@OT@@U?$hb_table_lazy_loader_t@Ukern@OT@@$0BH@$00@@Uhb_face_t@@$0BH@Uhb_blob_t@@@@QBEPAUhb_blob_t@@XZ 100613b0 f i hb-ot-layout.obj
 0001:000604e0       ?get_type@?$Extension@UExtensionSubst@GSUB_impl@Layout@OT@@@OT@@QBEIXZ 100614e0 f i hb-ot-layout.obj
 0001:000604e0       ?get_type@?$Extension@UExtensionPos@GPOS_impl@Layout@OT@@@OT@@QBEIXZ 100614e0 f i hb-ot-layout.obj
 0001:00060510       ?get_x_delta@Device@OT@@QBEHPAUhb_font_t@@ABUVariationStore@2@PAM@Z 10061510 f i hb-ot-layout.obj
 0001:000605e0       ?get_y_delta@Device@OT@@QBEHPAUhb_font_t@@ABUVariationStore@2@PAM@Z 100615e0 f i hb-ot-layout.obj
 0001:000606b0       ?hb_ot_layout_has_cross_kerning@@YA_NPAUhb_face_t@@@Z 100616b0 f   hb-ot-layout.obj
 0001:00060780       ?hb_ot_layout_has_kerning@@YA_NPAUhb_face_t@@@Z 10061780 f   hb-ot-layout.obj
 0001:000607c0       ?hb_ot_layout_has_machine_kerning@@YA_NPAUhb_face_t@@@Z 100617c0 f   hb-ot-layout.obj
 0001:00060890       ?hb_ot_layout_kern@@YAXPBUhb_ot_shape_plan_t@@PAUhb_font_t@@PAUhb_buffer_t@@@Z 10061890 f   hb-ot-layout.obj
 0001:00060930       ?hb_ot_layout_position_finish_offsets@@YAXPAUhb_font_t@@PAUhb_buffer_t@@@Z 10061930 f   hb-ot-layout.obj
 0001:00060a10       ?hb_ot_layout_position_start@@YAXPAUhb_font_t@@PAUhb_buffer_t@@@Z 10061a10 f   hb-ot-layout.obj
 0001:00060a40       ?hb_ot_layout_substitute_lookup@@YAXPAUhb_ot_apply_context_t@OT@@ABUSubstLookup@GSUB_impl@Layout@2@ABUhb_ot_layout_lookup_accelerator_t@2@@Z 10061a40 f   hb-ot-layout.obj
 0001:00060a50       ?hb_ot_layout_substitute_start@@YAXPAUhb_font_t@@PAUhb_buffer_t@@@Z 10061a50 f   hb-ot-layout.obj
 0001:00060a60       ?hb_ot_layout_table_find_feature@@YA_NPAUhb_face_t@@IIPAI@Z 10061a60 f   hb-ot-layout.obj
 0001:00060b90       ?is_blocklisted@GDEF@OT@@QBE_NPAUhb_blob_t@@PAUhb_face_t@@@Z 10061b90 f   hb-ot-layout.obj
 0001:00060f40       ?kern@?$hb_kern_machine_t@U?$KernSubTableFormat3@UKernAATSubTableHeader@OT@@@OT@@@OT@@QBEXPAUhb_font_t@@PAUhb_buffer_t@@I_N@Z 10061f40 f i hb-ot-layout.obj
 0001:000614f0       ?kern@?$hb_kern_machine_t@Uaccelerator_t@?$KerxSubTableFormat0@UKernAATSubTableHeader@OT@@@AAT@@@OT@@QBEXPAUhb_font_t@@PAUhb_buffer_t@@I_N@Z 100624f0 f i hb-ot-layout.obj
 0001:00061a10       ?kern@?$hb_kern_machine_t@Uaccelerator_t@?$KerxSubTableFormat0@UKernOTSubTableHeader@OT@@@AAT@@@OT@@QBEXPAUhb_font_t@@PAUhb_buffer_t@@I_N@Z 10062a10 f i hb-ot-layout.obj
 0001:00061f30       ?kern@?$hb_kern_machine_t@Uaccelerator_t@?$KerxSubTableFormat2@UKernAATSubTableHeader@OT@@@AAT@@@OT@@QBEXPAUhb_font_t@@PAUhb_buffer_t@@I_N@Z 10062f30 f i hb-ot-layout.obj
 0001:00062420       ?kern@?$hb_kern_machine_t@Uaccelerator_t@?$KerxSubTableFormat2@UKernOTSubTableHeader@OT@@@AAT@@@OT@@QBEXPAUhb_font_t@@PAUhb_buffer_t@@I_N@Z 10063420 f i hb-ot-layout.obj
 0001:00062c30       ___acrt_initialize         10063c30 f   MSVCRT:ucrt_stubs.obj
 0001:00062c30       ___vcrt_uninitialize_critical 10063c30 f   MSVCRT:ucrt_stubs.obj
 0001:00062c30       ___vcrt_uninitialize       10063c30 f   MSVCRT:ucrt_stubs.obj
 0001:00062c30       ___scrt_stub_for_acrt_thread_attach 10063c30 f   MSVCRT:ucrt_stubs.obj
 0001:00062c30       ___acrt_uninitialize_critical 10063c30 f   MSVCRT:ucrt_stubs.obj
 0001:00062c30       ___scrt_stub_for_acrt_uninitialize 10063c30 f   MSVCRT:ucrt_stubs.obj
 0001:00062c30       ___acrt_thread_detach      10063c30 f   MSVCRT:ucrt_stubs.obj
 0001:00062c30       ___vcrt_thread_detach      10063c30 f   MSVCRT:ucrt_stubs.obj
 0001:00062c30       ___acrt_uninitialize       10063c30 f   MSVCRT:ucrt_stubs.obj
 0001:00062c30       ___acrt_thread_attach      10063c30 f   MSVCRT:ucrt_stubs.obj
 0001:00062c30       ___scrt_stub_for_acrt_thread_detach 10063c30 f   MSVCRT:ucrt_stubs.obj
 0001:00062c30       ___scrt_stub_for_acrt_uninitialize_critical 10063c30 f   MSVCRT:ucrt_stubs.obj
 0001:00062c30       ___vcrt_thread_attach      10063c30 f   MSVCRT:ucrt_stubs.obj
 0001:00062c30       ___vcrt_initialize         10063c30 f   MSVCRT:ucrt_stubs.obj
 0001:00062c30       ___scrt_stub_for_acrt_initialize 10063c30 f   MSVCRT:ucrt_stubs.obj
 0001:00062dc0       ?position@hb_ot_map_t@@QBEXPBUhb_ot_shape_plan_t@@PAUhb_font_t@@PAUhb_buffer_t@@@Z 10063dc0 f   hb-ot-layout.obj
 0001:00063010       ?sanitize@?$ChainContextFormat2_5@USmallTypes@Layout@OT@@@OT@@QBE_NPAUhb_sanitize_context_t@@@Z 10064010 f i hb-ot-layout.obj
 0001:00063230       ?sanitize@?$ContextFormat2_5@USmallTypes@Layout@OT@@@OT@@QBE_NPAUhb_sanitize_context_t@@@Z 10064230 f i hb-ot-layout.obj
 0001:000633a0       ?sanitize@?$KerxSubTableFormat2@UKernAATSubTableHeader@OT@@@AAT@@QBE_NPAUhb_sanitize_context_t@@@Z 100643a0 f i hb-ot-layout.obj
 0001:000634f0       ?sanitize@?$KerxSubTableFormat2@UKernOTSubTableHeader@OT@@@AAT@@QBE_NPAUhb_sanitize_context_t@@@Z 100644f0 f i hb-ot-layout.obj
 0001:00063640       ?sanitize@?$KerxTable@UKernAAT@OT@@@AAT@@QBE_NPAUhb_sanitize_context_t@@@Z 10064640 f i hb-ot-layout.obj
 0001:00063830       ?sanitize@?$KerxTable@UKernOT@OT@@@AAT@@QBE_NPAUhb_sanitize_context_t@@@Z 10064830 f i hb-ot-layout.obj
 0001:00063a00       ?sanitize@?$MarkMarkPosFormat1_2@USmallTypes@Layout@OT@@@GPOS_impl@Layout@OT@@QBE_NPAUhb_sanitize_context_t@@@Z 10064a00 f i hb-ot-layout.obj
 0001:00063a00       ?sanitize@?$MarkBasePosFormat1_2@USmallTypes@Layout@OT@@@GPOS_impl@Layout@OT@@QBE_NPAUhb_sanitize_context_t@@@Z 10064a00 f i hb-ot-layout.obj
 0001:00063c00       ?sanitize@?$MarkLigPosFormat1_2@USmallTypes@Layout@OT@@@GPOS_impl@Layout@OT@@QBE_NPAUhb_sanitize_context_t@@@Z 10064c00 f i hb-ot-layout.obj
 0001:00063e00       ?sanitize@?$PairPosFormat1_3@USmallTypes@Layout@OT@@@GPOS_impl@Layout@OT@@QBE_NPAUhb_sanitize_context_t@@@Z 10064e00 f i hb-ot-layout.obj
 0001:00064010       ?sanitize@?$PairPosFormat2_4@USmallTypes@Layout@OT@@@GPOS_impl@Layout@OT@@QBE_NPAUhb_sanitize_context_t@@@Z 10065010 f i hb-ot-layout.obj
 0001:000642b0       ?sanitize@?$PairSet@USmallTypes@Layout@OT@@@GPOS_impl@Layout@OT@@QBE_NPAUhb_sanitize_context_t@@PBUsanitize_closure_t@1234@@Z 100652b0 f i hb-ot-layout.obj
 0001:00064420       ?sanitize@?$RecordListOf@UFeature@OT@@@OT@@QBE_NPAUhb_sanitize_context_t@@@Z 10065420 f i hb-ot-layout.obj
 0001:00064580       ?sanitize@?$Rule@USmallTypes@Layout@OT@@@OT@@QBE_NPAUhb_sanitize_context_t@@@Z 10065580 f i hb-ot-layout.obj
 0001:00064690       ?sanitize@?$SingleSubstFormat1_3@USmallTypes@Layout@OT@@@GSUB_impl@Layout@OT@@QBE_NPAUhb_sanitize_context_t@@@Z 10065690 f i hb-ot-layout.obj
 0001:000647b0       ?sanitize@AnchorFormat3@GPOS_impl@Layout@OT@@QBE_NPAUhb_sanitize_context_t@@@Z 100657b0 f i hb-ot-layout.obj
 0001:000648e0       ?sanitize@AnchorMatrix@GPOS_impl@Layout@OT@@QBE_NPAUhb_sanitize_context_t@@I@Z 100658e0 f i hb-ot-layout.obj
 0001:00064a70       ?sanitize@ChainContextFormat3@OT@@QBE_NPAUhb_sanitize_context_t@@@Z 10065a70 f i hb-ot-layout.obj
 0001:00064cc0       ?sanitize@ContextFormat3@OT@@QBE_NPAUhb_sanitize_context_t@@@Z 10065cc0 f i hb-ot-layout.obj
 0001:00064ec0       ?sanitize@CursivePosFormat1@GPOS_impl@Layout@OT@@QBE_NPAUhb_sanitize_context_t@@@Z 10065ec0 f i hb-ot-layout.obj
 0001:00065060       ?sanitize@Feature@OT@@QBE_NPAUhb_sanitize_context_t@@PBURecord_sanitize_closure_t@2@@Z 10066060 f i hb-ot-layout.obj
 0001:00065290       ?sanitize@FeatureParamsSize@OT@@QBE_NPAUhb_sanitize_context_t@@@Z 10066290 f i hb-ot-layout.obj
 0001:000653b0       ?sanitize@FeatureTableSubstitution@OT@@QBE_NPAUhb_sanitize_context_t@@@Z 100663b0 f i hb-ot-layout.obj
 0001:00065510       ?sanitize@FeatureVariations@OT@@QBE_NPAUhb_sanitize_context_t@@@Z 10066510 f i hb-ot-layout.obj
 0001:00065680       ?sanitize@GPOS@Layout@OT@@QBE_NPAUhb_sanitize_context_t@@@Z 10066680 f i hb-ot-layout.obj
 0001:000656c0       ?sanitize@GSUB@Layout@OT@@QBE_NPAUhb_sanitize_context_t@@@Z 100666c0 f i hb-ot-layout.obj
 0001:00065700       ?sanitize@KernAATSubTableHeader@OT@@QBE_NPAUhb_sanitize_context_t@@@Z 10066700 f i hb-ot-layout.obj
 0001:00065770       ?sanitize@KernOTSubTableHeader@OT@@QBE_NPAUhb_sanitize_context_t@@@Z 10066770 f i hb-ot-layout.obj
 0001:000657e0       ?sanitize@LangSys@OT@@QBE_NPAUhb_sanitize_context_t@@PBURecord_sanitize_closure_t@2@@Z 100667e0 f i hb-ot-layout.obj
 0001:00065860       ?sanitize@ReverseChainSingleSubstFormat1@GSUB_impl@Layout@OT@@QBE_NPAUhb_sanitize_context_t@@@Z 10066860 f i hb-ot-layout.obj
 0001:00065a50       ?sanitize@Script@OT@@QBE_NPAUhb_sanitize_context_t@@PBURecord_sanitize_closure_t@2@@Z 10066a50 f i hb-ot-layout.obj
 0001:00065be0       ?sanitize@SinglePosFormat1@GPOS_impl@Layout@OT@@QBE_NPAUhb_sanitize_context_t@@@Z 10066be0 f i hb-ot-layout.obj
 0001:00065dc0       ?sanitize@SinglePosFormat2@GPOS_impl@Layout@OT@@QBE_NPAUhb_sanitize_context_t@@@Z 10066dc0 f i hb-ot-layout.obj
 0001:00065f20       ?sanitize@kern@OT@@QBE_NPAUhb_sanitize_context_t@@@Z 10066f20 f i hb-ot-layout.obj
 0001:00065f70       ?sanitize_shallow@?$ArrayOf@UFeatureVariationRecord@OT@@U?$IntType@I$03@2@@OT@@QBE_NPAUhb_sanitize_context_t@@@Z 10066f70 f i hb-ot-layout.obj
 0001:00066030       ?sanitize_shallow@?$ArrayOf@UKernPair@AAT@@U?$BinSearchHeader@U?$IntType@G$01@OT@@@OT@@@OT@@QBE_NPAUhb_sanitize_context_t@@@Z 10067030 f i hb-ot-layout.obj
 0001:00066120       ?sanitize_shallow@?$HeadlessArrayOf@UHBGlyphID16@OT@@U?$IntType@G$01@2@@OT@@ABE_NPAUhb_sanitize_context_t@@@Z 10067120 f i hb-ot-layout.obj
 0001:000661d0       ?sanitize_value_devices@ValueFormat@GPOS_impl@Layout@OT@@ABE_NPAUhb_sanitize_context_t@@PBXPBU?$IntType@G$01@4@@Z 100671d0 f i hb-ot-layout.obj
 0001:000663b0       ?sanitize_values_stride_unsafe@ValueFormat@GPOS_impl@Layout@OT@@QBE_NPAUhb_sanitize_context_t@@PBXPBU?$IntType@G$01@4@II@Z 100673b0 f i hb-ot-layout.obj
 0001:00066400       ?substitute@hb_ot_map_t@@QBEXPBUhb_ot_shape_plan_t@@PAUhb_font_t@@PAUhb_buffer_t@@@Z 10067400 f   hb-ot-layout.obj
 0001:000664a0       ?transition@driver_context_t@?$KerxSubTableFormat1@UKernAATSubTableHeader@OT@@@AAT@@QAEXPAU?$StateTableDriver@UObsoleteTypes@AAT@@X@3@ABU?$Entry@X@3@@Z 100674a0 f i hb-ot-layout.obj
 0001:00066750       ?would_apply@?$ChainRuleSet@USmallTypes@Layout@OT@@@OT@@QBE_NPAUhb_would_apply_context_t@2@ABUChainContextApplyLookupContext@2@@Z 10067750 f i hb-ot-layout.obj
 0001:000668c0       ?would_apply@?$LigatureSubstFormat1_2@USmallTypes@Layout@OT@@@GSUB_impl@Layout@OT@@QBE_NPAUhb_would_apply_context_t@4@@Z 100678c0 f i hb-ot-layout.obj
 0001:00066aa0       ?would_apply@?$RuleSet@USmallTypes@Layout@OT@@@OT@@QBE_NPAUhb_would_apply_context_t@2@ABUContextApplyLookupContext@2@@Z 10067aa0 f i hb-ot-layout.obj
 0001:00066b90       _hb_ot_layout_collect_features_map 10067b90 f   hb-ot-layout.obj
 0001:00066cd0       _hb_ot_layout_feature_with_variations_get_lookups 10067cd0 f   hb-ot-layout.obj
 0001:00066d10       _hb_ot_layout_has_glyph_classes 10067d10 f   hb-ot-layout.obj
 0001:00066d70       _hb_ot_layout_has_positioning 10067d70 f   hb-ot-layout.obj
 0001:00066dc0       _hb_ot_layout_has_substitution 10067dc0 f   hb-ot-layout.obj
 0001:00066e10       _hb_ot_layout_language_find_feature 10067e10 f   hb-ot-layout.obj
 0001:00066f70       _hb_ot_layout_language_get_required_feature 10067f70 f   hb-ot-layout.obj
 0001:00067000       _hb_ot_layout_lookup_would_substitute 10068000 f   hb-ot-layout.obj
 0001:00067180       _hb_ot_layout_script_select_language 10068180 f   hb-ot-layout.obj
 0001:00067290       _hb_ot_layout_table_find_feature_variations 10068290 f   hb-ot-layout.obj
 0001:000672c0       _hb_ot_layout_table_get_lookup_count 100682c0 f   hb-ot-layout.obj
 0001:000672e0       _hb_ot_layout_table_select_script 100682e0 f   hb-ot-layout.obj
 0001:000674b0       ??0hb_ot_map_builder_t@@QAE@PAUhb_face_t@@ABUhb_segment_properties_t@@@Z 100684b0 f   hb-ot-map.obj
 0001:000675e0       ??1hb_ot_map_builder_t@@QAE@XZ 100685e0 f   hb-ot-map.obj
 0001:000676c0       ?add_feature@hb_ot_map_builder_t@@QAEXIW4hb_ot_map_feature_flags_t@@I@Z 100686c0 f   hb-ot-map.obj
 0001:000677a0       ?add_lookups@hb_ot_map_builder_t@@AAEXAAUhb_ot_map_t@@IIII_N111I@Z 100687a0 f   hb-ot-map.obj
 0001:00067990       ?add_pause@hb_ot_map_builder_t@@AAEXIP6A_NPBUhb_ot_shape_plan_t@@PAUhb_font_t@@PAUhb_buffer_t@@@Z@Z 10068990 f   hb-ot-map.obj
 0001:00067aa0       ?alloc@?$hb_vector_t@Ufeature_info_t@hb_ot_map_builder_t@@$0A@@@QAE_NI_N@Z 10068aa0 f i hb-ot-map.obj
 0001:00067b50       ?cmp@feature_info_t@hb_ot_map_builder_t@@SAHPBX0@Z 10068b50 f i hb-ot-map.obj
 0001:00067b80       ?cmp@feature_map_t@hb_ot_map_t@@SAHPBX0@Z 10068b80 f i hb-ot-map.obj
 0001:00067ba0       ?cmp@lookup_map_t@hb_ot_map_t@@SAHPBX0@Z 10068ba0 f i hb-ot-map.obj
 0001:00067bc0       ?compile@hb_ot_map_builder_t@@QAEXAAUhb_ot_map_t@@ABUhb_ot_shape_plan_key_t@@@Z 10068bc0 f   hb-ot-map.obj
 0001:00068610       ?has_feature@hb_ot_map_builder_t@@QAE_NI@Z 10069610 f   hb-ot-map.obj
 0001:00068660       ??$sanitize_blob@UMVAR@OT@@@hb_sanitize_context_t@@QAEPAUhb_blob_t@@PAU1@@Z 10069660 f i hb-ot-metrics.obj
 0001:000689a0       ?_hb_ot_metrics_get_position_common@@YA_NPAUhb_font_t@@W4hb_ot_metrics_tag_t@@PAH@Z 100699a0 f   hb-ot-metrics.obj
 0001:00068fb0       ?get@?$hb_lazy_loader_t@UMVAR@OT@@U?$hb_table_lazy_loader_t@UMVAR@OT@@$0BG@$00@@Uhb_face_t@@$0BG@Uhb_blob_t@@@@QBEPBUMVAR@OT@@XZ 10069fb0 f i hb-ot-metrics.obj
 0001:000690c0       ?get_var@MVAR@OT@@QBEMIPBHI@Z 1006a0c0 f i hb-ot-metrics.obj
 0001:000691f0       ?has_data@OS2@OT@@QBE_NXZ  1006a1f0 f i hb-ot-metrics.obj
 0001:00069250       ?sanitize@MVAR@OT@@QBE_NPAUhb_sanitize_context_t@@@Z 1006a250 f i hb-ot-metrics.obj
 0001:000693a0       ?_hb_ot_shape_fallback_kern@@YAXPBUhb_ot_shape_plan_t@@PAUhb_font_t@@PAUhb_buffer_t@@@Z 1006a3a0 f   hb-ot-shape-fallback.obj
 0001:00069450       ?_hb_ot_shape_fallback_mark_position@@YAXPBUhb_ot_shape_plan_t@@PAUhb_font_t@@PAUhb_buffer_t@@_N@Z 1006a450 f   hb-ot-shape-fallback.obj
 0001:00069560       ?_hb_ot_shape_fallback_mark_position_recategorize_marks@@YAXPBUhb_ot_shape_plan_t@@PAUhb_font_t@@PAUhb_buffer_t@@@Z 1006a560 f   hb-ot-shape-fallback.obj
 0001:000697c0       ?_hb_ot_shape_fallback_spaces@@YAXPBUhb_ot_shape_plan_t@@PAUhb_font_t@@PAUhb_buffer_t@@@Z 1006a7c0 f   hb-ot-shape-fallback.obj
 0001:00069a10       ?kern@?$hb_kern_machine_t@Uhb_ot_shape_fallback_kern_driver_t@@@OT@@QBEXPAUhb_font_t@@PAUhb_buffer_t@@I_N@Z 1006aa10 f i hb-ot-shape-fallback.obj
 0001:0006a860       ?_hb_ot_shape_normalize@@YAXPBUhb_ot_shape_plan_t@@PAUhb_buffer_t@@PAUhb_font_t@@@Z 1006b860 f   hb-ot-shape-normalize.obj
 0001:0006ba00       ??$bsearch@I$00$0A@@?$hb_vector_t@Ufeature_map_t@hb_ot_map_t@@$00@@QBEPBUfeature_map_t@hb_ot_map_t@@ABIPBU12@@Z 1006ca00 f i hb-ot-shape.obj
 0001:0006ba70       ?compile@hb_ot_shape_planner_t@@QAEXAAUhb_ot_shape_plan_t@@ABUhb_ot_shape_plan_key_t@@@Z 1006ca70 f   hb-ot-shape.obj
 0001:0006be30       ?fini@hb_ot_map_t@@QAEXXZ  1006ce30 f i hb-ot-shape.obj
 0001:0006bed0       ?fini@hb_ot_shape_plan_t@@QAEXXZ 1006ced0 f   hb-ot-shape.obj
 0001:0006bef0       ?get_1_mask@hb_ot_map_t@@QBEII@Z 1006cef0 f i hb-ot-shape.obj
 0001:0006bf10       ?has_glyph@hb_font_t@@QAE_NI@Z 1006cf10 f i hb-ot-shape.obj
 0001:0006da60       ?init0@hb_ot_shape_plan_t@@QAE_NPAUhb_face_t@@PBUhb_shape_plan_key_t@@@Z 1006ea60 f   hb-ot-shape.obj
 0001:0006dc20       __hb_ot_shape              1006ec20 f   hb-ot-shape.obj
 0001:0006dc70       ?data_create_arabic@@YAPAXPBUhb_ot_shape_plan_t@@@Z 1006ec70 f   hb-ot-shaper-arabic.obj
 0001:0006dd80       ?data_destroy_arabic@@YAXPAX@Z 1006ed80 f   hb-ot-shaper-arabic.obj
 0001:0006e1a0       ??$add_link@U?$OffsetTo@UCoverage@Common@Layout@OT@@U?$IntType@G$01@4@$00@OT@@@hb_serialize_context_t@@QAEXAAU?$OffsetTo@UCoverage@Common@Layout@OT@@U?$IntType@G$01@4@$00@OT@@IW4whence_t@0@I@Z 1006f1a0 f i hb-ot-shaper-arabic.obj
 0001:0006e1a0       ??$add_link@U?$OffsetTo@U?$Ligature@USmallTypes@Layout@OT@@@GSUB_impl@Layout@OT@@U?$IntType@G$01@4@$00@OT@@@hb_serialize_context_t@@QAEXAAU?$OffsetTo@U?$Ligature@USmallTypes@Layout@OT@@@GSUB_impl@Layout@OT@@U?$IntType@G$01@4@$00@OT@@IW4whence_t@0@I@Z 1006f1a0 f i hb-ot-shaper-arabic.obj
 0001:0006e1a0       ??$add_link@U?$OffsetTo@USubstLookupSubTable@GSUB_impl@Layout@OT@@U?$IntType@G$01@4@$00@OT@@@hb_serialize_context_t@@QAEXAAU?$OffsetTo@USubstLookupSubTable@GSUB_impl@Layout@OT@@U?$IntType@G$01@4@$00@OT@@IW4whence_t@0@I@Z 1006f1a0 f i hb-ot-shaper-arabic.obj
 0001:0006e1a0       ??$add_link@U?$OffsetTo@U?$LigatureSet@USmallTypes@Layout@OT@@@GSUB_impl@Layout@OT@@U?$IntType@G$01@4@$00@OT@@@hb_serialize_context_t@@QAEXAAU?$OffsetTo@U?$LigatureSet@USmallTypes@Layout@OT@@@GSUB_impl@Layout@OT@@U?$IntType@G$01@4@$00@OT@@IW4whence_t@0@I@Z 1006f1a0 f i hb-ot-shaper-arabic.obj
 0001:0006eb90       ??$copy@USubstLookup@GSUB_impl@Layout@OT@@@hb_serialize_context_t@@QBEPAUSubstLookup@GSUB_impl@Layout@OT@@XZ 1006fb90 f i hb-ot-shaper-arabic.obj
 0001:0006ebf0       ??$extend@ULookup@OT@@$$V@hb_serialize_context_t@@QAEPAULookup@OT@@PAU12@@Z 1006fbf0 f i hb-ot-shaper-arabic.obj
 0001:0006ec80       ??$extend_min@U?$CoverageFormat2_4@USmallTypes@Layout@OT@@@Common@Layout@OT@@@hb_serialize_context_t@@QAEPAU?$CoverageFormat2_4@USmallTypes@Layout@OT@@@Common@Layout@OT@@PAU1234@@Z 1006fc80 f i hb-ot-shaper-arabic.obj
 0001:0006ec80       ??$extend_min@U?$Ligature@USmallTypes@Layout@OT@@@GSUB_impl@Layout@OT@@@hb_serialize_context_t@@QAEPAU?$Ligature@USmallTypes@Layout@OT@@@GSUB_impl@Layout@OT@@PAU1234@@Z 1006fc80 f i hb-ot-shaper-arabic.obj
 0001:0006ecf0       ??$extend_min@U?$IntType@G$01@OT@@@hb_serialize_context_t@@QAEPAU?$IntType@G$01@OT@@AAU12@@Z 1006fcf0 f i hb-ot-shaper-arabic.obj
 0001:0006ecf0       ??$extend_min@U?$LigatureSet@USmallTypes@Layout@OT@@@GSUB_impl@Layout@OT@@@hb_serialize_context_t@@QAEPAU?$LigatureSet@USmallTypes@Layout@OT@@@GSUB_impl@Layout@OT@@PAU1234@@Z 1006fcf0 f i hb-ot-shaper-arabic.obj
 0001:0006ecf0       ??$extend_min@UCoverage@Common@Layout@OT@@@hb_serialize_context_t@@QAEPAUCoverage@Common@Layout@OT@@PAU1234@@Z 1006fcf0 f i hb-ot-shaper-arabic.obj
 0001:0006ed60       ??$extend_min@U?$LigatureSubstFormat1_2@USmallTypes@Layout@OT@@@GSUB_impl@Layout@OT@@@hb_serialize_context_t@@QAEPAU?$LigatureSubstFormat1_2@USmallTypes@Layout@OT@@@GSUB_impl@Layout@OT@@PAU1234@@Z 1006fd60 f i hb-ot-shaper-arabic.obj
 0001:0006ed60       ??$extend_min@ULookup@OT@@@hb_serialize_context_t@@QAEPAULookup@OT@@PAU12@@Z 1006fd60 f i hb-ot-shaper-arabic.obj
 0001:0006ed60       ??$extend_min@U?$SingleSubstFormat1_3@USmallTypes@Layout@OT@@@GSUB_impl@Layout@OT@@@hb_serialize_context_t@@QAEPAU?$SingleSubstFormat1_3@USmallTypes@Layout@OT@@@GSUB_impl@Layout@OT@@PAU1234@@Z 1006fd60 f i hb-ot-shaper-arabic.obj
 0001:0006ed60       ??$extend_min@U?$SingleSubstFormat2_4@USmallTypes@Layout@OT@@@GSUB_impl@Layout@OT@@@hb_serialize_context_t@@QAEPAU?$SingleSubstFormat2_4@USmallTypes@Layout@OT@@@GSUB_impl@Layout@OT@@PAU1234@@Z 1006fd60 f i hb-ot-shaper-arabic.obj
 0001:0006edd0       ??$extend_size@U?$ArrayOf@UHBGlyphID16@OT@@U?$IntType@G$01@2@@OT@@@hb_serialize_context_t@@QAEPAU?$ArrayOf@UHBGlyphID16@OT@@U?$IntType@G$01@2@@OT@@PAU12@I_N@Z 1006fdd0 f i hb-ot-shaper-arabic.obj
 0001:0006edd0       ??$extend_size@U?$HeadlessArrayOf@UHBGlyphID16@OT@@U?$IntType@G$01@2@@OT@@@hb_serialize_context_t@@QAEPAU?$HeadlessArrayOf@UHBGlyphID16@OT@@U?$IntType@G$01@2@@OT@@PAU12@I_N@Z 1006fdd0 f i hb-ot-shaper-arabic.obj
 0001:0006ef10       ??$serialize@U?$hb_map_iter_t@U?$hb_zip_iter_t@U?$hb_sorted_array_t@UHBGlyphID16@OT@@@@U?$hb_array_t@UHBGlyphID16@OT@@@@@@ABU<unnamed-type-hb_first>@@$00$0A@@@$0A@@?$CoverageFormat2_4@USmallTypes@Layout@OT@@@Common@Layout@OT@@AAE_NPAUhb_serialize_context_t@@U?$hb_map_iter_t@U?$hb_zip_iter_t@U?$hb_sorted_array_t@UHBGlyphID16@OT@@@@U?$hb_array_t@UHBGlyphID16@OT@@@@@@ABU<unnamed-type-hb_first>@@$00$0A@@@@Z 1006ff10 f i hb-ot-shaper-arabic.obj
 0001:0006f250       ??$serialize@U?$hb_map_iter_t@U?$hb_zip_iter_t@U?$hb_sorted_array_t@UHBGlyphID16@OT@@@@U?$hb_array_t@UHBGlyphID16@OT@@@@@@ABU<unnamed-type-hb_first>@@$00$0A@@@$0A@@Coverage@Common@Layout@OT@@QAE_NPAUhb_serialize_context_t@@U?$hb_map_iter_t@U?$hb_zip_iter_t@U?$hb_sorted_array_t@UHBGlyphID16@OT@@@@U?$hb_array_t@UHBGlyphID16@OT@@@@@@ABU<unnamed-type-hb_first>@@$00$0A@@@@Z 10070250 f i hb-ot-shaper-arabic.obj
 0001:0006f5f0       ??$serialize@U?$hb_sorted_array_t@$$CBUHBGlyphID16@OT@@@@$0A@@?$CoverageFormat2_4@USmallTypes@Layout@OT@@@Common@Layout@OT@@AAE_NPAUhb_serialize_context_t@@U?$hb_sorted_array_t@$$CBUHBGlyphID16@OT@@@@@Z 100705f0 f i hb-ot-shaper-arabic.obj
 0001:0006f7b0       ??$serialize@U?$hb_sorted_array_t@$$CBUHBGlyphID16@OT@@@@$0A@@Coverage@Common@Layout@OT@@QAE_NPAUhb_serialize_context_t@@U?$hb_sorted_array_t@$$CBUHBGlyphID16@OT@@@@@Z 100707b0 f i hb-ot-shaper-arabic.obj
 0001:0006f9b0       ??$serialize@U?$hb_zip_iter_t@U?$hb_sorted_array_t@UHBGlyphID16@OT@@@@U?$hb_array_t@UHBGlyphID16@OT@@@@@@$0A@@SingleSubst@GSUB_impl@Layout@OT@@QAE_NPAUhb_serialize_context_t@@U?$hb_zip_iter_t@U?$hb_sorted_array_t@UHBGlyphID16@OT@@@@U?$hb_array_t@UHBGlyphID16@OT@@@@@@@Z 100709b0 f i hb-ot-shaper-arabic.obj
 0001:0006fd70       ??$serialize_serialize@AAU?$hb_map_iter_t@U?$hb_zip_iter_t@U?$hb_sorted_array_t@UHBGlyphID16@OT@@@@U?$hb_array_t@UHBGlyphID16@OT@@@@@@ABU<unnamed-type-hb_first>@@$00$0A@@@@?$OffsetTo@UCoverage@Common@Layout@OT@@U?$IntType@G$01@4@$00@OT@@QAE_NPAUhb_serialize_context_t@@AAU?$hb_map_iter_t@U?$hb_zip_iter_t@U?$hb_sorted_array_t@UHBGlyphID16@OT@@@@U?$hb_array_t@UHBGlyphID16@OT@@@@@@ABU<unnamed-type-hb_first>@@$00$0A@@@@Z 10070d70 f i hb-ot-shaper-arabic.obj
 0001:0006fe20       ??$serialize_serialize@AAU?$hb_sorted_array_t@$$CBUHBGlyphID16@OT@@@@@?$OffsetTo@UCoverage@Common@Layout@OT@@U?$IntType@G$01@4@$00@OT@@QAE_NPAUhb_serialize_context_t@@AAU?$hb_sorted_array_t@$$CBUHBGlyphID16@OT@@@@@Z 10070e20 f i hb-ot-shaper-arabic.obj
 0001:0006fec0       ??$start_serialize@USubstLookup@GSUB_impl@Layout@OT@@@hb_serialize_context_t@@QAEPAUSubstLookup@GSUB_impl@Layout@OT@@XZ 10070ec0 f i hb-ot-shaper-arabic.obj
 0001:0006ff30       ??A?$ArrayOf@UManifestLookup@@U?$IntType@G$01@OT@@@OT@@QBEABUManifestLookup@@H@Z 10070f30 f i hb-ot-shaper-arabic.obj
 0001:0006ff60       ??D?$hb_iter_t@U?$hb_zip_iter_t@U?$hb_sorted_array_t@UHBGlyphID16@OT@@@@U?$hb_array_t@UHBGlyphID16@OT@@@@@@U?$hb_pair_t@AAUHBGlyphID16@OT@@AAU12@@@@@QAE?AU?$hb_pair_t@AAUHBGlyphID16@OT@@AAU12@@@XZ 10070f60 f i hb-ot-shaper-arabic.obj
 0001:00070f60       ?cmp@?$IntType@G$01@OT@@SAHPBU12@0@Z 10071f60 f i hb-ot-shaper-arabic.obj
 0001:00070fb0       ?cmp_range@?$RangeRecord@USmallTypes@Layout@OT@@@Common@Layout@OT@@SAHPBX0@Z 10071fb0 f i hb-ot-shaper-arabic.obj
 0001:00071050       ?discard_stale_objects@hb_serialize_context_t@@QAEXXZ 10072050 f i hb-ot-shaper-arabic.obj
 0001:00071200       ?end@?$hb_iter_t@U?$hb_map_iter_t@U?$hb_zip_iter_t@U?$hb_sorted_array_t@UHBGlyphID16@OT@@@@U?$hb_array_t@UHBGlyphID16@OT@@@@@@ABU<unnamed-type-hb_first>@@$00$0A@@@AAUHBGlyphID16@OT@@@@QBE?AU?$hb_map_iter_t@U?$hb_zip_iter_t@U?$hb_sorted_array_t@UHBGlyphID16@OT@@@@U?$hb_array_t@UHBGlyphID16@OT@@@@@@ABU<unnamed-type-hb_first>@@$00$0A@@@XZ 10072200 f i hb-ot-shaper-arabic.obj
 0001:00071450       ?pop_discard@hb_serialize_context_t@@QAEXXZ 10072450 f i hb-ot-shaper-arabic.obj
 0001:000714b0       ?push@?$hb_vector_t@Ulink_t@object_t@hb_serialize_context_t@@$0A@@@QAEPAUlink_t@object_t@hb_serialize_context_t@@XZ 100724b0 f i hb-ot-shaper-arabic.obj
 0001:00071590       ?safe_to_insert_tatweel@hb_buffer_t@@QAEXII@Z 10072590 f i hb-ot-shaper-arabic.obj
 0001:00071620       ?serialize@?$ArrayOf@UHBGlyphID16@OT@@U?$IntType@G$01@2@@OT@@QAE_NPAUhb_serialize_context_t@@I_N@Z 10072620 f i hb-ot-shaper-arabic.obj
 0001:00071710       ?serialize@?$HeadlessArrayOf@UHBGlyphID16@OT@@U?$IntType@G$01@2@@OT@@QAE_NPAUhb_serialize_context_t@@I_N@Z 10072710 f i hb-ot-shaper-arabic.obj
 0001:00071810       ?serialize@?$LigatureSet@USmallTypes@Layout@OT@@@GSUB_impl@Layout@OT@@QAE_NPAUhb_serialize_context_t@@U?$hb_array_t@$$CBUHBGlyphID16@OT@@@@U?$hb_array_t@$$CBI@@AAU6@@Z 10072810 f i hb-ot-shaper-arabic.obj
 0001:00071b50       ?serialize@?$LigatureSubstFormat1_2@USmallTypes@Layout@OT@@@GSUB_impl@Layout@OT@@QAE_NPAUhb_serialize_context_t@@U?$hb_sorted_array_t@$$CBUHBGlyphID16@OT@@@@U?$hb_array_t@$$CBI@@U?$hb_array_t@$$CBUHBGlyphID16@OT@@@@23@Z 10072b50 f i hb-ot-shaper-arabic.obj
 0001:00071e40       ?serialize@?$SortedArrayOf@U?$RangeRecord@USmallTypes@Layout@OT@@@Common@Layout@OT@@U?$IntType@G$01@4@@OT@@QAE_NPAUhb_serialize_context_t@@I@Z 10072e40 f i hb-ot-shaper-arabic.obj
 0001:00071f70       ?serialize@Lookup@OT@@QAE_NPAUhb_serialize_context_t@@III@Z 10072f70 f i hb-ot-shaper-arabic.obj
 0001:00072130       ?serialize_ligature@SubstLookup@GSUB_impl@Layout@OT@@QAE_NPAUhb_serialize_context_t@@IU?$hb_sorted_array_t@$$CBUHBGlyphID16@OT@@@@U?$hb_array_t@$$CBI@@U?$hb_array_t@$$CBUHBGlyphID16@OT@@@@23@Z 10073130 f i hb-ot-shaper-arabic.obj
 0001:00072280       ?setup_masks_arabic_plan@@YAXPBUarabic_shape_plan_t@@PAUhb_buffer_t@@W4hb_script_t@@@Z 10073280 f   hb-ot-shaper-arabic.obj
 0001:00072ea0       ?hb_indic_get_categories@@YAGI@Z 10073ea0 f   hb-ot-shaper-indic-table.obj
 0001:00073f80       ?find_syllables_indic@@YAXPAUhb_buffer_t@@@Z 10074f80 f i hb-ot-shaper-indic.obj
 0001:00074420       ?init@hb_indic_would_substitute_feature_t@@QAEXPBUhb_ot_map_t@@I_N@Z 10075420 f i hb-ot-shaper-indic.obj
 0001:00075450       ?would_substitute@hb_indic_would_substitute_feature_t@@QBE_NPBIIPAUhb_face_t@@@Z 10076450 f i hb-ot-shaper-indic.obj
 0001:00075800       ?find_syllables_khmer@@YAXPAUhb_buffer_t@@@Z 10076800 f i hb-ot-shaper-khmer.obj
 0001:00075ff0       ?find_syllables_myanmar@@YAXPAUhb_buffer_t@@@Z 10076ff0 f i hb-ot-shaper-myanmar.obj
 0001:00076740       ?hb_syllabic_clear_var@@YA_NPBUhb_ot_shape_plan_t@@PAUhb_font_t@@PAUhb_buffer_t@@@Z 10077740 f   hb-ot-shaper-syllabic.obj
 0001:00076750       ?hb_syllabic_insert_dotted_circles@@YA_NPAUhb_font_t@@PAUhb_buffer_t@@IIHH@Z 10077750 f   hb-ot-shaper-syllabic.obj
 0001:00079480       ?_hb_preprocess_text_vowel_constraints@@YAXPBUhb_ot_shape_plan_t@@PAUhb_buffer_t@@PAUhb_font_t@@@Z 1007a480 f   hb-ot-shaper-vowel-constraints.obj
 0001:0007c810       _hb_ot_tag_to_language     1007d810 f   hb-ot-tag.obj
 0001:0007c980       _hb_ot_tags_from_script_and_language 1007d980 f   hb-ot-tag.obj
 0001:0007cc50       ?get_instance@fvar@OT@@QBEPBUInstanceRecord@2@I@Z 1007dc50 f i hb-ot-var.obj
 0001:0007ccc0       ?map_coords@avar@OT@@QBEXPAHI@Z 1007dcc0 f i hb-ot-var.obj
 0001:0007d100       _hb_ot_var_named_instance_get_design_coords 1007e100 f   hb-ot-var.obj
 0001:0007d1c0       _hb_ot_var_normalize_coords 1007e1c0 f   hb-ot-var.obj
 0001:0007d350       ??$push@Uhb_outline_point_t@@@?$hb_vector_t@Uhb_outline_point_t@@$0A@@@QAEPAUhb_outline_point_t@@$$QAU1@@Z 1007e350 f i hb-outline.obj
 0001:0007d3c0       ?embolden@hb_outline_t@@QAEXMMMM@Z 1007e3c0 f   hb-outline.obj
 0001:0007d9f0       ?hb_outline_recording_pen_get_funcs@@YAPAUhb_draw_funcs_t@@XZ 1007e9f0 f   hb-outline.obj
 0001:0007dba0       ?replay@hb_outline_t@@QBEXPAUhb_draw_funcs_t@@PAX@Z 1007eba0 f   hb-outline.obj
 0001:0007e4e0       ?hb_paint_extents_get_funcs@@YAPAUhb_paint_funcs_t@@XZ 1007f4e0 f   hb-paint-extents.obj
 0001:0007eb30       ?paint@hb_paint_extents_context_t@@QAEXXZ 1007fb30 f i hb-paint-extents.obj
 0001:0007eba0       ?push_clip@hb_paint_extents_context_t@@QAEXUhb_extents_t@@@Z 1007fba0 f i hb-paint-extents.obj
 0001:0007ec30       ?transform_extents@hb_transform_t@@QBEXAAUhb_extents_t@@@Z 1007fc30 f i hb-paint-extents.obj
 0001:0007ef20       ?union_@hb_bounds_t@@QAEXABU1@@Z 1007ff20 f i hb-paint-extents.obj
 0001:0007f010       _hb_paint_funcs_create     10080010 f   hb-paint.obj
 0001:0007f100       _hb_paint_funcs_destroy    10080100 f   hb-paint.obj
 0001:0007f2e0       _hb_paint_funcs_get_empty  100802e0 f   hb-paint.obj
 0001:0007f2f0       _hb_paint_funcs_set_color_func 100802f0 f   hb-paint.obj
 0001:0007f3a0       _hb_paint_funcs_set_image_func 100803a0 f   hb-paint.obj
 0001:0007f450       _hb_paint_funcs_set_linear_gradient_func 10080450 f   hb-paint.obj
 0001:0007f500       _hb_paint_funcs_set_pop_clip_func 10080500 f   hb-paint.obj
 0001:0007f5b0       _hb_paint_funcs_set_pop_group_func 100805b0 f   hb-paint.obj
 0001:0007f660       _hb_paint_funcs_set_pop_transform_func 10080660 f   hb-paint.obj
 0001:0007f710       _hb_paint_funcs_set_push_clip_glyph_func 10080710 f   hb-paint.obj
 0001:0007f7c0       _hb_paint_funcs_set_push_clip_rectangle_func 100807c0 f   hb-paint.obj
 0001:0007f870       _hb_paint_funcs_set_push_group_func 10080870 f   hb-paint.obj
 0001:0007f920       _hb_paint_funcs_set_push_transform_func 10080920 f   hb-paint.obj
 0001:0007f9c0       _hb_paint_funcs_set_radial_gradient_func 100809c0 f   hb-paint.obj
 0001:0007fa70       _hb_paint_funcs_set_sweep_gradient_func 10080a70 f   hb-paint.obj
 0001:0007fb20       ??1hb_ot_map_t@@QAE@XZ     10080b20 f i hb-shape-plan.obj
 0001:0007fd40       ?init@hb_shape_plan_key_t@@QAE_N_NPAUhb_face_t@@PBUhb_segment_properties_t@@PBUhb_feature_t@@IPBHIPBQBD@Z 10080d40 f   hb-shape-plan.obj
 0001:00080090       _hb_shape_plan_create2     10081090 f   hb-shape-plan.obj
 0001:00080210       _hb_shape_plan_create_cached2 10081210 f   hb-shape-plan.obj
 0001:00080560       _hb_shape_plan_destroy     10081560 f   hb-shape-plan.obj
 0001:000805d0       _hb_shape_plan_execute     100815d0 f   hb-shape-plan.obj
 0001:00080610       _hb_shape_full             10081610 f   hb-shape.obj
 0001:000806f0       ?_hb_shapers_get@@YAPBUhb_shaper_entry_t@@XZ 100816f0 f   hb-shaper.obj
 0001:00080700       ?get_stored@?$hb_lazy_loader_t@Uhb_shaper_entry_t@@Uhb_shapers_lazy_loader_t@@X$0A@U1@@@QBEPAUhb_shaper_entry_t@@XZ 10081700 f i hb-shaper.obj
 0001:00080d70       _hb_ucd_get_unicode_funcs  10081d70 f   hb-ucd.obj
 0001:00080e50       ?_hb_unicode_is_emoji_Extended_Pictographic@@YA_NI@Z 10081e50 f   hb-unicode.obj
 0001:00080ef0       _hb_unicode_funcs_create   10081ef0 f   hb-unicode.obj
 0001:00080fb0       _hb_unicode_funcs_destroy  10081fb0 f   hb-unicode.obj
 0001:00081090       _hb_unicode_funcs_get_default 10082090 f   hb-unicode.obj
 0001:000810a0       _hb_unicode_funcs_get_empty 100820a0 f   hb-unicode.obj
 0001:000810b0       _hb_unicode_funcs_set_combining_class_func 100820b0 f   hb-unicode.obj
 0001:00081130       _hb_unicode_funcs_set_compose_func 10082130 f   hb-unicode.obj
 0001:000811b0       _hb_unicode_funcs_set_decompose_func 100821b0 f   hb-unicode.obj
 0001:00081230       _hb_unicode_funcs_set_general_category_func 10082230 f   hb-unicode.obj
 0001:000812b0       _hb_unicode_funcs_set_mirroring_func 100822b0 f   hb-unicode.obj
 0001:00081330       _hb_unicode_funcs_set_script_func 10082330 f   hb-unicode.obj
 0001:000813b0       _Java_sun_font_FileFontStrike__1getGlyphImageFromWindows@32 100823b0 f   lcdglyph.obj
 0001:00081d20       _Java_sun_font_FileFontStrike_initNative@8 10082d20 f   lcdglyph.obj
 0001:00081d50       _getHBScriptCode           10082d50 f   scriptMapping.obj
 0001:00081d70       _Java_sun_font_NullFontScaler_getGlyphImage@20 10082d70 f   sunFont.obj
 0001:00081d90       _Java_sun_font_NullFontScaler_getNullScalerContext@8 10082d90 f   sunFont.obj
 0001:00081db0       _Java_sun_font_StrikeCache_freeIntMemory@20 10082db0 f   sunFont.obj
 0001:00081e60       _Java_sun_font_StrikeCache_freeIntPointer@12 10082e60 f   sunFont.obj
 0001:00081e80       _Java_sun_font_StrikeCache_freeLongMemory@20 10082e80 f   sunFont.obj
 0001:00081f30       _Java_sun_font_StrikeCache_freeLongPointer@16 10082f30 f   sunFont.obj
 0001:00081f50       _Java_sun_font_StrikeCache_getGlyphCacheDescription@12 10082f50 f   sunFont.obj
 0001:00082070       _Java_sun_font_SunFontManager_initIDs@8 10083070 f   sunFont.obj
 0001:00082080       _getSunFontIDs             10083080 f   sunFont.obj
 0001:000826a0       _isNullScalerContext       100836a0 f   sunFont.obj
 0001:000826b0       _FT_Init_FreeType          100836b0 f   freetype:freetype.dll
 0001:000826b6       _FT_Done_FreeType          100836b6 f   freetype:freetype.dll
 0001:000826bc       _FT_New_Memory_Face        100836bc f   freetype:freetype.dll
 0001:000826c2       _FT_Open_Face              100836c2 f   freetype:freetype.dll
 0001:000826c8       _FT_Done_Face              100836c8 f   freetype:freetype.dll
 0001:000826ce       _FT_Set_Char_Size          100836ce f   freetype:freetype.dll
 0001:000826d4       _FT_Load_Glyph             100836d4 f   freetype:freetype.dll
 0001:000826da       _FT_Set_Transform          100836da f   freetype:freetype.dll
 0001:000826e0       _FT_Render_Glyph           100836e0 f   freetype:freetype.dll
 0001:000826e6       _FT_Get_Char_Index         100836e6 f   freetype:freetype.dll
 0001:000826ec       _FT_MulFix                 100836ec f   freetype:freetype.dll
 0001:000826f2       _FT_Matrix_Multiply        100836f2 f   freetype:freetype.dll
 0001:000826f8       _FT_Outline_Get_BBox       100836f8 f   freetype:freetype.dll
 0001:000826fe       _FT_Activate_Size          100836fe f   freetype:freetype.dll
 0001:00082704       _FT_Outline_Decompose      10083704 f   freetype:freetype.dll
 0001:0008270a       _FT_Outline_Get_CBox       1008370a f   freetype:freetype.dll
 0001:00082710       _FT_Outline_Translate      10083710 f   freetype:freetype.dll
 0001:00082716       _FT_GlyphSlot_Embolden     10083716 f   freetype:freetype.dll
 0001:0008271c       _FT_Library_SetLcdFilter   1008371c f   freetype:freetype.dll
 0001:00082722       _FT_Property_Set           10083722 f   freetype:freetype.dll
 0001:00082728       _JNU_ThrowArrayIndexOutOfBoundsException@8 10083728 f   java:java.dll
 0001:0008272e       _JNU_NewStringPlatform@8   1008372e f   java:java.dll
 0001:00082734       _SurfaceData_GetOps@8      10083734 f   awt:awt.dll
 0001:0008273a       _SurfaceData_IntersectBounds@8 1008373a f   awt:awt.dll
 0001:00082740       _GetNativePrim@8           10083740 f   awt:awt.dll
 0001:00082746       _GrPrim_Sg2dGetCompInfo@16 10083746 f   awt:awt.dll
 0001:0008274c       _GrPrim_Sg2dGetClip@12     1008374c f   awt:awt.dll
 0001:00082752       _GrPrim_Sg2dGetPixel@8     10083752 f   awt:awt.dll
 0001:00082758       _GrPrim_Sg2dGetEaRGB@8     10083758 f   awt:awt.dll
 0001:0008275e       _GrPrim_Sg2dGetLCDTextContrast@8 1008375e f   awt:awt.dll
 0001:00082764       _AccelGlyphCache_RemoveAllCellInfos 10083764 f   awt:awt.dll
 0001:0008276a       @__security_check_cookie@4 1008376a f   MSVCRT:secchk.obj
 0001:00082780       __ftoui3                   10083780 f   MSVCRT:ftol3.obj
 0001:0008278f       __ftoul3                   1008378f f   MSVCRT:ftol3.obj
 0001:0008279e       __ftol3                    1008379e f   MSVCRT:ftol3.obj
 0001:000827ab       __ftol3_NaN                100837ab f   MSVCRT:ftol3.obj
 0001:000827c3       __ftol3_work               100837c3 f   MSVCRT:ftol3.obj
 0001:00082849       __ftol3_common             10083849 f   MSVCRT:ftol3.obj
 0001:0008290b       __ftol3_arg_error          1008390b f   MSVCRT:ftol3.obj
 0001:0008291d       __ftol3_except             1008391d f   MSVCRT:ftol3.obj
 0001:00082961       __dtoui3                   10083961 f   MSVCRT:ftol3.obj
 0001:00082970       __dtoul3                   10083970 f   MSVCRT:ftol3.obj
 0001:0008297f       __dtol3                    1008397f f   MSVCRT:ftol3.obj
 0001:0008298c       __dtol3_NaN                1008398c f   MSVCRT:ftol3.obj
 0001:000829a9       __dtol3_work               100839a9 f   MSVCRT:ftol3.obj
 0001:00082a90       __ultod3                   10083a90 f   MSVCRT:ftol3.obj
 0001:00082ad0       __ltod3                    10083ad0 f   MSVCRT:ftol3.obj
 0001:00082b00       __allmul                   10083b00 f   MSVCRT:llmul.obj
 0001:00082b34       ___raise_securityfailure   10083b34 f   MSVCRT:gs_report.obj
 0001:00082b5c       ___report_gsfailure        10083b5c f   MSVCRT:gs_report.obj
 0001:00082c55       ___report_rangecheckfailure 10083c55 f   MSVCRT:gs_report.obj
 0001:00082c61       ___report_securityfailure  10083c61 f   MSVCRT:gs_report.obj
 0001:00082d30       __alldiv                   10083d30 f   MSVCRT:lldiv.obj
 0001:00082de0       __chkstk                   10083de0 f   MSVCRT:chkstk.obj
 0001:00082de0       __alloca_probe             10083de0 f   MSVCRT:chkstk.obj
 0001:00082e10       __ftol2_sse                10083e10 f   MSVCRT:ftol2.obj
 0001:00082e19       __ftol2_pentium4           10083e19 f   MSVCRT:ftol2.obj
 0001:00082e2c       __ftol2_sse_excpt          10083e2c f   MSVCRT:ftol2.obj
 0001:00082e50       __ftol2                    10083e50 f   MSVCRT:ftol2.obj
 0001:00082ed0       __alloca_probe_16          10083ed0 f   MSVCRT:alloca16.obj
 0001:00082ee6       __alloca_probe_8           10083ee6     MSVCRT:alloca16.obj
 0001:0008321c       __DllMainCRTStartup@12     1008421c f   MSVCRT:dll_dllmain.obj
 0001:0008323f       ___isa_available_init      1008423f f   MSVCRT:cpu_disp.obj
 0001:00083423       ___security_init_cookie    10084423 f   MSVCRT:gs_support.obj
 0001:0008346e       _DllMain@12                1008446e f   MSVCRT:dll_dllmain_stub.obj
 0001:00083490       ?__scrt_initialize_type_info@@YAXXZ 10084490 f   MSVCRT:tncleanup.obj
 0001:0008349c       ?__scrt_uninitialize_type_info@@YAXXZ 1008449c f   MSVCRT:tncleanup.obj
 0001:000834a8       ___local_stdio_scanf_options 100844a8 f i MSVCRT:default_local_stdio_options.obj
 0001:000834ae       ___scrt_initialize_default_local_stdio_options 100844ae f   MSVCRT:default_local_stdio_options.obj
 0001:0008350f       ___scrt_acquire_startup_lock 1008450f f   MSVCRT:utility.obj
 0001:00083541       ___scrt_dllmain_after_initialize_c 10084541 f   MSVCRT:utility.obj
 0001:0008356c       ___scrt_dllmain_before_initialize_c 1008456c f   MSVCRT:utility.obj
 0001:0008357a       ___scrt_dllmain_crt_thread_attach 1008457a f   MSVCRT:utility.obj
 0001:00083599       ___scrt_dllmain_crt_thread_detach 10084599 f   MSVCRT:utility.obj
 0001:000835a6       ___scrt_dllmain_exception_filter 100845a6 f   MSVCRT:utility.obj
 0001:000835da       ___scrt_dllmain_uninitialize_c 100845da f   MSVCRT:utility.obj
 0001:000835fd       ___scrt_dllmain_uninitialize_critical 100845fd f   MSVCRT:utility.obj
 0001:0008360a       ___scrt_initialize_crt     1008460a f   MSVCRT:utility.obj
 0001:00083643       ___scrt_initialize_onexit_tables 10084643 f   MSVCRT:utility.obj
 0001:000836e8       ___scrt_is_nonwritable_in_current_image 100846e8 f   MSVCRT:utility.obj
 0001:0008377c       ___scrt_release_startup_lock 1008477c f   MSVCRT:utility.obj
 0001:00083799       ___scrt_uninitialize_crt   10084799 f   MSVCRT:utility.obj
 0001:000837c1       ___scrt_get_dyn_tls_init_callback 100847c1 f   MSVCRT:dyn_tls_init.obj
 0001:000837c7       ___scrt_fastfail           100847c7 f   MSVCRT:utility_desktop.obj
 0001:000838e1       __crt_debugger_hook        100848e1 f   MSVCRT:utility_desktop.obj
 0001:000838e9       __RTC_Initialize           100848e9 f   MSVCRT:initsect.obj
 0001:00083915       __RTC_Terminate            10084915 f   MSVCRT:initsect.obj
 0001:00083950       __SEH_prolog4              10084950 f   MSVCRT:sehprolg4.obj
 0001:00083996       __SEH_epilog4              10084996 f   MSVCRT:sehprolg4.obj
 0001:000839ab       __except_handler4          100849ab f   MSVCRT:chandler4gs.obj
 0001:000839ce       __get_startup_argv_mode    100849ce f   MSVCRT:argv_mode.obj
 0001:000839d2       ___scrt_is_ucrt_dll_in_use 100849d2 f   MSVCRT:ucrt_detection.obj
 0001:000839de       _IsProcessorFeaturePresent@4 100849de f   kernel32:KERNEL32.dll
 0001:000839e4       _memset                    100849e4 f   vcruntime:VCRUNTIME140.dll
 0001:000839ea       _strrchr                   100849ea f   vcruntime:VCRUNTIME140.dll
 0001:000839f0       _wcsrchr                   100849f0 f   vcruntime:VCRUNTIME140.dll
 0001:000839f6       _wcsstr                    100849f6 f   vcruntime:VCRUNTIME140.dll
 0001:000839fc       _strstr                    100849fc f   vcruntime:VCRUNTIME140.dll
 0001:00083a02       _memcpy                    10084a02 f   vcruntime:VCRUNTIME140.dll
 0001:00083a08       _memmove                   10084a08 f   vcruntime:VCRUNTIME140.dll
 0001:00083a0e       _strchr                    10084a0e f   vcruntime:VCRUNTIME140.dll
 0001:00083a14       ___std_type_info_destroy_list 10084a14 f   vcruntime:VCRUNTIME140.dll
 0001:00083a1a       __except_handler4_common   10084a1a f   vcruntime:VCRUNTIME140.dll
 0001:00083a20       __libm_sse2_pow_precise    10084a20 f   ucrt:api-ms-win-crt-math-l1-1-0.dll
 0001:00083a26       _floor                     10084a26 f   ucrt:api-ms-win-crt-math-l1-1-0.dll
 0001:00083a2c       __libm_sse2_sqrt_precise   10084a2c f   ucrt:api-ms-win-crt-math-l1-1-0.dll
 0001:00083a32       _ceil                      10084a32 f   ucrt:api-ms-win-crt-math-l1-1-0.dll
 0001:00083a38       __libm_sse2_cos_precise    10084a38 f   ucrt:api-ms-win-crt-math-l1-1-0.dll
 0001:00083a3e       __libm_sse2_sin_precise    10084a3e f   ucrt:api-ms-win-crt-math-l1-1-0.dll
 0001:00083a44       __libm_sse2_tan_precise    10084a44 f   ucrt:api-ms-win-crt-math-l1-1-0.dll
 0001:00083a4a       __except1                  10084a4a f   ucrt:api-ms-win-crt-math-l1-1-0.dll
 0001:00083a50       __initterm                 10084a50 f   ucrt:api-ms-win-crt-runtime-l1-1-0.dll
 0001:00083a56       __initterm_e               10084a56 f   ucrt:api-ms-win-crt-runtime-l1-1-0.dll
 0001:00083a5c       __seh_filter_dll           10084a5c f   ucrt:api-ms-win-crt-runtime-l1-1-0.dll
 0001:00083a62       __configure_narrow_argv    10084a62 f   ucrt:api-ms-win-crt-runtime-l1-1-0.dll
 0001:00083a68       __initialize_narrow_environment 10084a68 f   ucrt:api-ms-win-crt-runtime-l1-1-0.dll
 0001:00083a6e       __initialize_onexit_table  10084a6e f   ucrt:api-ms-win-crt-runtime-l1-1-0.dll
 0001:00083a74       __execute_onexit_table     10084a74 f   ucrt:api-ms-win-crt-runtime-l1-1-0.dll
 0001:00083a7a       __cexit                    10084a7a f   ucrt:api-ms-win-crt-runtime-l1-1-0.dll
 0002:00000000       __imp__RegCloseKey@4       10085000     advapi32:ADVAPI32.dll
 0002:00000004       __imp__RegOpenKeyExA@20    10085004     advapi32:ADVAPI32.dll
 0002:00000008       __imp__RegQueryInfoKeyW@48 10085008     advapi32:ADVAPI32.dll
 0002:0000000c       __imp__RegEnumValueW@32    1008500c     advapi32:ADVAPI32.dll
 0002:00000010       \177ADVAPI32_NULL_THUNK_DATA 10085010     advapi32:ADVAPI32.dll
 0002:00000014       __imp__GetFontData@20      10085014     gdi32:GDI32.dll
 0002:00000018       __imp__GetDIBits@28        10085018     gdi32:GDI32.dll
 0002:0000001c       __imp__GetDeviceCaps@8     1008501c     gdi32:GDI32.dll
 0002:00000020       __imp__DeleteObject@4      10085020     gdi32:GDI32.dll
 0002:00000024       __imp__CreateFontIndirectW@4 10085024     gdi32:GDI32.dll
 0002:00000028       __imp__GetStockObject@4    10085028     gdi32:GDI32.dll
 0002:0000002c       __imp__CreateCompatibleBitmap@12 1008502c     gdi32:GDI32.dll
 0002:00000030       __imp__EnumFontFamiliesExW@20 10085030     gdi32:GDI32.dll
 0002:00000034       __imp__SetTextColor@8      10085034     gdi32:GDI32.dll
 0002:00000038       __imp__GetTextMetricsA@8   10085038     gdi32:GDI32.dll
 0002:0000003c       __imp__ExtTextOutW@32      1008503c     gdi32:GDI32.dll
 0002:00000040       __imp__GetGlyphOutlineA@28 10085040     gdi32:GDI32.dll
 0002:00000044       __imp__SelectObject@8      10085044     gdi32:GDI32.dll
 0002:00000048       __imp__SetBkColor@8        10085048     gdi32:GDI32.dll
 0002:0000004c       __imp__CreateCompatibleDC@4 1008504c     gdi32:GDI32.dll
 0002:00000050       __imp__SetMapMode@8        10085050     gdi32:GDI32.dll
 0002:00000054       \177GDI32_NULL_THUNK_DATA  10085054     gdi32:GDI32.dll
 0002:00000058       __imp__DeleteCriticalSection@4 10085058     kernel32:KERNEL32.dll
 0002:0000005c       __imp__LeaveCriticalSection@4 1008505c     kernel32:KERNEL32.dll
 0002:00000060       __imp__InitializeCriticalSection@4 10085060     kernel32:KERNEL32.dll
 0002:00000064       __imp__EnterCriticalSection@4 10085064     kernel32:KERNEL32.dll
 0002:00000068       __imp__GetWindowsDirectoryA@8 10085068     kernel32:KERNEL32.dll
 0002:0000006c       __imp__GetSystemDirectoryA@8 1008506c     kernel32:KERNEL32.dll
 0002:00000070       __imp__UnhandledExceptionFilter@4 10085070     kernel32:KERNEL32.dll
 0002:00000074       __imp__GetVersion@0        10085074     kernel32:KERNEL32.dll
 0002:00000078       __imp__SetUnhandledExceptionFilter@4 10085078     kernel32:KERNEL32.dll
 0002:0000007c       __imp__GetCurrentProcess@0 1008507c     kernel32:KERNEL32.dll
 0002:00000080       __imp__TerminateProcess@8  10085080     kernel32:KERNEL32.dll
 0002:00000084       __imp__IsProcessorFeaturePresent@4 10085084     kernel32:KERNEL32.dll
 0002:00000088       __imp__QueryPerformanceCounter@4 10085088     kernel32:KERNEL32.dll
 0002:0000008c       __imp__GetCurrentProcessId@0 1008508c     kernel32:KERNEL32.dll
 0002:00000090       __imp__GetCurrentThreadId@0 10085090     kernel32:KERNEL32.dll
 0002:00000094       __imp__GetSystemTimeAsFileTime@4 10085094     kernel32:KERNEL32.dll
 0002:00000098       __imp__DisableThreadLibraryCalls@4 10085098     kernel32:KERNEL32.dll
 0002:0000009c       __imp__InitializeSListHead@4 1008509c     kernel32:KERNEL32.dll
 0002:000000a0       __imp__IsDebuggerPresent@0 100850a0     kernel32:KERNEL32.dll
 0002:000000a4       \177KERNEL32_NULL_THUNK_DATA 100850a4     kernel32:KERNEL32.dll
 0002:000000a8       __imp__GetDesktopWindow@0  100850a8     user32:USER32.dll
 0002:000000ac       __imp__FillRect@12         100850ac     user32:USER32.dll
 0002:000000b0       __imp__ReleaseDC@8         100850b0     user32:USER32.dll
 0002:000000b4       __imp__GetWindowDC@4       100850b4     user32:USER32.dll
 0002:000000b8       __imp__SystemParametersInfoA@16 100850b8     user32:USER32.dll
 0002:000000bc       __imp__GetDC@4             100850bc     user32:USER32.dll
 0002:000000c0       \177USER32_NULL_THUNK_DATA 100850c0     user32:USER32.dll
 0002:000000c4       __imp__memset              100850c4     vcruntime:VCRUNTIME140.dll
 0002:000000c8       __imp__strrchr             100850c8     vcruntime:VCRUNTIME140.dll
 0002:000000cc       __imp__wcsrchr             100850cc     vcruntime:VCRUNTIME140.dll
 0002:000000d0       __imp__wcsstr              100850d0     vcruntime:VCRUNTIME140.dll
 0002:000000d4       __imp__strstr              100850d4     vcruntime:VCRUNTIME140.dll
 0002:000000d8       __imp__memcpy              100850d8     vcruntime:VCRUNTIME140.dll
 0002:000000dc       __imp____std_type_info_destroy_list 100850dc     vcruntime:VCRUNTIME140.dll
 0002:000000e0       __imp___except_handler4_common 100850e0     vcruntime:VCRUNTIME140.dll
 0002:000000e4       __imp__strchr              100850e4     vcruntime:VCRUNTIME140.dll
 0002:000000e8       __imp__memmove             100850e8     vcruntime:VCRUNTIME140.dll
 0002:000000ec       \177VCRUNTIME140_NULL_THUNK_DATA 100850ec     vcruntime:VCRUNTIME140.dll
 0002:000000f0       __imp__strtol              100850f0     ucrt:api-ms-win-crt-convert-l1-1-0.dll
 0002:000000f4       \177api-ms-win-crt-convert-l1-1-0_NULL_THUNK_DATA 100850f4     ucrt:api-ms-win-crt-convert-l1-1-0.dll
 0002:000000f8       __imp__getenv              100850f8     ucrt:api-ms-win-crt-environment-l1-1-0.dll
 0002:000000fc       \177api-ms-win-crt-environment-l1-1-0_NULL_THUNK_DATA 100850fc     ucrt:api-ms-win-crt-environment-l1-1-0.dll
 0002:00000100       __imp__realloc             10085100     ucrt:api-ms-win-crt-heap-l1-1-0.dll
 0002:00000104       __imp__malloc              10085104     ucrt:api-ms-win-crt-heap-l1-1-0.dll
 0002:00000108       __imp__free                10085108     ucrt:api-ms-win-crt-heap-l1-1-0.dll
 0002:0000010c       __imp__calloc              1008510c     ucrt:api-ms-win-crt-heap-l1-1-0.dll
 0002:00000110       \177api-ms-win-crt-heap-l1-1-0_NULL_THUNK_DATA 10085110     ucrt:api-ms-win-crt-heap-l1-1-0.dll
 0002:00000114       __imp___libm_sse2_cos_precise 10085114     ucrt:api-ms-win-crt-math-l1-1-0.dll
 0002:00000118       __imp___libm_sse2_pow_precise 10085118     ucrt:api-ms-win-crt-math-l1-1-0.dll
 0002:0000011c       __imp___except1            1008511c     ucrt:api-ms-win-crt-math-l1-1-0.dll
 0002:00000120       __imp___libm_sse2_tan_precise 10085120     ucrt:api-ms-win-crt-math-l1-1-0.dll
 0002:00000124       __imp___libm_sse2_sqrt_precise 10085124     ucrt:api-ms-win-crt-math-l1-1-0.dll
 0002:00000128       __imp__ceil                10085128     ucrt:api-ms-win-crt-math-l1-1-0.dll
 0002:0000012c       __imp___libm_sse2_sin_precise 1008512c     ucrt:api-ms-win-crt-math-l1-1-0.dll
 0002:00000130       __imp__floor               10085130     ucrt:api-ms-win-crt-math-l1-1-0.dll
 0002:00000134       __imp___hypotf             10085134     ucrt:api-ms-win-crt-math-l1-1-0.dll
 0002:00000138       \177api-ms-win-crt-math-l1-1-0_NULL_THUNK_DATA 10085138     ucrt:api-ms-win-crt-math-l1-1-0.dll
 0002:0000013c       __imp___cexit              1008513c     ucrt:api-ms-win-crt-runtime-l1-1-0.dll
 0002:00000140       __imp___execute_onexit_table 10085140     ucrt:api-ms-win-crt-runtime-l1-1-0.dll
 0002:00000144       __imp___initialize_onexit_table 10085144     ucrt:api-ms-win-crt-runtime-l1-1-0.dll
 0002:00000148       __imp___initialize_narrow_environment 10085148     ucrt:api-ms-win-crt-runtime-l1-1-0.dll
 0002:0000014c       __imp___errno              1008514c     ucrt:api-ms-win-crt-runtime-l1-1-0.dll
 0002:00000150       __imp___seh_filter_dll     10085150     ucrt:api-ms-win-crt-runtime-l1-1-0.dll
 0002:00000154       __imp___initterm_e         10085154     ucrt:api-ms-win-crt-runtime-l1-1-0.dll
 0002:00000158       __imp___initterm           10085158     ucrt:api-ms-win-crt-runtime-l1-1-0.dll
 0002:0000015c       __imp___configure_narrow_argv 1008515c     ucrt:api-ms-win-crt-runtime-l1-1-0.dll
 0002:00000160       \177api-ms-win-crt-runtime-l1-1-0_NULL_THUNK_DATA 10085160     ucrt:api-ms-win-crt-runtime-l1-1-0.dll
 0002:00000164       __imp____acrt_iob_func     10085164     ucrt:api-ms-win-crt-stdio-l1-1-0.dll
 0002:00000168       __imp____stdio_common_vsprintf 10085168     ucrt:api-ms-win-crt-stdio-l1-1-0.dll
 0002:0000016c       __imp____stdio_common_vfprintf 1008516c     ucrt:api-ms-win-crt-stdio-l1-1-0.dll
 0002:00000170       \177api-ms-win-crt-stdio-l1-1-0_NULL_THUNK_DATA 10085170     ucrt:api-ms-win-crt-stdio-l1-1-0.dll
 0002:00000174       __imp___stricmp            10085174     ucrt:api-ms-win-crt-string-l1-1-0.dll
 0002:00000174       __imp__stricmp             10085174     ucrt:api-ms-win-crt-string-l1-1-0.dll
 0002:00000178       __imp__strncpy             10085178     ucrt:api-ms-win-crt-string-l1-1-0.dll
 0002:0000017c       __imp__wcsicmp             1008517c     ucrt:api-ms-win-crt-string-l1-1-0.dll
 0002:0000017c       __imp___wcsicmp            1008517c     ucrt:api-ms-win-crt-string-l1-1-0.dll
 0002:00000180       __imp__strncmp             10085180     ucrt:api-ms-win-crt-string-l1-1-0.dll
 0002:00000184       \177api-ms-win-crt-string-l1-1-0_NULL_THUNK_DATA 10085184     ucrt:api-ms-win-crt-string-l1-1-0.dll
 0002:00000188       __imp__GrPrim_Sg2dGetClip@12 10085188     awt:awt.dll
 0002:0000018c       __imp__GrPrim_Sg2dGetCompInfo@16 1008518c     awt:awt.dll
 0002:00000190       __imp__GetNativePrim@8     10085190     awt:awt.dll
 0002:00000194       __imp__SurfaceData_IntersectBounds@8 10085194     awt:awt.dll
 0002:00000198       __imp__SurfaceData_GetOps@8 10085198     awt:awt.dll
 0002:0000019c       __imp__GrPrim_Sg2dGetPixel@8 1008519c     awt:awt.dll
 0002:000001a0       __imp__GrPrim_Sg2dGetEaRGB@8 100851a0     awt:awt.dll
 0002:000001a4       __imp__GrPrim_Sg2dGetLCDTextContrast@8 100851a4     awt:awt.dll
 0002:000001a8       __imp__AccelGlyphCache_RemoveAllCellInfos 100851a8     awt:awt.dll
 0002:000001ac       \177awt_NULL_THUNK_DATA    100851ac     awt:awt.dll
 0002:000001b0       __imp__FT_Property_Set     100851b0     freetype:freetype.dll
 0002:000001b4       __imp__FT_Library_SetLcdFilter 100851b4     freetype:freetype.dll
 0002:000001b8       __imp__FT_GlyphSlot_Embolden 100851b8     freetype:freetype.dll
 0002:000001bc       __imp__FT_New_Memory_Face  100851bc     freetype:freetype.dll
 0002:000001c0       __imp__FT_Outline_Get_CBox 100851c0     freetype:freetype.dll
 0002:000001c4       __imp__FT_Outline_Decompose 100851c4     freetype:freetype.dll
 0002:000001c8       __imp__FT_Activate_Size    100851c8     freetype:freetype.dll
 0002:000001cc       __imp__FT_Outline_Get_BBox 100851cc     freetype:freetype.dll
 0002:000001d0       __imp__FT_Matrix_Multiply  100851d0     freetype:freetype.dll
 0002:000001d4       __imp__FT_MulFix           100851d4     freetype:freetype.dll
 0002:000001d8       __imp__FT_Get_Char_Index   100851d8     freetype:freetype.dll
 0002:000001dc       __imp__FT_Render_Glyph     100851dc     freetype:freetype.dll
 0002:000001e0       __imp__FT_Set_Transform    100851e0     freetype:freetype.dll
 0002:000001e4       __imp__FT_Load_Glyph       100851e4     freetype:freetype.dll
 0002:000001e8       __imp__FT_Set_Char_Size    100851e8     freetype:freetype.dll
 0002:000001ec       __imp__FT_Done_FreeType    100851ec     freetype:freetype.dll
 0002:000001f0       __imp__FT_Outline_Translate 100851f0     freetype:freetype.dll
 0002:000001f4       __imp__FT_Done_Face        100851f4     freetype:freetype.dll
 0002:000001f8       __imp__FT_Open_Face        100851f8     freetype:freetype.dll
 0002:000001fc       __imp__FT_Init_FreeType    100851fc     freetype:freetype.dll
 0002:00000200       \177freetype_NULL_THUNK_DATA 10085200     freetype:freetype.dll
 0002:00000204       __imp__JNU_NewStringPlatform@8 10085204     java:java.dll
 0002:00000208       __imp__JNU_ThrowArrayIndexOutOfBoundsException@8 10085208     java:java.dll
 0002:0000020c       \177java_NULL_THUNK_DATA   1008520c     java:java.dll
 0002:00000210       ___guard_check_icall_fptr  10085210     MSVCRT:guard_support.obj
 0002:00000214       ___xc_a                    10085214     MSVCRT:initializers.obj
 0002:00000218       ___xc_z                    10085218     MSVCRT:initializers.obj
 0002:0000021c       ___xi_a                    1008521c     MSVCRT:initializers.obj
 0002:00000220       ___xi_z                    10085220     MSVCRT:initializers.obj
 0002:00000224       ___xl_a                    10085224     MSVCRT:tlssup.obj
 0002:00000228       ___xl_z                    10085228     MSVCRT:tlssup.obj
 0002:0000022c       ___xp_a                    1008522c     MSVCRT:initializers.obj
 0002:00000230       ___xp_z                    10085230     MSVCRT:initializers.obj
 0002:00000234       ___xt_a                    10085234     MSVCRT:initializers.obj
 0002:00000238       ___xt_z                    10085238     MSVCRT:initializers.obj
 0002:00000240       __real@3e2aaaad            10085240     DrawGlyphList.obj
 0002:00000244       __real@3f000000            10085244     DrawGlyphList.obj
 0002:00000248       __real@3ff0000000000000    10085248     DrawGlyphList.obj
 0002:00000250       __real@40400000            10085250     DrawGlyphList.obj
 0002:00000258       __real@4059000000000000    10085258     DrawGlyphList.obj
 0002:00000260       __real@406fe00000000000    10085260     DrawGlyphList.obj
 0002:00000268       ??_C@_0BM@DODCGPJL@sun?1font?1GlyphLayout$GVData@ 10085268     HBShaper.obj
 0002:00000284       ??_C@_01JPJNBJEM@I@        10085284     HBShaper.obj
 0002:00000288       ??_C@_06HHPHCOMB@_count@   10085288     HBShaper.obj
 0002:00000290       ??_C@_06PPHBKICC@_flags@   10085290     HBShaper.obj
 0002:00000298       ??_C@_02EBOMBDPA@?$FLI@    10085298     HBShaper.obj
 0002:0000029c       ??_C@_07PKNHOODJ@_glyphs@  1008529c     HBShaper.obj
 0002:000002a4       ??_C@_02MGHEAPDP@?$FLF@    100852a4     HBShaper.obj
 0002:000002a8       ??_C@_0L@BHNDECPI@_positions@ 100852a8     HBShaper.obj
 0002:000002b4       ??_C@_08MEOKMKLN@_indices@ 100852b4     HBShaper.obj
 0002:000002c0       ??_C@_03GAEACAIP@?$CI?$CJV@ 100852c0     HBShaper.obj
 0002:000002c4       ??_C@_04PAAMKIIE@grow@     100852c4     HBShaper.obj
 0002:000002c9       ??_C@_00CNPNBAHC@@         100852c9     HBShaper.obj
 0002:000002cc       ??_C@_0L@LCGIKEMB@HB_NODEVTX@ 100852cc     HBShaper.obj
 0002:000002d8       ??_C@_04HHMMLDJI@kern@     100852d8     HBShaper.obj
 0002:000002e0       ??_C@_05LLBOPDMO@?9kern@   100852e0     HBShaper.obj
 0002:000002e8       ??_C@_04BCEPKNGE@liga@     100852e8     HBShaper.obj
 0002:000002f0       ??_C@_05NOJNONDC@?9liga@   100852f0     HBShaper.obj
 0002:000002f8       __real@37800000            100852f8     HBShaper.obj
 0002:000002fc       __real@3f800000            100852fc     HBShaper.obj
 0002:00000300       __xmm@80000000800000008000000080000000 10085300     HBShaper.obj
 0002:00000374       ??_C@_11LOCGONAA@@         10085374     fontpath.obj
 0002:00000378       ??_C@_07GCCENIMJ@?2System@ 10085378     fontpath.obj
 0002:00000380       ??_C@_09FJGNFLHN@?2System32@ 10085380     fontpath.obj
 0002:0000038c       ??_C@_06MIJGMACG@?2Fonts@  1008538c     fontpath.obj
 0002:00000394       ??_C@_01ICJEACDI@?$DL@     10085394     fontpath.obj
 0002:00000398       ??_C@_17BCGMALNF@?$AA?5?$AA?$CG?$AA?5@ 10085398     fontpath.obj
 0002:000003a0       ??_C@_0BC@LEKPNIDO@java?1util?1HashMap@ 100853a0     fontpath.obj
 0002:000003b4       ??_C@_0DJ@FLFJBGBN@?$CILjava?1lang?1Object?$DLLjava?1lang?1O@ 100853b4     fontpath.obj
 0002:000003f0       ??_C@_03KMONJGDG@put@      100853f0     fontpath.obj
 0002:000003f4       ??_C@_0BG@DHOOFEJE@?$CILjava?1lang?1Object?$DL?$CJZ@ 100853f4     fontpath.obj
 0002:0000040c       ??_C@_0M@ILMAKOC@containsKey@ 1008540c     fontpath.obj
 0002:00000418       ??_C@_0BE@GPOIDJOH@java?1util?1ArrayList@ 10085418     fontpath.obj
 0002:0000042c       ??_C@_04PFANPMCN@?$CII?$CJV@ 1008542c     fontpath.obj
 0002:00000434       ??_C@_06FALKBLGB@?$DMinit?$DO@ 10085434     fontpath.obj
 0002:0000043c       ??_C@_03BDGOHNNK@add@      1008543c     fontpath.obj
 0002:00000440       ??_C@_0BB@FLFAIHG@java?1lang?1String@ 10085440     fontpath.obj
 0002:00000454       ??_C@_0CH@BHMNPKMP@?$CILjava?1util?1Locale?$DL?$CJLjava?1lang?1@ 10085454     fontpath.obj
 0002:0000047c       ??_C@_0M@IMBDOEKL@toLowerCase@ 1008547c     fontpath.obj
 0002:00000488       ??_C@_19OLAFNMII@?$AA?4?$AAt?$AAt?$AAf@ 10085488     fontpath.obj
 0002:00000494       ??_C@_19MKNEPBPF@?$AA?4?$AAo?$AAt?$AAf@ 10085494     fontpath.obj
 0002:000004b8       ??_C@_0BB@NIMAMPFF@invalidateScaler@ 100854b8     freetypeScaler.obj
 0002:000004cc       ??_C@_0BE@LLDKDDBI@FREETYPE_PROPERTIES@ 100854cc     freetypeScaler.obj
 0002:000004e0       ??_C@_08OKLLNAKL@truetype@ 100854e0     freetypeScaler.obj
 0002:000004ec       ??_C@_0BE@OJJAFABD@interpreter?9version@ 100854ec     freetypeScaler.obj
 0002:00000500       __real@00000000            10085500     freetypeScaler.obj
 0002:00000504       __real@3c800000            10085504     freetypeScaler.obj
 0002:00000508       __real@3ef0000000000000    10085508     freetypeScaler.obj
 0002:00000510       __real@3f90000000000000    10085510     freetypeScaler.obj
 0002:00000518       __real@4050000000000000    10085518     freetypeScaler.obj
 0002:00000520       __real@42800000            10085520     freetypeScaler.obj
 0002:00000524       __real@47800000            10085524     freetypeScaler.obj
 0002:00000528       __real@c7800000            10085528     freetypeScaler.obj
 0002:00000530       __xmm@00010000000000000000366a00010000 10085530     freetypeScaler.obj
 0002:00000540       __xmm@80000000000000008000000000000000 10085540     freetypeScaler.obj
 0002:00000a48       ?_Upper@?1??_Memory_order_upper_bound@std@@YA?AW4memory_order@2@W432@0@Z@4QAY05$$CBW432@A 10085a48     hb-aat-layout.obj
 0002:00000ad8       ??_C@_08EMNHGPIL@SANITIZE@ 10085ad8     hb-aat-layout.obj
 0002:00000ae4       ??_C@_0BL@LJCAAAA@start?5?$FL?$CFp?4?4?$CFp?$FN?5?$CI?$CFlu?5bytes?$CJ@ 10085ae4     hb-aat-layout.obj
 0002:00000b00       ??_C@_0BO@NFKLCDNJ@end?5?$FL?$CFp?4?4?$CFp?$FN?5?$CFu?5edit?5requests@ 10085b00     hb-aat-layout.obj
 0002:00000b20       ??_C@_02GIPFHKNO@OK@       10085b20     hb-aat-layout.obj
 0002:00000b24       ??_C@_0N@FLBMHONH@OUT?9OF?9RANGE@ 10085b24     hb-aat-layout.obj
 0002:00000b34       ??_C@_0DC@DHOCDOGD@check_range?5?$FL?$CFp?4?4?$CFp?$FN?5?$CI?$CFu?5bytes?$CJ@ 10085b34     hb-aat-layout.obj
 0002:00000b68       ??_C@_0DH@PGHLCKCM@check_range_fast?5?$FL?$CFp?4?4?$CFp?$FN?5?$CI?$CFu?5b@ 10085b68     hb-aat-layout.obj
 0002:00000ba0       ??_C@_07IICDHBMC@GRANTED@  10085ba0     hb-aat-layout.obj
 0002:00000ba8       ??_C@_06GONJNOIB@DENIED@   10085ba8     hb-aat-layout.obj
 0002:00000bb0       ??_C@_0DD@ENACFAKI@may_edit?$CI?$CFu?$CJ?5?$FL?$CFp?4?4?$CFp?$FN?5?$CI?$CFu?5bytes@ 10085bb0     hb-aat-layout.obj
 0002:00000be4       ??_C@_0BB@HBIIGPNG@start?5table?5morx@ 10085be4     hb-aat-layout.obj
 0002:00000bf8       ??_C@_0P@CBPBJJBN@end?5table?5morx@ 10085bf8     hb-aat-layout.obj
 0002:00000c08       ??_C@_0BB@NNDNCANK@start?5table?5mort@ 10085c08     hb-aat-layout.obj
 0002:00000c1c       ??_C@_0P@INEENGBB@end?5table?5mort@ 10085c1c     hb-aat-layout.obj
 0002:00000c2c       ??_C@_0BB@JBHFHKBC@start?5table?5kerx@ 10085c2c     hb-aat-layout.obj
 0002:00000c40       ??_C@_0P@MBAMIMNJ@end?5table?5kerx@ 10085c40     hb-aat-layout.obj
 0002:00000c50       ??_C@_0BC@JDHEBHPG@start?5subtable?5?$CFu@ 10085c50     hb-aat-layout.obj
 0002:00000c64       ??_C@_0BA@JPJCHFDI@end?5subtable?5?$CFu@ 10085c64     hb-aat-layout.obj
 0002:00000c74       ??_C@_0BH@HOIFGKFM@start?5chainsubtable?5?$CFu@ 10085c74     hb-aat-layout.obj
 0002:00000c8c       ??_C@_0BF@LIFFOAHA@end?5chainsubtable?5?$CFu@ 10085c8c     hb-aat-layout.obj
 0002:00000ca4       ??_C@_0L@PIONBGHN@start?5kern@ 10085ca4     hb-aat-layout.obj
 0002:00000cb0       ??_C@_08PMCHELIJ@end?5kern@ 10085cb0     hb-aat-layout.obj
 0002:00000cc0       __real@3fe999999999999a    10085cc0     hb-aat-layout.obj
 0002:00000cd0       ??_C@_04HDKFADDE@BLOB@     10085cd0     hb-blob.obj
 0002:00000cd8       ??_C@_0BH@NNGJHJOL@current?5data?5is?5?9?$DO?5?$CFp?6@ 10085cd8     hb-blob.obj
 0002:00000cf0       ??_C@_0DD@LDEEFHJD@bool?5__thiscall?5hb_blob_t?3?3try_@ 10085cf0     hb-blob.obj
 0002:00000d24       ??_C@_0BL@NAAIMIGO@dupped?5successfully?5?9?$DO?5?$CFp?6@ 10085d24     hb-blob.obj
 0002:00000d40       ??_C@_04CIMGMMMG@text@     10085d40     hb-buffer-serialize.obj
 0002:00000d48       ??_C@_04CLCAKCEI@json@     10085d48     hb-buffer-serialize.obj
 0002:00002798       ??_C@_02GMHACPFF@?$CFu@    10087798     hb-buffer-serialize.obj
 0002:0000279c       ??_C@_08ELFBALIN@?0?$CCcl?$CC?3?$CFu@ 1008779c     hb-buffer-serialize.obj
 0002:000027a8       ??_C@_04MAFNGINP@?$CCu?$CC?3@ 100877a8     hb-buffer-serialize.obj
 0002:000027b0       ??_C@_03LADEAJCH@?$DN?$CFu@ 100877b0     hb-buffer-serialize.obj
 0002:000027b4       ??_C@_06NGBPNBKB@U?$CL?$CF04X@ 100877b4     hb-buffer-serialize.obj
 0002:000027bc       ??_C@_09CPCAOBOK@harfbuzz?5@ 100877bc     hb-buffer-verify.obj
 0002:000027c8       ??_C@_01EEMJAFIK@?6@       100877c8     hb-buffer-verify.obj
 0002:000027cc       ??_C@_0DA@OHKIDNHD@buffer?5verify?5error?3?5clusters?5a@ 100877cc     hb-buffer-verify.obj
 0002:000027fc       ??_C@_0DC@KJMJOHEC@buffer?5verify?5error?3?5unsafe?9to?9@ 100877fc     hb-buffer-verify.obj
 0002:00002830       ??_C@_0DD@CKNGEJOG@buffer?5verify?5error?3?5unsafe?9to?9@ 10087830     hb-buffer-verify.obj
 0002:00002864       ??_C@_0CD@DIKIFAKO@buffer?5verify?5error?3?5text?5was?3?5@ 10087864     hb-buffer-verify.obj
 0002:00002890       ?minus_1@@3IB              10087890     hb-common.obj
 0002:00002894       ?_hb_Null_OT_CmapSubtableLongGroup@@3QBEB 10087894     hb-common.obj
 0002:00003120       ?_hb_Null_OT_Index@@3QBEB  10088120     hb-common.obj
 0002:00003124       ?_hb_Null_OT_VarIdx@@3QBEB 10088124     hb-common.obj
 0002:00003130       ?_hb_Null_AAT_Lookup@@3QBEB 10088130     hb-common.obj
 0002:00003134       ?_hb_Null_AAT_SettingName@@3QBEB 10088134     hb-common.obj
 0002:00003138       ?_hb_NullPool@@3QB_KB      10088138     hb-common.obj
 0002:000046cc       ?_hb_Null_OT_ClipRecord@@3QBEB 100896cc     hb-common.obj
 0002:000046d4       ?_hb_Null_OT_LangSys@@3QBEB 100896d4     hb-common.obj
 0002:000046dc       ?_hb_Null_OT_RangeRecord@@3QBEB 100896dc     hb-common.obj
 0002:000046e8       ??_C@_0L@PGCGEAJK@HB_OPTIONS@ 100896e8     hb-common.obj
 0002:000046f4       ??_C@_0BJ@EELCEACD@uniscribe?9bug?9compatible@ 100896f4     hb-common.obj
 0002:00004710       __real@38800000            10089710     hb-common.obj
 0002:00004714       __real@4f000000            10089714     hb-common.obj
 0002:00004718       __real@3eaaaaab            10089718     hb-draw.obj
 0002:00004728       ??_C@_0L@LHCHIOPJ@successful@ 10089728     hb-face-builder.obj
 0002:00004734       ??_C@_0N@KIEOCLDL@UNSUCCESSFUL@ 10089734     hb-face-builder.obj
 0002:00004744       ??_C@_0CF@PIDDOBFK@end?5?$FL?$CFp?4?4?$CFp?$FN?5serialized?5?$CFu?5byte@ 10089744     hb-face-builder.obj
 0002:0000476c       ??_C@_09EPPNEDIL@SERIALIZE@ 1008976c     hb-face-builder.obj
 0002:000056f0       __xmm@41f00000000000000000000000000000 1008a6f0     hb-font.obj
 0002:00005700       __xmm@7fffffffffffffff7fffffffffffffff 1008a700     hb-font.obj
 0002:00005868       __real@0010000000000000    1008a868     hb-number.obj
 0002:00005870       __real@4024000000000000    1008a870     hb-number.obj
 0002:00005878       __real@42f9999999999990    1008a878     hb-number.obj
 0002:00005880       __real@7fefffffffffffff    1008a880     hb-number.obj
 0002:00005888       __real@8010000000000000    1008a888     hb-number.obj
 0002:00005890       __real@bff0000000000000    1008a890     hb-number.obj
 0002:00005898       __real@ffefffffffffffff    1008a898     hb-number.obj
 0002:00007550       __xmm@41dfffffffc0000041dfffffffc00000 1008c550     hb-ot-cff1-table.obj
 0002:00007560       __xmm@c1e0000000000000c1e0000000000000 1008c560     hb-ot-cff1-table.obj
 0002:00007578       __real@40000000            1008c578     hb-ot-cff2-table.obj
 0002:0000d224       ??_C@_0BB@HNNCONOI@0123456789?4EE?$DP?9?$DP@ 10092224     hb-ot-font.obj
 0002:0000d238       __real@40490fdb            10092238     hb-ot-font.obj
 0002:0000d23c       __real@c0490fdb            1009223c     hb-ot-font.obj
 0002:0000d240       __xmm@3f80000000000000000000003f800000 10092240     hb-ot-font.obj
 0002:0000d250       __xmm@bf800000bf8000000000000000000000 10092250     hb-ot-font.obj
 0002:0000d260       __xmm@ffffffffffffffffffffffffffffffff 10092260     hb-ot-font.obj
 0002:0000da6c       ??_C@_0BN@IMAOBAG@recursing?5to?5lookup?5?$CFu?5at?5?$CFu@ 10092a6c     hb-ot-layout.obj
 0002:0000da8c       ??_C@_0BG@HECNAHM@recursed?5to?5lookup?5?$CFu@ 10092a8c     hb-ot-layout.obj
 0002:0000daa4       ??_C@_0BI@LEONKCCB@positioning?5glyph?5at?5?$CFu@ 10092aa4     hb-ot-layout.obj
 0002:0000dabc       ??_C@_0BH@NHBAIFPO@positioned?5glyph?5at?5?$CFu@ 10092abc     hb-ot-layout.obj
 0002:0000dad4       ??_C@_0CN@LEDGNLBP@cursive?5attaching?5glyph?5at?5?$CFu?5t@ 10092ad4     hb-ot-layout.obj
 0002:0000db04       ??_C@_0CM@NPOIGCBF@cursive?5attached?5glyph?5at?5?$CFu?5to@ 10092b04     hb-ot-layout.obj
 0002:0000db30       ??_C@_0CK@HCENOEA@attaching?5mark?5glyph?5at?5?$CFu?5to?5g@ 10092b30     hb-ot-layout.obj
 0002:0000db5c       ??_C@_0CJ@IBLNDIDG@attached?5mark?5glyph?5at?5?$CFu?5to?5gl@ 10092b5c     hb-ot-layout.obj
 0002:0000db88       ??_C@_0DG@CFBMBHJC@replacing?5glyph?5at?5?$CFu?5?$CIreverse?5@ 10092b88     hb-ot-layout.obj
 0002:0000dbc0       ??_C@_0DF@HANPKIIM@replaced?5glyph?5at?5?$CFu?5?$CIreverse?5c@ 10092bc0     hb-ot-layout.obj
 0002:0000dbf8       ??_C@_0BB@INONMPMF@start?5table?5kern@ 10092bf8     hb-ot-layout.obj
 0002:0000dc0c       ??_C@_0P@NNJEDJAO@end?5table?5kern@ 10092c0c     hb-ot-layout.obj
 0002:0000dc1c       ??_C@_0CH@IEHKJJLD@start?5table?5GSUB?5script?5tag?5?8?$CFc@ 10092c1c     hb-ot-layout.obj
 0002:0000dc44       ??_C@_0CF@EJFPDLF@end?5table?5GSUB?5script?5tag?5?8?$CFc?$CFc@ 10092c44     hb-ot-layout.obj
 0002:0000dc6c       ??_C@_0CH@GMBJPMNF@start?5table?5GPOS?5script?5tag?5?8?$CFc@ 10092c6c     hb-ot-layout.obj
 0002:0000dc94       ??_C@_0CF@OMPGJGND@end?5table?5GPOS?5script?5tag?5?8?$CFc?$CFc@ 10092c94     hb-ot-layout.obj
 0002:0000dcbc       ??_C@_0CD@BOMDBIAK@start?5lookup?5?$CFu?5feature?5?8?$CFc?$CFc?$CFc@ 10092cbc     hb-ot-layout.obj
 0002:0000dce0       ??_C@_0DO@IEOLAPEI@skipped?5lookup?5?$CFu?5feature?5?8?$CFc?$CFc@ 10092ce0     hb-ot-layout.obj
 0002:0000dd20       ??_C@_0CB@CHKBGOD@end?5lookup?5?$CFu?5feature?5?8?$CFc?$CFc?$CFc?$CFc@ 10092d20     hb-ot-layout.obj
 0002:0000dd44       ??_C@_0CM@MBFHEMDL@replacing?5glyph?5at?5?$CFu?5?$CIsingle?5s@ 10092d44     hb-ot-layout.obj
 0002:0000dd70       ??_C@_0CL@HNJEFGAB@replaced?5glyph?5at?5?$CFu?5?$CIsingle?5su@ 10092d70     hb-ot-layout.obj
 0002:0000dd9c       ??_C@_0BM@ILJLMNPF@try?5kerning?5glyphs?5at?5?$CFu?0?$CFu@ 10092d9c     hb-ot-layout.obj
 0002:0000ddb8       ??_C@_0BH@OPPMFNJB@kerned?5glyphs?5at?5?$CFu?0?$CFu@ 10092db8     hb-ot-layout.obj
 0002:0000ddd0       ??_C@_0BO@DMMODMBI@tried?5kerning?5glyphs?5at?5?$CFu?0?$CFu@ 10092dd0     hb-ot-layout.obj
 0002:0000ddf0       ??_C@_0CP@EIOKABLL@replacing?5glyph?5at?5?$CFu?5?$CIalternat@ 10092df0     hb-ot-layout.obj
 0002:0000de20       ??_C@_0CO@NDFGAIJA@replaced?5glyph?5at?5?$CFu?5?$CIalternate@ 10092e20     hb-ot-layout.obj
 0002:0000de50       ??_C@_0CO@BKNPNBH@replacing?5glyph?5at?5?$CFu?5?$CImultiple@ 10092e50     hb-ot-layout.obj
 0002:0000de80       ??_C@_0CN@NJGGGGNH@replaced?5glyph?5at?5?$CFu?5?$CImultiple?5@ 10092e80     hb-ot-layout.obj
 0002:0000deb0       ??_C@_0CN@NDMMJMPC@deleting?5glyph?5at?5?$CFu?5?$CImultiple?5@ 10092eb0     hb-ot-layout.obj
 0002:0000dee0       ??_C@_0CM@LFICHOPB@deleted?5glyph?5at?5?$CFu?5?$CImultiple?5s@ 10092ee0     hb-ot-layout.obj
 0002:0000df0c       ??_C@_0BI@MNHOPBOM@multiplying?5glyph?5at?5?$CFu@ 10092f0c     hb-ot-layout.obj
 0002:0000df24       ??_C@_0BI@MMDNIBFC@multiplied?5glyphs?5at?5?$CFs@ 10092f24     hb-ot-layout.obj
 0002:0000df3c       ??_C@_0CO@NFINLDBE@replacing?5glyph?5at?5?$CFu?5?$CIligature@ 10092f3c     hb-ot-layout.obj
 0002:0000df6c       ??_C@_0CN@NEGCINE@replaced?5glyph?5at?5?$CFu?5?$CIligature?5@ 10092f6c     hb-ot-layout.obj
 0002:0000df9c       ??_C@_0BG@PELKDOGC@ligating?5glyphs?5at?5?$CFs@ 10092f9c     hb-ot-layout.obj
 0002:0000dfb4       ??_C@_0BE@CENOONDG@ligated?5glyph?5at?5?$CFu@ 10092fb4     hb-ot-layout.obj
 0002:0000f334       ??_C@_0BE@JHLPALHA@start?5fallback?5mark@ 10094334     hb-ot-shape-fallback.obj
 0002:0000f348       ??_C@_0BC@GBHKPNCC@end?5fallback?5mark@ 10094348     hb-ot-shape-fallback.obj
 0002:0000f35c       ??_C@_0BE@OKOKJNMC@start?5fallback?5kern@ 1009435c     hb-ot-shape-fallback.obj
 0002:0000f370       ??_C@_0BC@BMCPGLJA@end?5fallback?5kern@ 10094370     hb-ot-shape-fallback.obj
 0002:0000f38c       ??_C@_0O@PHODME@start?5reorder@ 1009438c     hb-ot-shape-normalize.obj
 0002:0000f39c       ??_C@_0M@MGJODAHL@end?5reorder@ 1009439c     hb-ot-shape-normalize.obj
 0002:0000f420       ??_C@_0BJ@JCPBKLAK@start?5postprocess?9glyphs@ 10094420     hb-ot-shape.obj
 0002:0000f43c       ??_C@_0BH@KGKNGMEK@end?5postprocess?9glyphs@ 1009443c     hb-ot-shape.obj
 0002:0000f454       ??_C@_0BG@KEPPLGKM@start?5preprocess?9text@ 10094454     hb-ot-shape.obj
 0002:0000f46c       ??_C@_0BE@HIKMCIJG@end?5preprocess?9text@ 1009446c     hb-ot-shape.obj
 0002:0000f480       ??_C@_02IGGBGAC@ot@        10094480     hb-ot-shape.obj
 0002:0000f490       __xmm@00000007000000070000000700000007 10094490     hb-ot-shape.obj
 0002:0000f4c4       ?_hb_ot_shaper_arabic@@3Uhb_ot_shaper_t@@B 100944c4     hb-ot-shaper-arabic.obj
 0002:000106d0       ??_C@_09BJHPDKCP@measuring@ 100956d0     hb-ot-shaper-arabic.obj
 0002:000106dc       ??_C@_07MINDNCFJ@cutting@  100956dc     hb-ot-shaper-arabic.obj
 0002:000106e4       ??_C@_0BJ@CMFJBMOA@?$CFs?5stretch?5at?5?$CI?$CFu?0?$CFu?0?$CFu?$CJ@ 100956e4     hb-ot-shaper-arabic.obj
 0002:00010700       ??_C@_06DBDILMHG@ARABIC@   10095700     hb-ot-shaper-arabic.obj
 0002:00010710       ?_hb_ot_shaper_default@@3Uhb_ot_shaper_t@@B 10095710     hb-ot-shaper-default.obj
 0002:00010748       ?_hb_ot_shaper_dumber@@3Uhb_ot_shaper_t@@B 10095748     hb-ot-shaper-default.obj
 0002:00010788       ?_hb_ot_shaper_hangul@@3Uhb_ot_shaper_t@@B 10095788     hb-ot-shaper-hangul.obj
 0002:000107d8       ?_hb_ot_shaper_hebrew@@3Uhb_ot_shaper_t@@B 100957d8     hb-ot-shaper-hebrew.obj
 0002:000131d8       ?_hb_ot_shaper_indic@@3Uhb_ot_shaper_t@@B 100981d8     hb-ot-shaper-indic.obj
 0002:00013ec8       ??_C@_0BP@PFJNIBAL@start?5reordering?5indic?5initial@ 10098ec8     hb-ot-shaper-indic.obj
 0002:00013ee8       ??_C@_0BN@DEJECPK@end?5reordering?5indic?5initial@ 10098ee8     hb-ot-shaper-indic.obj
 0002:00013f08       ??_C@_0BN@BEFMFOMM@start?5reordering?5indic?5final@ 10098f08     hb-ot-shaper-indic.obj
 0002:00013f28       ??_C@_0BL@CMBCGANJ@end?5reordering?5indic?5final@ 10098f28     hb-ot-shaper-indic.obj
 0002:00013f50       ?_hb_ot_shaper_khmer@@3Uhb_ot_shaper_t@@B 10098f50     hb-ot-shaper-khmer.obj
 0002:00014540       ??_C@_0BH@LEEFGPFH@start?5reordering?5khmer@ 10099540     hb-ot-shaper-khmer.obj
 0002:00014558       ??_C@_0BF@HCJFOFHL@end?5reordering?5khmer@ 10099558     hb-ot-shaper-khmer.obj
 0002:00014578       ?_hb_ot_shaper_myanmar@@3Uhb_ot_shaper_t@@B 10099578     hb-ot-shaper-myanmar.obj
 0002:000145b0       ?_hb_ot_shaper_myanmar_zawgyi@@3Uhb_ot_shaper_t@@B 100995b0     hb-ot-shaper-myanmar.obj
 0002:00015050       ??_C@_0BJ@HDEFJBCC@start?5reordering?5myanmar@ 1009a050     hb-ot-shaper-myanmar.obj
 0002:0001506c       ??_C@_0BH@EHBJFGGC@end?5reordering?5myanmar@ 1009a06c     hb-ot-shaper-myanmar.obj
 0002:00015090       ??_C@_0EG@MEHLKFP@skipped?5inserting?5dotted?9circle@ 1009a090     hb-ot-shaper-syllabic.obj
 0002:000150d8       ??_C@_0BP@BAKDHKAL@start?5inserting?5dotted?9circles@ 1009a0d8     hb-ot-shaper-syllabic.obj
 0002:000150f8       ??_C@_0BN@OGHHLJPK@end?5inserting?5dotted?9circles@ 1009a0f8     hb-ot-shaper-syllabic.obj
 0002:00015120       ?_hb_ot_shaper_thai@@3Uhb_ot_shaper_t@@B 1009a120     hb-ot-shaper-thai.obj
 0002:000152d0       ?_hb_ot_shaper_use@@3Uhb_ot_shaper_t@@B 1009a2d0     hb-ot-shaper-use.obj
 0002:00017cec       ??_C@_0BF@INKMBGAO@start?5reordering?5USE@ 1009ccec     hb-ot-shaper-use.obj
 0002:00017d04       ??_C@_0BD@IDPODCA@end?5reordering?5USE@ 1009cd04     hb-ot-shaper-use.obj
 0002:0001a958       ??_C@_08LOEDBOED@?9fonnapa@ 1009f958     hb-ot-tag.obj
 0002:0001a964       ??_C@_08GMLKJDFJ@?9polyton@ 1009f964     hb-ot-tag.obj
 0002:0001a970       ??_C@_08NJCBHCMA@?9arevmda@ 1009f970     hb-ot-tag.obj
 0002:0001a97c       ??_C@_08DCLOKPKI@?9provenc@ 1009f97c     hb-ot-tag.obj
 0002:0001a988       ??_C@_07KBFBNAFC@?9fonipa@ 1009f988     hb-ot-tag.obj
 0002:0001a990       ??_C@_05BHGHNKKJ@?9geok@   1009f990     hb-ot-tag.obj
 0002:0001a998       ??_C@_05BCLFBOGB@?9syre@   1009f998     hb-ot-tag.obj
 0002:0001a9a0       ??_C@_05JFCNACKO@?9syrj@   1009f9a0     hb-ot-tag.obj
 0002:0001a9a8       ??_C@_05PBEBMHKK@?9syrn@   1009f9a8     hb-ot-tag.obj
 0002:0001a9b0       ??_C@_09GEIHALDG@rt?9lojban@ 1009f9b0     hb-ot-tag.obj
 0002:0001a9bc       ??_C@_0L@KFNBBKMN@do?9hant?9hk@ 1009f9bc     hb-ot-tag.obj
 0002:0001a9c8       ??_C@_0L@MHHGBNCC@do?9hant?9mo@ 1009f9c8     hb-ot-tag.obj
 0002:0001a9d4       ??_C@_0L@NNBHMAGE@jy?9hant?9hk@ 1009f9d4     hb-ot-tag.obj
 0002:0001a9e0       ??_C@_0L@LPLAMHIL@jy?9hant?9mo@ 1009f9e0     hb-ot-tag.obj
 0002:0001a9ec       ??_C@_0L@DBFOEPHG@mn?9hant?9hk@ 1009f9ec     hb-ot-tag.obj
 0002:0001a9f8       ??_C@_0L@FDPJEIJJ@mn?9hant?9mo@ 1009f9f8     hb-ot-tag.obj
 0002:0001aa04       ??_C@_0L@JBNLJICM@np?9hant?9hk@ 1009fa04     hb-ot-tag.obj
 0002:0001aa10       ??_C@_0L@PDHMJPMD@np?9hant?9mo@ 1009fa10     hb-ot-tag.obj
 0002:0001aa1c       ??_C@_0L@HOIMDHBF@px?9hant?9hk@ 1009fa1c     hb-ot-tag.obj
 0002:0001aa28       ??_C@_0L@BMCLDAPK@px?9hant?9mo@ 1009fa28     hb-ot-tag.obj
 0002:0001aa34       ??_C@_0L@PELJBBOA@sp?9hant?9hk@ 1009fa34     hb-ot-tag.obj
 0002:0001aa40       ??_C@_0L@JGBOBGAP@sp?9hant?9mo@ 1009fa40     hb-ot-tag.obj
 0002:0001aa4c       ??_C@_0L@LLINOOHJ@zh?9hant?9hk@ 1009fa4c     hb-ot-tag.obj
 0002:0001aa58       ??_C@_0L@NJCKOJJG@zh?9hant?9mo@ 1009fa58     hb-ot-tag.obj
 0002:0001aa64       ??_C@_0L@FJFBPFAA@zo?9hant?9hk@ 1009fa64     hb-ot-tag.obj
 0002:0001aa70       ??_C@_0L@DLPGPCOP@zo?9hant?9mo@ 1009fa70     hb-ot-tag.obj
 0002:0001aa7c       ??_C@_07GEDDMEMG@do?9hans@ 1009fa7c     hb-ot-tag.obj
 0002:0001aa84       ??_C@_07CLHCFCAB@do?9hant@ 1009fa84     hb-ot-tag.obj
 0002:0001aa8c       ??_C@_07HFLHHPAA@jy?9hans@ 1009fa8c     hb-ot-tag.obj
 0002:0001aa94       ??_C@_07DKPGOJMH@jy?9hant@ 1009fa94     hb-ot-tag.obj
 0002:0001aa9c       ??_C@_07NNALNEFJ@mn?9hans@ 1009fa9c     hb-ot-tag.obj
 0002:0001aaa4       ??_C@_07JCEKECJO@mn?9hant@ 1009faa4     hb-ot-tag.obj
 0002:0001aaac       ??_C@_07GEGFDECJ@np?9hans@ 1009faac     hb-ot-tag.obj
 0002:0001aab4       ??_C@_07CLCEKCOO@np?9hant@ 1009fab4     hb-ot-tag.obj
 0002:0001aabc       ??_C@_07DOLLFJFH@px?9hans@ 1009fabc     hb-ot-tag.obj
 0002:0001aac4       ??_C@_07HBPKMPJA@px?9hant@ 1009fac4     hb-ot-tag.obj
 0002:0001aacc       ??_C@_07IDNLBAND@sp?9hans@ 1009facc     hb-ot-tag.obj
 0002:0001aad4       ??_C@_07MMJKIGBE@sp?9hant@ 1009fad4     hb-ot-tag.obj
 0002:0001aadc       ??_C@_07MIKFNJFB@zh?9hans@ 1009fadc     hb-ot-tag.obj
 0002:0001aae4       ??_C@_07IHOEEPJG@zh?9hant@ 1009fae4     hb-ot-tag.obj
 0002:0001aaec       ??_C@_07NACOHNP@zo?9hans@  1009faec     hb-ot-tag.obj
 0002:0001aaf4       ??_C@_07ECEDHBBI@zo?9hant@ 1009faf4     hb-ot-tag.obj
 0002:0001aafc       ??_C@_03JFOJGEF@do?9@      1009fafc     hb-ot-tag.obj
 0002:0001ab00       ??_C@_03EMCOHPPE@?9hk@     1009fb00     hb-ot-tag.obj
 0002:0001ab04       ??_C@_03COIJHIBL@?9mo@     1009fb04     hb-ot-tag.obj
 0002:0001ab08       ??_C@_03LPGFHILN@?9tw@     1009fb08     hb-ot-tag.obj
 0002:0001ab0c       ??_C@_03PBCKDOLE@jy?9@     1009fb0c     hb-ot-tag.obj
 0002:0001ab10       ??_C@_03HFJELDPI@mn?9@     1009fb10     hb-ot-tag.obj
 0002:0001ab14       ??_C@_03HBJJJCGM@np?9@     1009fb14     hb-ot-tag.obj
 0002:0001ab18       ??_C@_03MPEMODHI@px?9@     1009fb18     hb-ot-tag.obj
 0002:0001ab1c       ??_C@_03NDOKBNCO@sp?9@     1009fb1c     hb-ot-tag.obj
 0002:0001ab20       ??_C@_03LMNHKAGM@zh?9@     1009fb20     hb-ot-tag.obj
 0002:0001ab24       ??_C@_03LJJILGOJ@zo?9@     1009fb24     hb-ot-tag.obj
 0002:0001ab28       ??_C@_0L@DLEENNLB@an?9hant?9hk@ 1009fb28     hb-ot-tag.obj
 0002:0001ab34       ??_C@_0L@FJODNKFO@an?9hant?9mo@ 1009fb34     hb-ot-tag.obj
 0002:0001ab40       ??_C@_07IKKEMBBG@an?9hans@ 1009fb40     hb-ot-tag.obj
 0002:0001ab48       ??_C@_07MFOFFHNB@an?9hant@ 1009fb48     hb-ot-tag.obj
 0002:0001ab50       ??_C@_06FCHMEGPO@a?9latg@  1009fb50     hb-ot-tag.obj
 0002:0001ab58       ??_C@_03DPECAMEA@an?9@     1009fb58     hb-ot-tag.obj
 0002:0001ab5c       ??_C@_0L@NNGNBGPF@ak?9hant?9hk@ 1009fb5c     hb-ot-tag.obj
 0002:0001ab68       ??_C@_0L@LPMKBBBK@ak?9hant?9mo@ 1009fb68     hb-ot-tag.obj
 0002:0001ab74       ??_C@_0L@MNNOKALL@sn?9hant?9hk@ 1009fb74     hb-ot-tag.obj
 0002:0001ab80       ??_C@_0L@KPHJKHFE@sn?9hant?9mo@ 1009fb80     hb-ot-tag.obj
 0002:0001ab8c       ??_C@_07NIJMOOLB@ak?9hans@ 1009fb8c     hb-ot-tag.obj
 0002:0001ab94       ??_C@_07JHNNHIHG@ak?9hant@ 1009fb94     hb-ot-tag.obj
 0002:0001ab9c       ??_C@_07LEDKPHEA@sn?9hans@ 1009fb9c     hb-ot-tag.obj
 0002:0001aba4       ??_C@_07PLHLGBIH@sn?9hant@ 1009fba4     hb-ot-tag.obj
 0002:0001abac       ??_C@_03DJIJMOKL@ak?9@     1009fbac     hb-ot-tag.obj
 0002:0001abb0       ??_C@_03MFFCJDFE@sn?9@     1009fbb0     hb-ot-tag.obj
 0002:0001abb4       ??_C@_07LCKCAAMB@?9navajo@ 1009fbb4     hb-ot-tag.obj
 0002:0001abbc       ??_C@_04DBACCPMA@?9hak@    1009fbbc     hb-ot-tag.obj
 0002:0001abc4       ??_C@_04MEKAPCKJ@?9lux@    1009fbc4     hb-ot-tag.obj
 0002:0001abcc       ??_C@_03HENGIEOJ@nw?9@     1009fbcc     hb-ot-tag.obj
 0002:0001abd0       ??_C@_03HCDPHGCD@?9th@     1009fbd0     hb-ot-tag.obj
 0002:0001abd4       ??_C@_05NKGDAJJP@o?9bok@   1009fbd4     hb-ot-tag.obj
 0002:0001abdc       ??_C@_05PFGJJNKA@o?9nyn@   1009fbdc     hb-ot-tag.obj
 0002:0001abe4       ??_C@_02GDBPPABP@o?9@      1009fbe4     hb-ot-tag.obj
 0002:0001abe8       ??_C@_03MNHNKBNA@?9md@     1009fbe8     hb-ot-tag.obj
 0002:0001abec       ??_C@_0L@PKCFBAOH@uu?9hant?9hk@ 1009fbec     hb-ot-tag.obj
 0002:0001abf8       ??_C@_0L@JIICBHAI@uu?9hant?9mo@ 1009fbf8     hb-ot-tag.obj
 0002:0001ac04       ??_C@_07BHIMDGPD@uu?9hans@ 1009fc04     hb-ot-tag.obj
 0002:0001ac0c       ??_C@_07FIMNKADE@uu?9hant@ 1009fc0c     hb-ot-tag.obj
 0002:0001ac14       ??_C@_03PAEKIABJ@uu?9@     1009fc14     hb-ot-tag.obj
 0002:0001ac18       ??_C@_07HAFCKKDN@ue?9hans@ 1009fc18     hb-ot-tag.obj
 0002:0001ac20       ??_C@_09CPANDNJE@h?9hant?9hk@ 1009fc20     hb-ot-tag.obj
 0002:0001ac2c       ??_C@_09ENKKDKHL@h?9hant?9mo@ 1009fc2c     hb-ot-tag.obj
 0002:0001ac38       ??_C@_09JKAGOIDE@h?9min?9nan@ 1009fc38     hb-ot-tag.obj
 0002:0001ac44       ??_C@_06NHLFEBO@h?9hans@   1009fc44     hb-ot-tag.obj
 0002:0001ac4c       ??_C@_06ECDKMCNJ@h?9hant@  1009fc4c     hb-ot-tag.obj
 0002:0001ac54       ??_C@_05OGPPKBIG@h?9min@   1009fc54     hb-ot-tag.obj
 0002:0001ac5c       ??_C@_02GGFAOGJK@h?9@      1009fc5c     hb-ot-tag.obj
 0002:0001ac60       ??_C@_03FHLPDODD@alt@      1009fc60     hb-ot-tag.obj
 0002:0001ac64       ??_C@_0M@EFNICDFC@und?9fonnapa@ 1009fc64     hb-ot-tag.obj
 0002:0001ac70       ??_C@_02FEKCJMIO@ar@       1009fc70     hb-ot-tag.obj
 0002:0001ac74       ??_C@_03OPDALMNL@rki@      1009fc74     hb-ot-tag.obj
 0002:0001ac78       ??_C@_03KDPNJBKG@ath@      1009fc78     hb-ot-tag.obj
 0002:0001ac7c       ??_C@_03BMIBANNE@ber@      1009fc7c     hb-ot-tag.obj
 0002:0001ac80       ??_C@_03IOJLFNKI@bik@      1009fc80     hb-ot-tag.obj
 0002:0001ac84       ??_C@_03JKGFGNIL@btk@      1009fc84     hb-ot-tag.obj
 0002:0001ac88       ??_C@_03IPGCLNMG@crp@      1009fc88     hb-ot-tag.obj
 0002:0001ac8c       ??_C@_03EHLLDHMO@crx@      1009fc8c     hb-ot-tag.obj
 0002:0001ac90       ??_C@_03JNELBMEE@doi@      1009fc90     hb-ot-tag.obj
 0002:0001ac94       ??_C@_03NGIHPGDB@din@      1009fc94     hb-ot-tag.obj
 0002:0001ac98       ??_C@_03OGODBGHE@prs@      1009fc98     hb-ot-tag.obj
 0002:0001ac9c       ??_C@_02JKLANEGN@dz@       1009fc9c     hb-ot-tag.obj
 0002:0001aca0       ??_C@_02FPBJDNE@et@        1009fca0     hb-ot-tag.obj
 0002:0001aca4       ??_C@_02DAACMLJJ@fa@       1009fca4     hb-ot-tag.obj
 0002:0001aca8       ??_C@_03MALPCFGN@gon@      1009fca8     hb-ot-tag.obj
 0002:0001acac       ??_C@_03NPJADACO@mrj@      1009fcac     hb-ot-tag.obj
 0002:0001acb0       ??_C@_03JLFIOBFF@hmn@      1009fcb0     hb-ot-tag.obj
 0002:0001acb4       ??_C@_03GDPBLHIG@hnd@      1009fcb4     hb-ot-tag.obj
 0002:0001acb8       ??_C@_03BLHHEDOB@hyw@      1009fcb8     hb-ot-tag.obj
 0002:0001acbc       ??_C@_03KPCANNMC@iba@      1009fcbc     hb-ot-tag.obj
 0002:0001acc0       ??_C@_03DPLAKBPE@ijo@      1009fcc0     hb-ot-tag.obj
 0002:0001acc4       ??_C@_02BFPAFLPB@iu@       1009fcc4     hb-ot-tag.obj
 0002:0001acc8       ??_C@_02MBLBGECO@ik@       1009fcc8     hb-ot-tag.obj
 0002:0001accc       ??_C@_0L@OOCAKEAN@und?9fonipa@ 1009fccc     hb-ot-tag.obj
 0002:0001acd8       ??_C@_07LBNNMAEP@ga?9Latg@ 1009fcd8     hb-ot-tag.obj
 0002:0001ace0       ??_C@_02OPKBKFNM@yi@       1009fce0     hb-ot-tag.obj
 0002:0001ace4       ??_C@_03IICPCEIM@kln@      1009fce4     hb-ot-tag.obj
 0002:0001ace8       ??_C@_08IBMBBMEF@und?9Geok@ 1009fce8     hb-ot-tag.obj
 0002:0001acf4       ??_C@_02FJDFBJFI@kr@       1009fcf4     hb-ot-tag.obj
 0002:0001acf8       ??_C@_03CJCPPGJN@okm@      1009fcf8     hb-ot-tag.obj
 0002:0001acfc       ??_C@_03PHBOGOJA@kok@      1009fcfc     hb-ot-tag.obj
 0002:0001ad00       ??_C@_02DNFJNMFM@kv@       1009fd00     hb-ot-tag.obj
 0002:0001ad04       ??_C@_03HOOHKHFD@kpe@      1009fd04     hb-ot-tag.obj
 0002:0001ad08       ??_C@_03GGIAOKIC@kar@      1009fd08     hb-ot-tag.obj
 0002:0001ad0c       ??_C@_03HCOHIEGC@uki@      1009fd0c     hb-ot-tag.obj
 0002:0001ad10       ??_C@_02BGHEIPJP@ku@       1009fd10     hb-ot-tag.obj
 0002:0001ad14       ??_C@_03EMDKIONB@mhr@      1009fd14     hb-ot-tag.obj
 0002:0001ad18       ??_C@_03DIMAAFM@luy@       1009fd18     hb-ot-tag.obj
 0002:0001ad1c       ??_C@_02DIBGMKNJ@lv@       1009fd1c     hb-ot-tag.obj
 0002:0001ad20       ??_C@_03FLEAGKJM@mwr@      1009fd20     hb-ot-tag.obj
 0002:0001ad24       ??_C@_02GKANIDPO@mg@       1009fd24     hb-ot-tag.obj
 0002:0001ad28       ??_C@_02EEKDFEKL@ms@       1009fd28     hb-ot-tag.obj
 0002:0001ad2c       ??_C@_02LLMPDILH@mn@       1009fd2c     hb-ot-tag.obj
 0002:0001ad30       ??_C@_03KFJMOIAD@man@      1009fd30     hb-ot-tag.obj
 0002:0001ad34       ??_C@_05KNLKPBHL@ro?9MD@   1009fd34     hb-ot-tag.obj
 0002:0001ad3c       ??_C@_06PALDGLND@mnw?9TH@  1009fd3c     hb-ot-tag.obj
 0002:0001ad44       ??_C@_03LHKJBKML@myn@      1009fd44     hb-ot-tag.obj
 0002:0001ad48       ??_C@_03OBHDOAGL@nah@      1009fd48     hb-ot-tag.obj
 0002:0001ad4c       ??_C@_02FKHNFPCF@ne@       1009fd4c     hb-ot-tag.obj
 0002:0001ad50       ??_C@_03JFNCHPFJ@njz@      1009fd50     hb-ot-tag.obj
 0002:0001ad54       ??_C@_02KAJCLHKP@no@       1009fd54     hb-ot-tag.obj
 0002:0001ad58       ??_C@_02NMCHCJNN@oj@       1009fd58     hb-ot-tag.obj
 0002:0001ad5c       ??_C@_02JDGGLPBK@om@       1009fd5c     hb-ot-tag.obj
 0002:0001ad60       ??_C@_02FAFNGEII@ps@       1009fd60     hb-ot-tag.obj
 0002:0001ad64       ??_C@_0L@LGMOIJP@el?9polyton@ 1009fd64     hb-ot-tag.obj
 0002:0001ad70       ??_C@_03JEELCJ@pro@        1009fd70     hb-ot-tag.obj
 0002:0001ad74       ??_C@_03PCCGKMAO@quh@      1009fd74     hb-ot-tag.obj
 0002:0001ad78       ??_C@_02HMFKJDJ@qu@        1009fd78     hb-ot-tag.obj
 0002:0001ad7c       ??_C@_03OJHLCDBG@qvi@      1009fd7c     hb-ot-tag.obj
 0002:0001ad80       ??_C@_03PBKCHIGA@qwh@      1009fd80     hb-ot-tag.obj
 0002:0001ad84       ??_C@_03MJIKGKMO@raj@      1009fd84     hb-ot-tag.obj
 0002:0001ad88       ??_C@_02LFKOONLL@ro@       1009fd88     hb-ot-tag.obj
 0002:0001ad8c       ??_C@_03IMFFNBAD@rom@      1009fd8c     hb-ot-tag.obj
 0002:0001ad90       ??_C@_02GACNLIFD@sq@       1009fd90     hb-ot-tag.obj
 0002:0001ad94       ??_C@_02ELAAOLJA@sr@       1009fd94     hb-ot-tag.obj
 0002:0001ad98       ??_C@_03KNGLMNJH@xnj@      1009fd98     hb-ot-tag.obj
 0002:0001ad9c       ??_C@_03OBBIGHDK@syr@      1009fd9c     hb-ot-tag.obj
 0002:0001ada0       ??_C@_08IEBDNIIN@und?9Syre@ 1009fda0     hb-ot-tag.obj
 0002:0001adac       ??_C@_08DILMEEC@und?9Syrj@ 1009fdac     hb-ot-tag.obj
 0002:0001adb8       ??_C@_08GHOHABEG@und?9Syrn@ 1009fdb8     hb-ot-tag.obj
 0002:0001adc4       ??_C@_03NHMNKOPE@tmh@      1009fdc4     hb-ot-tag.obj
 0002:0001adc8       ??_C@_03MDOLKBCN@xwo@      1009fdc8     hb-ot-tag.obj
 0002:0001adcc       ??_C@_05HCJKHBCC@zh?9HK@   1009fdcc     hb-ot-tag.obj
 0002:0001add4       ??_C@_07JGEPGFF@zh?9Hans@  1009fdd4     hb-ot-tag.obj
 0002:0001addc       ??_C@_07EGCFGAJC@zh?9Hant@ 1009fddc     hb-ot-tag.obj
 0002:0001ade4       ??_C@_05BADNHGMN@zh?9MO@   1009fde4     hb-ot-tag.obj
 0002:0001adec       ??_C@_03PPLJNHHL@zza@      1009fdec     hb-ot-tag.obj
 0002:0001adf0       ??_C@_05NFAFKFNN@?9hbsc@   1009fdf0     hb-ot-tag.obj
 0002:0001adf8       ??_C@_05MFLKHLFP@?9hbot@   1009fdf8     hb-ot-tag.obj
 0002:0001ae00       ??_C@_0M@MFILKOCI@x?9hbot?9?$CF08x@ 1009fe00     hb-ot-tag.obj
 0002:0001ae14       __real@46800000            1009fe14     hb-ot-var.obj
 0002:0001ae18       __real@bf700000            1009fe18     hb-outline.obj
 0002:0001ae2c       ??_C@_08LFBOCJLE@fallback@ 1009fe2c     hb-shape-plan.obj
 0002:0001ae38       ??_C@_0DF@MPFFHONM@face?$DN?$CFp?5num_features?$DN?$CFu?5num_coo@ 1009fe38     hb-shape-plan.obj
 0002:0001ae70       ??_C@_0MH@MMALGGGN@struct?5hb_shape_plan_t?5?$CK__cdecl@ 1009fe70     hb-shape-plan.obj
 0002:0001af38       ??_C@_0L@HJBOBLCO@SHAPE_PLAN@ 1009ff38     hb-shape-plan.obj
 0002:0001af44       ??_C@_0CP@GAFDBLDO@num_features?$DN?$CFu?5shaper_func?$DN?$CFp?0@ 1009ff44     hb-shape-plan.obj
 0002:0001af78       ??_C@_0JI@JOJJJOPA@bool?5__cdecl?5_hb_shape_plan_exe@ 1009ff78     hb-shape-plan.obj
 0002:0001b010       ??_C@_0CH@EAKAEIJM@face?$DN?$CFp?5num_features?$DN?$CFu?5shaper_@ 100a0010     hb-shape-plan.obj
 0002:0001b038       ??_C@_0MO@MGHFPDJG@struct?5hb_shape_plan_t?5?$CK__cdecl@ 100a0038     hb-shape-plan.obj
 0002:0001b13c       ??_C@_0P@GEOKODDH@HB_SHAPER_LIST@ 100a013c     hb-shaper.obj
 0002:0002eb70       ?_hb_modified_combining_class@@3QBEB 100b3b70     hb-unicode.obj
 0002:0002ec70       ??_C@_0BG@NKHBBPH@sun?1font?1TrueTypeFont@ 100b3c70     sunFont.obj
 0002:0002ec88       ??_C@_0BL@GAAGJDLL@?$CILjava?1nio?1ByteBuffer?$DLII?$CJI@ 100b3c88     sunFont.obj
 0002:0002eca4       ??_C@_09CKAKNPHP@readBlock@ 100b3ca4     sunFont.obj
 0002:0002ecb0       ??_C@_06JMOJDKIE@?$CIII?$CJ?$FLB@ 100b3cb0     sunFont.obj
 0002:0002ecb8       ??_C@_09IDIEPDPI@readBytes@ 100b3cb8     sunFont.obj
 0002:0002ecc4       ??_C@_0BD@OPLCIPMH@sun?1font?1Type1Font@ 100b3cc4     sunFont.obj
 0002:0002ecd8       ??_C@_0BJ@LMHMPPKE@?$CILjava?1nio?1ByteBuffer?$DL?$CJV@ 100b3cd8     sunFont.obj
 0002:0002ecf4       ??_C@_08CJNGBMAG@readFile@ 100b3cf4     sunFont.obj
 0002:0002ed00       ??_C@_0BM@DGICEJAA@java?1awt?1geom?1Point2D$Float@ 100b3d00     sunFont.obj
 0002:0002ed1c       ??_C@_05BHHDPELC@?$CIFF?$CJV@ 100b3d1c     sunFont.obj
 0002:0002ed24       ??_C@_01BIAFAFID@F@        100b3d24     sunFont.obj
 0002:0002ed28       ??_C@_01FJMABOPO@x@        100b3d28     sunFont.obj
 0002:0002ed2c       ??_C@_01EANLCPLP@y@        100b3d2c     sunFont.obj
 0002:0002ed30       ??_C@_0BH@ENELCGL@sun?1font?1StrikeMetrics@ 100b3d30     sunFont.obj
 0002:0002ed48       ??_C@_0O@LBAHCNJL@?$CIFFFFFFFFFF?$CJV@ 100b3d48     sunFont.obj
 0002:0002ed58       ??_C@_0CA@PDMBNICK@java?1awt?1geom?1Rectangle2D$Float@ 100b3d58     sunFont.obj
 0002:0002ed78       ??_C@_07PMCFNNPC@?$CIFFFF?$CJV@ 100b3d78     sunFont.obj
 0002:0002ed80       ??_C@_05IGKADHGO@width@    100b3d80     sunFont.obj
 0002:0002ed88       ??_C@_06LNLHEAAG@height@   100b3d88     sunFont.obj
 0002:0002ed90       ??_C@_0BK@COJNCHEM@java?1awt?1geom?1GeneralPath@ 100b3d90     sunFont.obj
 0002:0002edac       ??_C@_0L@MDPODKN@?$CII?$FLBI?$FLFI?$CJV@ 100b3dac     sunFont.obj
 0002:0002edb8       ??_C@_0BA@OKNBFGCN@sun?1font?1Font2D@ 100b3db8     sunFont.obj
 0002:0002edc8       ??_C@_04DIFHPCLD@?$CII?$CJI@ 100b3dc8     sunFont.obj
 0002:0002edd0       ??_C@_0M@NMGOHDEJ@charToGlyph@ 100b3dd0     sunFont.obj
 0002:0002eddc       ??_C@_05BKHNKL@?$CIII?$CJI@ 100b3ddc     sunFont.obj
 0002:0002ede4       ??_C@_0BF@NFJAPLLH@charToVariationGlyph@ 100b3de4     sunFont.obj
 0002:0002edfc       ??_C@_0BP@CBNLOFNN@?$CI?$CJLsun?1font?1CharToGlyphMapper?$DL@ 100b3dfc     sunFont.obj
 0002:0002ee1c       ??_C@_09DGCMEJKL@getMapper@ 100b3e1c     sunFont.obj
 0002:0002ee28       ??_C@_05IPLNOPFN@?$CII?$CJ?$FLB@ 100b3e28     sunFont.obj
 0002:0002ee30       ??_C@_0O@DBNIPDIH@getTableBytes@ 100b3e30     sunFont.obj
 0002:0002ee40       ??_C@_04DGAFFDEF@?$CIC?$CJZ@ 100b3e40     sunFont.obj
 0002:0002ee48       ??_C@_0L@PGEPPKMA@canDisplay@ 100b3e48     sunFont.obj
 0002:0002ee54       ??_C@_0BL@GAPGNAAC@sun?1font?1CharToGlyphMapper@ 100b3e54     sunFont.obj
 0002:0002ee70       ??_C@_0BI@GDBHNKM@sun?1font?1PhysicalStrike@ 100b3e70     sunFont.obj
 0002:0002ee88       ??_C@_0CB@IBGFEOCM@?$CII?$CJLjava?1awt?1geom?1Point2D$Float@ 100b3e88     sunFont.obj
 0002:0002eeac       ??_C@_0BA@FMKHNFIF@getGlyphMetrics@ 100b3eac     sunFont.obj
 0002:0002eebc       ??_C@_0CC@IBLMDHKA@?$CIII?$CJLjava?1awt?1geom?1Point2D$Floa@ 100b3ebc     sunFont.obj
 0002:0002eee0       ??_C@_0O@NHLNHECD@getGlyphPoint@ 100b3ee0     sunFont.obj
 0002:0002eef0       ??_C@_0CB@CONGGNHA@?$CILjava?1awt?1geom?1Point2D$Float?$DL?$CJ@ 100b3ef0     sunFont.obj
 0002:0002ef14       ??_C@_0M@MJABIGBP@adjustPoint@ 100b3f14     sunFont.obj
 0002:0002ef20       ??_C@_01LELAEKIP@J@        100b3f20     sunFont.obj
 0002:0002ef24       ??_C@_0P@DPIICNJB@pScalerContext@ 100b3f24     sunFont.obj
 0002:0002ef34       ??_C@_0BD@LPHBDEDB@sun?1font?1GlyphList@ 100b3f34     sunFont.obj
 0002:0002ef48       ??_C@_03BKCJCHLK@len@      100b3f48     sunFont.obj
 0002:0002ef4c       ??_C@_02GKMBEADD@?$FLJ@    100b3f4c     sunFont.obj
 0002:0002ef50       ??_C@_06IAHKIHIK@images@   100b3f50     sunFont.obj
 0002:0002ef58       ??_C@_01POHCFINO@Z@        100b3f58     sunFont.obj
 0002:0002ef5c       ??_C@_0N@CLHDJEN@usePositions@ 100b3f5c     sunFont.obj
 0002:0002ef6c       ??_C@_09HEJILCIA@positions@ 100b3f6c     sunFont.obj
 0002:0002ef78       ??_C@_0M@IOGNPDID@lcdRGBOrder@ 100b3f78     sunFont.obj
 0002:0002ef84       ??_C@_0N@OIMCCICM@lcdSubPixPos@ 100b3f84     sunFont.obj
 0002:0002f02c       __pDefaultRawDllMain       100b402c     MSVCRT:dll_dllmain.obj
 0002:0002f02c       __pRawDllMain              100b402c     MSVCRT:dll_dllmain.obj
 0002:0002f0a0       __load_config_used         100b40a0     MSVCRT:loadcfg.obj
 0002:0002f140       __tls_used                 100b4140     MSVCRT:tlssup.obj
 0002:0002f160       ___safe_se_handler_table   100b4160     <linker-defined>
 0002:0002f44c       ___rtc_iaa                 100b444c     MSVCRT:initsect.obj
 0002:0002f450       ___rtc_izz                 100b4450     MSVCRT:initsect.obj
 0002:0002f454       ___rtc_taa                 100b4454     MSVCRT:initsect.obj
 0002:0002f458       ___rtc_tzz                 100b4458     MSVCRT:initsect.obj
 0002:0002f45c       __tls_start                100b445c     MSVCRT:tlssup.obj
 0002:0002f45d       __tls_end                  100b445d     MSVCRT:tlssup.obj
 0002:0002fdbc       __IMPORT_DESCRIPTOR_freetype 100b4dbc     freetype:freetype.dll
 0002:0002fdd0       __IMPORT_DESCRIPTOR_java   100b4dd0     java:java.dll
 0002:0002fde4       __IMPORT_DESCRIPTOR_ADVAPI32 100b4de4     advapi32:ADVAPI32.dll
 0002:0002fdf8       __IMPORT_DESCRIPTOR_USER32 100b4df8     user32:USER32.dll
 0002:0002fe0c       __IMPORT_DESCRIPTOR_GDI32  100b4e0c     gdi32:GDI32.dll
 0002:0002fe20       __IMPORT_DESCRIPTOR_awt    100b4e20     awt:awt.dll
 0002:0002fe34       __IMPORT_DESCRIPTOR_KERNEL32 100b4e34     kernel32:KERNEL32.dll
 0002:0002fe48       __IMPORT_DESCRIPTOR_VCRUNTIME140 100b4e48     vcruntime:VCRUNTIME140.dll
 0002:0002fe5c       __IMPORT_DESCRIPTOR_api-ms-win-crt-heap-l1-1-0 100b4e5c     ucrt:api-ms-win-crt-heap-l1-1-0.dll
 0002:0002fe70       __IMPORT_DESCRIPTOR_api-ms-win-crt-math-l1-1-0 100b4e70     ucrt:api-ms-win-crt-math-l1-1-0.dll
 0002:0002fe84       __IMPORT_DESCRIPTOR_api-ms-win-crt-environment-l1-1-0 100b4e84     ucrt:api-ms-win-crt-environment-l1-1-0.dll
 0002:0002fe98       __IMPORT_DESCRIPTOR_api-ms-win-crt-convert-l1-1-0 100b4e98     ucrt:api-ms-win-crt-convert-l1-1-0.dll
 0002:0002feac       __IMPORT_DESCRIPTOR_api-ms-win-crt-stdio-l1-1-0 100b4eac     ucrt:api-ms-win-crt-stdio-l1-1-0.dll
 0002:0002fec0       __IMPORT_DESCRIPTOR_api-ms-win-crt-string-l1-1-0 100b4ec0     ucrt:api-ms-win-crt-string-l1-1-0.dll
 0002:0002fed4       __IMPORT_DESCRIPTOR_api-ms-win-crt-runtime-l1-1-0 100b4ed4     ucrt:api-ms-win-crt-runtime-l1-1-0.dll
 0002:0002fee8       __NULL_IMPORT_DESCRIPTOR   100b4ee8     freetype:freetype.dll
 0003:00000000       _defaultGammaLUT           100b6000     DrawGlyphList.obj
 0003:00000100       _defaultInvGammaLUT        100b6100     DrawGlyphList.obj
 0003:00000218       ?_hb_Null_hb_buffer_t@@3Uhb_buffer_t@@B 100b6218     hb-buffer.obj
 0003:000002c4       ?endchar_str@@3PBEB        100b62c4     hb-common.obj
 0003:000002c8       ?_hb_Null_hb_draw_funcs_t@@3Uhb_draw_funcs_t@@B 100b62c8     hb-draw.obj
 0003:000002f0       ?_hb_Null_hb_face_t@@3Uhb_face_t@@B 100b62f0     hb-face.obj
 0003:000003c8       ?_hb_Null_hb_font_funcs_t@@3Uhb_font_funcs_t@@B 100b63c8     hb-font.obj
 0003:00000428       ?_hb_Null_hb_font_t@@3Uhb_font_t@@B 100b6428     hb-font.obj
 0003:00000670       ?_hb_Null_hb_paint_funcs_t@@3Uhb_paint_funcs_t@@B 100b6670     hb-paint.obj
 0003:00000788       ?_hb_Null_hb_unicode_funcs_t@@3Uhb_unicode_funcs_t@@B 100b6788     hb-unicode.obj
 0003:000007f8       _MAX_ICU_SCRIPTCODE        100b67f8     scriptMapping.obj
 0003:00000800       _ICU_to_Harfbuzz_ScriptCode 100b6800     scriptMapping.obj
 0003:000008b8       ___security_cookie_complement 100b68b8     MSVCRT:gs_cookie.obj
 0003:000008bc       ___security_cookie         100b68bc     MSVCRT:gs_cookie.obj
 0003:000008c0       __fltused                  100b68c0     MSVCRT:fltused.obj
 0003:000008d0       ___isa_enabled             100b68d0     MSVCRT:cpu_disp.obj
 0003:000008d4       ___scrt_native_dllmain_reason 100b68d4     MSVCRT:utility.obj
 0003:000008e0       ___scrt_ucrt_dll_is_in_use 100b68e0     MSVCRT:ucrt_stubs.obj
 0003:00000928       ?_OptionsStorage@?1??__local_stdio_printf_options@@9@4_KA 100b6928     hb-buffer-serialize.obj
 0003:00000930       ?_hb_CrapPool@@3PA_KA      100b6930     hb-common.obj
 0003:00000bb0       ?_hb_options@@3Uhb_atomic_int_t@@A 100b6bb0     hb-common.obj
 0003:00000bdc       ?_hb_subset_accelerator_user_data_key@@3Uhb_user_data_key_t@@A 100b6bdc     hb-subset.obj
 0003:000010f4       __tls_index                100b70f4     MSVCRT:tlssup.obj
 0003:000010fc       ___isa_available           100b70fc     MSVCRT:cpu_disp.obj
 0003:00001100       ___favor                   100b7100     MSVCRT:cpu_disp.obj
 0003:00001108       ?__type_info_root_node@@3U__type_info_node@@A 100b7108     MSVCRT:tncleanup.obj
 0003:00001110       ?_OptionsStorage@?1??__local_stdio_scanf_options@@9@4_KA 100b7110     MSVCRT:default_local_stdio_options.obj
 0003:00001118       ___scrt_current_native_startup_state 100b7118     MSVCRT:utility.obj
 0003:0000111c       ___scrt_native_startup_lock 100b711c     MSVCRT:utility.obj
 0003:0000113c       ___scrt_debugger_hook_flag 100b713c     MSVCRT:utility_desktop.obj
 0003:00001140       _sunFontIDs                100b7140     <common>
 0003:000011e0       _lcdInvGammaLUT            100b71e0     <common>
 0003:00001440       _lcdGammaLUT               100b7440     <common>
 0003:0000169c       ___dyn_tls_init_callback   100b769c     <common>

 entry point at        0001:0008321c

 Static symbols

 0000:fff42000       .debug$S                   10000000     vcruntime:VCRUNTIME140.dll
 0000:fff42000       .debug$S                   10000000     gdi32:GDI32.dll
 0000:fff42000       .debug$S                   10000000     gdi32:GDI32.dll
 0000:fff42000       .debug$S                   10000000     gdi32:GDI32.dll
 0000:fff42000       .debug$S                   10000000     gdi32:GDI32.dll
 0000:fff42000       .debug$S                   10000000     gdi32:GDI32.dll
 0000:fff42000       .debug$S                   10000000     gdi32:GDI32.dll
 0000:fff42000       .debug$S                   10000000     gdi32:GDI32.dll
 0000:fff42000       .debug$S                   10000000     gdi32:GDI32.dll
 0000:fff42000       .debug$S                   10000000     gdi32:GDI32.dll
 0000:fff42000       .debug$S                   10000000     gdi32:GDI32.dll
 0000:fff42000       .debug$S                   10000000     gdi32:GDI32.dll
 0000:fff42000       .debug$S                   10000000     gdi32:GDI32.dll
 0000:fff42000       .debug$S                   10000000     gdi32:GDI32.dll
 0000:fff42000       .debug$S                   10000000     awt:awt.dll
 0000:fff42000       .debug$S                   10000000     awt:awt.dll
 0000:fff42000       .debug$S                   10000000     awt:awt.dll
 0000:fff42000       .debug$S                   10000000     awt:awt.dll
 0000:fff42000       .debug$S                   10000000     awt:awt.dll
 0000:fff42000       .debug$S                   10000000     awt:awt.dll
 0000:fff42000       .debug$S                   10000000     awt:awt.dll
 0000:fff42000       .debug$S                   10000000     awt:awt.dll
 0000:fff42000       .debug$S                   10000000     awt:awt.dll
 0000:fff42000       .debug$S                   10000000     gdi32:GDI32.dll
 0000:fff42000       .debug$S                   10000000     gdi32:GDI32.dll
 0000:fff42000       .debug$S                   10000000     user32:USER32.dll
 0000:fff42000       .debug$S                   10000000     user32:USER32.dll
 0000:fff42000       .debug$S                   10000000     user32:USER32.dll
 0000:fff42000       .debug$S                   10000000     user32:USER32.dll
 0000:fff42000       .debug$S                   10000000     user32:USER32.dll
 0000:fff42000       .debug$S                   10000000     user32:USER32.dll
 0000:fff42000       .debug$S                   10000000     advapi32:ADVAPI32.dll
 0000:fff42000       .debug$S                   10000000     advapi32:ADVAPI32.dll
 0000:fff42000       .debug$S                   10000000     advapi32:ADVAPI32.dll
 0000:fff42000       .debug$S                   10000000     advapi32:ADVAPI32.dll
 0000:fff42000       .debug$S                   10000000     java:java.dll
 0000:fff42000       .debug$S                   10000000     java:java.dll
 0000:fff42000       .debug$S                   10000000     freetype:freetype.dll
 0000:fff42000       .debug$S                   10000000     freetype:freetype.dll
 0000:fff42000       .debug$S                   10000000     freetype:freetype.dll
 0000:fff42000       .debug$S                   10000000     freetype:freetype.dll
 0000:fff42000       .debug$S                   10000000     fontmanager.exp
 0000:fff42000       .debug$S                   10000000     freetype:freetype.dll
 0000:fff42000       .debug$S                   10000000     freetype:freetype.dll
 0000:fff42000       .debug$S                   10000000     freetype:freetype.dll
 0000:fff42000       .debug$S                   10000000     freetype:freetype.dll
 0000:fff42000       .debug$S                   10000000     freetype:freetype.dll
 0000:fff42000       .debug$S                   10000000     freetype:freetype.dll
 0000:fff42000       .debug$S                   10000000     freetype:freetype.dll
 0000:fff42000       .debug$S                   10000000     freetype:freetype.dll
 0000:fff42000       .debug$S                   10000000     ucrt:api-ms-win-crt-string-l1-1-0.dll
 0000:fff42000       .debug$S                   10000000     ucrt:api-ms-win-crt-string-l1-1-0.dll
 0000:fff42000       .debug$S                   10000000     ucrt:api-ms-win-crt-runtime-l1-1-0.dll
 0000:fff42000       .debug$S                   10000000     ucrt:api-ms-win-crt-runtime-l1-1-0.dll
 0000:fff42000       .debug$S                   10000000     ucrt:api-ms-win-crt-runtime-l1-1-0.dll
 0000:fff42000       .debug$S                   10000000     ucrt:api-ms-win-crt-runtime-l1-1-0.dll
 0000:fff42000       .debug$S                   10000000     ucrt:api-ms-win-crt-runtime-l1-1-0.dll
 0000:fff42000       .debug$S                   10000000     ucrt:api-ms-win-crt-runtime-l1-1-0.dll
 0000:fff42000       .debug$S                   10000000     ucrt:api-ms-win-crt-runtime-l1-1-0.dll
 0000:fff42000       .debug$S                   10000000     ucrt:api-ms-win-crt-runtime-l1-1-0.dll
 0000:fff42000       .debug$S                   10000000     ucrt:api-ms-win-crt-runtime-l1-1-0.dll
 0000:fff42000       .debug$S                   10000000     ucrt:api-ms-win-crt-runtime-l1-1-0.dll
 0000:fff42000       .debug$S                   10000000     ucrt:api-ms-win-crt-runtime-l1-1-0.dll
 0000:fff42000       .debug$S                   10000000     ucrt:api-ms-win-crt-runtime-l1-1-0.dll
 0000:fff42000       .debug$S                   10000000     ucrt:api-ms-win-crt-math-l1-1-0.dll
 0000:fff42000       .debug$S                   10000000     ucrt:api-ms-win-crt-math-l1-1-0.dll
 0000:fff42000       .debug$S                   10000000     ucrt:api-ms-win-crt-math-l1-1-0.dll
 0000:fff42000       .debug$S                   10000000     ucrt:api-ms-win-crt-math-l1-1-0.dll
 0000:fff42000       .debug$S                   10000000     ucrt:api-ms-win-crt-math-l1-1-0.dll
 0000:fff42000       .debug$S                   10000000     ucrt:api-ms-win-crt-math-l1-1-0.dll
 0000:fff42000       .debug$S                   10000000     ucrt:api-ms-win-crt-math-l1-1-0.dll
 0000:fff42000       .debug$S                   10000000     ucrt:api-ms-win-crt-string-l1-1-0.dll
 0000:fff42000       .debug$S                   10000000     ucrt:api-ms-win-crt-convert-l1-1-0.dll
 0000:fff42000       .debug$S                   10000000     ucrt:api-ms-win-crt-convert-l1-1-0.dll
 0000:fff42000       .debug$S                   10000000     ucrt:api-ms-win-crt-runtime-l1-1-0.dll
 0000:fff42000       .debug$S                   10000000     ucrt:api-ms-win-crt-math-l1-1-0.dll
 0000:fff42000       .debug$S                   10000000     ucrt:api-ms-win-crt-string-l1-1-0.dll
 0000:fff42000       .debug$S                   10000000     ucrt:api-ms-win-crt-stdio-l1-1-0.dll
 0000:fff42000       .debug$S                   10000000     ucrt:api-ms-win-crt-stdio-l1-1-0.dll
 0000:fff42000       .debug$S                   10000000     ucrt:api-ms-win-crt-stdio-l1-1-0.dll
 0000:fff42000       .debug$S                   10000000     ucrt:api-ms-win-crt-stdio-l1-1-0.dll
 0000:fff42000       .debug$S                   10000000     ucrt:api-ms-win-crt-stdio-l1-1-0.dll
 0000:fff42000       .debug$S                   10000000     ucrt:api-ms-win-crt-stdio-l1-1-0.dll
 0000:fff42000       .debug$S                   10000000     ucrt:api-ms-win-crt-stdio-l1-1-0.dll
 0000:fff42000       .debug$S                   10000000     ucrt:api-ms-win-crt-stdio-l1-1-0.dll
 0000:fff42000       .debug$S                   10000000     ucrt:api-ms-win-crt-convert-l1-1-0.dll
 0000:fff42000       .debug$S                   10000000     ucrt:api-ms-win-crt-math-l1-1-0.dll
 0000:fff42000       .debug$S                   10000000     ucrt:api-ms-win-crt-heap-l1-1-0.dll
 0000:fff42000       .debug$S                   10000000     ucrt:api-ms-win-crt-environment-l1-1-0.dll
 0000:fff42000       .debug$S                   10000000     ucrt:api-ms-win-crt-heap-l1-1-0.dll
 0000:fff42000       .debug$S                   10000000     ucrt:api-ms-win-crt-math-l1-1-0.dll
 0000:fff42000       .debug$S                   10000000     ucrt:api-ms-win-crt-math-l1-1-0.dll
 0000:fff42000       .debug$S                   10000000     ucrt:api-ms-win-crt-heap-l1-1-0.dll
 0000:fff42000       .debug$S                   10000000     ucrt:api-ms-win-crt-heap-l1-1-0.dll
 0000:fff42000       .debug$S                   10000000     freetype:freetype.dll
 0000:fff42000       .debug$S                   10000000     vcruntime:VCRUNTIME140.dll
 0000:fff42000       .debug$S                   10000000     vcruntime:VCRUNTIME140.dll
 0000:fff42000       .debug$S                   10000000     vcruntime:VCRUNTIME140.dll
 0000:fff42000       .debug$S                   10000000     vcruntime:VCRUNTIME140.dll
 0000:fff42000       .debug$S                   10000000     vcruntime:VCRUNTIME140.dll
 0000:fff42000       .debug$S                   10000000     gdi32:GDI32.dll
 0000:fff42000       .debug$S                   10000000     vcruntime:VCRUNTIME140.dll
 0000:fff42000       .debug$S                   10000000     vcruntime:VCRUNTIME140.dll
 0000:fff42000       .debug$S                   10000000     vcruntime:VCRUNTIME140.dll
 0000:fff42000       .debug$S                   10000000     vcruntime:VCRUNTIME140.dll
 0000:fff42000       .debug$S                   10000000     freetype:freetype.dll
 0000:fff42000       .debug$S                   10000000     kernel32:KERNEL32.dll
 0000:fff42000       .debug$S                   10000000     kernel32:KERNEL32.dll
 0000:fff42000       .debug$S                   10000000     kernel32:KERNEL32.dll
 0000:fff42000       .debug$S                   10000000     kernel32:KERNEL32.dll
 0000:fff42000       .debug$S                   10000000     kernel32:KERNEL32.dll
 0000:fff42000       .debug$S                   10000000     kernel32:KERNEL32.dll
 0000:fff42000       .debug$S                   10000000     kernel32:KERNEL32.dll
 0000:fff42000       .debug$S                   10000000     kernel32:KERNEL32.dll
 0000:fff42000       .debug$S                   10000000     kernel32:KERNEL32.dll
 0000:fff42000       .debug$S                   10000000     kernel32:KERNEL32.dll
 0000:fff42000       .debug$S                   10000000     kernel32:KERNEL32.dll
 0000:fff42000       .debug$S                   10000000     kernel32:KERNEL32.dll
 0000:fff42000       .debug$S                   10000000     kernel32:KERNEL32.dll
 0000:fff42000       .debug$S                   10000000     kernel32:KERNEL32.dll
 0000:fff42000       .debug$S                   10000000     kernel32:KERNEL32.dll
 0000:fff42000       .debug$S                   10000000     kernel32:KERNEL32.dll
 0000:fff42000       .debug$S                   10000000     kernel32:KERNEL32.dll
 0000:fff42000       .debug$S                   10000000     kernel32:KERNEL32.dll
 0000:fff42000       .debug$S                   10000000     kernel32:KERNEL32.dll
 0000:fff42000       .debug$S                   10000000     kernel32:KERNEL32.dll
 0000:fff42000       .debug$S                   10000000     kernel32:KERNEL32.dll
 0000:fff42000       .debug$S                   10000000     kernel32:KERNEL32.dll
 0000:fff42000       .debug$S                   10000000     kernel32:KERNEL32.dll
 0000:fff42000       .debug$S                   10000000     kernel32:KERNEL32.dll
 0000:fff42000       .debug$S                   10000000     kernel32:KERNEL32.dll
 0000:fff42000       .debug$S                   10000000     kernel32:KERNEL32.dll
 0000:fff42000       .debug$S                   10000000     kernel32:KERNEL32.dll
 0000:fff42000       .debug$S                   10000000     freetype:freetype.dll
 0000:fff42000       .debug$S                   10000000     freetype:freetype.dll
 0000:fff42000       .debug$S                   10000000     freetype:freetype.dll
 0000:fff42000       .debug$S                   10000000     freetype:freetype.dll
 0000:fff42000       .debug$S                   10000000     freetype:freetype.dll
 0000:fff42000       .debug$S                   10000000     freetype:freetype.dll
 0001:00000240       _drawGlyphList             10001240 f   DrawGlyphList.obj
 0001:000003b0       _drawGlyphListLCD          100013b0 f   DrawGlyphList.obj
 0001:000013f0       _euclidianDistance         100023f0 f   HBShaper.obj
 0001:000019d0       _CheckFontFamilyProcW@16   100029d0 f   fontpath.obj
 0001:00001a20       _EnumFamilyNamesW@16       10002a20 f   fontpath.obj
 0001:00001d00       _EnumFontFacesInFamilyProcW@16 10002d00 f   fontpath.obj
 0001:00002540       _registerFontW             10003540 f   fontpath.obj
 0001:00002780       _moveTo                    10003780 f   freetypeScaler.obj
 0001:000027f0       _lineTo                    100037f0 f   freetypeScaler.obj
 0001:00002850       _conicTo                   10003850 f   freetypeScaler.obj
 0001:000028f0       _cubicTo                   100038f0 f   freetypeScaler.obj
 0001:000039a0       _ReadTTFontFileFunc        100049a0 f   freetypeScaler.obj
 0001:00003b00       _addToGP                   10004b00 f   freetypeScaler.obj
 0001:00003b40       _allocateSpaceForGP        10004b40 f   freetypeScaler.obj
 0001:00003c20       _freeNativeResources       10004c20 f   freetypeScaler.obj
 0001:00003c80       _getFTOutline              10004c80 f   freetypeScaler.obj
 0001:00003d40       _getGlyphImageNativeInternal 10004d40 f   freetypeScaler.obj
 0001:00004450       _setupFTContext            10005450 f   freetypeScaler.obj
 0001:00004770       ??$_hb_cmp_method@IU?$LookupSegmentSingle@U?$IntType@I$03@OT@@@AAT@@$$V@@YAHPBX0@Z 10005770 f   hb-aat-layout.obj
 0001:00004770       ??$_hb_cmp_method@IU?$LookupSegmentArray@U?$OffsetTo@U?$ArrayOf@UAnchor@AAT@@U?$IntType@I$03@OT@@@OT@@U?$IntType@G$01@2@$0A@@OT@@@AAT@@$$V@@YAHPBX0@Z 10005770 f   hb-aat-layout.obj
 0001:00004770       ??$_hb_cmp_method@IU?$LookupSegmentSingle@U?$OffsetTo@U?$ArrayOf@UAnchor@AAT@@U?$IntType@I$03@OT@@@OT@@U?$IntType@G$01@2@$0A@@OT@@@AAT@@$$V@@YAHPBX0@Z 10005770 f   hb-aat-layout.obj
 0001:00004770       ??$_hb_cmp_method@IU?$LookupSegmentArray@U?$IntType@G$01@OT@@@AAT@@$$V@@YAHPBX0@Z 10005770 f   hb-aat-layout.obj
 0001:00004770       ??$_hb_cmp_method@IU?$LookupSegmentArray@UHBGlyphID16@OT@@@AAT@@$$V@@YAHPBX0@Z 10005770 f   hb-aat-layout.obj
 0001:00004770       ??$_hb_cmp_method@IU?$LookupSegmentSingle@UHBGlyphID16@OT@@@AAT@@$$V@@YAHPBX0@Z 10005770 f   hb-aat-layout.obj
 0001:00004770       ??$_hb_cmp_method@IU?$LookupSegmentSingle@U?$IntType@G$01@OT@@@AAT@@$$V@@YAHPBX0@Z 10005770 f   hb-aat-layout.obj
 0001:00004770       ??$_hb_cmp_method@IU?$LookupSegmentArray@U?$IntType@I$03@OT@@@AAT@@$$V@@YAHPBX0@Z 10005770 f   hb-aat-layout.obj
 0001:000047b0       ??$_hb_cmp_method@IU?$LookupSingle@U?$IntType@G$01@OT@@@AAT@@$$V@@YAHPBX0@Z 100057b0 f   hb-aat-layout.obj
 0001:000047b0       ??$_hb_cmp_method@IU?$LookupSingle@U?$OffsetTo@U?$ArrayOf@UAnchor@AAT@@U?$IntType@I$03@OT@@@OT@@U?$IntType@G$01@2@$0A@@OT@@@AAT@@$$V@@YAHPBX0@Z 100057b0 f   hb-aat-layout.obj
 0001:000047b0       ??$_hb_cmp_method@IU?$LookupSingle@UHBGlyphID16@OT@@@AAT@@$$V@@YAHPBX0@Z 100057b0 f   hb-aat-layout.obj
 0001:000047b0       ??$_hb_cmp_method@IU?$LookupSingle@U?$IntType@I$03@OT@@@AAT@@$$V@@YAHPBX0@Z 100057b0 f   hb-aat-layout.obj
 0001:000047e0       ??$_hb_debug_msg@$0A@@@YAXPBDPBX0_NIH0ZZ 100057e0 f   hb-common.obj
 0001:000047e0       ?hb_paint_push_group_nil@@YAXPAUhb_paint_funcs_t@@PAX1@Z 100057e0 f   hb-paint.obj
 0001:000047e0       ?hb_paint_sweep_gradient_nil@@YAXPAUhb_paint_funcs_t@@PAXPAUhb_color_line_t@@MMMM1@Z 100057e0 f   hb-paint.obj
 0001:000047e0       ?hb_paint_radial_gradient_nil@@YAXPAUhb_paint_funcs_t@@PAXPAUhb_color_line_t@@MMMMMM1@Z 100057e0 f   hb-paint.obj
 0001:000047e0       ?hb_paint_linear_gradient_nil@@YAXPAUhb_paint_funcs_t@@PAXPAUhb_color_line_t@@MMMMMM1@Z 100057e0 f   hb-paint.obj
 0001:000047e0       ?_do_nothing@@YAXXZ        100057e0 f   hb-jdk-font.obj
 0001:000047e0       ?hb_paint_color_nil@@YAXPAUhb_paint_funcs_t@@PAXHI1@Z 100057e0 f   hb-paint.obj
 0001:000047e0       ??$_hb_debug_msg@$0A@@@YAXPBDPBX0_NIH0ZZ 100057e0 f   hb-ot-shaper-arabic.obj
 0001:000047e0       ?hb_paint_pop_group_nil@@YAXPAUhb_paint_funcs_t@@PAXW4hb_paint_composite_mode_t@@1@Z 100057e0 f   hb-paint.obj
 0001:000047e0       ?hb_paint_pop_clip_nil@@YAXPAUhb_paint_funcs_t@@PAX1@Z 100057e0 f   hb-paint.obj
 0001:000047e0       ??$_hb_debug_msg@$0A@@@YAXPBDPBX0_NIH0ZZ 100057e0 f   hb-shape-plan.obj
 0001:000047e0       ??$_hb_debug_msg@$0A@@@YAXPBDPBX0_NIH0ZZ 100057e0 f   hb-ot-font.obj
 0001:000047e0       ??$_hb_debug_msg@$0A@@@YAXPBDPBX0_NIH0ZZ 100057e0 f   hb-ot-face.obj
 0001:000047e0       ??$_hb_debug_msg@$0A@@@YAXPBDPBX0_NIH0ZZ 100057e0 f   hb-aat-layout.obj
 0001:000047e0       ??$_hb_debug_msg@$0A@@@YAXPBDPBX0_NIH0ZZ 100057e0 f   hb-face.obj
 0001:000047e0       ?hb_paint_push_clip_rectangle_nil@@YAXPAUhb_paint_funcs_t@@PAXMMMM1@Z 100057e0 f   hb-paint.obj
 0001:000047e0       ??$_hb_debug_msg@$0A@@@YAXPBDPBX0_NIH0ZZ 100057e0 f   hb-face-builder.obj
 0001:000047e0       ?hb_paint_push_clip_glyph_nil@@YAXPAUhb_paint_funcs_t@@PAXIPAUhb_font_t@@1@Z 100057e0 f   hb-paint.obj
 0001:000047e0       ?hb_paint_pop_transform_nil@@YAXPAUhb_paint_funcs_t@@PAX1@Z 100057e0 f   hb-paint.obj
 0001:000047e0       ??$_hb_debug_msg@$0A@@@YAXPBDPBX0_NIH0ZZ 100057e0 f   hb-ot-color.obj
 0001:000047e0       ?hb_draw_close_path_nil@@YAXPAUhb_draw_funcs_t@@PAXPAUhb_draw_state_t@@1@Z 100057e0 f   hb-draw.obj
 0001:000047e0       ?hb_draw_cubic_to_nil@@YAXPAUhb_draw_funcs_t@@PAXPAUhb_draw_state_t@@MMMMMM1@Z 100057e0 f   hb-draw.obj
 0001:000047e0       ?hb_font_paint_glyph_nil@@YAXPAUhb_font_t@@PAXIPAUhb_paint_funcs_t@@1II1@Z 100057e0 f   hb-font.obj
 0001:000047e0       ?hb_draw_line_to_nil@@YAXPAUhb_draw_funcs_t@@PAXPAUhb_draw_state_t@@MM1@Z 100057e0 f   hb-draw.obj
 0001:000047e0       ?hb_draw_move_to_nil@@YAXPAUhb_draw_funcs_t@@PAXPAUhb_draw_state_t@@MM1@Z 100057e0 f   hb-draw.obj
 0001:000047e0       ?hb_font_draw_glyph_nil@@YAXPAUhb_font_t@@PAXIPAUhb_draw_funcs_t@@11@Z 100057e0 f   hb-font.obj
 0001:000047e0       ?hb_paint_push_transform_nil@@YAXPAUhb_paint_funcs_t@@PAXMMMMMM1@Z 100057e0 f   hb-paint.obj
 0001:000047e0       ??$_hb_debug_msg@$0A@@@YAXPBDPBX0_NIH0ZZ 100057e0 f   hb-ot-layout.obj
 0001:000047e0       ??$_hb_debug_msg@$0A@@@YAXPBDPBX0_NIH0ZZ 100057e0 f   hb-ot-metrics.obj
 0001:000047e0       ??$_hb_debug_msg@$0A@@@YAXPBDPBX0_NIH0ZZ 100057e0 f   hb-font.obj
 0001:000047e0       ??$_hb_debug_msg@$0A@@@YAXPBDPBX0_NIH0ZZ 100057e0 f   hb-ot-shape-fallback.obj
 0001:000047e0       ??$_hb_debug_msg@$0A@@@YAXPBDPBX0_NIH0ZZ 100057e0 f   hb-blob.obj
 0001:00005970       $LN291                     10006970     hb-aat-layout.obj
 0001:00005c24       $LN291                     10006c24     hb-aat-layout.obj
 0001:00005ee4       $LN222                     10006ee4     hb-aat-layout.obj
 0001:000061ac       $LN274                     100071ac     hb-aat-layout.obj
 0001:00006394       $LN268                     10007394     hb-aat-layout.obj
 0001:000064dc       $LN160                     100074dc     hb-aat-layout.obj
 0001:00008800       ??$hb_bsearch_impl@$$CBXI$$V@@YA_NPAIABIPBXIIP6AH22@Z@Z 10009800 f   hb-aat-layout.obj
 0001:0000a8c4       $LN39                      1000b8c4     hb-aat-layout.obj
 0001:0000a8e0       ?_hb_grapheme_group_func@@YA_NABUhb_glyph_info_t@@0@Z 1000b8e0 f   hb-aat-layout.obj
 0001:0000a8e0       ?_hb_grapheme_group_func@@YA_NABUhb_glyph_info_t@@0@Z 1000b8e0 f   hb-ot-shape.obj
 0001:0000dee0       $LN130                     1000eee0     hb-aat-layout.obj
 0001:0000dee0       $LN130                     1000eee0     hb-aat-layout.obj
 0001:0000dee0       $LN130                     1000eee0     hb-aat-layout.obj
 0001:0000e104       $LN130                     1000f104     hb-aat-layout.obj
 0001:0000ee60       ?is_deleted_glyph@@YA_NPBUhb_glyph_info_t@@@Z 1000fe60 f   hb-aat-layout.obj
 0001:0000fd40       ?kerxTupleKern@AAT@@YAHHIPBXPAUhb_aat_apply_context_t@1@@Z 10010d40 f   hb-aat-layout.obj
 0001:000111d8       $LN411                     100121d8     hb-aat-layout.obj
 0001:00011428       $LN395                     10012428     hb-aat-layout.obj
 0001:000115fc       $LN330                     100125fc     hb-aat-layout.obj
 0001:00011844       $LN407                     10012844     hb-aat-layout.obj
 0001:000164f0       ??$sort_r_simple@$$V@@YAXPAXIIP6AHPBX1@Z@Z 100174f0 f   hb-aat-map.obj
 0001:000164f0       ??$sort_r_simple@$$V@@YAXPAXIIP6AHPBX1@Z@Z 100174f0 f   hb-ot-shaper-arabic.obj
 0001:000164f0       ??$sort_r_simple@$$V@@YAXPAXIIP6AHPBX1@Z@Z 100174f0 f   hb-ot-map.obj
 0001:000164f0       ??$sort_r_simple@$$V@@YAXPAXIIP6AHPBX1@Z@Z 100174f0 f   hb-ot-font.obj
 0001:000173f0       ?sort_r_swap@@YAXPIAD0I@Z  100183f0 f   hb-ot-font.obj
 0001:000173f0       ?sort_r_swap@@YAXPIAD0I@Z  100183f0 f   hb-ot-shaper-arabic.obj
 0001:000173f0       ?sort_r_swap@@YAXPIAD0I@Z  100183f0 f   hb-ot-map.obj
 0001:000173f0       ?sort_r_swap@@YAXPIAD0I@Z  100183f0 f   hb-aat-map.obj
 0001:000175a0       ?_hb_blob_destroy@@YAXPAX@Z 100185a0 f   hb-blob.obj
 0001:00017c70       ?buffer_verify_error@@YAXPAUhb_buffer_t@@PAUhb_font_t@@PBDZZ 10018c70 f   hb-buffer-verify.obj
 0001:00017cf0       ?buffer_verify_unsafe_to_break@@YA_NPAUhb_buffer_t@@0PAUhb_font_t@@PBUhb_feature_t@@IPBQBD@Z 10018cf0 f   hb-buffer-verify.obj
 0001:00017f80       ?buffer_verify_unsafe_to_concat@@YA_NPAUhb_buffer_t@@0PAUhb_font_t@@PBUhb_feature_t@@IPBQBD@Z 10018f80 f   hb-buffer-verify.obj
 0001:000184a0       ??$hb_buffer_add_utf@U?$hb_utf16_xe_t@G@@@@YAXPAUhb_buffer_t@@PBGHIH@Z 100194a0 f   hb-buffer.obj
 0001:0001fdd0       ?lang_find_or_insert@@YAPAUhb_language_item_t@@PBD@Z 10020dd0 f   hb-common.obj
 0001:0001ff90       ?parse_feature_value_postfix@@YA_NPAPBDPBDPAUhb_feature_t@@@Z 10020f90 f   hb-common.obj
 0001:000200f0       ?parse_one_feature@@YA_NPAPBDPBDPAUhb_feature_t@@@Z 100210f0 f   hb-common.obj
 0001:00020250       ?parse_space@@YA_NPAPBDPBD@Z 10021250 f   hb-common.obj
 0001:00020290       ?parse_tag@@YA_NPAPBDPBDPAI@Z 10021290 f   hb-common.obj
 0001:000217a0       ?_hb_draw_funcs_set_middle@@YA_NPAUhb_draw_funcs_t@@PAXP6AX1@Z@Z 100227a0 f   hb-draw.obj
 0001:00021800       ?hb_draw_quadratic_to_nil@@YAXPAUhb_draw_funcs_t@@PAXPAUhb_draw_state_t@@MMMM1@Z 10022800 f   hb-draw.obj
 0001:000225e0       ?fasthash64@@YA_KPBXI_K@Z  100235e0 f   hb-ot-shaper-arabic.obj
 0001:000225e0       ?fasthash64@@YA_KPBXI_K@Z  100235e0 f   hb-face-builder.obj
 0001:00022848       $LN54                      10023848     hb-ot-shaper-arabic.obj
 0001:00022848       $LN54                      10023848     hb-face-builder.obj
 0001:00022bc0       ?hb_memcmp@@YAHPBX0I@Z     10023bc0 f   hb-ot-font.obj
 0001:00022bc0       ?hb_memcmp@@YAHPBX0I@Z     10023bc0 f   hb-face-builder.obj
 0001:000232c0       ??$get_glyph_from_symbol@UCmapSubtable@OT@@$1?_hb_arabic_pua_simp_map@@YAII@Z@accelerator_t@cmap@OT@@KA_NPBXIPAI@Z 100242c0 f   hb-face.obj
 0001:00023300       ??$get_glyph_from_symbol@UCmapSubtable@OT@@$1?_hb_arabic_pua_trad_map@@YAII@Z@accelerator_t@cmap@OT@@KA_NPBXIPAI@Z 10024300 f   hb-face.obj
 0001:00023340       ??$get_glyph_from_symbol@UCmapSubtable@OT@@$1?_hb_symbol_pua_map@2@YAII@Z@accelerator_t@cmap@OT@@KA_NPBXIPAI@Z 10024340 f   hb-face.obj
 0001:00023390       ??$hb_object_create@Uhb_face_t@@$$V@@YAPAUhb_face_t@@XZ 10024390 f   hb-face.obj
 0001:00023540       ??$hb_object_set_user_data@Uhb_face_t@@@@YA_NPAUhb_face_t@@PAUhb_user_data_key_t@@PAXP6AX2@ZH@Z 10024540 f   hb-face.obj
 0001:00024110       ?_hb_arabic_pua_simp_map@@YAII@Z 10025110 f   hb-face.obj
 0001:00024190       ?_hb_arabic_pua_trad_map@@YAII@Z 10025190 f   hb-face.obj
 0001:000245bc       $LN110                     100255bc     hb-face.obj
 0001:000245d8       $LN105                     100255d8     hb-face.obj
 0001:00024aec       $LN380                     10025aec     hb-face.obj
 0001:00024b08       $LN374                     10025b08     hb-face.obj
 0001:00025b0c       $LN134                     10026b0c     hb-fallback-shape.obj
 0001:00025b20       $LN127                     10026b20     hb-fallback-shape.obj
 0001:00025b40       ?hb_unicode_eastasian_width_nil@@YAIPAUhb_unicode_funcs_t@@IPAX@Z 10026b40 f   hb-unicode.obj
 0001:00025b40       ?hb_jdk_get_glyph_h_origin@@YAHPAUhb_font_t@@PAXIPAH21@Z 10026b40 f   hb-jdk-font.obj
 0001:00025f80       ?_hb_font_create@@YAPAUhb_font_t@@PAUhb_face_t@@@Z 10026f80 f   hb-font.obj
 0001:00026080       ?_hb_font_funcs_set_middle@@YA_NPAUhb_font_funcs_t@@PAXP6AX1@Z@Z 10027080 f   hb-font.obj
 0001:00026360       ?hb_draw_close_path_default@@YAXPAUhb_draw_funcs_t@@PAXPAUhb_draw_state_t@@1@Z 10027360 f   hb-font.obj
 0001:00026390       ?hb_draw_cubic_to_default@@YAXPAUhb_draw_funcs_t@@PAXPAUhb_draw_state_t@@MMMMMM1@Z 10027390 f   hb-font.obj
 0001:00026470       ?hb_draw_line_to_default@@YAXPAUhb_draw_funcs_t@@PAXPAUhb_draw_state_t@@MM1@Z 10027470 f   hb-font.obj
 0001:000264f0       ?hb_draw_move_to_default@@YAXPAUhb_draw_funcs_t@@PAXPAUhb_draw_state_t@@MM1@Z 100274f0 f   hb-font.obj
 0001:00026550       ?hb_draw_quadratic_to_default@@YAXPAUhb_draw_funcs_t@@PAXPAUhb_draw_state_t@@MMMM1@Z 10027550 f   hb-font.obj
 0001:00026600       ?hb_font_draw_glyph_default@@YAXPAUhb_font_t@@PAXIPAUhb_draw_funcs_t@@11@Z 10027600 f   hb-font.obj
 0001:000266d0       ?hb_font_get_font_h_extents_default@@YAHPAUhb_font_t@@PAXPAUhb_font_extents_t@@1@Z 100276d0 f   hb-font.obj
 0001:000267b0       ?hb_font_get_font_h_extents_nil@@YAHPAUhb_font_t@@PAXPAUhb_font_extents_t@@1@Z 100277b0 f   hb-font.obj
 0001:000267b0       ?hb_font_get_font_v_extents_nil@@YAHPAUhb_font_t@@PAXPAUhb_font_extents_t@@1@Z 100277b0 f   hb-font.obj
 0001:000267d0       ?hb_font_get_font_v_extents_default@@YAHPAUhb_font_t@@PAXPAUhb_font_extents_t@@1@Z 100277d0 f   hb-font.obj
 0001:000268b0       ?hb_font_get_glyph_contour_point_default@@YAHPAUhb_font_t@@PAXIIPAH21@Z 100278b0 f   hb-font.obj
 0001:00026910       ?hb_font_get_glyph_contour_point_nil@@YAHPAUhb_font_t@@PAXIIPAH21@Z 10027910 f   hb-font.obj
 0001:00026930       ?hb_font_get_glyph_extents_default@@YAHPAUhb_font_t@@PAXIPAUhb_glyph_extents_t@@1@Z 10027930 f   hb-font.obj
 0001:000269f0       ?hb_font_get_glyph_extents_nil@@YAHPAUhb_font_t@@PAXIPAUhb_glyph_extents_t@@1@Z 100279f0 f   hb-font.obj
 0001:00026a00       ?hb_font_get_glyph_from_name_default@@YAHPAUhb_font_t@@PAXPBDHPAI1@Z 10027a00 f   hb-font.obj
 0001:00026a50       ?hb_font_get_variation_glyph_nil@@YAHPAUhb_font_t@@PAXIIPAI1@Z 10027a50 f   hb-font.obj
 0001:00026a50       ?hb_font_get_glyph_from_name_nil@@YAHPAUhb_font_t@@PAXPBDHPAI1@Z 10027a50 f   hb-font.obj
 0001:00026a60       ?hb_font_get_glyph_h_advance_default@@YAHPAUhb_font_t@@PAXI1@Z 10027a60 f   hb-font.obj
 0001:00026af0       ?hb_font_get_glyph_h_advance_nil@@YAHPAUhb_font_t@@PAXI1@Z 10027af0 f   hb-font.obj
 0001:00026b00       ?hb_font_get_glyph_h_advances_default@@YAXPAUhb_font_t@@PAXIPBIIPAHI1@Z 10027b00 f   hb-font.obj
 0001:00026be0       ?hb_font_get_glyph_h_kerning_default@@YAHPAUhb_font_t@@PAXII1@Z 10027be0 f   hb-font.obj
 0001:00026c40       ?hb_jdk_get_glyph_name@@YAHPAUhb_font_t@@PAXIPADI1@Z 10027c40 f   hb-jdk-font.obj
 0001:00026c40       ?hb_jdk_get_glyph_from_name@@YAHPAUhb_font_t@@PAXPBDHPAI1@Z 10027c40 f   hb-jdk-font.obj
 0001:00026c40       ?hb_paint_color_glyph_nil@@YAHPAUhb_paint_funcs_t@@PAXIPAUhb_font_t@@1@Z 10027c40 f   hb-paint.obj
 0001:00026c40       ?hb_paint_image_nil@@YAHPAUhb_paint_funcs_t@@PAXPAUhb_blob_t@@IIIMPAUhb_glyph_extents_t@@1@Z 10027c40 f   hb-paint.obj
 0001:00026c40       ?hb_font_get_glyph_v_kerning_nil@@YAHPAUhb_font_t@@PAXII1@Z 10027c40 f   hb-font.obj
 0001:00026c40       ?hb_jdk_get_glyph_v_origin@@YAHPAUhb_font_t@@PAXIPAH21@Z 10027c40 f   hb-jdk-font.obj
 0001:00026c40       ?hb_font_get_glyph_h_kerning_nil@@YAHPAUhb_font_t@@PAXII1@Z 10027c40 f   hb-font.obj
 0001:00026c40       ?hb_jdk_get_glyph_extents@@YAHPAUhb_font_t@@PAXIPAUhb_glyph_extents_t@@1@Z 10027c40 f   hb-jdk-font.obj
 0001:00026c40       ?hb_unicode_compose_nil@@YAHPAUhb_unicode_funcs_t@@IIPAIPAX@Z 10027c40 f   hb-unicode.obj
 0001:00026c40       ?hb_paint_custom_palette_color_nil@@YAHPAUhb_paint_funcs_t@@PAXIPAI1@Z 10027c40 f   hb-paint.obj
 0001:00026c40       ?hb_unicode_decompose_nil@@YAHPAUhb_unicode_funcs_t@@IPAI1PAX@Z 10027c40 f   hb-unicode.obj
 0001:00026c40       ?hb_unicode_decompose_compatibility_nil@@YAIPAUhb_unicode_funcs_t@@IPAIPAX@Z 10027c40 f   hb-unicode.obj
 0001:00026c40       ?hb_jdk_get_glyph_v_kerning@@YAHPAUhb_font_t@@PAXII1@Z 10027c40 f   hb-jdk-font.obj
 0001:00026c40       ?hb_jdk_get_glyph_h_kerning@@YAHPAUhb_font_t@@PAXII1@Z 10027c40 f   hb-jdk-font.obj
 0001:00026c40       ?hb_unicode_combining_class_nil@@YA?AW4hb_unicode_combining_class_t@@PAUhb_unicode_funcs_t@@IPAX@Z 10027c40 f   hb-unicode.obj
 0001:00026c50       ?hb_font_get_glyph_h_origin_default@@YAHPAUhb_font_t@@PAXIPAH21@Z 10027c50 f   hb-font.obj
 0001:00026cb0       ?hb_font_get_glyph_h_origin_nil@@YAHPAUhb_font_t@@PAXIPAH21@Z 10027cb0 f   hb-font.obj
 0001:00026cd0       ?hb_font_get_glyph_name_default@@YAHPAUhb_font_t@@PAXIPADI1@Z 10027cd0 f   hb-font.obj
 0001:00026d10       ?hb_font_get_glyph_name_nil@@YAHPAUhb_font_t@@PAXIPADI1@Z 10027d10 f   hb-font.obj
 0001:00026d30       ?hb_font_get_glyph_v_advance_default@@YAHPAUhb_font_t@@PAXI1@Z 10027d30 f   hb-font.obj
 0001:00026dc0       ?hb_font_get_glyph_v_advance_nil@@YAHPAUhb_font_t@@PAXI1@Z 10027dc0 f   hb-font.obj
 0001:00026dd0       ?hb_font_get_glyph_v_advances_default@@YAXPAUhb_font_t@@PAXIPBIIPAHI1@Z 10027dd0 f   hb-font.obj
 0001:00026eb0       ?hb_font_get_glyph_v_kerning_default@@YAHPAUhb_font_t@@PAXII1@Z 10027eb0 f   hb-font.obj
 0001:00026f10       ?hb_font_get_glyph_v_origin_default@@YAHPAUhb_font_t@@PAXIPAH21@Z 10027f10 f   hb-font.obj
 0001:00026f70       ?hb_font_get_glyph_v_origin_nil@@YAHPAUhb_font_t@@PAXIPAH21@Z 10027f70 f   hb-font.obj
 0001:00026f90       ?hb_font_get_nominal_glyph_default@@YAHPAUhb_font_t@@PAXIPAI1@Z 10027f90 f   hb-font.obj
 0001:00027010       ?hb_font_get_nominal_glyph_nil@@YAHPAUhb_font_t@@PAXIPAI1@Z 10028010 f   hb-font.obj
 0001:00027020       ?hb_font_get_nominal_glyphs_default@@YAIPAUhb_font_t@@PAXIPBIIPAII1@Z 10028020 f   hb-font.obj
 0001:000270d0       ?hb_font_get_variation_glyph_default@@YAHPAUhb_font_t@@PAXIIPAI1@Z 100280d0 f   hb-font.obj
 0001:00027110       ?hb_font_paint_glyph_default@@YAXPAUhb_font_t@@PAXIPAUhb_paint_funcs_t@@1II1@Z 10028110 f   hb-font.obj
 0001:000293d0       ?cleanupFontInfo@@YAXPAX@Z 1002a3d0 f   hb-jdk-font.obj
 0001:00029410       ?hb_jdk_get_glyph_contour_point@@YAHPAUhb_font_t@@PAXIIPAH21@Z 1002a410 f   hb-jdk-font.obj
 0001:000294e0       ?hb_jdk_get_glyph_h_advance@@YAHPAUhb_font_t@@PAXI1@Z 1002a4e0 f   hb-jdk-font.obj
 0001:00029560       ?hb_jdk_get_glyph_v_advance@@YAHPAUhb_font_t@@PAXI1@Z 1002a560 f   hb-jdk-font.obj
 0001:000295d0       ?hb_jdk_get_nominal_glyph@@YAHPAUhb_font_t@@PAXIPAI1@Z 1002a5d0 f   hb-jdk-font.obj
 0001:00029620       ?hb_jdk_get_variation_glyph@@YAHPAUhb_font_t@@PAXIIPAI1@Z 1002a620 f   hb-jdk-font.obj
 0001:00029680       ?reference_table@@YAPAUhb_blob_t@@PAUhb_face_t@@IPAX@Z 1002a680 f   hb-jdk-font.obj
 0001:000298e0       ?_pow10@@YANI@Z            1002a8e0 f   hb-number.obj
 0001:00029a60       ?strtod_rl@@YANPBDPAPBD@Z  1002aa60 f   hb-number.obj
 0001:00029d64       $LN77                      1002ad64     hb-number.obj
 0001:0002a0f0       ?_get_bounds@@YA_NPBUaccelerator_t@cff1@OT@@IAAUbounds_t@@_N@Z 1002b0f0 f   hb-ot-cff1-table.obj
 0001:0002a210       ?_get_path@@YA_NPBUaccelerator_t@cff1@OT@@PAUhb_font_t@@IAAUhb_draw_session_t@@_NPAUpoint_t@CFF@@@Z 1002b210 f   hb-ot-cff1-table.obj
 0001:0002a4c0       $LN19                      1002b4c0     hb-ot-cff1-table.obj
 0001:0002a4c0       $LN19                      1002b4c0     hb-ot-cff1-table.obj
 0001:0002a4d0       $LN16                      1002b4d0     hb-ot-cff1-table.obj
 0001:0002a4d0       $LN16                      1002b4d0     hb-ot-cff1-table.obj
 0001:0002ee3c       $LN31                      1002fe3c     hb-ot-cff1-table.obj
 0001:0002f324       $LN344                     10030324     hb-ot-cff1-table.obj
 0001:0002f37c       $LN337                     1003037c     hb-ot-cff1-table.obj
 0001:0002fd08       $LN648                     10030d08     hb-ot-cff1-table.obj
 0001:0002fd60       $LN638                     10030d60     hb-ot-cff1-table.obj
 0001:00030058       $LN179                     10031058     hb-ot-cff1-table.obj
 0001:00030068       $LN177                     10031068     hb-ot-cff1-table.obj
 0001:00038eac       $LN31                      10039eac     hb-ot-cff2-table.obj
 0001:00039358       $LN115                     1003a358     hb-ot-cff2-table.obj
 0001:00039368       $LN113                     1003a368     hb-ot-cff2-table.obj
 0001:00039548       $LN115                     1003a548     hb-ot-cff2-table.obj
 0001:00039558       $LN113                     1003a558     hb-ot-cff2-table.obj
 0001:00039970       $LN350                     1003a970     hb-ot-cff2-table.obj
 0001:000399c8       $LN341                     1003a9c8     hb-ot-cff2-table.obj
 0001:00039f44       $LN344                     1003af44     hb-ot-cff2-table.obj
 0001:00039f9c       $LN335                     1003af9c     hb-ot-cff2-table.obj
 0001:0003ebcc       $LN927                     1003fbcc     hb-ot-color.obj
 0001:00043590       ??$StructAtOffsetOrNull@U?$Subrs@U?$IntType@G$01@OT@@@CFF@@@CFF@@YAABU?$Subrs@U?$IntType@G$01@OT@@@0@PBXI@Z 10044590 f   hb-ot-font.obj
 0001:00043cb0       $LN589                     10044cb0     hb-ot-font.obj
 0001:000460f0       ??$sort_r_simple@PAX@@YAXPAXIIP6AHPBX10@Z0@Z 100470f0 f   hb-ot-font.obj
 0001:00047990       ?_hb_ot_font_destroy@@YAXPAX@Z 10048990 f   hb-ot-font.obj
 0001:000479b0       ?_hb_roundf@@YAMM@Z        100489b0 f   hb-ot-layout.obj
 0001:000479b0       ?_hb_roundf@@YAMM@Z        100489b0 f   hb-ot-font.obj
 0001:00048340       ?cff1_std_strings@@YA?AU?$hb_array_t@$$CBD@@I@Z 10049340 f   hb-ot-font.obj
 0001:00048500       ?format1_names@@YA?AU?$hb_array_t@$$CBD@@I@Z 10049500 f   hb-ot-font.obj
 0001:00049ed0       ?hb_ot_draw_glyph@@YAXPAUhb_font_t@@PAXIPAUhb_draw_funcs_t@@11@Z 1004aed0 f   hb-ot-font.obj
 0001:0004a200       ?hb_ot_get_font_h_extents@@YAHPAUhb_font_t@@PAXPAUhb_font_extents_t@@1@Z 1004b200 f   hb-ot-font.obj
 0001:0004a280       ?hb_ot_get_font_v_extents@@YAHPAUhb_font_t@@PAXPAUhb_font_extents_t@@1@Z 1004b280 f   hb-ot-font.obj
 0001:0004a2e0       ?hb_ot_get_glyph_extents@@YAHPAUhb_font_t@@PAXIPAUhb_glyph_extents_t@@1@Z 1004b2e0 f   hb-ot-font.obj
 0001:0004a3a0       ?hb_ot_get_glyph_from_name@@YAHPAUhb_font_t@@PAXPBDHPAI1@Z 1004b3a0 f   hb-ot-font.obj
 0001:0004a3f0       ?hb_ot_get_glyph_h_advances@@YAXPAUhb_font_t@@PAXIPBIIPAHI1@Z 1004b3f0 f   hb-ot-font.obj
 0001:0004a810       ?hb_ot_get_glyph_name@@YAHPAUhb_font_t@@PAXIPADI1@Z 1004b810 f   hb-ot-font.obj
 0001:0004a900       ?hb_ot_get_glyph_v_advances@@YAXPAUhb_font_t@@PAXIPBIIPAHI1@Z 1004b900 f   hb-ot-font.obj
 0001:0004ab80       ?hb_ot_get_glyph_v_origin@@YAHPAUhb_font_t@@PAXIPAH21@Z 1004bb80 f   hb-ot-font.obj
 0001:0004b060       ?hb_ot_get_nominal_glyph@@YAHPAUhb_font_t@@PAXIPAI1@Z 1004c060 f   hb-ot-font.obj
 0001:0004b0a0       ?hb_ot_get_nominal_glyphs@@YAIPAUhb_font_t@@PAXIPBIIPAII1@Z 1004c0a0 f   hb-ot-font.obj
 0001:0004b170       ?hb_ot_get_variation_glyph@@YAHPAUhb_font_t@@PAXIIPAI1@Z 1004c170 f   hb-ot-font.obj
 0001:0004b200       ?hb_ot_paint_glyph@@YAXPAUhb_font_t@@PAXIPAUhb_paint_funcs_t@@1II1@Z 1004c200 f   hb-ot-font.obj
 0001:0004bbf4       $LN147                     1004cbf4     hb-ot-font.obj
 0001:0004bbfc       $LN145                     1004cbfc     hb-ot-font.obj
 0001:0004c08c       $LN196                     1004d08c     hb-ot-font.obj
 0001:0004c09c       $LN192                     1004d09c     hb-ot-font.obj
 0001:0004c0b0       $LN197                     1004d0b0     hb-ot-font.obj
 0001:0004c0b8       $LN193                     1004d0b8     hb-ot-font.obj
 0001:0004f628       $LN240                     10050628     hb-ot-font.obj
 0001:0004f640       $LN233                     10050640     hb-ot-font.obj
 0001:0004f654       $LN241                     10050654     hb-ot-font.obj
 0001:0004f66c       $LN234                     1005066c     hb-ot-font.obj
 0001:0004f694       $LN242                     10050694     hb-ot-font.obj
 0001:00051500       ??$?UU?$hb_map_iter_t@U?$hb_array_t@$$CBUhb_applicable_t@hb_accelerate_subtables_context_t@OT@@@@V<lambda_77b345933307e1fb3f76492be2367557>@@$0A@$0A@@@ABU<unnamed-type-hb_any>@@$0A@@@YA_N$$QAU?$hb_map_iter_t@U?$hb_array_t@$$CBUhb_applicable_t@hb_accelerate_subtables_context_t@OT@@@@V<lambda_77b345933307e1fb3f76492be2367557>@@$0A@$0A@@@ABU<unnamed-type-hb_any>@@@Z 10052500 f   hb-ot-layout.obj
 0001:000515a0       ??$?UU?$hb_map_iter_t@U?$hb_array_t@$$CBUhb_applicable_t@hb_accelerate_subtables_context_t@OT@@@@V<lambda_f983cf953bf285b8455ade80df7cd301>@@$0A@$0A@@@ABU<unnamed-type-hb_any>@@$0A@@@YA_N$$QAU?$hb_map_iter_t@U?$hb_array_t@$$CBUhb_applicable_t@hb_accelerate_subtables_context_t@OT@@@@V<lambda_f983cf953bf285b8455ade80df7cd301>@@$0A@$0A@@@ABU<unnamed-type-hb_any>@@@Z 100525a0 f   hb-ot-layout.obj
 0001:00051640       ??$StructAfter@U?$ArrayOf@U?$IntType@G$01@OT@@U12@@OT@@U?$HeadlessArrayOf@U?$IntType@G$01@OT@@U12@@2@@@YAABU?$ArrayOf@U?$IntType@G$01@OT@@U12@@OT@@ABU?$HeadlessArrayOf@U?$IntType@G$01@OT@@U12@@1@@Z 10052640 f   hb-ot-layout.obj
 0001:00052280       ??$apply_string@UGSUBProxy@@@@YA_NPAUhb_ot_apply_context_t@OT@@ABUSubstLookup@GSUB_impl@Layout@1@ABUhb_ot_layout_lookup_accelerator_t@1@@Z 10053280 f   hb-ot-layout.obj
 0001:0005357c       $LN177                     1005457c     hb-ot-layout.obj
 0001:00053ba4       $LN659                     10054ba4     hb-ot-layout.obj
 0001:00053efc       $LN536                     10054efc     hb-ot-layout.obj
 0001:000540d8       $LN180                     100550d8     hb-ot-layout.obj
 0001:00054614       $LN347                     10055614     hb-ot-layout.obj
 0001:00054b94       $LN840                     10055b94     hb-ot-layout.obj
 0001:00055234       $LN484                     10056234     hb-ot-layout.obj
 0001:00056520       ??$would_match_input@U?$IntType@G$01@OT@@@OT@@YA_NPAUhb_would_apply_context_t@0@IQBU?$IntType@G$01@0@P6A_NAAUhb_glyph_info_t@@IPBX@Z3@Z 10057520 f   hb-ot-layout.obj
 0001:00056940       ?_hb_allocate_lig_id@@YAEPAUhb_buffer_t@@@Z 10057940 f   hb-ot-layout.obj
 0001:00056970       ?_hb_glyph_info_get_lig_comp@@YAIPBUhb_glyph_info_t@@@Z 10057970 f   hb-ot-layout.obj
 0001:00056990       ?_hb_glyph_info_is_zwj@@YA_NPBUhb_glyph_info_t@@@Z 10057990 f   hb-ot-layout.obj
 0001:000569b0       ?_hb_glyph_info_is_zwnj@@YA_NPBUhb_glyph_info_t@@@Z 100579b0 f   hb-ot-layout.obj
 0001:000569d0       ?_hb_ot_layout_set_glyph_props@@YAXPAUhb_font_t@@PAUhb_buffer_t@@@Z 100579d0 f   hb-ot-layout.obj
 0001:0005879c       $LN310                     1005979c     hb-ot-layout.obj
 0001:0005d66c       $LN408                     1005e66c     hb-ot-layout.obj
 0001:0005e160       ?apply_backward@@YA_NPAUhb_ot_apply_context_t@OT@@ABUhb_ot_layout_lookup_accelerator_t@2@I@Z 1005f160 f   hb-ot-layout.obj
 0001:0005e2a0       ?apply_forward@@YA_NPAUhb_ot_apply_context_t@OT@@ABUhb_ot_layout_lookup_accelerator_t@2@I@Z 1005f2a0 f   hb-ot-layout.obj
 0001:0005e4d0       ?apply_lookup@OT@@YAXPAUhb_ot_apply_context_t@1@IQAIIQBULookupRecord@1@I@Z 1005f4d0 f   hb-ot-layout.obj
 0001:0005f970       ?get_gsubgpos_table@@YAABUGSUBGPOS@OT@@PAUhb_face_t@@I@Z 10060970 f   hb-ot-layout.obj
 0001:00062910       ?ligate_input@OT@@YA_NPAUhb_ot_apply_context_t@1@IQBIIII@Z 10063910 f   hb-ot-layout.obj
 0001:00062c30       ?match_always@OT@@YA_NAAUhb_glyph_info_t@@IPBX@Z 10063c30 f   hb-ot-layout.obj
 0001:00062c40       ?match_class@OT@@YA_NAAUhb_glyph_info_t@@IPBX@Z 10063c40 f   hb-ot-layout.obj
 0001:00062c60       ?match_class_cached1@OT@@YA_NAAUhb_glyph_info_t@@IPBX@Z 10063c60 f   hb-ot-layout.obj
 0001:00062ca0       ?match_class_cached2@OT@@YA_NAAUhb_glyph_info_t@@IPBX@Z 10063ca0 f   hb-ot-layout.obj
 0001:00062ce0       ?match_class_cached@OT@@YA_NAAUhb_glyph_info_t@@IPBX@Z 10063ce0 f   hb-ot-layout.obj
 0001:00062d10       ?match_coverage@OT@@YA_NAAUhb_glyph_info_t@@IPBX@Z 10063d10 f   hb-ot-layout.obj
 0001:00062db0       ?match_glyph@OT@@YA_NAAUhb_glyph_info_t@@IPBX@Z 10063db0 f   hb-ot-layout.obj
 0001:00062e60       ?propagate_attachment_offsets@Layout@OT@@YAXPAUhb_glyph_position_t@@IIW4hb_direction_t@@I@Z 10063e60 f   hb-ot-layout.obj
 0001:00062f70       ?reverse_cursive_minor_offset@GPOS_impl@Layout@OT@@YAXPAUhb_glyph_position_t@@IW4hb_direction_t@@I@Z 10063f70 f   hb-ot-layout.obj
 0001:000639e4       $LN270                     100649e4     hb-ot-layout.obj
 0001:00068920       ?_fix_ascender_descender@@YAMMW4hb_ot_metrics_tag_t@@@Z 10069920 f   hb-ot-metrics.obj
 0001:0006966c       $LN60                      1006a66c     hb-ot-shape-fallback.obj
 0001:0006967c       $LN57                      1006a67c     hb-ot-shape-fallback.obj
 0001:0006971c       $LN61                      1006a71c     hb-ot-shape-fallback.obj
 0001:00069738       $LN58                      1006a738     hb-ot-shape-fallback.obj
 0001:000699d4       $LN76                      1006a9d4     hb-ot-shape-fallback.obj
 0001:000699ec       $LN69                      1006a9ec     hb-ot-shape-fallback.obj
 0001:00069f30       ?position_around_base@@YAXPBUhb_ot_shape_plan_t@@PAUhb_font_t@@PAUhb_buffer_t@@II_N@Z 1006af30 f   hb-ot-shape-fallback.obj
 0001:0006a340       ?position_cluster@@YAXPBUhb_ot_shape_plan_t@@PAUhb_font_t@@PAUhb_buffer_t@@II_N@Z 1006b340 f   hb-ot-shape-fallback.obj
 0001:0006a3c0       ?position_mark@@YAXPBUhb_ot_shape_plan_t@@PAUhb_font_t@@PAUhb_buffer_t@@AAUhb_glyph_extents_t@@II@Z 1006b3c0 f   hb-ot-shape-fallback.obj
 0001:0006a55c       $LN44                      1006b55c     hb-ot-shape-fallback.obj
 0001:0006a56c       $LN37                      1006b56c     hb-ot-shape-fallback.obj
 0001:0006a590       $LN45                      1006b590     hb-ot-shape-fallback.obj
 0001:0006a5a4       $LN38                      1006b5a4     hb-ot-shape-fallback.obj
 0001:0006a5d0       ?_hb_glyph_info_set_unicode_props@@YAXPAUhb_glyph_info_t@@PAUhb_buffer_t@@@Z 1006b5d0 f   hb-ot-shape-normalize.obj
 0001:0006a5d0       ?_hb_glyph_info_set_unicode_props@@YAXPAUhb_glyph_info_t@@PAUhb_buffer_t@@@Z 1006b5d0 f   hb-ot-shape.obj
 0001:0006a834       $LN112                     1006b834     hb-ot-shape.obj
 0001:0006a834       $LN112                     1006b834     hb-ot-shape-normalize.obj
 0001:0006a848       $LN106                     1006b848     hb-ot-shape-normalize.obj
 0001:0006a848       $LN106                     1006b848     hb-ot-shape.obj
 0001:0006b0e8       $LN399                     1006c0e8     hb-ot-shape-normalize.obj
 0001:0006b118       $LN372                     1006c118     hb-ot-shape-normalize.obj
 0001:0006b180       ?compare_combining_class@@YAHPBUhb_glyph_info_t@@0@Z 1006c180 f   hb-ot-shape-normalize.obj
 0001:0006b1d0       ?compose_unicode@@YA_NPBUhb_ot_shape_normalize_context_t@@IIPAI@Z 1006c1d0 f   hb-ot-shape-normalize.obj
 0001:0006b210       ?decompose@@YAIPBUhb_ot_shape_normalize_context_t@@_NI@Z 1006c210 f   hb-ot-shape-normalize.obj
 0001:0006b360       ?decompose_current_character@@YAXPBUhb_ot_shape_normalize_context_t@@_N@Z 1006c360 f   hb-ot-shape-normalize.obj
 0001:0006b5e0       $LN104                     1006c5e0     hb-ot-shape-normalize.obj
 0001:0006b610       $LN96                      1006c610     hb-ot-shape-normalize.obj
 0001:0006b670       ?decompose_unicode@@YA_NPBUhb_ot_shape_normalize_context_t@@IPAI1@Z 1006c670 f   hb-ot-shape-normalize.obj
 0001:0006b6b0       ?handle_variation_selector_cluster@@YAXPBUhb_ot_shape_normalize_context_t@@I_N@Z 1006c6b0 f   hb-ot-shape-normalize.obj
 0001:0006b970       ?output_char@@YAXPAUhb_buffer_t@@II@Z 1006c970 f   hb-ot-shape-normalize.obj
 0001:0006ba50       ?_hb_glyph_info_is_default_ignorable@@YA_NPBUhb_glyph_info_t@@@Z 1006ca50 f   hb-ot-shape.obj
 0001:0006bf50       ?hb_form_clusters@@YAXPAUhb_buffer_t@@@Z 1006cf50 f   hb-ot-shape.obj
 0001:0006c0c0       ?hb_ot_position@@YAXPBUhb_ot_shape_context_t@@@Z 1006d0c0 f   hb-ot-shape.obj
 0001:0006c210       ?hb_ot_position_plan@@YAXPBUhb_ot_shape_context_t@@@Z 1006d210 f   hb-ot-shape.obj
 0001:0006c470       ?hb_ot_rotate_chars@@YAXPBUhb_ot_shape_context_t@@@Z 1006d470 f   hb-ot-shape.obj
 0001:0006c72c       $LN90                      1006d72c     hb-ot-shape.obj
 0001:0006c740       $LN86                      1006d740     hb-ot-shape.obj
 0001:0006c820       $LN91                      1006d820     hb-ot-shape.obj
 0001:0006c834       $LN87                      1006d834     hb-ot-shape.obj
 0001:0006c848       $LN92                      1006d848     hb-ot-shape.obj
 0001:0006c8a4       $LN93                      1006d8a4     hb-ot-shape.obj
 0001:0006c8d8       $LN88                      1006d8d8     hb-ot-shape.obj
 0001:0006c940       ?hb_ot_shape_collect_features@@YAXPAUhb_ot_shape_planner_t@@PBUhb_feature_t@@I@Z 1006d940 f   hb-ot-shape.obj
 0001:0006cb30       ?hb_ot_shape_internal@@YAXPAUhb_ot_shape_context_t@@@Z 1006db30 f   hb-ot-shape.obj
 0001:0006cfb0       ?hb_ot_shape_setup_masks_fraction@@YAXPBUhb_ot_shape_context_t@@@Z 1006dfb0 f   hb-ot-shape.obj
 0001:0006d190       ?hb_ot_shaper_categorize@@YAPBUhb_ot_shaper_t@@PBUhb_ot_shape_planner_t@@@Z 1006e190 f   hb-ot-shape.obj
 0001:0006d680       ?hb_ot_substitute_pre@@YAXPBUhb_ot_shape_context_t@@@Z 1006e680 f   hb-ot-shape.obj
 0001:0006d840       ?hb_propagate_flags@@YAXPAUhb_buffer_t@@@Z 1006e840 f   hb-ot-shape.obj
 0001:0006dbc0       ?zero_mark_widths_by_gdef@@YAXPAUhb_buffer_t@@_N@Z 1006ebc0 f   hb-ot-shape.obj
 0001:0006dda0       ?collect_features_arabic@@YAXPAUhb_ot_shape_planner_t@@@Z 1006eda0 f   hb-ot-shaper-arabic.obj
 0001:0006def0       ?setup_masks_arabic@@YAXPBUhb_ot_shape_plan_t@@PAUhb_buffer_t@@PAUhb_font_t@@@Z 1006eef0 f   hb-ot-shaper-arabic.obj
 0001:0006df80       ?postprocess_glyphs_arabic@@YAXPBUhb_ot_shape_plan_t@@PAUhb_buffer_t@@PAUhb_font_t@@@Z 1006ef80 f   hb-ot-shaper-arabic.obj
 0001:0006df90       ?reorder_marks_arabic@@YAXPBUhb_ot_shape_plan_t@@PAUhb_buffer_t@@II@Z 1006ef90 f   hb-ot-shaper-arabic.obj
 0001:0006e210       ??$arabic_fallback_synthesize_lookup_ligature@$$BY00Uligature_3_set_t@@@@YAPAUSubstLookup@GSUB_impl@Layout@OT@@PBUhb_ot_shape_plan_t@@PAUhb_font_t@@AAY00$$CBUligature_3_set_t@@I@Z 1006f210 f   hb-ot-shaper-arabic.obj
 0001:0006e530       ??$arabic_fallback_synthesize_lookup_ligature@$$BY00Uligature_mark_set_t@@@@YAPAUSubstLookup@GSUB_impl@Layout@OT@@PBUhb_ot_shape_plan_t@@PAUhb_font_t@@AAY00$$CBUligature_mark_set_t@@I@Z 1006f530 f   hb-ot-shaper-arabic.obj
 0001:0006e850       ??$arabic_fallback_synthesize_lookup_ligature@$$BY0BC@Uligature_set_t@@@@YAPAUSubstLookup@GSUB_impl@Layout@OT@@PBUhb_ot_shape_plan_t@@PAUhb_font_t@@AAY0BC@$$CBUligature_set_t@@I@Z 1006f850 f   hb-ot-shaper-arabic.obj
 0001:0006ee50       ??$hb_stable_sort@UHBGlyphID16@OT@@U?$IntType@G$01@2@I@@YAXPAUHBGlyphID16@OT@@IP6AHPBU?$IntType@G$01@1@1@ZPAI@Z 1006fe50 f   hb-ot-shaper-arabic.obj
 0001:0006ffc0       ?apply_stch@@YAXPBUhb_ot_shape_plan_t@@PAUhb_buffer_t@@PAUhb_font_t@@@Z 10070fc0 f   hb-ot-shaper-arabic.obj
 0001:00070420       ?arabic_fallback_plan_create@@YAPAUarabic_fallback_plan_t@@PBUhb_ot_shape_plan_t@@PAUhb_font_t@@@Z 10071420 f   hb-ot-shaper-arabic.obj
 0001:000706d0       ?arabic_fallback_plan_destroy@@YAXPAUarabic_fallback_plan_t@@@Z 100716d0 f   hb-ot-shaper-arabic.obj
 0001:00070720       ?arabic_fallback_shape@@YA_NPBUhb_ot_shape_plan_t@@PAUhb_font_t@@PAUhb_buffer_t@@@Z 10071720 f   hb-ot-shaper-arabic.obj
 0001:00070860       ?arabic_fallback_synthesize_lookup_single@@YAPAUSubstLookup@GSUB_impl@Layout@OT@@PBUhb_ot_shape_plan_t@@PAUhb_font_t@@I@Z 10071860 f   hb-ot-shaper-arabic.obj
 0001:00070c00       ?arabic_joining@@YAXPAUhb_buffer_t@@@Z 10071c00 f   hb-ot-shaper-arabic.obj
 0001:00071040       ?deallocate_buffer_var@@YA_NPBUhb_ot_shape_plan_t@@PAUhb_font_t@@PAUhb_buffer_t@@@Z 10072040 f   hb-ot-shaper-arabic.obj
 0001:000712e0       ?get_joining_type@@YAIIW4hb_unicode_general_category_t@@@Z 100722e0 f   hb-ot-shaper-arabic.obj
 0001:00071404       $LN50                      10072404     hb-ot-shaper-arabic.obj
 0001:00071424       $LN48                      10072424     hb-ot-shaper-arabic.obj
 0001:00071530       ?record_stch@@YA_NPBUhb_ot_shape_plan_t@@PAUhb_font_t@@PAUhb_buffer_t@@@Z 10072530 f   hb-ot-shaper-arabic.obj
 0001:00072300       ?collect_features_hangul@@YAXPAUhb_ot_shape_planner_t@@@Z 10073300 f   hb-ot-shaper-hangul.obj
 0001:00072330       ?override_features_hangul@@YAXPAUhb_ot_shape_planner_t@@@Z 10073330 f   hb-ot-shaper-hangul.obj
 0001:00072350       ?data_create_hangul@@YAPAXPBUhb_ot_shape_plan_t@@@Z 10073350 f   hb-ot-shaper-hangul.obj
 0001:00072400       ?data_destroy_hangul@@YAXPAX@Z 10073400 f   hb-ot-shaper-hangul.obj
 0001:00072400       ?data_destroy_indic@@YAXPAX@Z 10073400 f   hb-ot-shaper-indic.obj
 0001:00072400       ?data_destroy_khmer@@YAXPAX@Z 10073400 f   hb-ot-shaper-khmer.obj
 0001:00072410       ?preprocess_text_hangul@@YAXPBUhb_ot_shape_plan_t@@PAUhb_buffer_t@@PAUhb_font_t@@@Z 10073410 f   hb-ot-shaper-hangul.obj
 0001:00072b20       ?setup_masks_hangul@@YAXPBUhb_ot_shape_plan_t@@PAUhb_buffer_t@@PAUhb_font_t@@@Z 10073b20 f   hb-ot-shaper-hangul.obj
 0001:00072b70       ?is_zero_width_char@@YA_NPAUhb_font_t@@I@Z 10073b70 f   hb-ot-shaper-hangul.obj
 0001:00072bb0       ?compose_hebrew@@YA_NPBUhb_ot_shape_normalize_context_t@@IIPAI@Z 10073bb0 f   hb-ot-shaper-hebrew.obj
 0001:00072d78       $LN45                      10073d78     hb-ot-shaper-hebrew.obj
 0001:00072d9c       $LN40                      10073d9c     hb-ot-shaper-hebrew.obj
 0001:00072db0       ?reorder_marks_hebrew@@YAXPBUhb_ot_shape_plan_t@@PAUhb_buffer_t@@II@Z 10073db0 f   hb-ot-shaper-hebrew.obj
 0001:0007301c       $LN61                      1007401c     hb-ot-shaper-indic-table.obj
 0001:00073038       $LN59                      10074038     hb-ot-shaper-indic-table.obj
 0001:00073050       ?collect_features_indic@@YAXPAUhb_ot_shape_planner_t@@@Z 10074050 f   hb-ot-shaper-indic.obj
 0001:00073100       ?override_features_indic@@YAXPAUhb_ot_shape_planner_t@@@Z 10074100 f   hb-ot-shaper-indic.obj
 0001:00073130       ?data_create_indic@@YAPAXPBUhb_ot_shape_plan_t@@@Z 10074130 f   hb-ot-shaper-indic.obj
 0001:00073280       ?setup_masks_indic@@YAXPBUhb_ot_shape_plan_t@@PAUhb_buffer_t@@PAUhb_font_t@@@Z 10074280 f   hb-ot-shaper-indic.obj
 0001:000732d0       ?preprocess_text_indic@@YAXPBUhb_ot_shape_plan_t@@PAUhb_buffer_t@@PAUhb_font_t@@@Z 100742d0 f   hb-ot-shaper-indic.obj
 0001:000732f0       ?decompose_indic@@YA_NPBUhb_ot_shape_normalize_context_t@@IPAI1@Z 100742f0 f   hb-ot-shaper-indic.obj
 0001:00073350       ?compose_indic@@YA_NPBUhb_ot_shape_normalize_context_t@@IIPAI@Z 10074350 f   hb-ot-shaper-indic.obj
 0001:00073400       ?_hb_next_syllable@@YAIPAUhb_buffer_t@@I@Z 10074400 f   hb-ot-shaper-indic.obj
 0001:00073430       ?final_reordering_indic@@YA_NPBUhb_ot_shape_plan_t@@PAUhb_font_t@@PAUhb_buffer_t@@@Z 10074430 f   hb-ot-shaper-indic.obj
 0001:000734d0       ?final_reordering_syllable_indic@@YAXPBUhb_ot_shape_plan_t@@PAUhb_buffer_t@@II@Z 100744d0 f   hb-ot-shaper-indic.obj
 0001:000743d4       $LN246                     100753d4     hb-ot-shaper-indic.obj
 0001:000744f0       ?initial_reordering_consonant_syllable@@YAXPBUhb_ot_shape_plan_t@@PAUhb_face_t@@PAUhb_buffer_t@@II@Z 100754f0 f   hb-ot-shaper-indic.obj
 0001:00075040       ?initial_reordering_indic@@YA_NPBUhb_ot_shape_plan_t@@PAUhb_font_t@@PAUhb_buffer_t@@@Z 10076040 f   hb-ot-shaper-indic.obj
 0001:00075154       $LN41                      10076154     hb-ot-shaper-indic.obj
 0001:00075170       ?is_joiner@@YA_NABUhb_glyph_info_t@@@Z 10076170 f   hb-ot-shaper-indic.obj
 0001:000751a0       ?is_one_of@@YA_NABUhb_glyph_info_t@@I@Z 100761a0 f   hb-ot-shaper-indic.obj
 0001:000751e0       ?setup_syllables_indic@@YA_NPBUhb_ot_shape_plan_t@@PAUhb_font_t@@PAUhb_buffer_t@@@Z 100761e0 f   hb-ot-shaper-indic.obj
 0001:000752b0       ?update_consonant_positions_indic@@YAXPBUhb_ot_shape_plan_t@@PAUhb_font_t@@PAUhb_buffer_t@@@Z 100762b0 f   hb-ot-shaper-indic.obj
 0001:000754b0       ?collect_features_khmer@@YAXPAUhb_ot_shape_planner_t@@@Z 100764b0 f   hb-ot-shaper-khmer.obj
 0001:00075550       ?override_features_khmer@@YAXPAUhb_ot_shape_planner_t@@@Z 10076550 f   hb-ot-shaper-khmer.obj
 0001:000755b0       ?data_create_khmer@@YAPAXPBUhb_ot_shape_plan_t@@@Z 100765b0 f   hb-ot-shaper-khmer.obj
 0001:00075660       ?setup_masks_khmer@@YAXPBUhb_ot_shape_plan_t@@PAUhb_buffer_t@@PAUhb_font_t@@@Z 10076660 f   hb-ot-shaper-khmer.obj
 0001:00075690       ?decompose_khmer@@YA_NPBUhb_ot_shape_normalize_context_t@@IPAI1@Z 10076690 f   hb-ot-shaper-khmer.obj
 0001:0007574c       $LN13                      1007674c     hb-ot-shaper-khmer.obj
 0001:00075770       ?compose_khmer@@YA_NPBUhb_ot_shape_normalize_context_t@@IIPAI@Z 10076770 f   hb-ot-shaper-khmer.obj
 0001:00075770       ?compose_use@@YA_NPBUhb_ot_shape_normalize_context_t@@IIPAI@Z 10076770 f   hb-ot-shaper-use.obj
 0001:00075b04       $LN154                     10076b04     hb-ot-shaper-khmer.obj
 0001:00075b40       ?reorder_consonant_syllable@@YAXPBUhb_ot_shape_plan_t@@PAUhb_face_t@@PAUhb_buffer_t@@II@Z 10076b40 f   hb-ot-shaper-khmer.obj
 0001:00075d30       ?reorder_khmer@@YA_NPBUhb_ot_shape_plan_t@@PAUhb_font_t@@PAUhb_buffer_t@@@Z 10076d30 f   hb-ot-shaper-khmer.obj
 0001:00075e30       ?setup_syllables_khmer@@YA_NPBUhb_ot_shape_plan_t@@PAUhb_font_t@@PAUhb_buffer_t@@@Z 10076e30 f   hb-ot-shaper-khmer.obj
 0001:00075f00       ?collect_features_myanmar@@YAXPAUhb_ot_shape_planner_t@@@Z 10076f00 f   hb-ot-shaper-myanmar.obj
 0001:00075fa0       ?setup_masks_myanmar@@YAXPBUhb_ot_shape_plan_t@@PAUhb_buffer_t@@PAUhb_font_t@@@Z 10076fa0 f   hb-ot-shaper-myanmar.obj
 0001:00075fd0       ?compare_myanmar_order@@YAHPBUhb_glyph_info_t@@0@Z 10076fd0 f   hb-ot-shaper-myanmar.obj
 0001:00076280       $LN131                     10077280     hb-ot-shaper-myanmar.obj
 0001:000762a0       ?initial_reordering_consonant_syllable@@YAXPAUhb_buffer_t@@II@Z 100772a0 f   hb-ot-shaper-myanmar.obj
 0001:00076590       ?reorder_myanmar@@YA_NPBUhb_ot_shape_plan_t@@PAUhb_font_t@@PAUhb_buffer_t@@@Z 10077590 f   hb-ot-shaper-myanmar.obj
 0001:00076670       ?setup_syllables_myanmar@@YA_NPBUhb_ot_shape_plan_t@@PAUhb_font_t@@PAUhb_buffer_t@@@Z 10077670 f   hb-ot-shaper-myanmar.obj
 0001:00076940       ?preprocess_text_thai@@YAXPBUhb_ot_shape_plan_t@@PAUhb_buffer_t@@PAUhb_font_t@@@Z 10077940 f   hb-ot-shaper-thai.obj
 0001:00076be0       ?do_thai_pua_shaping@@YAXPBUhb_ot_shape_plan_t@@PAUhb_buffer_t@@PAUhb_font_t@@@Z 10077be0 f   hb-ot-shaper-thai.obj
 0001:00076e10       ?thai_pua_shape@@YAIIW4thai_action_t@@PAUhb_font_t@@@Z 10077e10 f   hb-ot-shaper-thai.obj
 0001:00076ed0       $LN23                      10077ed0     hb-ot-shaper-thai.obj
 0001:00076ef0       ?collect_features_use@@YAXPAUhb_ot_shape_planner_t@@@Z 10077ef0 f   hb-ot-shaper-use.obj
 0001:00077030       ?data_create_use@@YAPAXPBUhb_ot_shape_plan_t@@@Z 10078030 f   hb-ot-shaper-use.obj
 0001:000770f0       ?data_destroy_use@@YAXPAX@Z 100780f0 f   hb-ot-shaper-use.obj
 0001:00077120       ?setup_masks_use@@YAXPBUhb_ot_shape_plan_t@@PAUhb_buffer_t@@PAUhb_font_t@@@Z 10078120 f   hb-ot-shaper-use.obj
 0001:000771d0       ?preprocess_text_use@@YAXPBUhb_ot_shape_plan_t@@PAUhb_buffer_t@@PAUhb_font_t@@@Z 100781d0 f   hb-ot-shaper-use.obj
 0001:000771e0       ??4?$machine_index_t@U?$hb_zip_iter_t@U?$hb_iota_iter_t@II@@U?$hb_filter_iter_t@U?$hb_filter_iter_t@U?$hb_zip_iter_t@U?$hb_iota_iter_t@II@@U?$hb_array_t@Uhb_glyph_info_t@@@@@@V<lambda_ce8f76acbbe9af6df8f1b6105ce8238a>@@ABU<unnamed-type-hb_second>@@$0A@@@V<lambda_daa85cc6b6d559953d3cb9980857ae51>@@ABU<unnamed-type-hb_identity>@@$0A@@@@@@@QAEXABU0@@Z 100781e0 f   hb-ot-shaper-use.obj
 0001:00077250       ??8?$machine_index_t@U?$hb_zip_iter_t@U?$hb_iota_iter_t@II@@U?$hb_filter_iter_t@U?$hb_filter_iter_t@U?$hb_zip_iter_t@U?$hb_iota_iter_t@II@@U?$hb_array_t@Uhb_glyph_info_t@@@@@@V<lambda_ce8f76acbbe9af6df8f1b6105ce8238a>@@ABU<unnamed-type-hb_second>@@$0A@@@V<lambda_daa85cc6b6d559953d3cb9980857ae51>@@ABU<unnamed-type-hb_identity>@@$0A@@@@@@@QBE_NABU0@@Z 10078250 f   hb-ot-shaper-use.obj
 0001:000772b0       ??D?$hb_iter_t@U?$hb_zip_iter_t@U?$hb_iota_iter_t@II@@U?$hb_filter_iter_t@U?$hb_filter_iter_t@U?$hb_zip_iter_t@U?$hb_iota_iter_t@II@@U?$hb_array_t@Uhb_glyph_info_t@@@@@@V<lambda_ce8f76acbbe9af6df8f1b6105ce8238a>@@ABU<unnamed-type-hb_second>@@$0A@@@V<lambda_daa85cc6b6d559953d3cb9980857ae51>@@ABU<unnamed-type-hb_identity>@@$0A@@@@@U?$hb_pair_t@IU?$hb_pair_t@IAAUhb_glyph_info_t@@@@@@@@QBE?AU?$hb_pair_t@IU?$hb_pair_t@IAAUhb_glyph_info_t@@@@@@XZ 100782b0 f   hb-ot-shaper-use.obj
 0001:000772f0       ??D?$hb_iter_t@U?$machine_index_t@U?$hb_zip_iter_t@U?$hb_iota_iter_t@II@@U?$hb_filter_iter_t@U?$hb_filter_iter_t@U?$hb_zip_iter_t@U?$hb_iota_iter_t@II@@U?$hb_array_t@Uhb_glyph_info_t@@@@@@V<lambda_ce8f76acbbe9af6df8f1b6105ce8238a>@@ABU<unnamed-type-hb_second>@@$0A@@@V<lambda_daa85cc6b6d559953d3cb9980857ae51>@@ABU<unnamed-type-hb_identity>@@$0A@@@@@@@U?$hb_pair_t@IU?$hb_pair_t@IAAUhb_glyph_info_t@@@@@@@@QAE?AU?$hb_pair_t@IU?$hb_pair_t@IAAUhb_glyph_info_t@@@@@@XZ 100782f0 f   hb-ot-shaper-use.obj
 0001:00077330       ??E?$hb_iter_t@U?$hb_filter_iter_t@U?$hb_filter_iter_t@U?$hb_zip_iter_t@U?$hb_iota_iter_t@II@@U?$hb_array_t@Uhb_glyph_info_t@@@@@@V<lambda_ce8f76acbbe9af6df8f1b6105ce8238a>@@ABU<unnamed-type-hb_second>@@$0A@@@V<lambda_daa85cc6b6d559953d3cb9980857ae51>@@ABU<unnamed-type-hb_identity>@@$0A@@@U?$hb_pair_t@IAAUhb_glyph_info_t@@@@@@QGAEAAU?$hb_filter_iter_t@U?$hb_filter_iter_t@U?$hb_zip_iter_t@U?$hb_iota_iter_t@II@@U?$hb_array_t@Uhb_glyph_info_t@@@@@@V<lambda_ce8f76acbbe9af6df8f1b6105ce8238a>@@ABU<unnamed-type-hb_second>@@$0A@@@V<lambda_daa85cc6b6d559953d3cb9980857ae51>@@ABU<unnamed-type-hb_identity>@@$0A@@@XZ 10078330 f   hb-ot-shaper-use.obj
 0001:00077410       ??F?$hb_iter_t@U?$hb_filter_iter_t@U?$hb_filter_iter_t@U?$hb_zip_iter_t@U?$hb_iota_iter_t@II@@U?$hb_array_t@Uhb_glyph_info_t@@@@@@V<lambda_ce8f76acbbe9af6df8f1b6105ce8238a>@@ABU<unnamed-type-hb_second>@@$0A@@@V<lambda_daa85cc6b6d559953d3cb9980857ae51>@@ABU<unnamed-type-hb_identity>@@$0A@@@U?$hb_pair_t@IAAUhb_glyph_info_t@@@@@@QGAEAAU?$hb_filter_iter_t@U?$hb_filter_iter_t@U?$hb_zip_iter_t@U?$hb_iota_iter_t@II@@U?$hb_array_t@Uhb_glyph_info_t@@@@@@V<lambda_ce8f76acbbe9af6df8f1b6105ce8238a>@@ABU<unnamed-type-hb_second>@@$0A@@@V<lambda_daa85cc6b6d559953d3cb9980857ae51>@@ABU<unnamed-type-hb_identity>@@$0A@@@XZ 10078410 f   hb-ot-shaper-use.obj
 0001:000774f0       ??F?$hb_iter_t@U?$machine_index_t@U?$hb_zip_iter_t@U?$hb_iota_iter_t@II@@U?$hb_filter_iter_t@U?$hb_filter_iter_t@U?$hb_zip_iter_t@U?$hb_iota_iter_t@II@@U?$hb_array_t@Uhb_glyph_info_t@@@@@@V<lambda_ce8f76acbbe9af6df8f1b6105ce8238a>@@ABU<unnamed-type-hb_second>@@$0A@@@V<lambda_daa85cc6b6d559953d3cb9980857ae51>@@ABU<unnamed-type-hb_identity>@@$0A@@@@@@@U?$hb_pair_t@IU?$hb_pair_t@IAAUhb_glyph_info_t@@@@@@@@QAE?AU?$machine_index_t@U?$hb_zip_iter_t@U?$hb_iota_iter_t@II@@U?$hb_filter_iter_t@U?$hb_filter_iter_t@U?$hb_zip_iter_t@U?$hb_iota_iter_t@II@@U?$hb_array_t@Uhb_glyph_info_t@@@@@@V<lambda_ce8f76acbbe9af6df8f1b6105ce8238a>@@ABU<unnamed-type-hb_second>@@$0A@@@V<lambda_daa85cc6b6d559953d3cb9980857ae51>@@ABU<unnamed-type-hb_identity>@@$0A@@@@@@@H@Z 100784f0 f   hb-ot-shaper-use.obj
 0001:00077540       ??H?$hb_iter_t@U?$machine_index_t@U?$hb_zip_iter_t@U?$hb_iota_iter_t@II@@U?$hb_filter_iter_t@U?$hb_filter_iter_t@U?$hb_zip_iter_t@U?$hb_iota_iter_t@II@@U?$hb_array_t@Uhb_glyph_info_t@@@@@@V<lambda_ce8f76acbbe9af6df8f1b6105ce8238a>@@ABU<unnamed-type-hb_second>@@$0A@@@V<lambda_daa85cc6b6d559953d3cb9980857ae51>@@ABU<unnamed-type-hb_identity>@@$0A@@@@@@@U?$hb_pair_t@IU?$hb_pair_t@IAAUhb_glyph_info_t@@@@@@@@QBE?AU?$machine_index_t@U?$hb_zip_iter_t@U?$hb_iota_iter_t@II@@U?$hb_filter_iter_t@U?$hb_filter_iter_t@U?$hb_zip_iter_t@U?$hb_iota_iter_t@II@@U?$hb_array_t@Uhb_glyph_info_t@@@@@@V<lambda_ce8f76acbbe9af6df8f1b6105ce8238a>@@ABU<unnamed-type-hb_second>@@$0A@@@V<lambda_daa85cc6b6d559953d3cb9980857ae51>@@ABU<unnamed-type-hb_identity>@@$0A@@@@@@@I@Z 10078540 f   hb-ot-shaper-use.obj
 0001:000775b0       ??Y?$hb_iter_t@U?$hb_zip_iter_t@U?$hb_iota_iter_t@II@@U?$hb_filter_iter_t@U?$hb_filter_iter_t@U?$hb_zip_iter_t@U?$hb_iota_iter_t@II@@U?$hb_array_t@Uhb_glyph_info_t@@@@@@V<lambda_ce8f76acbbe9af6df8f1b6105ce8238a>@@ABU<unnamed-type-hb_second>@@$0A@@@V<lambda_daa85cc6b6d559953d3cb9980857ae51>@@ABU<unnamed-type-hb_identity>@@$0A@@@@@U?$hb_pair_t@IU?$hb_pair_t@IAAUhb_glyph_info_t@@@@@@@@QGAEAAU?$hb_zip_iter_t@U?$hb_iota_iter_t@II@@U?$hb_filter_iter_t@U?$hb_filter_iter_t@U?$hb_zip_iter_t@U?$hb_iota_iter_t@II@@U?$hb_array_t@Uhb_glyph_info_t@@@@@@V<lambda_ce8f76acbbe9af6df8f1b6105ce8238a>@@ABU<unnamed-type-hb_second>@@$0A@@@V<lambda_daa85cc6b6d559953d3cb9980857ae51>@@ABU<unnamed-type-hb_identity>@@$0A@@@@@I@Z 100785b0 f   hb-ot-shaper-use.obj
 0001:000775f0       ??Z?$hb_iter_t@U?$hb_zip_iter_t@U?$hb_iota_iter_t@II@@U?$hb_filter_iter_t@U?$hb_filter_iter_t@U?$hb_zip_iter_t@U?$hb_iota_iter_t@II@@U?$hb_array_t@Uhb_glyph_info_t@@@@@@V<lambda_ce8f76acbbe9af6df8f1b6105ce8238a>@@ABU<unnamed-type-hb_second>@@$0A@@@V<lambda_daa85cc6b6d559953d3cb9980857ae51>@@ABU<unnamed-type-hb_identity>@@$0A@@@@@U?$hb_pair_t@IU?$hb_pair_t@IAAUhb_glyph_info_t@@@@@@@@QGAEAAU?$hb_zip_iter_t@U?$hb_iota_iter_t@II@@U?$hb_filter_iter_t@U?$hb_filter_iter_t@U?$hb_zip_iter_t@U?$hb_iota_iter_t@II@@U?$hb_array_t@Uhb_glyph_info_t@@@@@@V<lambda_ce8f76acbbe9af6df8f1b6105ce8238a>@@ABU<unnamed-type-hb_second>@@$0A@@@V<lambda_daa85cc6b6d559953d3cb9980857ae51>@@ABU<unnamed-type-hb_identity>@@$0A@@@@@I@Z 100785f0 f   hb-ot-shaper-use.obj
 0001:00077630       ?__forward__@?$hb_iter_fallback_mixin_t@U?$hb_filter_iter_t@U?$hb_filter_iter_t@U?$hb_zip_iter_t@U?$hb_iota_iter_t@II@@U?$hb_array_t@Uhb_glyph_info_t@@@@@@V<lambda_ce8f76acbbe9af6df8f1b6105ce8238a>@@ABU<unnamed-type-hb_second>@@$0A@@@V<lambda_daa85cc6b6d559953d3cb9980857ae51>@@ABU<unnamed-type-hb_identity>@@$0A@@@U?$hb_pair_t@IAAUhb_glyph_info_t@@@@@@QAEXI@Z 10078630 f   hb-ot-shaper-use.obj
 0001:00077820       ?__item__@?$hb_filter_iter_t@U?$hb_zip_iter_t@U?$hb_iota_iter_t@II@@U?$hb_array_t@Uhb_glyph_info_t@@@@@@V<lambda_ce8f76acbbe9af6df8f1b6105ce8238a>@@ABU<unnamed-type-hb_second>@@$0A@@@QBE?AU?$hb_pair_t@IAAUhb_glyph_info_t@@@@XZ 10078820 f   hb-ot-shaper-use.obj
 0001:00077870       ?__rewind__@?$hb_iter_fallback_mixin_t@U?$hb_filter_iter_t@U?$hb_filter_iter_t@U?$hb_zip_iter_t@U?$hb_iota_iter_t@II@@U?$hb_array_t@Uhb_glyph_info_t@@@@@@V<lambda_ce8f76acbbe9af6df8f1b6105ce8238a>@@ABU<unnamed-type-hb_second>@@$0A@@@V<lambda_daa85cc6b6d559953d3cb9980857ae51>@@ABU<unnamed-type-hb_identity>@@$0A@@@U?$hb_pair_t@IAAUhb_glyph_info_t@@@@@@QAEXI@Z 10078870 f   hb-ot-shaper-use.obj
 0001:00077a60       ?_hb_clear_substitution_flags@@YA_NPBUhb_ot_shape_plan_t@@PAUhb_font_t@@PAUhb_buffer_t@@@Z 10078a60 f   hb-ot-shaper-use.obj
 0001:00077a90       ?find_syllables_use@@YAXPAUhb_buffer_t@@@Z 10078a90 f   hb-ot-shaper-use.obj
 0001:00078c0c       $LN2071                    10079c0c     hb-ot-shaper-use.obj
 0001:00078c70       ?record_pref_use@@YA_NPBUhb_ot_shape_plan_t@@PAUhb_font_t@@PAUhb_buffer_t@@@Z 10079c70 f   hb-ot-shaper-use.obj
 0001:00078d00       ?record_rphf_use@@YA_NPBUhb_ot_shape_plan_t@@PAUhb_font_t@@PAUhb_buffer_t@@@Z 10079d00 f   hb-ot-shaper-use.obj
 0001:00078db0       ?reorder_syllable_use@@YAXPAUhb_buffer_t@@II@Z 10079db0 f   hb-ot-shaper-use.obj
 0001:00079000       ?reorder_use@@YA_NPBUhb_ot_shape_plan_t@@PAUhb_font_t@@PAUhb_buffer_t@@@Z 1007a000 f   hb-ot-shaper-use.obj
 0001:000790d0       ?setup_syllables_use@@YA_NPBUhb_ot_shape_plan_t@@PAUhb_font_t@@PAUhb_buffer_t@@@Z 1007a0d0 f   hb-ot-shaper-use.obj
 0001:00079240       ?setup_topographical_masks@@YAXPBUhb_ot_shape_plan_t@@PAUhb_buffer_t@@@Z 1007a240 f   hb-ot-shaper-use.obj
 0001:00079460       $LN120                     1007a460     hb-ot-shaper-use.obj
 0001:00079468       $LN114                     1007a468     hb-ot-shaper-use.obj
 0001:00079e60       $LN399                     1007ae60     hb-ot-shaper-vowel-constraints.obj
 0001:00079e78       $LN380                     1007ae78     hb-ot-shaper-vowel-constraints.obj
 0001:00079ea4       $LN400                     1007aea4     hb-ot-shaper-vowel-constraints.obj
 0001:00079eac       $LN381                     1007aeac     hb-ot-shaper-vowel-constraints.obj
 0001:00079ecc       $LN401                     1007aecc     hb-ot-shaper-vowel-constraints.obj
 0001:00079ed4       $LN382                     1007aed4     hb-ot-shaper-vowel-constraints.obj
 0001:00079ee4       $LN402                     1007aee4     hb-ot-shaper-vowel-constraints.obj
 0001:00079ef4       $LN383                     1007aef4     hb-ot-shaper-vowel-constraints.obj
 0001:00079f00       $LN403                     1007af00     hb-ot-shaper-vowel-constraints.obj
 0001:00079f14       $LN384                     1007af14     hb-ot-shaper-vowel-constraints.obj
 0001:00079f58       $LN404                     1007af58     hb-ot-shaper-vowel-constraints.obj
 0001:00079f6c       $LN385                     1007af6c     hb-ot-shaper-vowel-constraints.obj
 0001:00079f7c       $LN405                     1007af7c     hb-ot-shaper-vowel-constraints.obj
 0001:00079f84       $LN386                     1007af84     hb-ot-shaper-vowel-constraints.obj
 0001:00079f9c       $LN406                     1007af9c     hb-ot-shaper-vowel-constraints.obj
 0001:00079fac       $LN387                     1007afac     hb-ot-shaper-vowel-constraints.obj
 0001:00079fd8       $LN407                     1007afd8     hb-ot-shaper-vowel-constraints.obj
 0001:00079fe4       $LN388                     1007afe4     hb-ot-shaper-vowel-constraints.obj
 0001:0007a020       ?_output_with_dotted_circle@@YAXPAUhb_buffer_t@@@Z 1007b020 f   hb-ot-shaper-vowel-constraints.obj
 0001:0007a0b0       ?TOLOWER@@YAEE@Z           1007b0b0 f   hb-ot-tag.obj
 0001:0007a0d0       ?TOUPPER@@YAEE@Z           1007b0d0 f   hb-ot-tag.obj
 0001:0007a0f0       ?hb_ot_ambiguous_tag_to_language@@YAPBUhb_language_impl_t@@I@Z 1007b0f0 f   hb-ot-tag.obj
 0001:0007a910       ?hb_ot_tags_from_complex_language@@YA_NPBD0PAI1@Z 1007b910 f   hb-ot-tag.obj
 0001:0007c3ac       $LN414                     1007d3ac     hb-ot-tag.obj
 0001:0007c3e0       $LN375                     1007d3e0     hb-ot-tag.obj
 0001:0007c400       ?hb_ot_tags_from_language@@YAXPBD0PAI1@Z 1007d400 f   hb-ot-tag.obj
 0001:0007c5e0       ?lang_matches@@YA_NPBD00I@Z 1007d5e0 f   hb-ot-tag.obj
 0001:0007c620       ?parse_private_use_subtag@@YA_NPBDPAI10P6AEE@Z@Z 1007d620 f   hb-ot-tag.obj
 0001:0007c7a0       ?subtag_matches@@YA_NPBD00I@Z 1007d7a0 f   hb-ot-tag.obj
 0001:0007d920       ?hb_outline_recording_pen_close_path@@YAXPAUhb_draw_funcs_t@@PAXPAUhb_draw_state_t@@1@Z 1007e920 f   hb-outline.obj
 0001:0007d960       ?hb_outline_recording_pen_cubic_to@@YAXPAUhb_draw_funcs_t@@PAXPAUhb_draw_state_t@@MMMMMM1@Z 1007e960 f   hb-outline.obj
 0001:0007dac0       ?hb_outline_recording_pen_line_to@@YAXPAUhb_draw_funcs_t@@PAXPAUhb_draw_state_t@@MM1@Z 1007eac0 f   hb-outline.obj
 0001:0007db00       ?hb_outline_recording_pen_move_to@@YAXPAUhb_draw_funcs_t@@PAXPAUhb_draw_state_t@@MM1@Z 1007eb00 f   hb-outline.obj
 0001:0007db40       ?hb_outline_recording_pen_quadratic_to@@YAXPAUhb_draw_funcs_t@@PAXPAUhb_draw_state_t@@MMMM1@Z 1007eb40 f   hb-outline.obj
 0001:0007e1ac       $LN260                     1007f1ac     hb-outline.obj
 0001:0007e1c0       ?hb_draw_extents_cubic_to@@YAXPAUhb_draw_funcs_t@@PAXPAUhb_draw_state_t@@MMMMMM1@Z 1007f1c0 f   hb-paint-extents.obj
 0001:0007e340       ?hb_draw_extents_move_to@@YAXPAUhb_draw_funcs_t@@PAXPAUhb_draw_state_t@@MM1@Z 1007f340 f   hb-paint-extents.obj
 0001:0007e340       ?hb_draw_extents_line_to@@YAXPAUhb_draw_funcs_t@@PAXPAUhb_draw_state_t@@MM1@Z 1007f340 f   hb-paint-extents.obj
 0001:0007e3d0       ?hb_draw_extents_quadratic_to@@YAXPAUhb_draw_funcs_t@@PAXPAUhb_draw_state_t@@MMMM1@Z 1007f3d0 f   hb-paint-extents.obj
 0001:0007e620       ?hb_paint_extents_paint_radial_gradient@@YAXPAUhb_paint_funcs_t@@PAXPAUhb_color_line_t@@MMMMMM1@Z 1007f620 f   hb-paint-extents.obj
 0001:0007e620       ?hb_paint_extents_paint_color@@YAXPAUhb_paint_funcs_t@@PAXHI1@Z 1007f620 f   hb-paint-extents.obj
 0001:0007e620       ?hb_paint_extents_paint_sweep_gradient@@YAXPAUhb_paint_funcs_t@@PAXPAUhb_color_line_t@@MMMM1@Z 1007f620 f   hb-paint-extents.obj
 0001:0007e620       ?hb_paint_extents_paint_linear_gradient@@YAXPAUhb_paint_funcs_t@@PAXPAUhb_color_line_t@@MMMMMM1@Z 1007f620 f   hb-paint-extents.obj
 0001:0007e630       ?hb_paint_extents_paint_image@@YAHPAUhb_paint_funcs_t@@PAXPAUhb_blob_t@@IIIMPAUhb_glyph_extents_t@@1@Z 1007f630 f   hb-paint-extents.obj
 0001:0007e6b0       ?hb_paint_extents_pop_clip@@YAXPAUhb_paint_funcs_t@@PAX1@Z 1007f6b0 f   hb-paint-extents.obj
 0001:0007e6c0       ?hb_paint_extents_pop_group@@YAXPAUhb_paint_funcs_t@@PAXW4hb_paint_composite_mode_t@@1@Z 1007f6c0 f   hb-paint-extents.obj
 0001:0007e81c       $LN62                      1007f81c     hb-paint-extents.obj
 0001:0007e840       ?hb_paint_extents_pop_transform@@YAXPAUhb_paint_funcs_t@@PAX1@Z 1007f840 f   hb-paint-extents.obj
 0001:0007e850       ?hb_paint_extents_push_clip_glyph@@YAXPAUhb_paint_funcs_t@@PAXIPAUhb_font_t@@1@Z 1007f850 f   hb-paint-extents.obj
 0001:0007e940       ?hb_paint_extents_push_clip_rectangle@@YAXPAUhb_paint_funcs_t@@PAXMMMM1@Z 1007f940 f   hb-paint-extents.obj
 0001:0007e990       ?hb_paint_extents_push_group@@YAXPAUhb_paint_funcs_t@@PAX1@Z 1007f990 f   hb-paint-extents.obj
 0001:0007e9c0       ?hb_paint_extents_push_transform@@YAXPAUhb_paint_funcs_t@@PAXMMMMMM1@Z 1007f9c0 f   hb-paint-extents.obj
 0001:0007efb0       ?_hb_paint_funcs_set_middle@@YA_NPAUhb_paint_funcs_t@@PAXP6AX1@Z@Z 1007ffb0 f   hb-paint.obj
 0001:0007fbd0       ?_hb_shape_plan_execute_internal@@YA_NPAUhb_shape_plan_t@@PAUhb_font_t@@PAUhb_buffer_t@@PBUhb_feature_t@@I@Z 10080bd0 f   hb-shape-plan.obj
 0001:000808b0       ?hb_ucd_combining_class@@YA?AW4hb_unicode_combining_class_t@@PAUhb_unicode_funcs_t@@IPAX@Z 100818b0 f   hb-ucd.obj
 0001:00080910       ?hb_ucd_compose@@YAHPAUhb_unicode_funcs_t@@IIPAIPAX@Z 10081910 f   hb-ucd.obj
 0001:00080aa0       ?hb_ucd_decompose@@YAHPAUhb_unicode_funcs_t@@IPAI1PAX@Z 10081aa0 f   hb-ucd.obj
 0001:00080c30       ?hb_ucd_general_category@@YA?AW4hb_unicode_general_category_t@@PAUhb_unicode_funcs_t@@IPAX@Z 10081c30 f   hb-ucd.obj
 0001:00080c90       ?hb_ucd_mirroring@@YAIPAUhb_unicode_funcs_t@@IPAX@Z 10081c90 f   hb-ucd.obj
 0001:00080d00       ?hb_ucd_script@@YA?AW4hb_script_t@@PAUhb_unicode_funcs_t@@IPAX@Z 10081d00 f   hb-ucd.obj
 0001:00080ec0       ?hb_unicode_general_category_nil@@YA?AW4hb_unicode_general_category_t@@PAUhb_unicode_funcs_t@@IPAX@Z 10081ec0 f   hb-unicode.obj
 0001:00080ed0       ?hb_unicode_mirroring_nil@@YAIPAUhb_unicode_funcs_t@@IPAX@Z 10081ed0 f   hb-unicode.obj
 0001:00080ee0       ?hb_unicode_script_nil@@YA?AW4hb_script_t@@PAUhb_unicode_funcs_t@@IPAX@Z 10081ee0 f   hb-unicode.obj
 0001:000820b0       _initFontIDs               100830b0 f   sunFont.obj
 0001:00082780       $$000000                   10083780     MSVCRT:ftol3.obj
 0001:00082b00       $$000000                   10083b00     MSVCRT:llmul.obj
 0001:00082d30       $$000000                   10083d30     MSVCRT:lldiv.obj
 0001:00082de0       $$000000                   10083de0     MSVCRT:chkstk.obj
 0001:00082e10       $$000000                   10083e10     MSVCRT:ftol2.obj
 0001:00082ed0       $$000000                   10083ed0     MSVCRT:alloca16.obj
 0001:00082efc       ?dllmain_crt_dispatch@@YGHQAUHINSTANCE__@@KQAX@Z 10083efc f   MSVCRT:dll_dllmain.obj
 0001:00082f4f       ?dllmain_crt_process_attach@@YAHQAUHINSTANCE__@@QAX@Z 10083f4f f   MSVCRT:dll_dllmain.obj
 0001:00083059       ?dllmain_crt_process_detach@@YAH_N@Z 10084059 f   MSVCRT:dll_dllmain.obj
 0001:000830eb       ?dllmain_dispatch@@YAHQAUHINSTANCE__@@KQAX@Z 100840eb f   MSVCRT:dll_dllmain.obj
 0001:000831f1       ?dllmain_raw@@YGHQAUHINSTANCE__@@KQAX@Z 100841f1 f   MSVCRT:dll_dllmain.obj
 0001:000833d6       ___get_entropy             100843d6 f   MSVCRT:gs_support.obj
 0001:000834cb       ?find_pe_section@@YAPAU_IMAGE_SECTION_HEADER@@QAEI@Z 100844cb f   MSVCRT:utility.obj
 0001:00083950       $$000000                   10084950     MSVCRT:sehprolg4.obj
 0002:00000310       _FONTKEY_NT                10085310     fontpath.obj
 0002:00000344       ?TTSUFFIX@?1??RegistryToBaseTTNameW@@9@9 10085344     fontpath.obj
 0002:0000035c       ?OTSUFFIX@?1??RegistryToBaseTTNameW@@9@9 1008535c     fontpath.obj
 0002:000004a0       ?outline_funcs@?1??addToGP@@9@9 100854a0     freetypeScaler.obj
 0002:00000550       ?table_tags@@3QBIB         10085550     gsubgpos-context.obj
 0002:00000558       ?hb_identity@@3U<unnamed-type-hb_identity>@@B 10085558     gsubgpos-context.obj
 0002:00000559       ?hb_ridentity@@3U<unnamed-type-hb_ridentity>@@B 10085559     gsubgpos-context.obj
 0002:0000055a       ?hb_swap@@3U<unnamed-type-hb_swap>@@B 1008555a     gsubgpos-context.obj
 0002:00000560       ?table_tags@@3QBIB         10085560     hb-aat-layout.obj
 0002:00000568       ?feature_mappings@@3QBUhb_aat_feature_mapping_t@@B 10085568     hb-aat-layout.obj
 0002:00000cc8       ?table_tags@@3QBIB         10085cc8     hb-aat-map.obj
 0002:00000d50       ?_deserialize_json_trans_keys@@3QBEB 10085d50     hb-buffer-serialize.obj
 0002:00000dc8       ?_deserialize_json_key_spans@@3QBDB 10085dc8     hb-buffer-serialize.obj
 0002:00000e08       ?_deserialize_json_index_offsets@@3QBFB 10085e08     hb-buffer-serialize.obj
 0002:00000e80       ?_deserialize_json_indicies@@3QBDB 10085e80     hb-buffer-serialize.obj
 0002:00001bb0       ?_deserialize_json_trans_targs@@3QBDB 10086bb0     hb-buffer-serialize.obj
 0002:00001c18       ?_deserialize_json_trans_actions@@3QBDB 10086c18     hb-buffer-serialize.obj
 0002:00001c7c       ?_deserialize_text_glyphs_trans_keys@@3QBEB 10086c7c     hb-buffer-serialize.obj
 0002:00001cb4       ?_deserialize_text_glyphs_key_spans@@3QBDB 10086cb4     hb-buffer-serialize.obj
 0002:00001cd0       ?_deserialize_text_glyphs_index_offsets@@3QBFB 10086cd0     hb-buffer-serialize.obj
 0002:00001d08       ?_deserialize_text_glyphs_indicies@@3QBDB 10086d08     hb-buffer-serialize.obj
 0002:000023d8       ?_deserialize_text_glyphs_trans_targs@@3QBDB 100873d8     hb-buffer-serialize.obj
 0002:00002418       ?_deserialize_text_glyphs_trans_actions@@3QBDB 10087418     hb-buffer-serialize.obj
 0002:00002458       ?_deserialize_text_glyphs_eof_actions@@3QBDB 10087458     hb-buffer-serialize.obj
 0002:00002474       ?_deserialize_text_unicode_trans_keys@@3QBEB 10087474     hb-buffer-serialize.obj
 0002:00002488       ?_deserialize_text_unicode_key_spans@@3QBDB 10087488     hb-buffer-serialize.obj
 0002:00002494       ?_deserialize_text_unicode_index_offsets@@3QBFB 10087494     hb-buffer-serialize.obj
 0002:000024a8       ?_deserialize_text_unicode_indicies@@3QBDB 100874a8     hb-buffer-serialize.obj
 0002:0000276c       ?_deserialize_text_unicode_trans_targs@@3QBDB 1008776c     hb-buffer-serialize.obj
 0002:0000277c       ?_deserialize_text_unicode_trans_actions@@3QBDB 1008777c     hb-buffer-serialize.obj
 0002:0000278c       ?_deserialize_text_unicode_eof_actions@@3QBDB 1008778c     hb-buffer-serialize.obj
 0002:00002888       ?table_tags@@3QBIB         10087888     hb-buffer.obj
 0002:000028a0       ?_hb_arabic_u8@@3QBEB      100878a0     hb-common.obj
 0002:00002a70       ?_hb_arabic_u16@@3QBGB     10087a70     hb-common.obj
 0002:00003010       ?direction_strings@@3QAY03$$CBDA 10088010     hb-common.obj
 0002:00003020       ?canon_map@@3QBDB          10088020     hb-common.obj
 0002:00003122       ?static_endchar_str@@3QBEB 10088122     hb-common.obj
 0002:00003128       ?table_tags@@3QBIB         10088128     hb-common.obj
 0002:000033b8       ?_hb_ms_language_map@@3QBUhb_ot_language_map_t@@B 100883b8     hb-common.obj
 0002:00003b38       ?_hb_mac_language_map@@3QBUhb_ot_language_map_t@@B 10088b38     hb-common.obj
 0002:00003ee0       ?_hb_os2_unicode_ranges@OT@@3QBUOS2Range@1@B 10088ee0     hb-common.obj
 0002:0000471c       ?table_tags@@3QBIB         1008971c     hb-face-builder.obj
 0002:00004724       ?hb_identity@@3U<unnamed-type-hb_identity>@@B 10089724     hb-face-builder.obj
 0002:00004725       ?hb_ridentity@@3U<unnamed-type-hb_ridentity>@@B 10089725     hb-face-builder.obj
 0002:00004778       ?table_tags@@3QBIB         10089778     hb-face.obj
 0002:00004780       ?_hb_os2_unicode_ranges@OT@@3QBUOS2Range@1@B 10089780     hb-face.obj
 0002:00004f70       ?_hb_arabic_u8@@3QBEB      10089f70     hb-face.obj
 0002:00005140       ?_hb_arabic_u16@@3QBGB     1008a140     hb-face.obj
 0002:000056e0       ?table_tags@@3QBIB         1008a6e0     hb-fallback-shape.obj
 0002:000056e8       ?table_tags@@3QBIB         1008a6e8     hb-font.obj
 0002:00005710       ?hb_identity@@3U<unnamed-type-hb_identity>@@B 1008a710     hb-map.obj
 0002:00005711       ?hb_ridentity@@3U<unnamed-type-hb_ridentity>@@B 1008a711     hb-map.obj
 0002:00005718       ?_double_parser_trans_keys@@3QBEB 1008a718     hb-number.obj
 0002:0000572c       ?_double_parser_key_spans@@3QBDB 1008a72c     hb-number.obj
 0002:00005738       ?_double_parser_index_offsets@@3QBEB 1008a738     hb-number.obj
 0002:00005748       ?_double_parser_indicies@@3QBDB 1008a748     hb-number.obj
 0002:00005808       ?_double_parser_trans_targs@@3QBDB 1008a808     hb-number.obj
 0002:00005814       ?_double_parser_trans_actions@@3QBDB 1008a814     hb-number.obj
 0002:00005820       ?_powers_of_10@?1??_pow10@@YANI@Z@4QBNB 1008a820     hb-number.obj
 0002:000058a0       ?table_tags@@3QBIB         1008a8a0     hb-ot-cff1-table.obj
 0002:000058a8       ?standard_encoding_to_code@@3QBEB 1008a8a8     hb-ot-cff1-table.obj
 0002:00005940       ?expert_encoding_to_code@@3QBEB 1008a940     hb-ot-cff1-table.obj
 0002:00005ac0       ?expert_charset_to_sid@@3QBGB 1008aac0     hb-ot-cff1-table.obj
 0002:00005c10       ?expert_subset_charset_to_sid@@3QBGB 1008ac10     hb-ot-cff1-table.obj
 0002:00005cc0       ?expert_charset_sid_to_gid@@3QBUsid_to_gid_t@@B 1008acc0     hb-ot-cff1-table.obj
 0002:00005f58       ?expert_subset_charset_sid_to_gid@@3QBUsid_to_gid_t@@B 1008af58     hb-ot-cff1-table.obj
 0002:000060b0       ?standard_encoding_to_sid@@3QBEB 1008b0b0     hb-ot-cff1-table.obj
 0002:000061b0       ?cff1_std_strings_msgstr@@3Tcff1_std_strings_msgstr_t@@B 1008b1b0     hb-ot-cff1-table.obj
 0002:00006f28       ?cff1_std_strings_msgidx@@3QBIB 1008bf28     hb-ot-cff1-table.obj
 0002:00007570       ?table_tags@@3QBIB         1008c570     hb-ot-cff2-table.obj
 0002:0000757c       ?table_tags@@3QBIB         1008c57c     hb-ot-color.obj
 0002:00007588       ?_hb_os2_unicode_ranges@OT@@3QBUOS2Range@1@B 1008c588     hb-ot-face.obj
 0002:00007d78       ?_hb_arabic_u8@@3QBEB      1008cd78     hb-ot-face.obj
 0002:00007f48       ?_hb_arabic_u16@@3QBGB     1008cf48     hb-ot-face.obj
 0002:000084e8       ?format1_names_msgstr@@3Tformat1_names_msgstr_t@@B 1008d4e8     hb-ot-face.obj
 0002:00008c28       ?format1_names_msgidx@@3QBIB 1008dc28     hb-ot-face.obj
 0002:00009038       ?cff1_std_strings_msgstr@@3Tcff1_std_strings_msgstr_t@@B 1008e038     hb-ot-face.obj
 0002:00009db0       ?cff1_std_strings_msgidx@@3QBIB 1008edb0     hb-ot-face.obj
 0002:0000a3d0       ?table_tags@@3QBIB         1008f3d0     hb-ot-face.obj
 0002:0000a3d8       ?cff1_std_strings_msgstr@@3Tcff1_std_strings_msgstr_t@@B 1008f3d8     hb-ot-font.obj
 0002:0000b150       ?cff1_std_strings_msgidx@@3QBIB 10090150     hb-ot-font.obj
 0002:0000b770       ?table_tags@@3QBIB         10090770     hb-ot-font.obj
 0002:0000b778       ?_hb_os2_unicode_ranges@OT@@3QBUOS2Range@1@B 10090778     hb-ot-font.obj
 0002:0000bf68       ?_hb_arabic_u8@@3QBEB      10090f68     hb-ot-font.obj
 0002:0000c138       ?_hb_arabic_u16@@3QBGB     10091138     hb-ot-font.obj
 0002:0000c6d8       ?format1_names_msgstr@@3Tformat1_names_msgstr_t@@B 100916d8     hb-ot-font.obj
 0002:0000ce18       ?format1_names_msgidx@@3QBIB 10091e18     hb-ot-font.obj
 0002:0000d270       ?_hb_os2_unicode_ranges@OT@@3QBUOS2Range@1@B 10092270     hb-ot-layout.obj
 0002:0000da5c       ?table_tags@@3QBIB         10092a5c     hb-ot-layout.obj
 0002:0000da64       ?hb_identity@@3U<unnamed-type-hb_identity>@@B 10092a64     hb-ot-layout.obj
 0002:0000da65       ?hb_first@@3U<unnamed-type-hb_first>@@B 10092a65     hb-ot-layout.obj
 0002:0000da66       ?hb_second@@3U<unnamed-type-hb_second>@@B 10092a66     hb-ot-layout.obj
 0002:0000da67       ?hb_add@@3U<unnamed-type-hb_add>@@B 10092a67     hb-ot-layout.obj
 0002:0000da68       ?hb_zip@@3U<unnamed-type-hb_zip>@@B 10092a68     hb-ot-layout.obj
 0002:0000da69       ?hb_any@@3U<unnamed-type-hb_any>@@B 10092a69     hb-ot-layout.obj
 0002:0000dfc8       ?table_tags@@3QBIB         10092fc8     hb-ot-map.obj
 0002:0000dfd0       ?table_tags@@3QBIB         10092fd0     hb-ot-math.obj
 0002:0000dfd8       ?table_tags@@3QBIB         10092fd8     hb-ot-meta.obj
 0002:0000dfe0       ?table_tags@@3QBIB         10092fe0     hb-ot-metrics.obj
 0002:0000dfe8       ?_hb_os2_unicode_ranges@OT@@3QBUOS2Range@1@B 10092fe8     hb-ot-metrics.obj
 0002:0000e7d8       ?format1_names_msgstr@@3Tformat1_names_msgstr_t@@B 100937d8     hb-ot-metrics.obj
 0002:0000ef18       ?format1_names_msgidx@@3QBIB 10093f18     hb-ot-metrics.obj
 0002:0000f324       ?table_tags@@3QBIB         10094324     hb-ot-name.obj
 0002:0000f32c       ?table_tags@@3QBIB         1009432c     hb-ot-shape-fallback.obj
 0002:0000f384       ?table_tags@@3QBIB         10094384     hb-ot-shape-normalize.obj
 0002:0000f3a8       ?table_tags@@3QBIB         100943a8     hb-ot-shape.obj
 0002:0000f3b0       ?common_features@@3QBUhb_ot_map_feature_t@@B 100943b0     hb-ot-shape.obj
 0002:0000f3e8       ?horizontal_features@@3QBUhb_ot_map_feature_t@@B 100943e8     hb-ot-shape.obj
 0002:0000f4a0       ?table_tags@@3QBIB         100944a0     hb-ot-shaper-arabic.obj
 0002:0000f4a8       ?arabic_fallback_features@@3QBIB 100944a8     hb-ot-shaper-arabic.obj
 0002:0000f4fc       ?ligature_3_table@@3QBUligature_3_set_t@@B 100944fc     hb-ot-shaper-arabic.obj
 0002:0000f510       ?joining_table@@3QBEB      10094510     hb-ot-shaper-arabic.obj
 0002:0000faa8       ?shaping_table@@3QAY03$$CBGA 10094aa8     hb-ot-shaper-arabic.obj
 0002:00010040       ?ligature_table@@3QBUligature_set_t@@B 10095040     hb-ot-shaper-arabic.obj
 0002:00010454       ?ligature_mark_table@@3QBUligature_mark_set_t@@B 10095454     hb-ot-shaper-arabic.obj
 0002:0001046c       ?arabic_features@@3QBIB    1009546c     hb-ot-shaper-arabic.obj
 0002:00010490       ?arabic_state_table@@3QAY05$$CBUarabic_state_table_entry@@A 10095490     hb-ot-shaper-arabic.obj
 0002:00010538       ?arabic_win1256_gsub_lookups@@3U0@B 10095538     hb-ot-shaper-arabic.obj
 0002:000106ca       ?hb_identity@@3U<unnamed-type-hb_identity>@@B 100956ca     hb-ot-shaper-arabic.obj
 0002:000106cb       ?hb_first@@3U<unnamed-type-hb_first>@@B 100956cb     hb-ot-shaper-arabic.obj
 0002:000106cc       ?hb_second@@3U<unnamed-type-hb_second>@@B 100956cc     hb-ot-shaper-arabic.obj
 0002:000106cd       ?hb_add@@3U<unnamed-type-hb_add>@@B 100956cd     hb-ot-shaper-arabic.obj
 0002:00010708       ?table_tags@@3QBIB         10095708     hb-ot-shaper-default.obj
 0002:00010780       ?table_tags@@3QBIB         10095780     hb-ot-shaper-hangul.obj
 0002:000107c0       ?hangul_features@@3QBIB    100957c0     hb-ot-shaper-hangul.obj
 0002:000107d0       ?table_tags@@3QBIB         100957d0     hb-ot-shaper-hebrew.obj
 0002:00010810       ?sDageshForms@?1??compose_hebrew@@YA_NPBUhb_ot_shape_normalize_context_t@@IIPAI@Z@4QBIB 10095810     hb-ot-shaper-hebrew.obj
 0002:00010880       ?table_tags@@3QBIB         10095880     hb-ot-shaper-indic-table.obj
 0002:00010888       ?_indic_syllable_machine_trans_keys@@3QBEB 10095888     hb-ot-shaper-indic-table.obj
 0002:000109a0       ?_indic_syllable_machine_key_spans@@3QBDB 100959a0     hb-ot-shaper-indic-table.obj
 0002:00010a30       ?_indic_syllable_machine_index_offsets@@3QBFB 10095a30     hb-ot-shaper-indic-table.obj
 0002:00010b48       ?_indic_syllable_machine_indicies@@3QBEB 10095b48     hb-ot-shaper-indic-table.obj
 0002:000110e8       ?_indic_syllable_machine_trans_targs@@3QBEB 100960e8     hb-ot-shaper-indic-table.obj
 0002:00011180       ?_indic_syllable_machine_trans_actions@@3QBDB 10096180     hb-ot-shaper-indic-table.obj
 0002:00011218       ?_indic_syllable_machine_to_state_actions@@3QBDB 10096218     hb-ot-shaper-indic-table.obj
 0002:000112a8       ?_indic_syllable_machine_from_state_actions@@3QBDB 100962a8     hb-ot-shaper-indic-table.obj
 0002:00011338       ?_indic_syllable_machine_eof_trans@@3QBFB 10096338     hb-ot-shaper-indic-table.obj
 0002:00011450       ?_khmer_syllable_machine_trans_keys@@3QBEB 10096450     hb-ot-shaper-indic-table.obj
 0002:000114a8       ?_khmer_syllable_machine_key_spans@@3QBDB 100964a8     hb-ot-shaper-indic-table.obj
 0002:000114d8       ?_khmer_syllable_machine_index_offsets@@3QBFB 100964d8     hb-ot-shaper-indic-table.obj
 0002:00011530       ?_khmer_syllable_machine_indicies@@3QBDB 10096530     hb-ot-shaper-indic-table.obj
 0002:000118f0       ?_khmer_syllable_machine_trans_targs@@3QBDB 100968f0     hb-ot-shaper-indic-table.obj
 0002:00011924       ?_khmer_syllable_machine_trans_actions@@3QBDB 10096924     hb-ot-shaper-indic-table.obj
 0002:00011958       ?_khmer_syllable_machine_to_state_actions@@3QBDB 10096958     hb-ot-shaper-indic-table.obj
 0002:00011984       ?_khmer_syllable_machine_from_state_actions@@3QBDB 10096984     hb-ot-shaper-indic-table.obj
 0002:000119b0       ?_khmer_syllable_machine_eof_trans@@3QBFB 100969b0     hb-ot-shaper-indic-table.obj
 0002:00011a08       ?_myanmar_syllable_machine_trans_keys@@3QBEB 10096a08     hb-ot-shaper-indic-table.obj
 0002:00011a78       ?_myanmar_syllable_machine_key_spans@@3QBDB 10096a78     hb-ot-shaper-indic-table.obj
 0002:00011ab0       ?_myanmar_syllable_machine_index_offsets@@3QBFB 10096ab0     hb-ot-shaper-indic-table.obj
 0002:00011b20       ?_myanmar_syllable_machine_indicies@@3QBDB 10096b20     hb-ot-shaper-indic-table.obj
 0002:000122f0       ?_myanmar_syllable_machine_trans_targs@@3QBDB 100972f0     hb-ot-shaper-indic-table.obj
 0002:00012330       ?_myanmar_syllable_machine_trans_actions@@3QBDB 10097330     hb-ot-shaper-indic-table.obj
 0002:00012370       ?_myanmar_syllable_machine_to_state_actions@@3QBDB 10097370     hb-ot-shaper-indic-table.obj
 0002:000123a8       ?_myanmar_syllable_machine_from_state_actions@@3QBDB 100973a8     hb-ot-shaper-indic-table.obj
 0002:000123e0       ?_myanmar_syllable_machine_eof_trans@@3QBFB 100973e0     hb-ot-shaper-indic-table.obj
 0002:00012450       ?indic_table@@3QBGB        10097450     hb-ot-shaper-indic-table.obj
 0002:000131d0       ?table_tags@@3QBIB         100981d0     hb-ot-shaper-indic.obj
 0002:00013210       ?_indic_syllable_machine_trans_keys@@3QBEB 10098210     hb-ot-shaper-indic.obj
 0002:00013328       ?_indic_syllable_machine_key_spans@@3QBDB 10098328     hb-ot-shaper-indic.obj
 0002:000133b8       ?_indic_syllable_machine_index_offsets@@3QBFB 100983b8     hb-ot-shaper-indic.obj
 0002:000134d0       ?_indic_syllable_machine_indicies@@3QBEB 100984d0     hb-ot-shaper-indic.obj
 0002:00013a70       ?_indic_syllable_machine_trans_targs@@3QBEB 10098a70     hb-ot-shaper-indic.obj
 0002:00013b08       ?_indic_syllable_machine_trans_actions@@3QBDB 10098b08     hb-ot-shaper-indic.obj
 0002:00013ba0       ?_indic_syllable_machine_to_state_actions@@3QBDB 10098ba0     hb-ot-shaper-indic.obj
 0002:00013c30       ?_indic_syllable_machine_from_state_actions@@3QBDB 10098c30     hb-ot-shaper-indic.obj
 0002:00013cc0       ?_indic_syllable_machine_eof_trans@@3QBFB 10098cc0     hb-ot-shaper-indic.obj
 0002:00013dd8       ?indic_configs@@3QBUindic_config_t@@B 10098dd8     hb-ot-shaper-indic.obj
 0002:00013f48       ?table_tags@@3QBIB         10098f48     hb-ot-shaper-khmer.obj
 0002:00013f88       ?_khmer_syllable_machine_trans_keys@@3QBEB 10098f88     hb-ot-shaper-khmer.obj
 0002:00013fe0       ?_khmer_syllable_machine_key_spans@@3QBDB 10098fe0     hb-ot-shaper-khmer.obj
 0002:00014010       ?_khmer_syllable_machine_index_offsets@@3QBFB 10099010     hb-ot-shaper-khmer.obj
 0002:00014068       ?_khmer_syllable_machine_indicies@@3QBDB 10099068     hb-ot-shaper-khmer.obj
 0002:00014428       ?_khmer_syllable_machine_trans_targs@@3QBDB 10099428     hb-ot-shaper-khmer.obj
 0002:0001445c       ?_khmer_syllable_machine_trans_actions@@3QBDB 1009945c     hb-ot-shaper-khmer.obj
 0002:00014490       ?_khmer_syllable_machine_to_state_actions@@3QBDB 10099490     hb-ot-shaper-khmer.obj
 0002:000144bc       ?_khmer_syllable_machine_from_state_actions@@3QBDB 100994bc     hb-ot-shaper-khmer.obj
 0002:000144e8       ?_khmer_syllable_machine_eof_trans@@3QBFB 100994e8     hb-ot-shaper-khmer.obj
 0002:00014570       ?table_tags@@3QBIB         10099570     hb-ot-shaper-myanmar.obj
 0002:000145e8       ?_myanmar_syllable_machine_trans_keys@@3QBEB 100995e8     hb-ot-shaper-myanmar.obj
 0002:00014658       ?_myanmar_syllable_machine_key_spans@@3QBDB 10099658     hb-ot-shaper-myanmar.obj
 0002:00014690       ?_myanmar_syllable_machine_index_offsets@@3QBFB 10099690     hb-ot-shaper-myanmar.obj
 0002:00014700       ?_myanmar_syllable_machine_indicies@@3QBDB 10099700     hb-ot-shaper-myanmar.obj
 0002:00014ed0       ?_myanmar_syllable_machine_trans_targs@@3QBDB 10099ed0     hb-ot-shaper-myanmar.obj
 0002:00014f10       ?_myanmar_syllable_machine_trans_actions@@3QBDB 10099f10     hb-ot-shaper-myanmar.obj
 0002:00014f50       ?_myanmar_syllable_machine_to_state_actions@@3QBDB 10099f50     hb-ot-shaper-myanmar.obj
 0002:00014f88       ?_myanmar_syllable_machine_from_state_actions@@3QBDB 10099f88     hb-ot-shaper-myanmar.obj
 0002:00014fc0       ?_myanmar_syllable_machine_eof_trans@@3QBFB 10099fc0     hb-ot-shaper-myanmar.obj
 0002:00015030       ?myanmar_basic_features@@3QBIB 1009a030     hb-ot-shaper-myanmar.obj
 0002:00015040       ?myanmar_other_features@@3QBIB 1009a040     hb-ot-shaper-myanmar.obj
 0002:00015084       ?table_tags@@3QBIB         1009a084     hb-ot-shaper-syllabic.obj
 0002:00015118       ?table_tags@@3QBIB         1009a118     hb-ot-shaper-thai.obj
 0002:00015158       ?thai_above_state_machine@@3QAY02$$CBUthai_above_state_machine_edge_t@@A 1009a158     hb-ot-shaper-thai.obj
 0002:000151b8       ?thai_below_state_machine@@3QAY02$$CBUthai_below_state_machine_edge_t@@A 1009a1b8     hb-ot-shaper-thai.obj
 0002:00015200       ?SD_mappings@?1??thai_pua_shape@@YAIIW4thai_action_t@@PAUhb_font_t@@@Z@4QBUthai_pua_mapping_t@?1??1@YAII01@Z@B 1009a200     hb-ot-shaper-thai.obj
 0002:00015238       ?SDL_mappings@?1??thai_pua_shape@@YAIIW4thai_action_t@@PAUhb_font_t@@@Z@4QBUthai_pua_mapping_t@?1??1@YAII01@Z@B 1009a238     hb-ot-shaper-thai.obj
 0002:00015260       ?SL_mappings@?1??thai_pua_shape@@YAIIW4thai_action_t@@PAUhb_font_t@@@Z@4QBUthai_pua_mapping_t@?1??1@YAII01@Z@B 1009a260     hb-ot-shaper-thai.obj
 0002:000152b0       ?RD_mappings@?1??thai_pua_shape@@YAIIW4thai_action_t@@PAUhb_font_t@@@Z@4QBUthai_pua_mapping_t@?1??1@YAII01@Z@B 1009a2b0     hb-ot-shaper-thai.obj
 0002:000152c8       ?table_tags@@3QBIB         1009a2c8     hb-ot-shaper-use.obj
 0002:00015308       ?_use_syllable_machine_trans_keys@@3QBEB 1009a308     hb-ot-shaper-use.obj
 0002:00015408       ?_use_syllable_machine_key_spans@@3QBDB 1009a408     hb-ot-shaper-use.obj
 0002:00015488       ?_use_syllable_machine_index_offsets@@3QBFB 1009a488     hb-ot-shaper-use.obj
 0002:00015588       ?_use_syllable_machine_indicies@@3QBEB 1009a588     hb-ot-shaper-use.obj
 0002:000166c0       ?_use_syllable_machine_trans_targs@@3QBDB 1009b6c0     hb-ot-shaper-use.obj
 0002:00016750       ?_use_syllable_machine_trans_actions@@3QBDB 1009b750     hb-ot-shaper-use.obj
 0002:000167e0       ?_use_syllable_machine_to_state_actions@@3QBDB 1009b7e0     hb-ot-shaper-use.obj
 0002:00016860       ?_use_syllable_machine_from_state_actions@@3QBDB 1009b860     hb-ot-shaper-use.obj
 0002:000168e0       ?_use_syllable_machine_eof_trans@@3QBFB 1009b8e0     hb-ot-shaper-use.obj
 0002:000169e0       ?hb_use_u8@@3QBEB          1009b9e0     hb-ot-shaper-use.obj
 0002:00017658       ?hb_use_u16@@3QBGB         1009c658     hb-ot-shaper-use.obj
 0002:00017ca8       ?use_basic_features@@3QBIB 1009cca8     hb-ot-shaper-use.obj
 0002:00017cc4       ?use_topographical_features@@3QBIB 1009ccc4     hb-ot-shaper-use.obj
 0002:00017cd4       ?use_other_features@@3QBIB 1009ccd4     hb-ot-shaper-use.obj
 0002:00017ce8       ?hb_identity@@3U<unnamed-type-hb_identity>@@B 1009cce8     hb-ot-shaper-use.obj
 0002:00017ce9       ?hb_second@@3U<unnamed-type-hb_second>@@B 1009cce9     hb-ot-shaper-use.obj
 0002:00017d18       ?table_tags@@3QBIB         1009cd18     hb-ot-shaper-vowel-constraints.obj
 0002:00017d20       ?ot_languages2@@3QBULangTag@@B 1009cd20     hb-ot-tag.obj
 0002:00018378       ?ot_languages3@@3QBULangTag@@B 1009d378     hb-ot-tag.obj
 0002:0001ae0c       ?table_tags@@3QBIB         1009fe0c     hb-ot-var.obj
 0002:0001ae1c       ?table_tags@@3QBIB         1009fe1c     hb-paint.obj
 0002:0001ae24       ?table_tags@@3QBIB         1009fe24     hb-shape-plan.obj
 0002:0001b108       ?table_tags@@3QBIB         100a0108     hb-shape.obj
 0002:0001b110       ?nil_shaper_list@@3QBQBDB  100a0110     hb-shape.obj
 0002:0001b114       ?_hb_all_shapers@@3QBUhb_shaper_entry_t@@B 100a0114     hb-shaper.obj
 0002:0001b150       ?table_tags@@3QBIB         100a0150     hb-static.obj
 0002:0001b158       ?_hb_os2_unicode_ranges@OT@@3QBUOS2Range@1@B 100a0158     hb-static.obj
 0002:0001b948       ?_hb_arabic_u8@@3QBEB      100a0948     hb-static.obj
 0002:0001bb18       ?_hb_arabic_u16@@3QBGB     100a0b18     hb-static.obj
 0002:0001c0b8       ?_hb_os2_unicode_ranges@OT@@3QBUOS2Range@1@B 100a10b8     hb-style.obj
 0002:0001c8a4       ?table_tags@@3QBIB         100a18a4     hb-style.obj
 0002:0001c8b0       ?format1_names_msgstr@@3Tformat1_names_msgstr_t@@B 100a18b0     hb-style.obj
 0002:0001cff0       ?format1_names_msgidx@@3QBIB 100a1ff0     hb-style.obj
 0002:0001d3fc       ?table_tags@@3QBIB         100a23fc     hb-subset-cff-common.obj
 0002:0001d408       ?table_tags@@3QBIB         100a2408     hb-subset-cff1.obj
 0002:0001d410       ?cff1_std_strings_msgstr@@3Tcff1_std_strings_msgstr_t@@B 100a2410     hb-subset-cff1.obj
 0002:0001e188       ?cff1_std_strings_msgidx@@3QBIB 100a3188     hb-subset-cff1.obj
 0002:0001e7a8       ?hb_identity@@3U<unnamed-type-hb_identity>@@B 100a37a8     hb-subset-cff1.obj
 0002:0001e7a9       ?hb_swap@@3U<unnamed-type-hb_swap>@@B 100a37a9     hb-subset-cff1.obj
 0002:0001e7ac       ?table_tags@@3QBIB         100a37ac     hb-subset-cff2.obj
 0002:0001e7b4       ?hb_identity@@3U<unnamed-type-hb_identity>@@B 100a37b4     hb-subset-cff2.obj
 0002:0001e7b5       ?hb_swap@@3U<unnamed-type-hb_swap>@@B 100a37b5     hb-subset-cff2.obj
 0002:0001e7b8       ?table_tags@@3QBIB         100a37b8     hb-subset-input.obj
 0002:0001e7c0       ?table_tags@@3QBIB         100a37c0     hb-subset-plan.obj
 0002:0001e7c8       ?_hb_os2_unicode_ranges@OT@@3QBUOS2Range@1@B 100a37c8     hb-subset-plan.obj
 0002:0001efb8       ?_hb_arabic_u8@@3QBEB      100a3fb8     hb-subset-plan.obj
 0002:0001f188       ?_hb_arabic_u16@@3QBGB     100a4188     hb-subset-plan.obj
 0002:0001f728       ?cff1_std_strings_msgstr@@3Tcff1_std_strings_msgstr_t@@B 100a4728     hb-subset-plan.obj
 0002:000204a0       ?cff1_std_strings_msgidx@@3QBIB 100a54a0     hb-subset-plan.obj
 0002:00020ac0       ?hb_identity@@3U<unnamed-type-hb_identity>@@B 100a5ac0     hb-subset-plan.obj
 0002:00020ac1       ?hb_ridentity@@3U<unnamed-type-hb_ridentity>@@B 100a5ac1     hb-subset-plan.obj
 0002:00020ac2       ?hb_bool@@3U<unnamed-type-hb_bool>@@B 100a5ac2     hb-subset-plan.obj
 0002:00020ac3       ?hb_hash@@3U<unnamed-type-hb_hash>@@B 100a5ac3     hb-subset-plan.obj
 0002:00020ac4       ?hb_swap@@3U<unnamed-type-hb_swap>@@B 100a5ac4     hb-subset-plan.obj
 0002:00020ac5       ?hb_first@@3U<unnamed-type-hb_first>@@B 100a5ac5     hb-subset-plan.obj
 0002:00020ac6       ?hb_second@@3U<unnamed-type-hb_second>@@B 100a5ac6     hb-subset-plan.obj
 0002:00020ac7       ?hb_add@@3U<unnamed-type-hb_add>@@B 100a5ac7     hb-subset-plan.obj
 0002:00020ac8       ?hb_iter@@3U<unnamed-type-hb_iter>@@B 100a5ac8     hb-subset-plan.obj
 0002:00020ac9       ?hb_zip@@3U<unnamed-type-hb_zip>@@B 100a5ac9     hb-subset-plan.obj
 0002:00020aca       ?hb_enumerate@@3U<unnamed-type-hb_enumerate>@@B 100a5aca     hb-subset-plan.obj
 0002:00020ad0       ?cff1_std_strings_msgstr@@3Tcff1_std_strings_msgstr_t@@B 100a5ad0     hb-subset.obj
 0002:00021848       ?cff1_std_strings_msgidx@@3QBIB 100a6848     hb-subset.obj
 0002:00021e68       ?table_tags@@3QBIB         100a6e68     hb-subset.obj
 0002:00021e70       ?format1_names_msgstr@@3Tformat1_names_msgstr_t@@B 100a6e70     hb-subset.obj
 0002:000225b0       ?format1_names_msgidx@@3QBIB 100a75b0     hb-subset.obj
 0002:000229c0       ?_hb_os2_unicode_ranges@OT@@3QBUOS2Range@1@B 100a79c0     hb-subset.obj
 0002:000231b0       ?_hb_arabic_u8@@3QBEB      100a81b0     hb-subset.obj
 0002:00023380       ?_hb_arabic_u16@@3QBGB     100a8380     hb-subset.obj
 0002:00023920       ?hb_identity@@3U<unnamed-type-hb_identity>@@B 100a8920     hb-subset.obj
 0002:00023921       ?hb_ridentity@@3U<unnamed-type-hb_ridentity>@@B 100a8921     hb-subset.obj
 0002:00023922       ?hb_hash@@3U<unnamed-type-hb_hash>@@B 100a8922     hb-subset.obj
 0002:00023923       ?hb_swap@@3U<unnamed-type-hb_swap>@@B 100a8923     hb-subset.obj
 0002:00023924       ?hb_first@@3U<unnamed-type-hb_first>@@B 100a8924     hb-subset.obj
 0002:00023925       ?hb_second@@3U<unnamed-type-hb_second>@@B 100a8925     hb-subset.obj
 0002:00023926       ?hb_add@@3U<unnamed-type-hb_add>@@B 100a8926     hb-subset.obj
 0002:00023927       ?hb_iter@@3U<unnamed-type-hb_iter>@@B 100a8927     hb-subset.obj
 0002:00023928       ?hb_len@@3U<unnamed-type-hb_len>@@B 100a8928     hb-subset.obj
 0002:00023929       ?hb_zip@@3U<unnamed-type-hb_zip>@@B 100a8929     hb-subset.obj
 0002:0002392a       ?hb_enumerate@@3U<unnamed-type-hb_enumerate>@@B 100a892a     hb-subset.obj
 0002:0002392b       ?hb_take@@3U<unnamed-type-hb_take>@@B 100a892b     hb-subset.obj
 0002:0002392c       ?hb_all@@3U<unnamed-type-hb_all>@@B 100a892c     hb-subset.obj
 0002:00023930       ?_hb_ucd_sc_map@@3QBW4hb_script_t@@B 100a8930     hb-ucd.obj
 0002:00023bc8       ?_hb_ucd_dm1_p0_map@@3QBGB 100a8bc8     hb-ucd.obj
 0002:00024240       ?_hb_ucd_dm1_p2_map@@3QBGB 100a9240     hb-ucd.obj
 0002:00024320       ?_hb_ucd_dm2_u32_map@@3QBIB 100a9320     hb-ucd.obj
 0002:00024d18       ?_hb_ucd_dm2_u64_map@@3QB_KB 100a9d18     hb-ucd.obj
 0002:00025938       ?_hb_ucd_u8@@3QBEB         100aa938     hb-ucd.obj
 0002:00029f18       ?_hb_ucd_u16@@3QBGB        100aef18     hb-ucd.obj
 0002:0002e818       ?_hb_ucd_i16@@3QBFB        100b3818     hb-ucd.obj
 0002:0002e9a0       ?_hb_emoji_u8@@3QBEB       100b39a0     hb-unicode.obj
 0002:0002efa0       _Int32ToUInt32             100b3fa0     MSVCRT:ftol3.obj
 0002:0002efa8       _DP2to32                   100b3fa8     MSVCRT:ftol3.obj
 0002:0002efb0       _MantissaMask              100b3fb0     MSVCRT:ftol3.obj
 0002:0002efb8       _IntegerBit                100b3fb8     MSVCRT:ftol3.obj
 0002:0002efc0       _SignBit64                 100b3fc0     MSVCRT:ftol3.obj
 0002:0002efc8       _MinFP64                   100b3fc8     MSVCRT:ftol3.obj
 0002:0002efd0       _MinInt64                  100b3fd0     MSVCRT:ftol3.obj
 0002:0002efd8       _MaxInt64                  100b3fd8     MSVCRT:ftol3.obj
 0002:0002efe0       _MaxUInt64                 100b3fe0     MSVCRT:ftol3.obj
 0002:0002efe8       _MaxFP32                   100b3fe8     MSVCRT:ftol3.obj
 0002:0002eff0       _MinFP32                   100b3ff0     MSVCRT:ftol3.obj
 0002:0002eff8       _MinSubInexact             100b3ff8     MSVCRT:ftol3.obj
 0002:0002f000       _FpExcptTable              100b4000     MSVCRT:ftol3.obj
 0002:0002f010       _i1075                     100b4010     MSVCRT:ftol3.obj
 0002:0002f014       _i1087                     100b4014     MSVCRT:ftol3.obj
 0002:0002f018       _x0800                     100b4018     MSVCRT:ftol3.obj
 0002:0002f01c       _x17FF                     100b401c     MSVCRT:ftol3.obj
 0002:0002f020       _CWMask                    100b4020     MSVCRT:ftol3.obj
 0002:0002f024       _GS_ExceptionPointers      100b4024     MSVCRT:gs_report.obj
 0002:0002f460       __sehtable$?dllmain_crt_process_attach@@YAHQAUHINSTANCE__@@QAX@Z 100b4460     MSVCRT:dll_dllmain.obj
 0002:0002f480       __sehtable$?dllmain_crt_process_detach@@YAH_N@Z 100b4480     MSVCRT:dll_dllmain.obj
 0002:0002f4a0       __sehtable$?dllmain_dispatch@@YAHQAUHINSTANCE__@@KQAX@Z 100b44a0     MSVCRT:dll_dllmain.obj
 0002:0002f4c0       __sehtable$___scrt_is_nonwritable_in_current_image 100b44c0     MSVCRT:utility.obj
 0002:0002f4e0       .edata                     100b44e0     fontmanager.exp
 0002:0002f508       rgpv                       100b4508     fontmanager.exp
 0002:0002f598       rgszName                   100b4598     fontmanager.exp
 0002:0002f628       rgwOrd                     100b4628     fontmanager.exp
 0002:0002f670       szName                     100b4670     fontmanager.exp
 0002:0002f680       $N00001                    100b4680     fontmanager.exp
 0002:0002f6ae       $N00002                    100b46ae     fontmanager.exp
 0002:0002f6e9       $N00003                    100b46e9     fontmanager.exp
 0002:0002f725       $N00004                    100b4725     fontmanager.exp
 0002:0002f750       $N00005                    100b4750     fontmanager.exp
 0002:0002f78f       $N00006                    100b478f     fontmanager.exp
 0002:0002f7c8       $N00007                    100b47c8     fontmanager.exp
 0002:0002f802       $N00008                    100b4802     fontmanager.exp
 0002:0002f83d       $N00009                    100b483d     fontmanager.exp
 0002:0002f875       $N00010                    100b4875     fontmanager.exp
 0002:0002f8ae       $N00011                    100b48ae     fontmanager.exp
 0002:0002f8e9       $N00012                    100b48e9     fontmanager.exp
 0002:0002f92a       $N00013                    100b492a     fontmanager.exp
 0002:0002f965       $N00014                    100b4965     fontmanager.exp
 0002:0002f99e       $N00015                    100b499e     fontmanager.exp
 0002:0002f9df       $N00016                    100b49df     fontmanager.exp
 0002:0002fa1e       $N00017                    100b4a1e     fontmanager.exp
 0002:0002fa56       $N00018                    100b4a56     fontmanager.exp
 0002:0002fa8f       $N00019                    100b4a8f     fontmanager.exp
 0002:0002fabc       $N00020                    100b4abc     fontmanager.exp
 0002:0002faf2       $N00021                    100b4af2     fontmanager.exp
 0002:0002fb21       $N00022                    100b4b21     fontmanager.exp
 0002:0002fb56       $N00023                    100b4b56     fontmanager.exp
 0002:0002fb82       $N00024                    100b4b82     fontmanager.exp
 0002:0002fbaf       $N00025                    100b4baf     fontmanager.exp
 0002:0002fbdc       $N00026                    100b4bdc     fontmanager.exp
 0002:0002fc0a       $N00027                    100b4c0a     fontmanager.exp
 0002:0002fc41       $N00028                    100b4c41     fontmanager.exp
 0002:0002fc69       $N00029                    100b4c69     fontmanager.exp
 0002:0002fc96       $N00030                    100b4c96     fontmanager.exp
 0002:0002fcc4       $N00031                    100b4cc4     fontmanager.exp
 0002:0002fcec       $N00032                    100b4cec     fontmanager.exp
 0002:0002fd26       $N00033                    100b4d26     fontmanager.exp
 0002:0002fd62       $N00034                    100b4d62     fontmanager.exp
 0002:0002fd98       $N00035                    100b4d98     fontmanager.exp
 0002:0002fda6       $N00036                    100b4da6     fontmanager.exp
 0002:0003029e       .idata$6                   100b529e     freetype:freetype.dll
 0002:000302f6       .idata$6                   100b52f6     java:java.dll
 0002:00030342       .idata$6                   100b5342     advapi32:ADVAPI32.dll
 0002:000303aa       .idata$6                   100b53aa     user32:USER32.dll
 0002:000304ce       .idata$6                   100b54ce     gdi32:GDI32.dll
 0002:000305dc       .idata$6                   100b55dc     awt:awt.dll
 0002:000307a8       .idata$6                   100b57a8     kernel32:KERNEL32.dll
 0002:00030840       .idata$6                   100b5840     vcruntime:VCRUNTIME140.dll
 0002:00030a56       .idata$6                   100b5a56     ucrt:api-ms-win-crt-heap-l1-1-0.dll
 0002:00030a76       .idata$6                   100b5a76     ucrt:api-ms-win-crt-math-l1-1-0.dll
 0002:00030a96       .idata$6                   100b5a96     ucrt:api-ms-win-crt-environment-l1-1-0.dll
 0002:00030abc       .idata$6                   100b5abc     ucrt:api-ms-win-crt-convert-l1-1-0.dll
 0002:00030ade       .idata$6                   100b5ade     ucrt:api-ms-win-crt-stdio-l1-1-0.dll
 0002:00030afe       .idata$6                   100b5afe     ucrt:api-ms-win-crt-string-l1-1-0.dll
 0002:00030b20       .idata$6                   100b5b20     ucrt:api-ms-win-crt-runtime-l1-1-0.dll
 0003:00000200       _gvdClassName              100b6200     HBShaper.obj
 0003:00000204       ?PADBYTES@?1??getGlyphImageNativeInternal@@9@9 100b6204     freetypeScaler.obj
 0003:00000208       ?_hb_buffer_serialize_formats@@3PAPBDA 100b6208     hb-buffer-serialize.obj
 0003:000004b8       ?_hb_draw_funcs_default@@3Uhb_draw_funcs_t@@B 100b64b8     hb-font.obj
 0003:000004e0       ?_hb_font_funcs_default@@3Uhb_font_funcs_t@@B 100b64e0     hb-font.obj
 0003:00000540       ?modifier_combining_marks@@3PAIA 100b6540     hb-ot-shaper-arabic.obj
 0003:00000578       ?indic_features@@3QBUhb_ot_map_feature_t@@B 100b6578     hb-ot-shaper-indic.obj
 0003:00000600       ?khmer_features@@3QBUhb_ot_map_feature_t@@B 100b6600     hb-ot-shaper-khmer.obj
 0003:00000648       ?thai_above_start_state@@3PAW4thai_above_state_t@@A 100b6648     hb-ot-shaper-thai.obj
 0003:0000065c       ?thai_below_start_state@@3PAW4thai_below_state_t@@A 100b665c     hb-ot-shaper-thai.obj
 0003:000006c0       ?known_tables@@3PAIA       100b66c0     hb-subset.obj
 0003:00000900       _gvdClass                  100b6900     HBShaper.obj
 0003:00000904       _gvdCountFID               100b6904     HBShaper.obj
 0003:00000908       _gvdFlagsFID               100b6908     HBShaper.obj
 0003:0000090c       _gvdGlyphsFID              100b690c     HBShaper.obj
 0003:00000910       _gvdPositionsFID           100b6910     HBShaper.obj
 0003:00000914       _gvdIndicesFID             100b6914     HBShaper.obj
 0003:00000918       _gvdGrowMID                100b6918     HBShaper.obj
 0003:0000091c       _jniInited                 100b691c     HBShaper.obj
 0003:00000920       _screenDC                  100b6920     fontpath.obj
 0003:00000924       _invalidateScalerMID       100b6924     freetypeScaler.obj
 0003:00000bb4       ?langs@@3U?$hb_atomic_ptr_t@Uhb_language_item_t@@@@A 100b6bb4     hb-common.obj
 0003:00000bb8       ?jdk_ffuncs@?1??_hb_jdk_get_font_funcs@@YAPAUhb_font_funcs_t@@XZ@4PAU2@A 100b6bb8     hb-jdk-font.obj
 0003:00000bbc       ?static_ot_funcs@@3Uhb_ot_font_funcs_lazy_loader_t@@A 100b6bbc     hb-ot-font.obj
 0003:00000bc0       ?hb_ot_font_cmap_cache_user_data_key@@3Uhb_user_data_key_t@@A 100b6bc0     hb-ot-font.obj
 0003:00000bc4       ?last_tag_idx@?4??hb_ot_tags_from_language@@YAXPBD0PAI1@Z@4Uhb_atomic_int_t@@A 100b6bc4     hb-ot-tag.obj
 0003:00000bc8       ?static_outline_recording_pen_funcs@@3Uhb_outline_recording_pen_funcs_lazy_loader_t@@A 100b6bc8     hb-outline.obj
 0003:00000bcc       ?static_draw_extents_funcs@@3Uhb_draw_extents_funcs_lazy_loader_t@@A 100b6bcc     hb-paint-extents.obj
 0003:00000bd0       ?static_paint_extents_funcs@@3Uhb_paint_extents_funcs_lazy_loader_t@@A 100b6bd0     hb-paint-extents.obj
 0003:00000bd4       ?static_shaper_list@@3Uhb_shaper_list_lazy_loader_t@@A 100b6bd4     hb-shape.obj
 0003:00000bd8       ?static_shapers@@3Uhb_shapers_lazy_loader_t@@A 100b6bd8     hb-shaper.obj
 0003:00000be0       ?static_ucd_funcs@@3Uhb_ucd_unicode_funcs_lazy_loader_t@@A 100b6be0     hb-ucd.obj
 0003:00000be8       _igLUTable                 100b6be8     lcdglyph.obj
 0003:00000dcc       _theNullScalerContext      100b6dcc     sunFont.obj
 0003:00000dd0       _initialisedFontIDs        100b6dd0     sunFont.obj
 0003:00000dd8       _GS_ExceptionRecord        100b6dd8     MSVCRT:gs_report.obj
 0003:00000e28       _GS_ContextRecord          100b6e28     MSVCRT:gs_report.obj
 0003:000010f8       ?__proc_attached@@3HA      100b70f8     MSVCRT:dll_dllmain.obj
 0003:00001120       ?is_initialized_as_dll@@3_NA 100b7120     MSVCRT:utility.obj
 0003:00001121       ?module_local_atexit_table_initialized@@3_NA 100b7121     MSVCRT:utility.obj
 0003:00001124       ?module_local_atexit_table@@3U_onexit_table_t@@A 100b7124     MSVCRT:utility.obj
 0003:00001130       ?module_local_at_quick_exit_table@@3U_onexit_table_t@@A 100b7130     MSVCRT:utility.obj
 0004:00000060       $R000000                   100b8060     fontmanager.dll.res
